
 Start         Length     Name                   Class
 0001:00000000 0005DF6CH .text                   CODE
 0002:00000000 00001370H .data                   DATA
 0002:00001370 00000C29H .bss                    BSS


Detailed map of segments

 0001:00000000 000053CB C=CODE     S=.text    G=(none)   M=System   ACBP=A9
 0001:000053CC 000001CC C=CODE     S=.text    G=(none)   M=SysInit  ACBP=A9
 0001:00005598 00000078 C=CODE     S=.text    G=(none)   M=Types    ACBP=A9
 0001:00005610 00000CA0 C=CODE     S=.text    G=(none)   M=Windows  ACBP=A9
 0001:000062B0 00000310 C=CODE     S=.text    G=(none)   M=SysConst ACBP=A9
 0001:000065C0 00006564 C=CODE     S=.text    G=(none)   M=SysUtils ACBP=A9
 0001:0000CB24 00000038 C=CODE     S=.text    G=(none)   M=Messages ACBP=A9
 0001:0000CB5C 000007FB C=CODE     S=.text    G=(none)   M=VarUtils ACBP=A9
 0001:0000D358 00005B12 C=CODE     S=.text    G=(none)   M=Variants ACBP=A9
 0001:00012E6C 00000120 C=CODE     S=.text    G=(none)   M=RTLConsts ACBP=A9
 0001:00012F8C 000007E8 C=CODE     S=.text    G=(none)   M=TypInfo  ACBP=A9
 0001:00013774 0000017C C=CODE     S=.text    G=(none)   M=ActiveX  ACBP=A9
 0001:000138F0 0000973E C=CODE     S=.text    G=(none)   M=Classes  ACBP=A9
 0001:0001D030 00000088 C=CODE     S=.text    G=(none)   M=Math     ACBP=A9
 0001:0001D0B8 00000290 C=CODE     S=.text    G=(none)   M=Consts   ACBP=A9
 0001:0001D348 000072D7 C=CODE     S=.text    G=(none)   M=Graphics ACBP=A9
 0001:00024620 000002B8 C=CODE     S=.text    G=(none)   M=Contnrs  ACBP=A9
 0001:000248D8 000000F4 C=CODE     S=.text    G=(none)   M=CommCtrl ACBP=A9
 0001:000249CC 00000787 C=CODE     S=.text    G=(none)   M=MultiMon ACBP=A9
 0001:00025154 00000038 C=CODE     S=.text    G=(none)   M=Imm      ACBP=A9
 0001:0002518C 00000FF8 C=CODE     S=.text    G=(none)   M=HelpIntfs ACBP=A9
 0001:00026184 00000038 C=CODE     S=.text    G=(none)   M=WinSpool ACBP=A9
 0001:000261BC 00000044 C=CODE     S=.text    G=(none)   M=Printers ACBP=A9
 0001:00026200 0000031F C=CODE     S=.text    G=(none)   M=FlatSB   ACBP=A9
 0001:00026520 000001A4 C=CODE     S=.text    G=(none)   M=SyncObjs ACBP=A9
 0001:000266C4 000009BB C=CODE     S=.text    G=(none)   M=UxTheme  ACBP=A9
 0001:00027080 00000038 C=CODE     S=.text    G=(none)   M=RichEdit ACBP=A9
 0001:000270B8 00000038 C=CODE     S=.text    G=(none)   M=ToolWin  ACBP=A9
 0001:000270F0 00000038 C=CODE     S=.text    G=(none)   M=ShellAPI ACBP=A9
 0001:00027128 00000038 C=CODE     S=.text    G=(none)   M=RegStr   ACBP=A9
 0001:00027160 00000038 C=CODE     S=.text    G=(none)   M=WinInet  ACBP=A9
 0001:00027198 00000038 C=CODE     S=.text    G=(none)   M=UrlMon   ACBP=A9
 0001:000271D0 00000038 C=CODE     S=.text    G=(none)   M=ShlObj   ACBP=A9
 0001:00027208 00000038 C=CODE     S=.text    G=(none)   M=CommDlg  ACBP=A9
 0001:00027240 00000038 C=CODE     S=.text    G=(none)   M=Dlgs     ACBP=A9
 0001:00027278 0000066D C=CODE     S=.text    G=(none)   M=Dialogs  ACBP=A9
 0001:000278E8 00000652 C=CODE     S=.text    G=(none)   M=ExtCtrls ACBP=A9
 0001:00027F3C 00000038 C=CODE     S=.text    G=(none)   M=ComStrs  ACBP=A9
 0001:00027F74 00000094 C=CODE     S=.text    G=(none)   M=Clipbrd  ACBP=A9
 0001:00028008 00000038 C=CODE     S=.text    G=(none)   M=StrUtils ACBP=A9
 0001:00028040 000000F5 C=CODE     S=.text    G=(none)   M=Buttons  ACBP=A9
 0001:00028138 00000038 C=CODE     S=.text    G=(none)   M=ExtDlgs  ACBP=A9
 0001:00028170 00000068 C=CODE     S=.text    G=(none)   M=IniFiles ACBP=A9
 0001:000281D8 00000068 C=CODE     S=.text    G=(none)   M=Registry ACBP=A9
 0001:00028240 0000006C C=CODE     S=.text    G=(none)   M=Mapi     ACBP=A9
 0001:000282AC 00000058 C=CODE     S=.text    G=(none)   M=ExtActns ACBP=A9
 0001:00028304 00000038 C=CODE     S=.text    G=(none)   M=ListActns ACBP=A9
 0001:0002833C 00000180 C=CODE     S=.text    G=(none)   M=ComCtrls ACBP=A9
 0001:000284BC 00000A0C C=CODE     S=.text    G=(none)   M=Themes   ACBP=A9
 0001:00028EC8 00000038 C=CODE     S=.text    G=(none)   M=StdCtrls ACBP=A9
 0001:00028F00 00000168 C=CODE     S=.text    G=(none)   M=StdActns ACBP=A9
 0001:00029068 00000D1F C=CODE     S=.text    G=(none)   M=WinHelpViewer ACBP=A9
 0001:00029D88 00010467 C=CODE     S=.text    G=(none)   M=Controls ACBP=A9
 0001:0003A1F0 00001292 C=CODE     S=.text    G=(none)   M=ActnList ACBP=A9
 0001:0003B484 000016E4 C=CODE     S=.text    G=(none)   M=ImgList  ACBP=A9
 0001:0003CB68 000066AD C=CODE     S=.text    G=(none)   M=Menus    ACBP=A9
 0001:00043218 0000C3BC C=CODE     S=.text    G=(none)   M=Forms    ACBP=A9
 0001:0004F5D4 00000038 C=CODE     S=.text    G=(none)   M=DirectDraw ACBP=A9
 0001:0004F60C 00000060 C=CODE     S=.text    G=(none)   M=MMSystem ACBP=A9
 0001:0004F66C 00000038 C=CODE     S=.text    G=(none)   M=DXTypes  ACBP=A9
 0001:0004F6A4 00000074 C=CODE     S=.text    G=(none)   M=DirectSound ACBP=A9
 0001:0004F718 00000038 C=CODE     S=.text    G=(none)   M=Direct3D9 ACBP=A9
 0001:0004F750 00000060 C=CODE     S=.text    G=(none)   M=ComConst ACBP=A9
 0001:0004F7B0 00000FA5 C=CODE     S=.text    G=(none)   M=ComObj   ACBP=A9
 0001:00050758 00000260 C=CODE     S=.text    G=(none)   M=DirectShow9 ACBP=A9
 0001:000509B8 00000038 C=CODE     S=.text    G=(none)   M=WMF9     ACBP=A9
 0001:000509F0 000006C8 C=CODE     S=.text    G=(none)   M=DSUtil   ACBP=A9
 0001:000510B8 0000A7B0 C=CODE     S=.text    G=(none)   M=BaseClass ACBP=A9
 0001:0005B868 00000494 C=CODE     S=.text    G=(none)   M=formRenderer ACBP=A9
 0001:0005BCFC 00001FF0 C=CODE     S=.text    G=(none)   M=VidRenderer ACBP=A9
 0001:0005DCEC 0000027D C=CODE     S=.text    G=(none)   M=VideoRenderer ACBP=A9
 0002:00000000 0000009C C=DATA     S=.data    G=DGROUP   M=System   ACBP=A9
 0002:0000009C 00000030 C=DATA     S=.data    G=DGROUP   M=SysInit  ACBP=A9
 0002:000000CC 00000250 C=DATA     S=.data    G=DGROUP   M=SysUtils ACBP=A9
 0002:0000031C 00000008 C=DATA     S=.data    G=DGROUP   M=VarUtils ACBP=A9
 0002:00000324 0000008E C=DATA     S=.data    G=DGROUP   M=Variants ACBP=A9
 0002:000003B4 0000000C C=DATA     S=.data    G=DGROUP   M=TypInfo  ACBP=A9
 0002:000003C0 00000010 C=DATA     S=.data    G=DGROUP   M=ActiveX  ACBP=A9
 0002:000003D0 00000064 C=DATA     S=.data    G=DGROUP   M=Classes  ACBP=A9
 0002:00000434 00000304 C=DATA     S=.data    G=DGROUP   M=Graphics ACBP=A9
 0002:00000738 00000004 C=DATA     S=.data    G=DGROUP   M=Printers ACBP=A9
 0002:0000073C 00000074 C=DATA     S=.data    G=DGROUP   M=Dialogs  ACBP=A9
 0002:000007B0 00000178 C=DATA     S=.data    G=DGROUP   M=ExtCtrls ACBP=A9
 0002:00000928 0000002C C=DATA     S=.data    G=DGROUP   M=Buttons  ACBP=A9
 0002:00000954 00000008 C=DATA     S=.data    G=DGROUP   M=IniFiles ACBP=A9
 0002:0000095C 00000008 C=DATA     S=.data    G=DGROUP   M=Registry ACBP=A9
 0002:00000964 00000008 C=DATA     S=.data    G=DGROUP   M=Mapi     ACBP=A9
 0002:0000096C 00000018 C=DATA     S=.data    G=DGROUP   M=ComCtrls ACBP=A9
 0002:00000984 00000068 C=DATA     S=.data    G=DGROUP   M=Themes   ACBP=A9
 0002:000009EC 0000013C C=DATA     S=.data    G=DGROUP   M=Controls ACBP=A9
 0002:00000B28 00000020 C=DATA     S=.data    G=DGROUP   M=ImgList  ACBP=A9
 0002:00000B48 000000EC C=DATA     S=.data    G=DGROUP   M=Menus    ACBP=A9
 0002:00000C34 0000011C C=DATA     S=.data    G=DGROUP   M=Forms    ACBP=A9
 0002:00000D50 00000030 C=DATA     S=.data    G=DGROUP   M=ComObj   ACBP=A9
 0002:00000D80 00000150 C=DATA     S=.data    G=DGROUP   M=DirectShow9 ACBP=A9
 0002:00000ED0 0000000C C=DATA     S=.data    G=DGROUP   M=DSUtil   ACBP=A9
 0002:00000EDC 0000000C C=DATA     S=.data    G=DGROUP   M=BaseClass ACBP=A9
 0002:00000EE8 00000010 C=DATA     S=.data    G=DGROUP   M=VidRenderer ACBP=A9
 0002:00002000 00000664 C=BSS      S=.bss     G=DGROUP   M=System   ACBP=A9
 0002:00002664 00000014 C=BSS      S=.bss     G=DGROUP   M=SysInit  ACBP=A9
 0002:00002678 00000004 C=BSS      S=.bss     G=DGROUP   M=Types    ACBP=A9
 0002:0000267C 00000004 C=BSS      S=.bss     G=DGROUP   M=Windows  ACBP=A9
 0002:00002680 00000004 C=BSS      S=.bss     G=DGROUP   M=SysConst ACBP=A9
 0002:00002684 00000120 C=BSS      S=.bss     G=DGROUP   M=SysUtils ACBP=A9
 0002:000027A4 00000004 C=BSS      S=.bss     G=DGROUP   M=Messages ACBP=A9
 0002:000027A8 0000005C C=BSS      S=.bss     G=DGROUP   M=VarUtils ACBP=A9
 0002:00002804 00000040 C=BSS      S=.bss     G=DGROUP   M=Variants ACBP=A9
 0002:00002844 00000004 C=BSS      S=.bss     G=DGROUP   M=RTLConsts ACBP=A9
 0002:00002848 00000004 C=BSS      S=.bss     G=DGROUP   M=TypInfo  ACBP=A9
 0002:0000284C 00000004 C=BSS      S=.bss     G=DGROUP   M=ActiveX  ACBP=A9
 0002:00002850 00000040 C=BSS      S=.bss     G=DGROUP   M=Classes  ACBP=A9
 0002:00002890 00000004 C=BSS      S=.bss     G=DGROUP   M=Math     ACBP=A9
 0002:00002894 00000004 C=BSS      S=.bss     G=DGROUP   M=Consts   ACBP=A9
 0002:00002898 00000060 C=BSS      S=.bss     G=DGROUP   M=Graphics ACBP=A9
 0002:000028F8 00000004 C=BSS      S=.bss     G=DGROUP   M=Contnrs  ACBP=A9
 0002:000028FC 00000004 C=BSS      S=.bss     G=DGROUP   M=CommCtrl ACBP=A9
 0002:00002900 00000031 C=BSS      S=.bss     G=DGROUP   M=MultiMon ACBP=A9
 0002:00002934 00000004 C=BSS      S=.bss     G=DGROUP   M=Imm      ACBP=A9
 0002:00002938 00000008 C=BSS      S=.bss     G=DGROUP   M=HelpIntfs ACBP=A9
 0002:00002940 00000004 C=BSS      S=.bss     G=DGROUP   M=WinSpool ACBP=A9
 0002:00002944 00000004 C=BSS      S=.bss     G=DGROUP   M=Printers ACBP=A9
 0002:00002948 00000034 C=BSS      S=.bss     G=DGROUP   M=FlatSB   ACBP=A9
 0002:0000297C 00000004 C=BSS      S=.bss     G=DGROUP   M=SyncObjs ACBP=A9
 0002:00002980 000000CC C=BSS      S=.bss     G=DGROUP   M=UxTheme  ACBP=A9
 0002:00002A4C 00000004 C=BSS      S=.bss     G=DGROUP   M=RichEdit ACBP=A9
 0002:00002A50 00000004 C=BSS      S=.bss     G=DGROUP   M=ToolWin  ACBP=A9
 0002:00002A54 00000004 C=BSS      S=.bss     G=DGROUP   M=ShellAPI ACBP=A9
 0002:00002A58 00000004 C=BSS      S=.bss     G=DGROUP   M=RegStr   ACBP=A9
 0002:00002A5C 00000004 C=BSS      S=.bss     G=DGROUP   M=WinInet  ACBP=A9
 0002:00002A60 00000004 C=BSS      S=.bss     G=DGROUP   M=UrlMon   ACBP=A9
 0002:00002A64 00000004 C=BSS      S=.bss     G=DGROUP   M=ShlObj   ACBP=A9
 0002:00002A68 00000004 C=BSS      S=.bss     G=DGROUP   M=CommDlg  ACBP=A9
 0002:00002A6C 00000004 C=BSS      S=.bss     G=DGROUP   M=Dlgs     ACBP=A9
 0002:00002A70 0000000C C=BSS      S=.bss     G=DGROUP   M=Dialogs  ACBP=A9
 0002:00002A7C 00000004 C=BSS      S=.bss     G=DGROUP   M=ExtCtrls ACBP=A9
 0002:00002A80 00000004 C=BSS      S=.bss     G=DGROUP   M=ComStrs  ACBP=A9
 0002:00002A84 0000000C C=BSS      S=.bss     G=DGROUP   M=Clipbrd  ACBP=A9
 0002:00002A90 00000004 C=BSS      S=.bss     G=DGROUP   M=StrUtils ACBP=A9
 0002:00002A94 00000030 C=BSS      S=.bss     G=DGROUP   M=Buttons  ACBP=A9
 0002:00002AC4 00000004 C=BSS      S=.bss     G=DGROUP   M=ExtDlgs  ACBP=A9
 0002:00002AC8 00000004 C=BSS      S=.bss     G=DGROUP   M=IniFiles ACBP=A9
 0002:00002ACC 00000004 C=BSS      S=.bss     G=DGROUP   M=Registry ACBP=A9
 0002:00002AD0 00000004 C=BSS      S=.bss     G=DGROUP   M=Mapi     ACBP=A9
 0002:00002AD4 00000009 C=BSS      S=.bss     G=DGROUP   M=ExtActns ACBP=A9
 0002:00002AE0 00000004 C=BSS      S=.bss     G=DGROUP   M=ListActns ACBP=A9
 0002:00002AE4 00000010 C=BSS      S=.bss     G=DGROUP   M=ComCtrls ACBP=A9
 0002:00002AF4 00000008 C=BSS      S=.bss     G=DGROUP   M=Themes   ACBP=A9
 0002:00002AFC 00000004 C=BSS      S=.bss     G=DGROUP   M=StdCtrls ACBP=A9
 0002:00002B00 00000004 C=BSS      S=.bss     G=DGROUP   M=StdActns ACBP=A9
 0002:00002B04 00000014 C=BSS      S=.bss     G=DGROUP   M=WinHelpViewer ACBP=A9
 0002:00002B18 00000080 C=BSS      S=.bss     G=DGROUP   M=Controls ACBP=A9
 0002:00002B98 00000004 C=BSS      S=.bss     G=DGROUP   M=ActnList ACBP=A9
 0002:00002B9C 0000000C C=BSS      S=.bss     G=DGROUP   M=ImgList  ACBP=A9
 0002:00002BA8 00000010 C=BSS      S=.bss     G=DGROUP   M=Menus    ACBP=A9
 0002:00002BB8 00000020 C=BSS      S=.bss     G=DGROUP   M=Forms    ACBP=A9
 0002:00002BD8 00000004 C=BSS      S=.bss     G=DGROUP   M=DirectDraw ACBP=A9
 0002:00002BDC 00000004 C=BSS      S=.bss     G=DGROUP   M=MMSystem ACBP=A9
 0002:00002BE0 00000004 C=BSS      S=.bss     G=DGROUP   M=DXTypes  ACBP=A9
 0002:00002BE4 00000004 C=BSS      S=.bss     G=DGROUP   M=DirectSound ACBP=A9
 0002:00002BE8 00000004 C=BSS      S=.bss     G=DGROUP   M=Direct3D9 ACBP=A9
 0002:00002BEC 00000004 C=BSS      S=.bss     G=DGROUP   M=ComConst ACBP=A9
 0002:00002BF0 00000011 C=BSS      S=.bss     G=DGROUP   M=ComObj   ACBP=A9
 0002:00002C04 00000004 C=BSS      S=.bss     G=DGROUP   M=DirectShow9 ACBP=A9
 0002:00002C08 00000004 C=BSS      S=.bss     G=DGROUP   M=WMF9     ACBP=A9
 0002:00002C0C 00000004 C=BSS      S=.bss     G=DGROUP   M=DSUtil   ACBP=A9
 0002:00002C10 00000010 C=BSS      S=.bss     G=DGROUP   M=BaseClass ACBP=A9
 0002:00002C20 00000004 C=BSS      S=.bss     G=DGROUP   M=formRenderer ACBP=A9
 0002:00002C24 00000004 C=BSS      S=.bss     G=DGROUP   M=VidRenderer ACBP=A9


  Address         Publics by Name

 0002:00002A60       .1
 0002:00002BEC       .1
 0002:00002A5C       .1
 0002:00002968       .1
 0002:00002A68       .1
 0002:00002A58       .1
 0002:00002A54       .1
 0002:00002A6C       .1
 0002:00002A4C       .1
 0002:00002BE8       .1
 0002:000027A4       .1
 0002:00002894       .1
 0002:00002844       .1
 0002:00002B0C       .1
 0002:00002670       .1
 0002:00002A80       .1
 0002:00002678       .1
 0002:00002BE4       .1
 0002:00002BE0       .1
 0002:00002934       .1
 0002:00002A3C       .1
 0002:00002A64       .1
 0002:00002680       .1
 0002:00002C08       .1
 0002:00002920       .1
 0002:00002BD8       .1
 0002:00002A90       .1
 0002:00002AD0       .1
 0002:000028FC       .1
 0002:00002C0C       .11
 0002:00002A70       .11
 0002:0000289C       .12
 0002:00002A7C       .12
 0002:00002AF4       .2
 0002:00002C24       .2
 0002:00002938       .2
 0002:00002C20       .2
 0002:00002A88       .2
 0002:00002890       .2
 0002:000028F8       .21
 0002:00002AC4       .3
 0002:00002944       .3
 0002:00002940       .3
 0002:0000267C       .3
 0002:00002B9C       .3
 0002:0000284C       .3
 0002:00002C04       .31
 0002:00002794       .35
 0002:00002AE4       .36
 0002:00002A50       .4
 0002:00002A94       .4
 0002:00002BF0       .41
 0002:00002BC0       .41
 0002:00002AFC       .42
 0002:0000285C       .45
 0002:00002ACC       .5
 0002:00002800       .5
 0002:000025BC       .5
 0002:00002848       .6
 0002:0000297C       .6
 0002:00002BDC       .7
 0002:00002AD4       .72
 0002:00002B20       .72
 0002:00002B00       .73
 0002:00002C10       .74
 0002:00002AE0       .8
 0002:00002AC8       .8
 0002:00002B98       .8
 0002:00002824       .81
 0002:00002BB0       .9
 0001:00001CC8       @AbstractError
 0001:00002808       @AfterConstruction
 0001:0000264C       @AsClass
 0001:000032A8       @Assert
 0001:00001E30       @AStrCmp
 0001:00002818       @BeforeDestruction
 0001:000023CC       @BoundErr
 0001:00002698       @CallDynaInst
 0001:000027B0       @ClassCreate
 0001:00002800       @ClassDestroy
 0001:00001D38       @Close
 0001:00001BF4       @Copy
 0001:00003FA0       @CopyArray
 0001:00003E84       @CopyRecord
 0001:0000410C       @DispCallByIDError
 0001:0000DE7C       @DispInvokeError
 0001:000040A8       @Dispose
 0001:00002C94       @DoneExcept
 0001:000045FC       @DynArrayAsg
 0001:000045C0       @DynArrayClear
 0001:000043E0       @DynArrayHigh
 0001:000043D8       @DynArrayLength
 0001:000045B4       @DynArraySetLength
 0001:00002D7C       @ExceptionHandler
 0001:00001EA0       @FillChar
 0001:00003E60       @Finalize
 0001:00003D74       @FinalizeArray
 0001:00003D28       @FinalizeRecord
 0001:000023C0       @FpuInit
 0001:000022FC       @FpuMaskInit
 0001:00001A68       @FreeMem
 0001:00001A38       @GetMem
 0001:000054CC       @GetTls
 0001:00003290       @Halt
 0001:000031B0       @Halt0
 0001:0000292C       @HandleAnyException
 0001:00002BE0       @HandleFinally
 0001:00002A58       @HandleOnException
 0001:00003D1C       @Initialize
 0001:00003C88       @InitializeArray
 0001:00003C58       @InitializeRecord
 0001:00003058       @InitImports
 0001:00005518       @InitLib
 0001:00003030       @InitResStringImports
 0001:0000300C       @InitResStrings
 0001:0000307C       @InitWideStrings
 0001:00004D88       @IntfAddRef
 0001:00004D58       @IntfCast
 0001:00004D14       @IntfClear
 0001:00004D2C       @IntfCopy
 0001:00002628       @IsClass
 0001:000022CC       @isNECWindows
 0001:00003778       @LStrAddRef
 0001:000032EC       @LStrArrayClr
 0001:0000331C       @LStrAsg
 0001:00003590       @LStrCat
 0001:000035D4       @LStrCat3
 0001:00003648       @LStrCatN
 0001:000032C8       @LStrClr
 0001:000036D4       @LStrCmp
 0001:000037E8       @LStrCopy
 0001:00003828       @LStrDelete
 0001:00003538       @LStrFromArray
 0001:000034B0       @LStrFromChar
 0001:000034C0       @LStrFromPChar
 0001:000033B8       @LStrFromPCharLen
 0001:000034F0       @LStrFromPWChar
 0001:00003424       @LStrFromPWCharLen
 0001:0000352C       @LStrFromString
 0001:00003550       @LStrFromWStr
 0001:00003870       @LStrInsert
 0001:00003360       @LStrLAsg
 0001:00003588       @LStrLen
 0001:000038CC       @LStrPos
 0001:00003914       @LStrSetLength
 0001:00003788       @LStrToPChar
 0001:00003564       @LStrToString
 0001:00004094       @New
 0001:0000338C       @NewAnsiString
 0001:00003980       @NewWideString
 0001:00001FE0       @Pow10
 0001:00001DAC       @PStrCmp
 0001:00001D90       @PStrNCpy
 0001:00002C40       @RaiseAgain
 0001:00002C18       @RaiseExcept
 0001:00001A88       @ReallocMem
 0001:00001CBC       @ROUND
 0001:0000329C       @RunError
 0001:00001FC4       @SetEq
 0001:00002F44       @StartLib
 0001:000002AC       @strlen
 0001:00002CC4       @TryFinallyExit
 0001:000037E0       @UniqueStringA
 0001:000041B4       @ValInt64
 0001:00001EC0       @ValLong
 0001:000125C0       @VarAddRef
 0001:0000E770       @VarCast
 0001:0000E168       @VarClear
 0001:00003D5C       @VarClr
 0001:0000E17C       @VarClr
 0001:00003E6C       @VarCopy
 0001:0000E4A4       @VarCopy
 0001:000124A0       @VarFromBool
 0001:0001232C       @VarFromByte
 0001:000124F0       @VarFromCurr
 0001:00012448       @VarFromCurrency
 0001:00012474       @VarFromDate
 0001:00012594       @VarFromDisp
 0001:0001241C       @VarFromDouble
 0001:000122D0       @VarFromInt
 0001:000123CC       @VarFromInt64
 0001:0001230C       @VarFromInteger
 0001:00012568       @VarFromIntf
 0001:0001236C       @VarFromLongWord
 0001:00012504       @VarFromLStr
 0001:000124C8       @VarFromReal
 0001:0001238C       @VarFromShortInt
 0001:000123F8       @VarFromSingle
 0001:000123AC       @VarFromSmallInt
 0001:000124DC       @VarFromTDateTime
 0001:0001234C       @VarFromWord
 0001:00012530       @VarFromWStr
 0001:0000DED0       @VarNull
 0001:0000FBF4       @VarToBoolean
 0001:0000F034       @VarToByte
 0001:00010DB8       @VarToCurrency
 0001:00010850       @VarToDate
 0001:00012224       @VarToDisp
 0001:000100FC       @VarToDouble
 0001:0000F5F8       @VarToInt64
 0001:0000EB34       @VarToInteger
 0001:00012158       @VarToIntf
 0001:0000F2AC       @VarToLongWord
 0001:0001146C       @VarToLStr
 0001:0000EF84       @VarToShortInt
 0001:00010478       @VarToSingle
 0001:0000F0DC       @VarToSmallInt
 0001:0000F1D4       @VarToWord
 0001:00011B8C       @VarToWStr
 0001:00003C38       @WStrAddRef
 0001:000039C0       @WStrArrayClr
 0001:000039E4       @WStrAsg
 0001:000039A8       @WStrClr
 0001:00003B20       @WStrCmp
 0001:00003BA4       @WStrCopy
 0001:00003AF4       @WStrFromLStr
 0001:00003A08       @WStrFromPCharLen
 0001:00003AB8       @WStrFromPWChar
 0001:00003A94       @WStrFromPWCharLen
 0001:00003B14       @WStrLen
 0001:00003BF0       @WStrSetLength
 0001:00003B04       @WStrToPWChar
 0001:00001FA0       @_CLenToPasStr
 0001:00001F94       @_CToPasStr
 0001:00001BC4       @_IOTest
 0001:00004138       @_lldiv
 0001:00004114       @_llmul
 0001:0002C5AC       AbsMin
 0001:0000AEA4       AbstractErrorHandler
 0002:0000202C       AbstractErrorProc
 0002:0000014C       AccessMode
 0001:00001B24       AcquireExceptionObject
 0001:00015C00       ActivateClassGroup
 0001:00005B1C       ActivateKeyboardLayout
 0002:00002B54       ActiveDrag
 0001:000138E8       ActiveX
 0001:0003B458       ActnList
 0001:0000040C       AddBlockAfter
 0002:000003D0       AddDataModule
 0001:00018CC0       AddFinished
 0001:0003E79C       AddIn
 0001:00004B6C       AddModuleUnloadProc
 0001:00004B7C       AddModuleUnloadProc
 0001:00018CF8       AddNotFinished
 0001:0001971C       AddSubComponentsToLoaded
 0001:000209A8       AdjustColor
 0001:00045818       Adjustment
 0001:00005B24       AdjustWindowRectEx
 0002:00000C0C       Alignments
 0002:00000C1C       Alignments
 0001:00031B50       AlignWork
 0001:0004C75C       AlignWork
 0001:0001CE10       AllocateHWnd
 0001:0000719C       AllocMem
 0002:000025B4       AllocMemCount
 0002:000025B8       AllocMemSize
 0001:00024418       AllocPatternBitmap
 0001:000053FC       AllocTlsBuffer
 0001:0005274C       AMGetWideString
 0002:000009F8       AnchorAlign
 0002:000009EC       AnimateWindowProc
 0002:00000AF4       AnimationStyle
 0001:00007324       AnsiCompareStr
 0001:0000735C       AnsiCompareText
 0001:0000796C       AnsiLastChar
 0001:00005B2C       AnsiLower
 0001:0000B7BC       AnsiPos
 0001:00043024       AnsiSameCaption
 0001:00007394       AnsiSameText
 0001:000073AC       AnsiStrLIComp
 0001:0000B7F8       AnsiStrPos
 0001:0000B8B8       AnsiStrRScan
 0001:0000B900       AnsiStrScan
 0001:00005188       AnsiToUtf8
 0001:000120E0       AnyToIntf
 0001:00008DE0       AppendChars
 0001:000091AC       AppendFormat
 0001:00008E44       AppendNumber
 0001:00008E24       AppendString
 0002:00002BB8       Application
 0002:000003E0       ApplicationHandleException
 0002:000003E8       ApplicationShowException
 0002:00000D48       AppVisible
 0001:0000AE88       AssertErrorHandler
 0002:00002024       AssertErrorProc
 0001:0001323C       AssignLongStr
 0001:000135E0       AssignVariant
 0002:0000260C       avail
 0001:00007A68       BackfillGetDiskFreeSpaceEx
 0001:0002F104       BackgroundClipped
 0001:0000CDEC       BackupVarBoolFromStr
 0001:0000CF4C       BackupVarBStrFromBool
 0001:0000CE6C       BackupVarBStrFromCy
 0001:0000CEDC       BackupVarBStrFromDate
 0001:0000CD80       BackupVarCyFromStr
 0001:0000CD14       BackupVarDateFromStr
 0001:0000CBD0       BackupVarI4FromStr
 0001:0000CB7C       BackupVariantChangeTypeEx
 0001:0000CC3C       BackupVarR4FromStr
 0001:0000CCA8       BackupVarR8FromStr
 0001:0005B860       BaseClass
 0001:00015F58       BeginGlobalLoading
 0001:00005B34       BeginPaint
 0001:000209B4       BetterSize
 0001:0003F630       BiDiDraw
 0001:00005964       BitBlt
 0002:00000928       BitBtnCaptions
 0002:00002A98       BitBtnGlyphs
 0002:000006EC       BitmapCanvasList
 0002:000028B4       BitmapImageLock
 0001:0000CBB8       BiUnimplemented
 0002:00000408       BlockCode
 0002:000025E4       blockDescBlockList
 0002:000025E8       blockDescFreeList
 0002:000003B4       BooleanIdents
 0002:00000330       BooleanToStringRule
 0001:00007804       BoolToStr
 0001:000111F4       BoolToWStrViaOS
 0001:00014F18       Bounds
 0001:000055BC       Bounds
 0002:00000BB4       Breaks
 0002:000028EC       BrushManager
 0001:00041E04       BuildImage
 0002:00000784       ButtonCaptions
 0002:00000758       ButtonNames
 0002:00000C30       Buttons
 0001:00028110       Buttons
 0001:00020180       BytesPerScanline
 0001:000204E4       ByteSwapColors
 0001:0000B560       ByteToCharIndex
 0001:0000B538       ByteToCharLen
 0001:0000B4FC       ByteType
 0001:0000B484       ByteTypeTest
 0002:00002BA0       CachedComCtrlVer
 0001:0001CD4C       CalcJmpOffset
 0001:000394E0       CalcSplitterPos
 0001:00005B3C       CallNextHookEx
 0001:0000BFD8       CallTerminateProcs
 0001:00005B44       CallWindowProc
 0001:0002D5E4       CancelDrag
 0002:00002B68       CanvasList
 0002:000028F0       CanvasList
 0002:00000744       Captions
 0002:00000AB0       CaptureControl
 0002:00000B54       cBooleanToItemAutoFlag
 0002:00002A86       CF_COMPONENT
 0002:00002A84       CF_PICTURE
 0002:0000281C       ChangeAnyProc
 0001:000033E8       CharFromWChar
 0001:0000B744       CharLength
 0001:00005B4C       CharNext
 0001:0000022C       CharNext
 0001:0001EB04       CharsetToIdent
 0001:0000B64C       CharToByteIndex
 0001:0000B6B0       CharToByteLen
 0001:00005B54       CharToOemA
 0001:00020F70       CheckBool
 0001:0005C524       CheckConnected
 0001:000028A8       CheckJmp
 0001:00005B5C       CheckMenuItem
 0002:00000BA4       Checks
 0001:00019758       CheckSubComponents
 0001:0001BB24       CheckSynchronize
 0001:00045254       CheckTaskWindow
 0001:0002D298       CheckUndock
 0001:0000B378       CheckWin32Version
 0002:00000334       CInvalidCustomVariantType
 0002:00000B58       cItemAutoFlagToBoolean
 0002:00000B50       cItemAutoFlagToMenu
 0001:0001CF9C       Classes
 0001:000159C4       ClassNotFound
 0002:00002818       ClearAnyProc
 0001:0001E384       ClearColor
 0001:00050438       ClearExcepInfo
 0001:000128FC       ClearVariantTypeList
 0001:00005B64       ClientToScreen
 0001:00036AC8       ClientToWindow
 0002:000006E4       ClipboardFormats
 0001:00027FB0       Clipbrd
 0001:0000570C       CloseHandle
 0002:00002984       CloseThemeData
 0002:00000EE8       CLSID_DelphiVideoRenderer
 0002:00000E60       CLSID_FilterMapper
 0002:00000E90       CLSID_FilterMapper2
 0002:00000E80       CLSID_LegacyAmFilterCategory
 0002:00000EA0       CLSID_MemoryAllocator
 0002:00000E70       CLSID_VideoRenderer
 0002:00002040       CmdLine
 0002:0000203C       CmdShow
 0002:00000B4C       cMenuAutoFlagToItem
 0001:0000CBC4       CmpUnimplemented
 0002:00000D58       CoAddRefServerProcess
 0001:00013860       CoCreateInstance
 0002:00000D50       CoCreateInstanceEx
 0002:00000D68       CoInitFlags
 0001:00013848       CoInitialize
 0002:00000D54       CoInitializeEx
 0001:00013858       CoLockObjectExternal
 0002:00000464       Colors
 0001:0001E8FC       ColorToIdent
 0002:000007B0       ColorToPretyName
 0001:0001E8EC       ColorToRGB
 0002:00002BF8       ComClassManagerVar
 0001:0004F7A8       ComConst
 0002:00002AF0       ComCtlVersion
 0001:000284B4       ComCtrls
 0002:00002BB4       CommandPool
 0001:000249C4       CommCtrl
 0001:00027238       CommDlg
 0001:0000078C       Commit
 0002:00002628       committedRoot
 0001:00050700       ComObj
 0001:0003DD80       CompareFront
 0001:0000728C       CompareMem
 0001:0000725C       CompareStr
 0001:00005714       CompareString
 0001:0000571C       CompareStringA
 0001:00005724       CompareStringW
 0001:000072AC       CompareText
 0001:0000772C       CompareWith
 0001:0005793C       CompatibleTimeSetEvent
 0001:00019838       ComponentCreated
 0001:00027F6C       ComStrs
 0001:0001D340       Consts
 0001:000248D0       Contnrs
 0002:00002B26       ControlAtom
 0002:00002B2C       ControlAtomString
 0001:0004A000       ControlHasHelp
 0001:0003A160       Controls
 0001:0000A88C       ConvertAddr
 0001:00008F38       ConvertEraString
 0001:00007178       ConvertErrorFmt
 0001:000090A4       ConvertYearString
 0001:000043E8       CopyArray
 0001:00021A48       CopyBitmap
 0001:00022110       CopyBitmapAsMask
 0001:00050A18       CopyMediaType
 0001:00006034       CopyMemory
 0001:000220AC       CopyPalette
 0002:00000988       Copyright
 0001:00040EB0       CopyToBest
 0002:00000D5C       CoReleaseServerProcess
 0002:00000D60       CoResumeClassObjects
 0002:00000D64       CoSuspendClassObjects
 0001:00013870       CoTaskMemAlloc
 0001:00013878       CoTaskMemFree
 0001:00013850       CoUninitialize
 0001:0000B5BC       CountChars
 0002:000028CC       CounterLock
 0002:00000338       CRangeToType
 0001:0000ADCC       CreateAssertException
 0001:0000AF54       CreateAVObject
 0001:0000596C       CreateBitmap
 0001:00005974       CreateBrushIndirect
 0001:0000597C       CreateCompatibleBitmap
 0001:00005984       CreateCompatibleDC
 0001:000198B8       CreateComponent
 0001:00005994       CreateDIBitmap
 0001:0000598C       CreateDIBSection
 0001:0000572C       CreateEvent
 0001:00005734       CreateFile
 0001:0000599C       CreateFontIndirect
 0001:000059A4       CreateHalftonePalette
 0001:00005B6C       CreateIcon
 0001:0000ACF8       CreateInOutError
 0001:00005B74       CreateMenu
 0001:000059AC       CreatePalette
 0001:000059B4       CreatePenIndirect
 0001:00005B7C       CreatePopupMenu
 0001:0004FB98       CreateRegKey
 0001:000059BC       CreateSolidBrush
 0001:0002053C       CreateSystemPalette
 0001:0000573C       CreateThread
 0001:00006128       CreateWindow
 0001:000060D0       CreateWindowEx
 0002:000009F0       CreationControl
 0002:0000073C       CreationControl
 0002:000003A0       CRelationshipToBoolean
 0002:0000031C       CResult
 0002:00000144       cSimpleBoolStrs
 0002:0000034C       CText
 0002:00000AEC       Ctl3DStyles
 0002:00002620       curAlloc
 0002:0000268C       CurrencyDecimals
 0002:00002688       CurrencyFormat
 0002:00002684       CurrencyString
 0001:00008DCC       CurrentYear
 0001:00008958       CurrToStr
 0001:00011184       CurrToWStrViaOS
 0002:00000CCC       CursorMap
 0002:00000A00       Cursors
 0001:0002BE84       CursorToIdent
 0002:00000CBC       cUseAlpha
 0002:00000CC4       cUseColorKey
 0001:00007480       CvtInt
 0001:000074EC       CvtInt64
 0002:00000184       CWNear
 0002:0000268D       DateSeparator
 0001:000099E0       DateTimeToStr
 0001:00009984       DateTimeToString
 0001:00008A18       DateTimeToTimeStamp
 0001:000111BC       DateToWStrViaOS
 0001:00008DA4       DayOfWeek
 0002:00000180       DCon10
 0002:00000460       DDBsOnly
 0001:0001CEC4       DeallocateHWnd
 0002:00000028       DebugHook
 0002:0000268B       DecimalSeparator
 0001:00008D84       DecodeDate
 0001:00008C34       DecodeDateFully
 0001:00008ACC       DecodeTime
 0001:0000084C       Decommit
 0001:00000F78       DecommitFree
 0002:000025FC       decommittedRoot
 0001:0004D398       Default
 0001:00047C80       Default
 0002:00000020       Default8087CW
 0002:000009F4       DefaultDockTreeClass
 0002:000025C0       DefaultUserCodePage
 0002:000006B4       DefBrushData
 0002:00000434       DefFontData
 0001:00005B84       DefFrameProc
 0002:00000210       DefLongDayNames
 0002:000001C4       DefLongMonthNames
 0001:00005B8C       DefMDIChildProc
 0002:00000694       DefPenData
 0002:000001F4       DefShortDayNames
 0002:00000194       DefShortMonthNames
 0001:00005B94       DefWindowProc
 0001:00004654       DelayLoadResourceModule
 0001:00000468       DeleteBlock
 0001:00000378       DeleteCriticalSection
 0001:00005744       DeleteCriticalSection
 0001:000059C4       DeleteDC
 0001:00000D60       DeleteFree
 0001:00050A00       DeleteMediaType
 0001:00005B9C       DeleteMenu
 0001:000059CC       DeleteObject
 0001:0004FC30       DeleteRegKey
 0001:00021604       DeselectBitmap
 0001:00005BA4       DestroyCursor
 0001:00005BAC       DestroyIcon
 0001:00028040       DestroyLocals
 0001:00005BB4       DestroyMenu
 0001:00005BBC       DestroyWindow
 0001:00029A3C       DialogEnumerationTester
 0001:000278A8       Dialogs
 0002:000006F0       DIBPalSizes
 0002:0000008C       dig
 0001:0004F748       Direct3D9
 0001:0004F604       DirectDraw
 0001:000509B0       DirectShow9
 0001:0004F710       DirectSound
 0001:00045090       DisableTaskWindows
 0001:0004FE4C       DispatchInvoke
 0001:0005042C       DispatchInvokeError
 0001:00005BC4       DispatchMessage
 0001:0004B2E0       DispatchShortCut
 0001:00050448       DispCall
 0001:0005052C       DispCallByID
 0002:00002000       DispCallByIDProc
 0001:00050358       DispCallError
 0001:0000715C       DivMod
 0001:00027270       Dlgs
 0001:0005283C       DllCanUnloadNow
 0001:000527F4       DllGetClassObject
 0002:0000266C       DllProc
 0001:00052858       DllRegisterServer
 0001:00052874       DllUnregisterServer
 0001:000319E0       DoAlign
 0001:0004C610       DoAlign
 0001:00035984       DoCalcConstraints
 0002:00002B5C       DockSiteList
 0001:00041AD0       DoClick
 0001:000330B8       DoControlMsg
 0001:00045040       DoDisableWindow
 0001:0002CBC4       DoDragOver
 0001:000377B4       DoFindControlZone
 0001:00045194       DoFindWindow
 0001:00037D40       DoFindZone
 0001:00037838       DoForEach
 0001:00039144       DoGetNextLimit
 0001:00045008       DoneApplication
 0001:00039EA4       DoneControls
 0001:0000B288       DoneExceptions
 0001:0004965C       DoNestedActivation
 0001:0001BAE4       DoneThreadSynchronization
 0001:0004E530       DoOnHelp
 0001:0004C460       DoPosition
 0001:000315A0       DoPosition
 0001:0003876C       DoPrune
 0001:00038C44       DoSaveZone
 0001:00038E48       DoSetNewBounds
 0002:000003BC       DotSep
 0001:000211C8       DoWrite
 0001:00016D8C       DoWrite
 0001:0003C3E0       DoWrite
 0001:000326A0       DoWriteDesignSize
 0001:000301F8       DoWriteIsControl
 0002:00002B40       DragCapture
 0002:00002B34       DragControl
 0001:0002D30C       DragDone
 0001:0002CB74       DragFindTarget
 0001:0002CB48       DragFindWindow
 0002:00002B58       DragImageList
 0001:0002CF64       DragInit
 0001:0002D0D4       DragInitControl
 0002:00002B3C       DragInternalObject
 0001:0002CA90       DragMessage
 0002:00002B38       DragObject
 0002:00002B64       DragSave
 0002:00002B4C       DragSaveCursor
 0002:00002B44       DragStartPos
 0002:00002B50       DragThreshold
 0001:0002CC94       DragTo
 0001:0004D3D4       DrawAppIcon
 0001:000382D8       DrawCloseButton
 0001:00005BCC       DrawEdge
 0001:00005BD4       DrawFrameControl
 0001:00038330       DrawGrabberLine
 0001:00005BDC       DrawIcon
 0001:00005BE4       DrawIconEx
 0002:00000B28       DrawingStyles
 0001:00005BEC       DrawMenuBar
 0001:00042E40       DrawMenuItem
 0001:00005BF4       DrawText
 0002:00002988       DrawThemeBackground
 0002:000029AC       DrawThemeEdge
 0002:000029B0       DrawThemeIcon
 0002:00002A34       DrawThemeParentBackground
 0002:0000298C       DrawThemeText
 0001:000510A4       DSUtil
 0001:000589E4       DumbItDownFor95
 0001:00020000       DupBits
 0001:0004F69C       DXTypes
 0001:00004400       DynArrayClear
 0001:00004408       DynArraySetLength
 0002:00000C14       EdgeStyle
 0002:00000ADC       EdgeStyles
 0001:0000ACCC       EHeapException.FreeInstance
 0002:00002804       EmptyParam
 0002:000000CC       EmptyStr
 0002:000000D0       EmptyWideStr
 0001:00005BFC       EnableMenuItem
 0002:00000BAC       Enables
 0001:00005C04       EnableScrollBar
 0001:00045144       EnableTaskWindows
 0002:00002A1C       EnableThemeDialogTexture
 0002:00002A38       EnableTheming
 0001:00005C0C       EnableWindow
 0001:00015FE0       EndGlobalLoading
 0001:00059960       EndOfStreamTimer
 0001:00005C14       EndPaint
 0001:00050B40       EnlargedUnsignedDivide
 0001:00000368       EnterCriticalSection
 0001:0000574C       EnterCriticalSection
 0001:00005754       EnumCalendarInfoA
 0002:0000291C       EnumDisplayMonitors
 0001:0000A500       EnumEraNames
 0001:0000A53C       EnumEraYearOffsets
 0001:00048244       EnumMonitorsProc
 0001:00005C1C       EnumThreadWindows
 0001:00019068       EnumValue
 0001:00005C24       EnumWindows
 0001:0004FAA0       EOleException.Create
 0001:0004F9D0       EOleSysError.Create
 0001:00005C2C       EqualRect
 0002:00002754       EraNames
 0001:00009C58       EraToYear
 0002:00002770       EraYearOffsets
 0002:00000064       errCaption
 0001:00015568       Error
 0001:00001BB8       Error
 0001:0001884C       Error
 0001:0003DAD0       Error
 0002:00000004       ErrorAddr
 0001:00001B6C       ErrorAt
 0001:0000AD78       ErrorHandler
 0002:0000022C       ErrorMap
 0002:00002008       ErrorProc
 0002:000023E8       ErrOutput
 0001:00001AF8       ExceptAddr
 0002:0000200C       ExceptClsProc
 0001:0000B1F4       ExceptHandler
 0001:0000AAF8       Exception.Create
 0001:0000AB34       Exception.CreateFmt
 0001:0000AC84       Exception.CreateHelp
 0001:0000ABB4       Exception.CreateRes
 0001:0000ABF0       Exception.CreateResFmt
 0002:0000201C       ExceptionClass
 0001:0000A898       ExceptionErrorMessage
 0002:00000264       ExceptMap
 0001:00001AD8       ExceptObject
 0002:00002010       ExceptObjProc
 0002:00002004       ExceptProc
 0001:000059D4       ExcludeClipRect
 0002:00000000       ExitCode
 0001:000030F4       ExitDll
 0002:00002048       ExitProc
 0001:00000234       ExitProcess
 0002:00002028       ExitProcessProc
 0001:000054A8       ExitProcessTLS
 0001:00005480       ExitThreadTLS
 0001:00007A2C       ExpandFileName
 0001:000282FC       ExtActns
 0001:00027F0C       ExtCtrls
 0001:00028168       ExtDlgs
 0001:000079F4       ExtractFileName
 0002:00002C18       FactoryCount
 0001:000138AC       Failed
 0002:00002790       FalseBoolStrs
 0002:00002A8C       FClipboard
 0002:00000174       FCon1E18
 0001:00007964       FileClose
 0001:000078A8       FileCreate
 0001:000078CC       FileCreate
 0002:000006E8       FileFormats
 0002:00000008       FileMode
 0001:00007850       FileOpen
 0001:000078D4       FileRead
 0002:000003F8       FilerSignature
 0001:0000792C       FileSeek
 0001:00007900       FileWrite
 0001:00000E98       FillAfterGap
 0001:00000E38       FillBeforeGap
 0001:00000F38       FillerSizeAfterGap
 0001:00000EC0       FillerSizeBeforeGap
 0001:00005C34       FillRect
 0001:0003A0F8       Finalization
 0001:00029030       Finalization
 0001:0004F534       Finalization
 0001:0005B814       Finalization
 0001:000055D8       Finalization
 0001:0003CB30       Finalization
 0001:0001CEEC       Finalization
 0001:000281F0       Finalization
 0001:0002784C       Finalization
 0001:00005560       Finalization
 0001:00027EC4       Finalization
 0001:00012F54       Finalization
 0001:00028254       Finalization
 0001:00006588       Finalization
 0001:000052A4       Finalization
 0001:00006278       Finalization
 0001:000138B8       Finalization
 0001:0000D318       Finalization
 0001:00027010       Finalization
 0001:00012D48       Finalization
 0001:00027F74       Finalization
 0001:00027080       Finalization
 0001:00050680       Finalization
 0001:0000C924       Finalization
 0001:0005BCC4       Finalization
 0001:000270B8       Finalization
 0001:00028008       Finalization
 0001:0005DC64       Finalization
 0001:0005DCEC       Finalization
 0001:0000CB24       Finalization
 0001:00028E7C       Finalization
 0001:00050980       Finalization
 0001:00025114       Finalization
 0001:00025154       Finalization
 0001:000509B8       Finalization
 0001:0003B428       Finalization
 0001:000270F0       Finalization
 0001:00027128       Finalization
 0001:00028EC8       Finalization
 0001:00027160       Finalization
 0001:0005105C       Finalization
 0001:0004F718       Finalization
 0001:00029CB4       Finalization
 0001:000280D8       Finalization
 0001:0004F778       Finalization
 0001:000248A0       Finalization
 0001:00027198       Finalization
 0001:0002613C       Finalization
 0001:0004F6E0       Finalization
 0001:00026184       Finalization
 0001:0001D310       Finalization
 0001:000261BC       Finalization
 0001:00028138       Finalization
 0001:0004F66C       Finalization
 0001:0002843C       Finalization
 0001:000271D0       Finalization
 0001:00028304       Finalization
 0001:0004F634       Finalization
 0001:00028188       Finalization
 0001:00027208       Finalization
 0001:00027240       Finalization
 0001:0004F5D4       Finalization
 0001:000282AC       Finalization
 0001:00024450       Finalization
 0001:0001D080       Finalization
 0001:0002668C       Finalization
 0001:000264E0       Finalization
 0001:00043120       Finalization
 0001:00027F3C       Finalization
 0001:00024994       Finalization
 0001:0001371C       Finalization
 0001:000043F8       FinalizeArray
 0001:00002E64       FinalizeUnits
 0001:00041890       Find
 0001:000046E4       FindBS
 0001:00015A84       FindClass
 0001:0000464C       FindClassHInstance
 0001:00000244       FindClose
 0001:00000DF4       FindCommitted
 0001:0002BC64       FindControl
 0001:00037F6C       FindControlAtPos
 0001:00012BA0       FindCustomVariantType
 0001:00012C58       FindCustomVariantType
 0001:0002D630       FindDragTarget
 0001:00019A68       FindExistingComponent
 0001:0000024C       FindFirstFile
 0001:00015E70       FindGlobalComponent
 0001:000452A0       FindGlobalComponent
 0002:00002868       FindGlobalComponentProcs
 0001:00004624       FindHInstance
 0001:00015D18       FindIdentToInt
 0002:00002A78       FindMsg
 0001:00018BF8       FindNestedComponent
 0001:0003DA98       FindPopupControl
 0001:0000CFE0       FindProc
 0001:0000575C       FindResource
 0001:0000469C       FindResourceHInstance
 0001:0004ED64       FindScanline
 0001:000451F8       FindTopMostWindow
 0001:0001A94C       FindUniqueName
 0001:0002D5FC       FindVCLWindow
 0001:00005C3C       FindWindow
 0001:00029A94       FindWinHelp
 0001:000219FC       FixupBitFields
 0002:00000C24       Flags
 0002:000027A0       FLanguages
 0001:00026510       FlatSB
 0002:00002948       FlatSB_EnableScrollBar
 0002:00002954       FlatSB_GetScrollInfo
 0002:00002958       FlatSB_GetScrollPos
 0002:00002950       FlatSB_GetScrollRange
 0002:00002960       FlatSB_SetScrollInfo
 0002:0000295C       FlatSB_SetScrollPos
 0001:00026200       FlatSB_SetScrollProp
 0002:00002964       FlatSB_SetScrollRange
 0002:0000294C       FlatSB_ShowScrollBar
 0001:000085E8       FloatToDecimal
 0001:00008928       FloatToStr
 0001:00008314       FloatToText
 0001:00001D2C       Flush
 0002:00000188       FMSecsPerDay
 0001:00008208       FmtStr
 0002:00000C40       FocusCount
 0002:00000C3C       FocusMessages
 0002:00000604       FontCharsets
 0002:000028E4       FontManager
 0001:00045274       ForegroundTask
 0002:00000190       Format
 0001:000081F4       Format
 0001:00007DE4       FormatBuf
 0001:00007DD8       FormatClearStr
 0001:00007D5C       FormatError
 0002:0000016C       FormatErrorStrs
 0001:00005764       FormatMessage
 0001:00007DB4       FormatVarToStr
 0002:00000EB0       FORMAT_VideoInfo
 0001:0005BCF4       formRenderer
 0001:0004F590       Forms
 0001:00001FD8       FPower10
 0002:00000738       FPrinter
 0001:00005C44       FrameRect
 0001:000509F0       FreeAndNil
 0001:0000C504       FreeAndNil
 0001:00000AF4       FreeCommitted
 0001:0000112C       FreeCurAlloc
 0001:0002D6F0       FreeDeviceContext
 0001:0002D7AC       FreeDeviceContexts
 0001:0001CCB8       FreeIntConstList
 0001:00000254       FreeLibrary
 0001:0000576C       FreeLibrary
 0001:00050AEC       FreeMediaType
 0001:00021558       FreeMemoryContexts
 0001:0001CDEC       FreeObjectInstance
 0001:0000578C       FreeResource
 0001:000006C4       FreeSpace
 0001:0000C004       FreeTerminateProcs
 0001:000266C4       FreeThemeLibrary
 0002:00002AEC       FRichEditModule
 0001:0001FFF0       GDICheck
 0001:0001FF48       GDIError
 0001:00001CB4       Get8087CW
 0001:00005794       GetACP
 0001:00005C4C       GetActiveWindow
 0001:0004CAEC       GetAnimation
 0001:000059DC       GetBitmapBits
 0001:00000380       GetBlockDesc
 0001:000059E4       GetBrushOrgEx
 0001:00005C54       GetCapture
 0001:0002BF2C       GetCaptureControl
 0001:00015A30       GetClass
 0001:00005C5C       GetClassInfo
 0001:00005C64       GetClassName
 0001:00005C6C       GetClientRect
 0001:000059EC       GetClipBox
 0001:0000031C       GetCmdShow
 0001:0003B5F8       GetColor
 0001:000283DC       GetComCtlVersion
 0001:0000025C       GetCommandLine
 0001:00000908       GetCommitted
 0001:000009B0       GetCommittedAt
 0001:00032C6C       GetControlAtPos
 0001:00008E90       GetCount
 0001:0000579C       GetCPInfo
 0001:000059F4       GetCurrentPositionEx
 0001:000057A4       GetCurrentProcessId
 0002:00002A2C       GetCurrentThemeName
 0001:000057AC       GetCurrentThread
 0001:0000030C       GetCurrentThreadId
 0001:000057B4       GetCurrentThreadId
 0001:0000602C       GetCurrentTime
 0001:00005C74       GetCursor
 0001:0004ED74       GetCursorHeightMargin
 0001:00005C7C       GetCursorPos
 0001:00008EC0       GetDate
 0001:000057BC       GetDateFormat
 0001:00009B70       GetDateOrder
 0001:00005C84       GetDC
 0001:00005C8C       GetDCEx
 0001:000059FC       GetDCOrgEx
 0001:00024058       GetDefFontCharSet
 0001:00005C94       GetDesktopWindow
 0001:00005A14       GetDeviceCaps
 0001:00020F58       GetDIB
 0001:00005A04       GetDIBColorTable
 0001:00005A0C       GetDIBits
 0001:00020EA0       GetDIBSizes
 0001:00020160       GetDInColors
 0001:000057C4       GetDiskFreeSpaceA
 0002:00000140       GetDiskFreeSpaceEx
 0001:00039224       GetDockAlign
 0001:0002C8D4       GetDockSiteAtPos
 0001:0002CC00       GetDropCtl
 0001:00002668       GetDynaMethod
 0001:00012FC4       GetEnumNameValue
 0001:00013010       GetEnumValue
 0001:0000A5B4       GetEraNamesAndYearOffsets
 0001:00009C04       GetEraYearOffset
 0001:00013898       GetErrorInfo
 0001:0000AF3C       GetExceptionClass
 0001:0000B128       GetExceptionObject
 0001:000159B8       GetFieldClassTable
 0001:0000B398       GetFileVersion
 0001:0000594C       GetFileVersionInfo
 0001:00005954       GetFileVersionInfoSize
 0001:00005C9C       GetFocus
 0001:0001EB24       GetFontData
 0001:00005CA4       GetForegroundWindow
 0001:0000BBAC       GetFormatSettings
 0001:000057CC       GetFullPathName
 0001:0001E06C       GetHashCode
 0001:0004A038       GetHelpInfo
 0001:000255D4       GetHelpSystem
 0001:0004C8D0       GetHint
 0001:0004C908       GetHintControl
 0001:00042FC0       GetHotkey
 0001:00005CAC       GetIconInfo
 0001:000501C4       GetIDsOfNames
 0001:00005CC4       GetKeyboardLayout
 0001:00005CCC       GetKeyboardLayoutList
 0001:00005CD4       GetKeyboardState
 0001:000022C4       GetKeyboardType
 0001:00005CB4       GetKeyNameText
 0001:00005CBC       GetKeyState
 0001:00005CDC       GetLastActivePopup
 0001:000374EC       GetLastChildZone
 0001:000057D4       GetLastError
 0001:0000A378       GetLocaleChar
 0001:000057E4       GetLocaleInfo
 0001:00000264       GetLocaleInfo
 0001:0000A32C       GetLocaleStr
 0001:000057DC       GetLocalTime
 0001:0002BEE8       GetLongHint
 0001:00005CE4       GetMenu
 0001:00049FC0       GetMenuHelpContext
 0001:00005CEC       GetMenuItemCount
 0001:00005CF4       GetMenuItemID
 0001:00005CFC       GetMenuItemInfo
 0001:000400DC       GetMenuSize
 0001:00005D04       GetMenuState
 0001:00005D0C       GetMenuString
 0001:000057EC       GetModuleFileName
 0001:0000026C       GetModuleFileName
 0001:000057F4       GetModuleHandle
 0001:00000274       GetModuleHandle
 0002:00002910       GetMonitorInfo
 0002:00002914       GetMonitorInfoA
 0002:00002918       GetMonitorInfoW
 0001:0000A3DC       GetMonthDayNames
 0001:00005D14       GetNextWindow
 0001:00005A1C       GetObject
 0001:000130E4       GetOrdProp
 0001:00005A24       GetPaletteEntries
 0001:00005D1C       GetParent
 0001:0004546C       GetParentForm
 0001:00005A2C       GetPixel
 0001:000057FC       GetProcAddress
 0001:0000027C       GetProcAddress
 0001:00005D24       GetProp
 0001:00013074       GetPropInfo
 0001:00005D2C       GetQueueStatus
 0001:0004592C       GetRealScrollPosition
 0001:0003B5D8       GetRGBColor
 0001:00005D34       GetScrollInfo
 0001:00005D3C       GetScrollPos
 0001:00005D44       GetScrollRange
 0001:0002BEA4       GetShortHint
 0001:000005E8       GetSpace
 0001:0000064C       GetSpaceAt
 0001:0003DB28       GetSpecialName
 0001:00000284       GetStartupInfo
 0001:00005804       GetStdHandle
 0001:00000204       GetStdHandle
 0001:00005A34       GetStockObject
 0001:0000580C       GetStringTypeEx
 0001:00005D4C       GetSubMenu
 0001:00005D54       GetSysColor
 0001:00005D5C       GetSysColorBrush
 0001:00005814       GetSystemInfo
 0001:00005D64       GetSystemMenu
 0001:00005D6C       GetSystemMetrics
 0002:00002900       GetSystemMetrics
 0001:00005A3C       GetSystemPaletteEntries
 0001:00005A44       GetTextExtentPoint32
 0001:00005A4C       GetTextMetrics
 0002:00002A24       GetThemeAppProperties
 0002:00002990       GetThemeBackgroundContentRect
 0002:00002994       GetThemeBackgroundExtent
 0002:000029A4       GetThemeBackgroundRegion
 0002:000029C8       GetThemeBool
 0002:000029BC       GetThemeColor
 0002:00002A30       GetThemeDocumentationProperty
 0002:000029D0       GetThemeEnumValue
 0002:000029F0       GetThemeFilename
 0002:000029D8       GetThemeFont
 0002:000029CC       GetThemeInt
 0002:000029E4       GetThemeIntList
 0002:000029E0       GetThemeMargins
 0002:000029C0       GetThemeMetric
 0002:00002998       GetThemePartSize
 0002:000029D4       GetThemePosition
 0002:000029E8       GetThemePropertyOrigin
 0002:000029DC       GetThemeRect
 0002:000029C4       GetThemeString
 0002:000029FC       GetThemeSysBool
 0002:000029F4       GetThemeSysColor
 0002:000029F8       GetThemeSysColorBrush
 0002:00002A04       GetThemeSysFont
 0002:00002A0C       GetThemeSysInt
 0002:00002A00       GetThemeSysSize
 0002:00002A08       GetThemeSysString
 0002:0000299C       GetThemeTextExtent
 0002:000029A0       GetThemeTextMetrics
 0001:0000028C       GetThreadLocale
 0001:0000581C       GetThreadLocale
 0001:00005824       GetThreadPriority
 0001:0000582C       GetTickCount
 0001:00008EF8       GetTime
 0001:00005408       GetTlsSize
 0001:0004D0B0       GetTopMostWindows
 0001:0002C034       GetTopParent
 0001:00005D74       GetTopWindow
 0001:00012FB8       GetTypeData
 0001:00005834       GetVersion
 0001:00000314       GetVersion
 0001:0000583C       GetVersionEx
 0001:00005D7C       GetWindow
 0001:00005D84       GetWindowDC
 0001:00005D8C       GetWindowLong
 0001:00005A54       GetWindowOrgEx
 0001:00005D94       GetWindowPlacement
 0001:00005D9C       GetWindowRect
 0001:00005DA4       GetWindowText
 0002:00002A18       GetWindowTheme
 0001:00005DAC       GetWindowThreadProcessId
 0001:00005DB4       GetWindowThreadProcessId
 0001:00005844       GlobalAddAtom
 0001:0000584C       GlobalAlloc
 0001:00006048       GlobalAllocPtr
 0001:00005854       GlobalDeleteAtom
 0001:0000585C       GlobalFindAtom
 0002:0000286C       GlobalFixupList
 0001:00018D40       GlobalFixupReferences
 0001:00005864       GlobalFree
 0001:00006074       GlobalFreePtr
 0001:00005874       GlobalHandle
 0001:0000586C       GlobalLock
 0002:00002850       GlobalNameSpace
 0001:0000587C       GlobalReAlloc
 0001:00006058       GlobalReAllocPtr
 0001:00005884       GlobalUnlock
 0001:00024524       Graphics
 0001:00015BAC       GroupDescendentsWith
 0001:0004FB6C       GUIDToString
 0002:00000E30       GUID_NULL
 0002:000003C0       GUID_NULL
 0001:0000DDF8       HandleConversionException
 0001:0004A240       HandleEdge
 0001:0001A1A4       HandleException
 0002:00000024       HeapAllocFlags
 0002:000025C8       heapErrorCode
 0002:000025CC       heapLock
 0001:0002617C       HelpIntfs
 0002:0000293C       HelpManager
 0002:00002A74       HelpMsg
 0002:00002B10       HelpViewer
 0002:00002B14       HelpViewerIntf
 0002:0000013C       HexDisplayPrefix
 0001:000392A0       HideZone
 0002:00002668       HInstance
 0002:00002BCC       HintDoneEvent
 0001:0004C9D8       HintGetMsgHook
 0002:00002BD0       HintHook
 0001:0004C97C       HintMouseThread
 0002:00002BD4       HintThread
 0002:00002BC8       HintThreadID
 0001:0004C928       HintTimerProc
 0002:00000C34       HintWindowClass
 0002:000029A8       HitTestThemeBackground
 0001:00006028       HiWord
 0001:0004CA1C       HookHintHooks
 0001:00006180       HwndMSWheel
 0002:00000BC8       IBreaks
 0002:00000BD4       IChecks
 0002:00000BDC       IDefaults
 0001:0001EB14       IdentToCharset
 0001:0001E90C       IdentToColor
 0001:0002BE94       IdentToCursor
 0001:00015D94       IdentToInt
 0002:00000BE4       IEnables
 0001:00040E80       IfHotkeyAvailable
 0002:00000D80       IID_IBaseFilter
 0002:00000DE0       IID_IMediaEventSink
 0002:00000E00       IID_IMediaPosition
 0002:00000D90       IID_IMediaSample2
 0002:00000DC0       IID_IMediaSeeking
 0002:00000DA0       IID_IMemAllocator
 0002:00000DB0       IID_IMemInputPin
 0002:00000DD0       IID_IQualityControl
 0002:00000E20       IID_IQualProp
 0002:00000E10       IID_IVideoWindow
 0002:00002BA4       ImageListWriteExProc
 0001:000248F0       ImageList_Add
 0001:00024910       ImageList_AddIcon
 0001:00024934       ImageList_BeginDrag
 0001:000248D8       ImageList_Create
 0001:000248E0       ImageList_Destroy
 0001:00024944       ImageList_DragEnter
 0001:0002494C       ImageList_DragLeave
 0001:00024954       ImageList_DragMove
 0001:00024964       ImageList_DragShowNolock
 0001:0002491C       ImageList_Draw
 0001:00024924       ImageList_DrawEx
 0001:0002493C       ImageList_EndDrag
 0001:00024908       ImageList_GetBkColor
 0001:0002496C       ImageList_GetDragImage
 0001:00024984       ImageList_GetIconSize
 0001:000248E8       ImageList_GetImageCount
 0001:00024974       ImageList_Read
 0001:0002492C       ImageList_Remove
 0001:000248F8       ImageList_ReplaceIcon
 0001:00024900       ImageList_SetBkColor
 0001:0002495C       ImageList_SetDragCursorImage
 0001:0002498C       ImageList_SetIconSize
 0001:0002497C       ImageList_Write
 0002:00000B38       Images
 0001:0003CB60       ImgList
 0001:00025184       Imm
 0002:00000B1C       IMM32DLL
 0001:00039E90       Imm32IsIME
 0002:0000018C       IMSecsPerDay
 0001:0000E184       InBounds
 0001:0000DEE4       InBounds
 0001:0000E1B4       Increment
 0001:0000DF14       Increment
 0001:00005DC4       InflateRect
 0001:000281D0       IniFiles
 0001:00000B88       InitAllocator
 0001:000249CC       InitAnApi
 0002:00002928       InitApis
 0001:00050608       InitComObj
 0001:0001603C       InitComponent
 0002:00002638       InitContext
 0001:00039F2C       InitControls
 0001:0002409C       InitDefFontData
 0001:0000C030       InitDriveSpacePtr
 0001:0000B204       InitExceptions
 0001:0002625C       InitFlatSB
 0001:000276F8       InitGlobals
 0001:00020D58       InitializeBitmapInfoHeader
 0001:0000588C       InitializeCriticalSection
 0001:00000360       InitializeCriticalSection
 0002:000025C4       initialized
 0001:00026234       InitializeFlatSB
 0001:0000550C       InitializeModule
 0001:0000D00C       InitializeVarUtils
 0001:00039B30       InitIMM32
 0001:000160E4       InitInheritedComponent
 0001:0000B9BC       InitLeadBytes
 0001:000250A8       InitMultiMonStubs
 0001:0000B308       InitPlatformId
 0002:00002044       InitProc
 0001:00005454       InitProcessTLS
 0001:0004F4A8       InitProcs
 0001:00024020       InitScreenLogPixels
 0001:0000BA34       InitSysLocale
 0001:00026884       InitThemeLibrary
 0001:0001BAB0       InitThreadSynchronization
 0001:00005410       InitThreadTLS
 0001:00002ED4       InitUnits
 0001:0002BB78       InitWndProc
 0002:00000ABC       InnerStyles
 0002:00002050       Input
 0001:00005DBC       InSendMessage
 0001:0004C400       InsertBefore
 0001:00031514       InsertBefore
 0001:00001034       InsertFree
 0001:00040F34       InsertHotkeyFarEastFormat
 0001:00005DCC       InsertMenu
 0001:00005DD4       InsertMenuItem
 0002:00002888       InstBlockList
 0002:0000288C       InstFreeList
 0002:00002860       IntConstList
 0001:00000304       InterlockedDecrement
 0001:00005774       InterlockedDecrement
 0001:0000C098       InterlockedDecrement
 0001:0000577C       InterlockedExchange
 0001:0000C0A4       InterlockedExchange
 0001:0000C0AC       InterlockedExchangeAdd
 0001:0000C08C       InterlockedIncrement
 0001:000002FC       InterlockedIncrement
 0001:00005784       InterlockedIncrement
 0001:0001DFF8       InternalDeletePalette
 0001:00001CE4       InternalFlush
 0001:00000E74       InternalFreeMem
 0001:00020EA8       InternalGetDIB
 0001:00020E3C       InternalGetDIBSizes
 0001:00015ED4       InternalReadComponentRes
 0002:00002AF8       InternalServices
 0001:00003794       InternalUniqueString
 0001:00005A5C       IntersectClipRect
 0001:00005DDC       IntersectRect
 0001:000075E0       IntToHex
 0001:00015DD4       IntToIdent
 0001:000075B8       IntToStr
 0001:000074CC       IntToStr
 0001:00005DE4       InvalidateRect
 0001:0001FEDC       InvalidBitmap
 0001:0001FEC4       InvalidGraphic
 0001:0001FEE8       InvalidIcon
 0001:0001FEAC       InvalidOperation
 0001:00014F40       InvalidPoint
 0002:0000279C       InvalidPointer
 0001:00002514       InvokeImplGetter
 0001:00001C38       IOResult
 0002:00000C04       IOwnerDraw
 0002:00000BEC       IRadios
 0002:00000BFC       IRTL
 0001:000453FC       IsAccel
 0001:00042114       IsAccelChar
 0002:00002A14       IsAppThemed
 0001:0002C68C       IsBeforeTargetWindow
 0002:00000EDC       IsCheckedVersion
 0001:00005DEC       IsChild
 0002:0000204C       IsConsole
 0001:0002CAE8       IsDelphiHandle
 0001:00005DF4       IsDialogMessage
 0002:00000BF4       ISeparators
 0001:00013840       IsEqualGUID
 0001:00005DFC       IsIconic
 0001:00042170       IsInitialChar
 0001:00008B28       IsLeapYear
 0002:00002038       IsLibrary
 0002:0000204D       IsMultiThread
 0001:00036F50       IsOrientationSet
 0001:0005B4D4       isqrt
 0001:00005E04       IsRectEmpty
 0001:0002C890       IsSiteChildOfClient
 0002:00002A10       IsThemeActive
 0002:000029B8       IsThemeBackgroundPartiallyTransparent
 0002:00002A20       IsThemeDialogTextureEnabled
 0002:000029B4       IsThemePartDefined
 0002:00000EE0       IsTimeKillSynchronousFlagAvailable
 0001:00015EB0       IsUniqueGlobalComponentName
 0002:00002854       IsUniqueGlobalComponentNameProc
 0001:0000741C       IsValidIdent
 0001:0000BA1C       IsWesternGroup
 0001:00005E0C       IsWindow
 0001:00005E14       IsWindowEnabled
 0001:00005E1C       IsWindowVisible
 0001:00005E24       IsZoomed
 0001:0003DEF4       Iterate
 0001:0003DF54       IterateMenus
 0002:0000002C       JITEnable
 0001:000453B0       KeyboardStateToShiftState
 0001:00045374       KeyDataToShiftState
 0001:00045320       KeysToShiftState
 0001:00005E2C       KillTimer
 0001:000079A4       LastDelimiter
 0001:0000B948       LCIDToCodePage
 0001:00005230       LCIDToCodePage
 0002:0000011C       LeadBytes
 0001:00000370       LeaveCriticalSection
 0001:00005894       LeaveCriticalSection
 0002:00000DF0       LIBID_QuartzTypeLib
 0002:00000034       LibModuleList
 0001:00005A64       LineTo
 0001:00028334       ListActns
 0001:0002D678       ListAdd
 0001:0002D6A0       ListRemove
 0002:00002752       ListSeparator
 0001:00050B60       llMulDiv
 0001:00005E34       LoadBitmap
 0001:0004FC48       LoadComExProcs
 0001:00005E3C       LoadCursor
 0001:00005E44       LoadIcon
 0001:00005E4C       LoadKeyboardLayout
 0001:0000589C       LoadLibrary
 0001:00000294       LoadLibraryEx
 0001:00013890       LoadRegTypeLib
 0001:000058A4       LoadResource
 0001:000048E8       LoadResourceModule
 0001:000051D8       LoadResString
 0001:00005E54       LoadString
 0001:0000029C       LoadString
 0001:00013888       LoadTypeLib
 0001:00000340       LocalAlloc
 0001:000053CC       LocalAlloc
 0001:00000348       LocalFree
 0001:000053D4       LocalFree
 0001:0000A3A0       LocalGetLocaleStr
 0002:00002A48       Lock
 0001:000058AC       LockResource
 0002:00002694       LongDateFormat
 0002:00002728       LongDayNames
 0002:000026DC       LongMonthNames
 0002:000026A8       LongTimeFormat
 0001:0000720C       LowerCase
 0001:00005944       lstrcpy
 0001:000002A4       lstrcpyn
 0002:00002828       LVarTypes
 0002:0000282C       LVarTypeSync
 0002:00002030       MainInstance
 0002:00002034       MainThreadID
 0001:00000404       MakeEmpty
 0001:00003098       MakeErrorMessage
 0002:00000B08       MakeLast
 0001:0000601C       MakeLong
 0001:0001CD54       MakeObjectInstance
 0001:00006088       MakeROP4
 0001:000060C0       MakeWParam
 0001:0000AEBC       MapException
 0001:000282A4       Mapi
 0002:00000964       MAPIDLL
 0002:00000968       MAPIModule
 0001:00002CDC       MapToRunError
 0001:00005E5C       MapVirtualKey
 0001:00005E64       MapWindowPoints
 0002:00000B40       Mask
 0001:00005A6C       MaskBlt
 0001:0001D0B0       Math
 0001:0001D078       Max
 0001:00047CCC       MaximizedChildren
 0002:00000ED0       MAX_TIME
 0002:00000E50       MEDIASUBTYPE_RGB24
 0002:00000E40       MEDIATYPE_Video
 0002:0000003C       MemoryManager
 0002:00000B5C       MenuKeyCaps
 0001:00043190       Menus
 0001:0000049C       MergeBlockAfter
 0001:00001178       MergeCommit
 0001:0000023C       MessageBox
 0001:00005E6C       MessageBox
 0001:0000CB54       Messages
 0001:0001D038       Min
 0001:0001D030       Min
 0001:00016748       Min
 0001:00030E9C       MinVar
 0002:00002930       MMAvailable
 0001:0004F664       MMSystem
 0002:00000B20       ModeMap
 0001:000499CC       ModifySystemMenu
 0002:000000A4       Module
 0002:00002665       ModuleIsCpp
 0002:00002664       ModuleIsLib
 0001:0001CD24       ModuleUnload
 0002:00000038       ModuleUnloadList
 0002:0000290C       MonitorFromPoint
 0002:00002908       MonitorFromRect
 0002:00002904       MonitorFromWindow
 0002:000000EC       MonthDays
 0002:00002B18       Mouse
 0001:00001C58       Move
 0001:00005A74       MoveToEx
 0001:00005E74       MoveWindow
 0001:0002D6C0       MoveWindowOrg
 0002:00000EE4       MsgId
 0001:00005E7C       MsgWaitForMultipleObjects
 0001:00057998       MSR_INTEGER
 0001:000058B4       MulDiv
 0001:000058BC       MultiByteToWideChar
 0001:000002B4       MultiByteToWideChar
 0001:0004EF34       MultiLineWidth
 0001:00025144       MultiMon
 0002:00002C00       NeedToUninitialize
 0002:00002689       NegCurrFormat
 0001:00001204       NewCommit
 0001:00001230       NewCommitAt
 0002:00002B1C       NewStyleControls
 0001:0000B780       NextCharIndex
 0001:00036F34       NextVisibleZone
 0002:000003FC       NilMethod
 0002:00000030       NoErrMsg
 0001:0003ED08       NormalDraw
 0001:00002894       NotifyAnyExcept
 0001:00002868       NotifyExcept
 0001:000028C8       NotifyExceptFinally
 0001:00015FB0       NotifyGlobalLoading
 0001:00004C24       NotifyModuleUnload
 0001:00002844       NotifyNonDelphiException
 0001:00002880       NotifyOnExcept
 0001:00002828       NotifyReRaise
 0001:000028F0       NotifyTerminate
 0001:0000290C       NotifyUnhandled
 0001:00041AC0       NthParentOf
 0001:00012D40       Null
 0002:00000328       NullAsStringValue
 0002:00000324       NullStrictConvert
 0002:00002C14       ObjectCount
 0001:0002BC30       ObjectFromHWnd
 0001:00005E84       OemToAnsi
 0001:00005E8C       OffsetRect
 0001:0004FB54       OleCheck
 0001:0004FB38       OleError
 0001:000040C4       OleStrToStrVar
 0002:00002BF4       OleUninitializing
 0002:00002980       OpenThemeData
 0002:00000B00       OrientArray
 0002:00000ACC       OuterStyles
 0002:00002798       OutOfMemory
 0001:0001FEF4       OutOfResources
 0002:0000221C       Output
 0002:0000032C       PackVarCreation
 0002:000006F8       Pal16
 0001:0001E400       PaletteChanged
 0001:000206EC       PaletteFromDIBColorTable
 0001:00020790       PaletteToDIBColorTable
 0002:000006F4       PalSize
 0001:00037318       ParentNotLast
 0001:00005A7C       PatBlt
 0002:000028F4       PatternManager
 0001:00005E94       PeekMessage
 0002:000028E8       PenManager
 0002:000006C4       PenModes
 0002:000006A4       PenStyles
 0001:00014EC8       Point
 0001:000055B4       Point
 0001:00015300       PointerInModule
 0001:0003268C       PointsEqual
 0001:000060A8       PointToSmallPoint
 0002:00002BA8       PopupList
 0001:0005B9F4       PossiblyEatMessage
 0001:00005E9C       PostMessage
 0001:00005EA4       PostQuitMessage
 0001:00005EAC       PostThreadMessage
 0001:000261F8       Printers
 0001:0004B0E0       ProcessExecute
 0001:0004562C       ProcessHorz
 0001:0004B1E0       ProcessUpdate
 0001:00045698       ProcessVert
 0001:0001903C       PropertyNotFound
 0001:0001A2A4       PropPathError
 0002:00000C64       Props
 0001:00019030       PropValueError
 0001:00005EB4       PtInRect
 0002:000000A0       PtrToNil
 0001:000082D0       PutExponent
 0002:00002B60       QualifyingSites
 0001:0000AE78       RaiseAssertException
 0001:00018050       RaiseException
 0001:000502A4       RaiseException
 0001:0000020C       RaiseException
 0002:00002014       RaiseExceptionProc
 0001:0000BF2C       RaiseLastOSError
 0001:00050190       RaiseNameException
 0001:00038088       ReadControlName
 0001:0001B4E4       ReadCustomVariant
 0001:00019018       ReadError
 0001:000058C4       ReadFile
 0001:00020A44       ReadIcon
 0001:00005A84       RealizePalette
 0001:00019858       Recover
 0001:00005598       Rect
 0001:00014EF0       Rect
 0001:00005A8C       RectVisible
 0001:00005EBC       RedrawWindow
 0002:00002820       RefAnyProc
 0002:00002A44       ReferenceCount
 0001:000056DC       RegCloseKey
 0001:000002BC       RegCloseKey
 0001:000056E4       RegCreateKeyEx
 0001:000056EC       RegDeleteKey
 0002:00002864       RegGroups
 0001:00005EC4       RegisterClass
 0001:00015AA4       RegisterClass
 0001:00005ECC       RegisterClipboardFormat
 0001:0002CA30       RegisterDockSite
 0001:00015E18       RegisterFindGlobalComponentProc
 0001:00015CEC       RegisterIntegerConsts
 0001:00004C80       RegisterModule
 0001:00025550       RegisterViewer
 0001:00005ED4       RegisterWindowMessage
 0001:00028238       Registry
 0001:000002C4       RegOpenKeyEx
 0001:000056F4       RegOpenKeyEx
 0001:000002CC       RegQueryValueEx
 0001:000056FC       RegQueryValueEx
 0001:00005704       RegSetValueEx
 0001:00027158       RegStr
 0001:00005EDC       ReleaseCapture
 0001:00005EE4       ReleaseDC
 0002:00000048       reMap
 0002:0000261C       remBytes
 0001:00000524       RemoveBlock
 0002:000003D8       RemoveDataModule
 0001:00018EE8       RemoveFixupReferences
 0001:00018F94       RemoveFixups
 0001:0001928C       RemoveGlobalFixup
 0001:00005EEC       RemoveMenu
 0001:00004B9C       RemoveModuleUnloadProc
 0001:00004B74       RemoveModuleUnloadProc
 0001:00005EF4       RemoveProp
 0001:000058CC       ResetEvent
 0001:0001BAFC       ResetSyncEvent
 0001:00001768       ResizeInPlace
 0001:00005A94       RestoreDC
 0001:00044FB4       RestoreFocusState
 0001:0003DAC8       ReturnAddr
 0001:00016274       ReturnAddr
 0001:00016EEC       ReturnAddr
 0001:00020470       RGBQuadToTriple
 0001:00020428       RGBTripleToQuad
 0001:000270B0       RichEdit
 0002:00002B30       RM_GetObjectInstance
 0002:00002BC4       RM_TaskbarCreated
 0002:00002618       rover
 0002:0000096C       RTFConversionFormat
 0001:00012F84       RTLConsts
 0001:00000214       RtlUnwind
 0002:00002018       RTLUnwindProc
 0002:0000006C       runErrMsg
 0001:00001B60       RunErrorAt
 0001:0000CFC0       SafeArrayCreate
 0001:0000CFC8       SafeArrayGetLBound
 0001:0000CFD0       SafeArrayGetUBound
 0001:0000CFD8       SafeArrayPtrOfIndex
 0001:0004FD4C       SafeCallError
 0002:00002020       SafeCallErrorProc
 0001:0000C5D0       SafeLoadLibrary
 0001:00007300       SameText
 0001:00005A9C       SaveDC
 0001:00044FA4       SaveFocusState
 0002:00002BFC       SaveInitProc
 0001:000099F4       ScanBlanks
 0001:00009B38       ScanChar
 0001:00009CB4       ScanDate
 0001:00009A18       ScanNumber
 0001:00009AAC       ScanString
 0001:00009FF8       ScanTime
 0001:00009BBC       ScanToNumber
 0002:00002BBC       Screen
 0002:000028A0       ScreenLogPixels
 0001:00005EFC       ScreenToClient
 0001:000457E4       ScrollBarVisible
 0001:00005F04       ScrollWindow
 0001:00001264       SearchSmallBlocks
 0001:00005AA4       SelectObject
 0001:00005AAC       SelectPalette
 0001:0002BCC0       SendAppMessage
 0001:00045234       SendFocusMessage
 0001:00005F0C       SendMessage
 0002:00000BC0       Separators
 0001:00001CA4       Set8087CW
 0001:00005F14       SetActiveWindow
 0001:0004CB1C       SetAnimation
 0001:00005AB4       SetBkColor
 0001:00005ABC       SetBkMode
 0001:00005AC4       SetBrushOrgEx
 0001:00005F1C       SetCapture
 0001:0002BF54       SetCaptureControl
 0001:00005F24       SetClassLong
 0001:000128CC       SetClearVarToEmptyParam
 0001:000199C8       SetCompName
 0001:00005F2C       SetCursor
 0001:00005ACC       SetDIBColorTable
 0001:000058D4       SetEndOfFile
 0001:000058DC       SetErrorMode
 0001:000058E4       SetEvent
 0001:00002E1C       SetExceptionHandler
 0001:000058EC       SetFilePointer
 0001:000133E8       SetFloatProp
 0001:00005F34       SetFocus
 0001:00005F3C       SetForegroundWindow
 0001:00039DB4       SetImeMode
 0001:00001BE4       SetInOutRes
 0001:0001366C       SetInt64Prop
 0001:000136A8       SetInterfaceProp
 0001:0001A584       SetInterfaceReference
 0001:0001A4A0       SetIntIdent
 0001:000058F4       SetLastError
 0002:00000C38       SetLayeredWindowAttributes
 0001:00013250       SetLongStrProp
 0001:00005F44       SetMenu
 0001:00005F4C       SetMenuItemInfo
 0001:00013634       SetMethodProp
 0001:0001A4E8       SetObjectIdent
 0001:00013158       SetOrdProp
 0001:00005F54       SetParent
 0001:00005AD4       SetPixel
 0001:00005F5C       SetProp
 0001:00005F64       SetRect
 0001:00005ADC       SetROP2
 0001:00005F6C       SetScrollInfo
 0001:00005F74       SetScrollPos
 0001:00005F7C       SetScrollRange
 0001:000131B4       SetShortStrProp
 0001:00013208       SetShortStrPropAsLongStr
 0001:00005AE4       SetStretchBltMode
 0001:000132E8       SetStrProp
 0001:000197D0       SetSubComponentState
 0001:00005AEC       SetTextColor
 0002:00002A28       SetThemeAppProperties
 0001:000058FC       SetThreadLocale
 0001:00005904       SetThreadPriority
 0001:00005F84       SetTimer
 0001:000128B4       SetVarAsError
 0001:000135F4       SetVariantProp
 0001:0001A528       SetVariantReference
 0001:00005AF4       SetViewportOrgEx
 0001:0004EA38       SetVisible
 0001:00013314       SetWideStrProp
 0001:00013290       SetWideStrPropAsLongStr
 0001:00005F8C       SetWindowLong
 0001:00005AFC       SetWindowOrgEx
 0001:00005F94       SetWindowPlacement
 0001:00005F9C       SetWindowPos
 0001:00005FA4       SetWindowsHookEx
 0002:000029EC       SetWindowTheme
 0002:00000158       ShareMode
 0001:00027120       ShellAPI
 0002:00002AE8       ShellModule
 0001:00027200       ShlObj
 0001:0003DAF0       ShortCut
 0002:00002BAC       ShortCutItems
 0001:0003DB7C       ShortCutToText
 0002:00002690       ShortDateFormat
 0002:0000270C       ShortDayNames
 0002:000026AC       ShortMonthNames
 0002:000026A4       ShortTimeFormat
 0002:00000CB0       ShowCommands
 0002:00000C98       ShowCommands
 0002:00000CA4       ShowCommands
 0001:00005FAC       ShowCursor
 0001:0000AA30       ShowException
 0002:00000D4C       ShowFlags
 0002:00000AB4       ShowFlags
 0001:00044FBC       ShowMDIClientEdge
 0001:00005FB4       ShowOwnedPopups
 0001:00005FBC       ShowScrollBar
 0001:00005FC4       ShowWindow
 0001:0004CB44       ShowWinNoAnimate
 0001:00039320       ShowZone
 0002:00000B14       SizeCursors
 0001:0000590C       SizeofResource
 0001:0001B018       SkipBinary
 0001:0001B048       SkipCollection
 0001:0001AFF0       SkipList
 0001:00005914       Sleep
 0001:0000BF24       Sleep
 0001:00014EE0       SmallPoint
 0001:00006094       SmallPointToPoint
 0002:00002624       smallTab
 0002:000025EC       spaceRoot
 0001:00015B60       StartClassGroup
 0001:00029060       StdActns
 0001:00028EF8       StdCtrls
 0001:0001CD2C       StdWndProc
 0002:000028A8       StockBrush
 0002:000028AC       StockFont
 0002:000028B0       StockIcon
 0002:000028A4       StockPen
 0001:00007CF0       StrAlloc
 0001:00007D04       StrBufSize
 0001:0000B520       StrByteType
 0001:0000B710       StrCharLength
 0001:00007BD4       StrComp
 0001:00007B24       StrCopy
 0001:00007D4C       StrDispose
 0001:0003C2AC       StreamsEqual
 0001:00007B00       StrEnd
 0001:00005B04       StretchBlt
 0001:00005B0C       StretchDIBits
 0001:0000815C       StrFmt
 0001:00007BF8       StrIComp
 0001:00013868       StringFromCLSID
 0001:00017EEC       StringListCompareStrings
 0001:000040E8       StringToOleStr
 0001:00042F28       StripHotkey
 0001:00007B4C       StrLCopy
 0001:00007AE8       StrLen
 0001:000081A8       StrLFmt
 0001:00007C38       StrLIComp
 0001:00007B14       StrMove
 0001:00007D18       StrNew
 0001:0000B730       StrNextChar
 0001:00007B80       StrPCopy
 0001:00007BAC       StrPLCopy
 0001:00007C9C       StrPos
 0001:00007C7C       StrScan
 0001:00007608       StrToInt
 0001:00007644       StrToIntDef
 0001:00028038       StrUtils
 0002:00000C8C       Styles
 0001:000138A0       Succeeded
 0001:0000C514       Supports
 0001:0000C538       Supports
 0002:00002858       SyncEvent
 0002:00000404       SyncList
 0001:000266BC       SyncObjs
 0001:000002E4       SysAllocStringLen
 0001:000065B8       SysConst
 0002:00000C5C       SysConsts
 0002:00000C54       SysConsts
 0001:0000A2E0       SysErrorMessage
 0001:00001590       SysFreeMem
 0001:000002F4       SysFreeString
 0001:00013880       SysFreeString
 0001:000013E4       SysGetMem
 0001:00005590       SysInit
 0002:00002744       SysLocale
 0001:0000196C       SysReallocMem
 0001:000002EC       SysReAllocStringLen
 0001:000052F8       System
 0002:00002898       SystemPalette16
 0001:00020654       SystemPaletteOverride
 0001:00005FCC       SystemParametersInfo
 0001:0000CAA4       SysUtils
 0001:0003AC48       TActionLink.IsCaptionLinked
 0001:0003AC5C       TActionLink.IsCheckedLinked
 0001:0003AC70       TActionLink.IsEnabledLinked
 0001:0003AC84       TActionLink.IsGroupIndexLinked
 0001:0003AC98       TActionLink.IsHelpContextLinked
 0001:0003ACAC       TActionLink.IsHelpLinked
 0001:0003ACC0       TActionLink.IsHintLinked
 0001:0003ACD4       TActionLink.IsImageIndexLinked
 0001:0003ACE8       TActionLink.IsShortCutLinked
 0001:0003ACFC       TActionLink.IsVisibleLinked
 0001:0003AD10       TActionLink.SetAutoCheck
 0001:0003AD14       TActionLink.SetCaption
 0001:0003AD18       TActionLink.SetChecked
 0001:0003AD1C       TActionLink.SetEnabled
 0001:0003AD20       TActionLink.SetGroupIndex
 0001:0003AD24       TActionLink.SetHelpContext
 0001:0003AD28       TActionLink.SetHelpKeyword
 0001:0003AD2C       TActionLink.SetHelpType
 0001:0003AD30       TActionLink.SetHint
 0001:0003AD34       TActionLink.SetImageIndex
 0001:0003AD38       TActionLink.SetShortCut
 0001:0003AD3C       TActionLink.SetVisible
 0001:0004EFF8       TApplication.ActivateHint
 0001:0004DCEC       TApplication.BringToFront
 0001:0004ED3C       TApplication.CancelHint
 0001:0004D2D4       TApplication.CheckIniChange
 0001:0004D050       TApplication.ControlDestroyed
 0001:0004CB84       TApplication.Create
 0001:0004CEA0       TApplication.CreateHandle
 0001:0004CD84       TApplication.Destroy
 0001:0004F3C8       TApplication.DispatchAction
 0001:0004E708       TApplication.DoActionIdle
 0001:0004E76C       TApplication.DoMouseIdle
 0001:0004D120       TApplication.DoNormalizeTopMosts
 0001:0004F458       TApplication.ExecuteAction
 0001:0004F38C       TApplication.GetCurrentHelpFile
 0001:0004DB20       TApplication.GetIconHandle
 0001:0004DD28       TApplication.GetTitle
 0001:0004E0F8       TApplication.HandleException
 0001:0004DFD8       TApplication.HandleMessage
 0001:0004E6B0       TApplication.HelpCommand
 0001:0004E628       TApplication.HelpContext
 0001:0004E598       TApplication.HelpKeyword
 0001:0004ECF8       TApplication.HideHint
 0001:0004EBB0       TApplication.HintMouseMessage
 0001:0004ECC0       TApplication.HintTimerExpired
 0001:0004DFFC       TApplication.HookMainWindow
 0001:0004F504       TApplication.HookSynchronizeWakeup
 0001:0004E940       TApplication.IconChanged
 0001:0004E7E4       TApplication.Idle
 0001:0004E3C8       TApplication.InvokeHelp
 0001:0004DD74       TApplication.IsDlgMsg
 0001:0004DEA0       TApplication.IsHintMsg
 0001:0004DDE8       TApplication.IsKeyMsg
 0001:0004DD98       TApplication.IsMDIMsg
 0001:0004DED4       TApplication.IsShortCut
 0001:0004E188       TApplication.MessageBox
 0001:0004DB3C       TApplication.Minimize
 0001:0004D1FC       TApplication.ModalFinished
 0001:0004D1D0       TApplication.ModalStarted
 0001:0004D230       TApplication.NormalizeAllTopMosts
 0001:0004D228       TApplication.NormalizeTopMosts
 0001:0004E904       TApplication.NotifyForms
 0001:0004DF40       TApplication.ProcessMessage
 0001:0004DBEC       TApplication.Restore
 0001:0004D238       TApplication.RestoreTopMosts
 0001:0004E9A4       TApplication.SetHint
 0001:0004E6B8       TApplication.SetShowHint
 0001:0004D32C       TApplication.SettingChange
 0001:0004E2F0       TApplication.ShowException
 0001:0004EB44       TApplication.StartHintTimer
 0001:0004EB88       TApplication.StopHintTimer
 0001:0004E0E4       TApplication.Terminate
 0001:0004E058       TApplication.UnhookMainWindow
 0001:0004F514       TApplication.UnhookSynchronizeWakeup
 0001:0004F480       TApplication.UpdateAction
 0001:0004EA94       TApplication.UpdateVisible
 0001:0004D2BC       TApplication.UseRightToLeftAlignment
 0001:0004D2A4       TApplication.UseRightToLeftReading
 0001:0004EB1C       TApplication.ValidateHelpSystem
 0001:0004F4F4       TApplication.WakeMainThread
 0001:0004D420       TApplication.WndProc
 0002:00000C44       TaskActiveWindow
 0002:00000C4C       TaskFirstTopMost
 0002:00000C48       TaskFirstWindow
 0002:00000C50       TaskWindowList
 0001:0002C3A4       TBaseDragControlObject.Assign
 0001:0002C380       TBaseDragControlObject.Create
 0001:0002C3D0       TBaseDragControlObject.EndDrag
 0001:0002C3FC       TBaseDragControlObject.Finished
 0001:0001C730       TBasicAction.Change
 0001:0001C5CC       TBasicAction.Create
 0001:0001C610       TBasicAction.Destroy
 0001:0001C69C       TBasicAction.Execute
 0001:0001C66C       TBasicAction.ExecuteTarget
 0001:0001C668       TBasicAction.HandlesTarget
 0001:0001C670       TBasicAction.Notification
 0001:0001C744       TBasicAction.RegisterChanges
 0001:0001C790       TBasicAction.SetActionComponent
 0001:0001C6D4       TBasicAction.SetOnExecute
 0001:0001C750       TBasicAction.UnRegisterChanges
 0001:0001C6B8       TBasicAction.Update
 0001:0001C698       TBasicAction.UpdateTarget
 0001:0001C51C       TBasicActionLink.AssignClient
 0001:0001C554       TBasicActionLink.Change
 0001:0001C4D8       TBasicActionLink.Create
 0001:0001C520       TBasicActionLink.Destroy
 0001:0001C56C       TBasicActionLink.Execute
 0001:0001C5B4       TBasicActionLink.IsOnExecuteLinked
 0001:0001C588       TBasicActionLink.SetAction
 0001:0001C5B8       TBasicActionLink.SetOnExecute
 0001:0001C5C0       TBasicActionLink.Update
 0001:000577FC       TBCAMEvent.Create
 0001:00057848       TBCAMEvent.destroy
 0001:000578E4       TBCAMEvent.Reset
 0001:000578F0       TBCAMEvent.SetEv
 0001:00056734       TBCBaseDispatch.GetIDsOfNames
 0001:000567B0       TBCBaseDispatch.GetTypeInfo
 0001:000568A0       TBCBaseDispatch.GetTypeInfoCount
 0001:00053304       TBCBaseFilter.Create
 0001:00053438       TBCBaseFilter.CreateFromFactory
 0001:00053490       TBCBaseFilter.destroy
 0001:000534D0       TBCBaseFilter.EnumPins
 0001:00053518       TBCBaseFilter.FindPin
 0001:00053674       TBCBaseFilter.GetClassID
 0001:00053690       TBCBaseFilter.GetPinVersion
 0001:00053694       TBCBaseFilter.GetState
 0001:000536A8       TBCBaseFilter.GetSyncSource
 0001:00053708       TBCBaseFilter.IsActive
 0001:0005376C       TBCBaseFilter.JoinFilterGraph
 0001:000538C8       TBCBaseFilter.NotifyEvent
 0001:00053954       TBCBaseFilter.Pause
 0001:00053A04       TBCBaseFilter.QueryFilterInfo
 0001:00053A94       TBCBaseFilter.QueryVendorInfo
 0001:00053AA0       TBCBaseFilter.Register
 0001:00053BCC       TBCBaseFilter.Run
 0001:00053CBC       TBCBaseFilter.SetSyncSource
 0001:00053D44       TBCBaseFilter.Stop
 0001:00053DF8       TBCBaseFilter.StreamTime
 0001:00053E3C       TBCBaseFilter.Unregister
 0001:00055884       TBCBaseInputPin.BeginFlush
 0001:00055948       TBCBaseInputPin.BreakConnect
 0001:00055980       TBCBaseInputPin.CheckStreaming
 0001:00055A28       TBCBaseInputPin.Create
 0001:00055AEC       TBCBaseInputPin.Destroy
 0001:00055B28       TBCBaseInputPin.EndFlush
 0001:00055BF4       TBCBaseInputPin.GetAllocator
 0001:00055D10       TBCBaseInputPin.GetAllocatorRequirements
 0001:00055D1C       TBCBaseInputPin.Inactive
 0001:00055D44       TBCBaseInputPin.Notify
 0001:00055D84       TBCBaseInputPin.NotifyAllocator
 0001:00055E24       TBCBaseInputPin.Receive
 0001:00056060       TBCBaseInputPin.ReceiveCanBlock
 0001:000561F4       TBCBaseInputPin.ReceiveMultiple
 0001:00056234       TBCBaseInputPin.SampleProps
 0001:00053084       TBCBaseObject.Create
 0001:000530F8       TBCBaseObject.Destroy
 0001:00053120       TBCBaseObject.FreeInstance
 0001:00053130       TBCBaseObject.NewInstance
 0001:00054378       TBCBasePin.Active
 0001:0005437C       TBCBasePin.AgreeMediaType
 0001:00054518       TBCBasePin.AttemptConnection
 0001:000546E4       TBCBasePin.BreakConnect
 0001:000546E8       TBCBasePin.CheckConnect
 0001:000547DC       TBCBasePin.CompleteConnect
 0001:0005480C       TBCBasePin.Connect
 0001:00054970       TBCBasePin.ConnectedTo
 0001:000549A4       TBCBasePin.ConnectionMediaType
 0001:00054A40       TBCBasePin.Create
 0001:00054BE4       TBCBasePin.destroy
 0001:00054CA0       TBCBasePin.Disconnect
 0001:00054D08       TBCBasePin.DisconnectInternal
 0001:00054DB4       TBCBasePin.DisplayPinInfo
 0001:00054DDC       TBCBasePin.DisplayTypeInfo
 0001:00054E04       TBCBasePin.EndOfStream
 0001:00054E10       TBCBasePin.EnumMediaTypes
 0001:00054E58       TBCBasePin.GetMediaType
 0001:00054E60       TBCBasePin.GetMediaTypeVersion
 0001:00054E64       TBCBasePin.Inactive
 0001:00054E6C       TBCBasePin.IsConnected
 0001:00054E74       TBCBasePin.IsStopped
 0001:00054E80       TBCBasePin.NewSegment
 0001:00054EC4       TBCBasePin.NonDelegatingAddRef
 0001:00054F50       TBCBasePin.NonDelegatingRelease
 0001:00054FDC       TBCBasePin.Notify
 0001:00055020       TBCBasePin.QueryAccept
 0001:00055048       TBCBasePin.QueryDirection
 0001:0005505C       TBCBasePin.QueryId
 0001:00055074       TBCBasePin.QueryInternalConnections
 0001:0005508C       TBCBasePin.QueryPinInfo
 0001:00055100       TBCBasePin.ReceiveConnection
 0001:0005533C       TBCBasePin.Run
 0001:00055348       TBCBasePin.SetMediaType
 0001:00055368       TBCBasePin.SetSink
 0001:000553F4       TBCBasePin.TryMediaTypes
 0001:0005632C       TBCBasePropertyPage.Activate
 0001:00056394       TBCBasePropertyPage.Apply
 0001:00056654       TBCBasePropertyPage.Create
 0001:000563E0       TBCBasePropertyPage.Deactivate
 0001:000566FC       TBCBasePropertyPage.Destroy
 0001:00056444       TBCBasePropertyPage.GetPageInfo
 0001:000564DC       TBCBasePropertyPage.Help
 0001:000564E8       TBCBasePropertyPage.IsPageDirty
 0001:00056504       TBCBasePropertyPage.Move
 0001:0005654C       TBCBasePropertyPage.SetObjects
 0001:0005659C       TBCBasePropertyPage.SetPageSite
 0001:000565E4       TBCBasePropertyPage.Show
 0001:00056648       TBCBasePropertyPage.TranslateAccelerator
 0001:00058D60       TBCBaseRenderer.Active
 0001:00058C28       TBCBaseRenderer.BeginFlush
 0001:00058D88       TBCBaseRenderer.BreakConnect
 0001:00058F60       TBCBaseRenderer.CancelNotification
 0001:000598F8       TBCBaseRenderer.ClearPendingSample
 0001:00058CF0       TBCBaseRenderer.CompleteConnect
 0001:00058190       TBCBaseRenderer.CompleteStateChange
 0001:000579DC       TBCBaseRenderer.Create
 0001:00057B4C       TBCBaseRenderer.Destroy
 0001:00058C60       TBCBaseRenderer.EndFlush
 0001:00058BF4       TBCBaseRenderer.EndOfStream
 0001:00058ADC       TBCBaseRenderer.FindPin
 0001:00059288       TBCBaseRenderer.GetCurrentSample
 0001:00057C74       TBCBaseRenderer.GetMediaPositionInterface
 0001:000588A4       TBCBaseRenderer.GetPin
 0001:0005889C       TBCBaseRenderer.GetPinCount
 0001:00057F74       TBCBaseRenderer.GetRealState
 0001:00058E00       TBCBaseRenderer.GetSampleTimes
 0001:00058158       TBCBaseRenderer.GetState
 0001:0005922C       TBCBaseRenderer.HaveCurrentSample
 0001:00058D64       TBCBaseRenderer.Inactive
 0001:00057DE0       TBCBaseRenderer.JoinFilterGraph
 0001:00057E4C       TBCBaseRenderer.NonDelegatingQueryInterface
 0001:00059A90       TBCBaseRenderer.NotifyEndOfStream
 0001:0005820C       TBCBaseRenderer.NotReady
 0001:000581D8       TBCBaseRenderer.OnReceiveFirstSample
 0001:00059F40       TBCBaseRenderer.OnRenderEnd
 0001:00059F18       TBCBaseRenderer.OnRenderStart
 0001:00059F68       TBCBaseRenderer.OnStartStreaming
 0001:00059F6C       TBCBaseRenderer.OnStopStreaming
 0001:00059F74       TBCBaseRenderer.OnWaitEnd
 0001:00059F70       TBCBaseRenderer.OnWaitStart
 0001:000583D4       TBCBaseRenderer.Pause
 0001:000592E4       TBCBaseRenderer.PrepareReceive
 0001:00059F78       TBCBaseRenderer.PrepareRender
 0001:00058200       TBCBaseRenderer.Ready
 0001:00059620       TBCBaseRenderer.Receive
 0001:000591AC       TBCBaseRenderer.Render
 0001:00059C28       TBCBaseRenderer.ResetEndOfStream
 0001:00059CAC       TBCBaseRenderer.ResetEndOfStreamTimer
 0001:00058618       TBCBaseRenderer.Run
 0001:00059024       TBCBaseRenderer.ScheduleSample
 0001:000599D8       TBCBaseRenderer.SendEndOfStream
 0001:00058D84       TBCBaseRenderer.SetMediaType
 0001:00059EC0       TBCBaseRenderer.SetRepaintStatus
 0001:00058F24       TBCBaseRenderer.ShouldDrawSampleNow
 0001:00058F58       TBCBaseRenderer.SignalTimerFired
 0001:00057E98       TBCBaseRenderer.SourceThreadCanWait
 0001:00059CCC       TBCBaseRenderer.StartStreaming
 0001:00058218       TBCBaseRenderer.Stop
 0001:00059E44       TBCBaseRenderer.StopStreaming
 0001:00059970       TBCBaseRenderer.TimerCallback
 0001:00057F24       TBCBaseRenderer.WaitForReceiveToComplete
 0001:00057EB4       TBCBaseRenderer.WaitForRenderTime
 0001:0005A5BC       TBCBaseVideoRenderer.Create
 0001:0005A66C       TBCBaseVideoRenderer.Destroy
 0001:0005B540       TBCBaseVideoRenderer.GetStdDev
 0001:0005B310       TBCBaseVideoRenderer.get_AvgFrameRate
 0001:0005B428       TBCBaseVideoRenderer.get_AvgSyncOffset
 0001:0005B698       TBCBaseVideoRenderer.get_DevSyncOffset
 0001:0005B2A8       TBCBaseVideoRenderer.get_FramesDrawn
 0001:0005B240       TBCBaseVideoRenderer.get_FramesDroppedInRenderer
 0001:0005B6CC       TBCBaseVideoRenderer.get_Jitter
 0001:0005B77C       TBCBaseVideoRenderer.JoinFilterGraph
 0001:0005B700       TBCBaseVideoRenderer.NonDelegatingQueryInterface
 0001:0005AAF8       TBCBaseVideoRenderer.Notify
 0001:0005A978       TBCBaseVideoRenderer.OnDirectRender
 0001:0005AA28       TBCBaseVideoRenderer.OnRenderEnd
 0001:0005A9D8       TBCBaseVideoRenderer.OnRenderStart
 0001:0005A7FC       TBCBaseVideoRenderer.PreparePerformanceData
 0001:0005A80C       TBCBaseVideoRenderer.RecordFrameLateness
 0001:0005A6FC       TBCBaseVideoRenderer.ResetStreamingTimes
 0001:0005B1E4       TBCBaseVideoRenderer.ScheduleSample
 0001:0005AB6C       TBCBaseVideoRenderer.SendQuality
 0001:0005AAA4       TBCBaseVideoRenderer.SetSink
 0001:0005ADB4       TBCBaseVideoRenderer.ShouldDrawSampleNow
 0001:0005A940       TBCBaseVideoRenderer.ThrottleWait
 0001:00052890       TBCClassFactory.CreateFilter
 0001:00052944       TBCClassFactory.CreateInstance
 0001:00052E60       TBCClassFactory.LockServer
 0001:00052EA0       TBCClassFactory.QueryInterface
 0001:00052B78       TBCClassFactory.RegisterFilter
 0001:00052D60       TBCClassFactory.RegisterFilter
 0001:000529C8       TBCClassFactory.UpdateRegistry
 0001:00052E38       TBCClassFactory._AddRef
 0001:00052E4C       TBCClassFactory._Release
 0001:000562B4       TBCCritSec.Create
 0001:000562EC       TBCCritSec.CritCheckIn
 0001:000562F0       TBCCritSec.Destroy
 0001:00056314       TBCCritSec.Lock
 0001:00056320       TBCCritSec.UnLock
 0001:0005558C       TBCEnumMediaTypes.AreWeOutOfSync
 0001:000555A4       TBCEnumMediaTypes.Clone
 0001:00055608       TBCEnumMediaTypes.Create
 0001:000556D8       TBCEnumMediaTypes.Destroy
 0001:00055708       TBCEnumMediaTypes.Next
 0001:00055810       TBCEnumMediaTypes.Reset
 0001:00055830       TBCEnumMediaTypes.Skip
 0001:00054360       TBCEnumPins.AreWeOutOfSync
 0001:000540F4       TBCEnumPins.Clone
 0001:00053F68       TBCEnumPins.Create
 0001:000540BC       TBCEnumPins.Destroy
 0001:00054158       TBCEnumPins.Next
 0001:00054334       TBCEnumPins.Refresh
 0001:00054300       TBCEnumPins.Reset
 0001:000542C4       TBCEnumPins.Skip
 0001:00052EC8       TBCFilterTemplate.AddObjectFactory
 0001:00052ED4       TBCFilterTemplate.Create
 0001:00052EFC       TBCFilterTemplate.Destroy
 0001:00052F40       TBCFilterTemplate.GetFactoryFromClassID
 0001:00052F70       TBCFilterTemplate.RegisterServer
 0001:000568B4       TBCMediaPosition.Create
 0001:00056950       TBCMediaPosition.Destroy
 0001:00056980       TBCMediaPosition.GetIDsOfNames
 0001:000569AC       TBCMediaPosition.GetTypeInfo
 0001:000569D4       TBCMediaPosition.GetTypeInfoCount
 0001:000569EC       TBCMediaPosition.Invoke
 0001:00052728       TBCMediaType.InitMediaType
 0001:000526F4       TBCMediaType.IsPartiallySpecified
 0001:00052650       TBCMediaType.MatchesPartial
 0001:00056A8C       TBCPosPassThru.CheckCapabilities
 0001:00056AF8       TBCPosPassThru.ConvertTimeFormat
 0001:00056B70       TBCPosPassThru.Create
 0001:00056C80       TBCPosPassThru.GetAvailable
 0001:00056CF0       TBCPosPassThru.GetCapabilities
 0001:00056D5C       TBCPosPassThru.GetCurrentPosition
 0001:00056DEC       TBCPosPassThru.GetDuration
 0001:00056E58       TBCPosPassThru.GetMediaTime
 0001:00056E60       TBCPosPassThru.GetPeerSeeking
 0001:00056F14       TBCPosPassThru.GetPositions
 0001:00056F84       TBCPosPassThru.GetPreroll
 0001:00056FF0       TBCPosPassThru.GetRate
 0001:0005705C       TBCPosPassThru.GetStopPosition
 0001:000570C8       TBCPosPassThru.GetTimeFormat
 0001:00057134       TBCPosPassThru.IsFormatSupported
 0001:000571A0       TBCPosPassThru.IsUsingTimeFormat
 0001:0005720C       TBCPosPassThru.QueryPreferredFormat
 0001:00057278       TBCPosPassThru.SetPositions
 0001:000572F0       TBCPosPassThru.SetRate
 0001:00057374       TBCPosPassThru.SetTimeFormat
 0001:0005A560       TBCRendererInputPin.Active
 0001:0005A158       TBCRendererInputPin.BeginFlush
 0001:0005A490       TBCRendererInputPin.BreakConnect
 0001:0005A550       TBCRendererInputPin.CheckMediaType
 0001:0005A4C0       TBCRendererInputPin.CompleteConnect
 0001:00059F7C       TBCRendererInputPin.Create
 0001:0005A224       TBCRendererInputPin.EndFlush
 0001:0005A098       TBCRendererInputPin.EndOfStream
 0001:0005A570       TBCRendererInputPin.Inactive
 0001:0005A440       TBCRendererInputPin.InheritedReceive
 0001:0005A530       TBCRendererInputPin.QueryId
 0001:0005A2CC       TBCRendererInputPin.Receive
 0001:0005A584       TBCRendererInputPin.SetMediaType
 0001:000573E0       TBCRendererPosPassThru.Create
 0001:000574B4       TBCRendererPosPassThru.destroy
 0001:000574E4       TBCRendererPosPassThru.EOS
 0001:0005757C       TBCRendererPosPassThru.GetMediaTime
 0001:0005762C       TBCRendererPosPassThru.RegisterMediaTime
 0001:00057784       TBCRendererPosPassThru.ResetMediaTime
 0001:00053234       TBCUnknown.Create
 0001:000532C0       TBCUnknown.CreateFromFactory
 0001:00053220       TBCUnknown.GetOwner
 0001:000531E4       TBCUnknown.NonDelegatingAddRef
 0001:000531BC       TBCUnknown.NonDelegatingQueryInterface
 0001:000531F8       TBCUnknown.NonDelegatingRelease
 0001:00053148       TBCUnknown.QueryInterface
 0001:00053174       TBCUnknown._AddRef
 0001:00053198       TBCUnknown._Release
 0001:000223C0       TBitmap.Assign
 0001:0002259C       TBitmap.Changed
 0001:00022578       TBitmap.Changing
 0001:000224B8       TBitmap.CopyImage
 0001:0002231C       TBitmap.Create
 0001:00022384       TBitmap.Destroy
 0001:00022A28       TBitmap.DIBNeeded
 0001:000225A8       TBitmap.Dormant
 0001:0002261C       TBitmap.Draw
 0001:00022A9C       TBitmap.FreeContext
 0001:0002286C       TBitmap.FreeImage
 0001:000228EC       TBitmap.GetCanvas
 0001:000228D0       TBitmap.GetEmpty
 0001:00022934       TBitmap.GetHandle
 0001:00022958       TBitmap.GetHandleType
 0001:00022984       TBitmap.GetHeight
 0001:00022994       TBitmap.GetMaskHandle
 0001:000229A8       TBitmap.GetMonochrome
 0001:000229C4       TBitmap.GetPalette
 0001:000229D8       TBitmap.GetTransparentColor
 0001:00022A20       TBitmap.GetWidth
 0001:00022AAC       TBitmap.HandleNeeded
 0001:00022C64       TBitmap.LoadFromClipboardFormat
 0001:00022CE8       TBitmap.LoadFromStream
 0001:00022B4C       TBitmap.MaskHandleNeeded
 0001:00022D0C       TBitmap.NewImage
 0001:00022BAC       TBitmap.PaletteNeeded
 0001:00022E0C       TBitmap.ReadData
 0001:00022E34       TBitmap.ReadDIB
 0001:0002339C       TBitmap.ReadStream
 0001:00023ACC       TBitmap.SaveToClipboardFormat
 0001:00023AC4       TBitmap.SaveToStream
 0001:0002340C       TBitmap.SetHandle
 0001:000234D0       TBitmap.SetHandleType
 0001:00023608       TBitmap.SetHeight
 0001:0002365C       TBitmap.SetMonochrome
 0001:000236DC       TBitmap.SetPalette
 0001:000237B0       TBitmap.SetWidth
 0001:00023804       TBitmap.WriteData
 0001:0002380C       TBitmap.WriteStream
 0001:00021680       TBitmapCanvas.Create
 0001:00021788       TBitmapCanvas.CreateHandle
 0001:000216BC       TBitmapCanvas.Destroy
 0001:000216E8       TBitmapCanvas.FreeContext
 0001:00021898       TBitmapImage.Destroy
 0001:000218F4       TBitmapImage.FreeHandle
 0001:00016700       TBits.Destroy
 0001:00016730       TBits.Error
 0001:00016824       TBits.OpenBit
 0001:000167F8       TBits.SetBit
 0001:00016754       TBits.SetSize
 0001:0001F438       TBrush.Assign
 0001:0001F3D0       TBrush.Create
 0001:0001F410       TBrush.Destroy
 0001:0001F570       TBrush.GetColor
 0001:0001F4E0       TBrush.GetData
 0001:0001F5AC       TBrush.GetHandle
 0001:0001F68C       TBrush.GetStyle
 0001:0001F54C       TBrush.SetBitmap
 0001:0001F578       TBrush.SetColor
 0001:0001F4FC       TBrush.SetData
 0001:0001F694       TBrush.SetStyle
 0001:0001FE8C       TCanvas.BrushChanged
 0001:0001FD60       TCanvas.Changed
 0001:0001FD4C       TCanvas.Changing
 0001:0001F7E8       TCanvas.CopyRect
 0001:0001F6C8       TCanvas.Create
 0001:0001FDD0       TCanvas.CreateBrush
 0001:0001FD74       TCanvas.CreateFont
 0001:0001FC80       TCanvas.CreateHandle
 0001:0001FDA0       TCanvas.CreatePen
 0001:0001FC24       TCanvas.DeselectHandles
 0001:0001F78C       TCanvas.Destroy
 0001:0001F870       TCanvas.Draw
 0001:0001F91C       TCanvas.FillRect
 0001:0001FE4C       TCanvas.FontChanged
 0001:0001FC04       TCanvas.GetHandle
 0001:0001FB4C       TCanvas.GetPenPos
 0001:0001FB90       TCanvas.GetPixel
 0001:0001F958       TCanvas.LineTo
 0001:0001F990       TCanvas.Lock
 0001:0001F9B8       TCanvas.MoveTo
 0001:0001FE6C       TCanvas.PenChanged
 0001:0001FCD8       TCanvas.RequiredState
 0001:0001FB40       TCanvas.SetBrush
 0001:0001FB24       TCanvas.SetFont
 0001:0001FC84       TCanvas.SetHandle
 0001:0001FB34       TCanvas.SetPen
 0001:0001FB70       TCanvas.SetPenPos
 0001:0001FBBC       TCanvas.SetPixel
 0001:0001F9E4       TCanvas.StretchDraw
 0001:0001FA20       TCanvas.TextExtent
 0001:0001FA80       TCanvas.TextHeight
 0001:0001FA64       TCanvas.TextWidth
 0001:0001FAA0       TCanvas.TryLock
 0001:0001FAFC       TCanvas.Unlock
 0001:0003CB18       TChangeLink.Change
 0001:0003CAE4       TChangeLink.Destroy
 0001:000157D4       TClassFinder.Create
 0001:00015900       TClassFinder.Destroy
 0001:00015930       TClassFinder.GetClass
 0001:00016B24       TCollection.Add
 0001:00016B44       TCollection.Clear
 0001:000273E4       TCommonDialog.Create
 0001:00027488       TCommonDialog.DefaultHandler
 0001:0002742C       TCommonDialog.Destroy
 0001:0002762C       TCommonDialog.DoClose
 0001:00027640       TCommonDialog.DoShow
 0001:000274C0       TCommonDialog.MainWndProc
 0001:00027460       TCommonDialog.MessageHook
 0001:00027558       TCommonDialog.TaskModalDialog
 0001:00027514       TCommonDialog.WMDestroy
 0001:0002752C       TCommonDialog.WMInitDialog
 0001:00027544       TCommonDialog.WMNCDestroy
 0001:0002750C       TCommonDialog.WndProc
 0001:0001BD88       TComponent.BeforeDestruction
 0001:0001C2A8       TComponent.ChangeName
 0001:0001BCC4       TComponent.Create
 0001:0001C03C       TComponent.DefineProperties
 0001:0001BD10       TComponent.Destroy
 0001:0001BF0C       TComponent.DestroyComponents
 0001:0001BF64       TComponent.Destroying
 0001:0001C3E4       TComponent.ExecuteAction
 0001:0001C1CC       TComponent.FindComponent
 0001:0001BD94       TComponent.FreeNotification
 0001:0001C0D0       TComponent.GetChildOwner
 0001:0001C0D4       TComponent.GetChildParent
 0001:0001C0C8       TComponent.GetChildren
 0001:0001C2BC       TComponent.GetComponent
 0001:0001C2E8       TComponent.GetComponentCount
 0001:0001C0D8       TComponent.GetNamePath
 0001:0001C0EC       TComponent.GetOwner
 0001:0001C0F4       TComponent.GetParentComponent
 0001:0001C0C4       TComponent.HasParent
 0001:0001BE28       TComponent.Insert
 0001:0001BE7C       TComponent.InsertComponent
 0001:0001C4D4       TComponent.IntfGetComponent
 0001:0001C114       TComponent.Loaded
 0001:0001BFE0       TComponent.Notification
 0001:0001C120       TComponent.PaletteCreated
 0001:0001C454       TComponent.QueryInterface
 0001:0001BDE8       TComponent.ReadLeft
 0001:0001C124       TComponent.ReadState
 0001:0001BDFC       TComponent.ReadTop
 0001:0001BE54       TComponent.Remove
 0001:0001BED4       TComponent.RemoveComponent
 0001:0001BFC4       TComponent.RemoveFreeNotification
 0001:0001BFA0       TComponent.RemoveNotification
 0001:0001C434       TComponent.SafeCallException
 0001:0001C0F0       TComponent.SetChildOrder
 0001:0001C2F8       TComponent.SetComponentIndex
 0001:0001C34C       TComponent.SetDesigning
 0001:0001C21C       TComponent.SetName
 0001:0001C0F8       TComponent.SetParentComponent
 0001:0001C39C       TComponent.SetReference
 0001:0001C40C       TComponent.UpdateAction
 0001:0001C108       TComponent.Updated
 0001:0001C44C       TComponent.UpdateRegistry
 0001:0001C0FC       TComponent.Updating
 0001:0001C1B4       TComponent.ValidateContainer
 0001:0001C1C8       TComponent.ValidateInsert
 0001:0001C134       TComponent.ValidateRename
 0001:0001BE10       TComponent.WriteLeft
 0001:0001C12C       TComponent.WriteState
 0001:0001BE1C       TComponent.WriteTop
 0001:0001C494       TComponent._AddRef
 0001:0001C4B4       TComponent._Release
 0001:0003A6E4       TContainedAction.Destroy
 0001:0003A850       TContainedAction.Execute
 0001:0003A718       TContainedAction.GetIndex
 0001:0003A734       TContainedAction.GetParentComponent
 0001:0003A744       TContainedAction.HasParent
 0001:0003A730       TContainedAction.IsCategoryStored
 0001:0003A754       TContainedAction.ReadState
 0001:0003A7FC       TContainedAction.SetActionList
 0001:0003A7D0       TContainedAction.SetCategory
 0001:0003A788       TContainedAction.SetIndex
 0001:0003A824       TContainedAction.SetParentComponent
 0001:0003A8A8       TContainedAction.Update
 0001:00030C10       TControl.ActionChange
 0001:00030FBC       TControl.AdjustSize
 0001:00030DF0       TControl.AssignTo
 0001:0002F3CC       TControl.BeginAutoDrag
 0001:0002F3E4       TControl.BeginDrag
 0001:0002EFA8       TControl.BringToFront
 0001:0002FDBC       TControl.CalcCursorPos
 0001:0002FF24       TControl.CalcDockSizes
 0001:0002FCBC       TControl.CanAutoSize
 0001:0002FCC0       TControl.CanResize
 0001:0002E990       TControl.ChangeScale
 0001:00030480       TControl.CheckNewSize
 0001:00030278       TControl.Click
 0001:0002E89C       TControl.ClientToScreen
 0001:000309C4       TControl.CMBiDiModeChanged
 0001:0003090C       TControl.CMColorChanged
 0001:00030A98       TControl.CMDesignHitTest
 0001:000308FC       TControl.CMEnabledChanged
 0001:00030BB0       TControl.CMFloat
 0001:00030904       TControl.CMFontChanged
 0001:00031008       TControl.CMHintShow
 0001:00030A60       TControl.CMHitTest
 0001:00030A68       TControl.CMMouseEnter
 0001:00030A80       TControl.CMMouseLeave
 0001:00030968       TControl.CMMouseWheel
 0001:00030944       TControl.CMParentBiDiModeChanged
 0001:00030914       TControl.CMParentColorChanged
 0001:00030A0C       TControl.CMParentFontChanged
 0001:000309E4       TControl.CMParentShowHintChanged
 0001:00030A3C       TControl.CMSysFontChanged
 0001:000308D4       TControl.CMVisibleChanged
 0001:0002FD8C       TControl.ConstrainedResize
 0001:0002DE84       TControl.Create
 0001:00030AA0       TControl.CreateFloatingDockSite
 0001:000302E4       TControl.DblClick
 0001:0002F7F8       TControl.DefaultDockImage
 0001:00030150       TControl.DefaultHandler
 0001:00030228       TControl.DefineProperties
 0001:0002FDE8       TControl.DesignWndProc
 0001:0002DF5C       TControl.Destroy
 0001:00030D0C       TControl.DoActionChange
 0001:0002FCF0       TControl.DoCanAutoSize
 0001:0002FD5C       TControl.DoCanResize
 0001:0002E588       TControl.Dock
 0001:0002F63C       TControl.DockTrackNoTarget
 0001:0002FE1C       TControl.DoConstrainedResize
 0001:0002FCB0       TControl.DoConstraintsChange
 0001:0003115C       TControl.DoContextPopup
 0001:0002E694       TControl.DoDock
 0001:0002F94C       TControl.DoDragMsg
 0001:0002F650       TControl.DoEndDock
 0001:0002F540       TControl.DoEndDrag
 0001:0003033C       TControl.DoMouseDown
 0001:0003069C       TControl.DoMouseUp
 0001:0002F69C       TControl.DoMouseWheel
 0001:0002F760       TControl.DoMouseWheelDown
 0001:0002F7AC       TControl.DoMouseWheelUp
 0001:0002F67C       TControl.DoStartDock
 0001:0002F520       TControl.DoStartDrag
 0001:0002F4A8       TControl.DragCanceled
 0001:0002F4F4       TControl.DragDrop
 0001:0002F4AC       TControl.Dragging
 0001:0002F4B8       TControl.DragOver
 0001:0002F924       TControl.DrawDragDockImage
 0001:00030FDC       TControl.DrawTextBiDiModeFlagsReadingOnly
 0001:0002F938       TControl.EraseDragDockImage
 0001:0002EE24       TControl.FontChanged
 0001:0002E0C8       TControl.GetAction
 0001:00030D30       TControl.GetActionLinkClass
 0001:0002E724       TControl.GetBoundsRect
 0001:0002E7CC       TControl.GetClientHeight
 0001:0002E80C       TControl.GetClientOrigin
 0001:0002E770       TControl.GetClientRect
 0001:0002E788       TControl.GetClientWidth
 0001:0002F37C       TControl.GetControlsAlignment
 0001:0002F05C       TControl.GetDeviceContext
 0001:00030ED8       TControl.GetDockEdge
 0001:0002E010       TControl.GetDragImages
 0001:0002E014       TControl.GetEnabled
 0001:00030F88       TControl.GetFloating
 0001:00030FB4       TControl.GetFloatingDockSiteClass
 0001:0002EF70       TControl.GetMouseCapture
 0001:0002E018       TControl.GetPalette
 0001:0002E024       TControl.GetParentComponent
 0001:0003047C       TControl.GetPopupMenu
 0001:0002ED74       TControl.GetText
 0001:0002ECF8       TControl.GetTextBuf
 0001:0002ECE8       TControl.GetTextLen
 0001:0002ED04       TControl.GetUndockHeight
 0001:0002ED18       TControl.GetUndockWidth
 0001:0002E01C       TControl.HasParent
 0001:00030FF8       TControl.InitiateAction
 0001:0002F21C       TControl.Invalidate
 0001:0002F190       TControl.InvalidateControl
 0001:0002E174       TControl.IsAnchorsStored
 0001:0002EE98       TControl.IsBiDiModeStored
 0001:0002EF04       TControl.IsColorStored
 0001:00030D38       TControl.IsEnabledStored
 0001:0002EE78       TControl.IsFontStored
 0001:00030D78       TControl.IsHelpContextStored
 0001:00030D58       TControl.IsHintStored
 0001:0002EE8C       TControl.IsShowHintStored
 0001:00030D98       TControl.IsVisibleStored
 0001:00030DB8       TControl.Loaded
 0001:0002FA3C       TControl.ManualDock
 0001:0002FC1C       TControl.ManualFloat
 0001:00030304       TControl.MouseDown
 0001:000305BC       TControl.MouseMove
 0001:00030664       TControl.MouseUp
 0001:0002F22C       TControl.MouseWheelHandler
 0001:0002E254       TControl.Notification
 0001:0002E050       TControl.PaletteChanged
 0001:0002FEF0       TControl.Perform
 0001:0002F56C       TControl.PositionDockRect
 0001:000301D8       TControl.ReadIsControl
 0001:0002E1C0       TControl.ReadState
 0001:0002F284       TControl.Repaint
 0001:0002E190       TControl.RequestAlign
 0001:0002E1A0       TControl.Resize
 0001:0002E8C8       TControl.ScreenToClient
 0001:0002E8F4       TControl.SendCancelMode
 0001:0002E924       TControl.SendDockNotification
 0001:0002E0F8       TControl.SetAction
 0001:0002E298       TControl.SetAlign
 0001:0002E0D8       TControl.SetAnchors
 0001:0002EB44       TControl.SetAutoSize
 0001:0002EE08       TControl.SetBiDiMode
 0001:0002E340       TControl.SetBounds
 0001:0002E744       TControl.SetBoundsRect
 0001:0002E7E4       TControl.SetClientHeight
 0001:0002EC00       TControl.SetClientSize
 0001:0002E7A0       TControl.SetClientWidth
 0001:0002EEE8       TControl.SetColor
 0001:00031190       TControl.SetConstraints
 0001:0002EF54       TControl.SetCursor
 0001:0002E18C       TControl.SetDragMode
 0001:0002ECD0       TControl.SetEnabled
 0001:0002EE68       TControl.SetFont
 0001:0002E564       TControl.SetHeight
 0001:0002E6EC       TControl.SetHelpContext
 0001:0002E700       TControl.SetHelpKeyword
 0001:0002E4F4       TControl.SetLeft
 0001:0002EF80       TControl.SetMouseCapture
 0001:0002EB5C       TControl.SetName
 0001:0002EC48       TControl.SetParent
 0001:0002EF30       TControl.SetParentBiDiMode
 0001:0002EF0C       TControl.SetParentColor
 0001:0002E028       TControl.SetParentComponent
 0001:0002EEA0       TControl.SetParentFont
 0001:0002ED2C       TControl.SetPopupMenu
 0001:0002EEC4       TControl.SetShowHint
 0001:0002EDA4       TControl.SetText
 0001:0002ED50       TControl.SetTextBuf
 0001:0002E518       TControl.SetTop
 0001:0002EC94       TControl.SetVisible
 0001:0002E540       TControl.SetWidth
 0001:0002F038       TControl.SetZOrder
 0001:0002EFB8       TControl.SetZOrderPosition
 0001:0002F270       TControl.Update
 0001:0002E3D8       TControl.UpdateAnchorRules
 0001:0002FF94       TControl.UpdateBoundsRect
 0001:0002F398       TControl.UseRightToLeftAlignment
 0001:0002F380       TControl.UseRightToLeftReading
 0001:0002F3B0       TControl.UseRightToLeftScrollBar
 0001:0002FFB8       TControl.VisibleChanging
 0001:000307E4       TControl.WMCancelMode
 0001:00031034       TControl.WMContextMenu
 0001:00030428       TControl.WMLButtonDblClk
 0001:000303C0       TControl.WMLButtonDown
 0001:000306D4       TControl.WMLButtonUp
 0001:00030594       TControl.WMMButtonDblClk
 0001:0003056C       TControl.WMMButtonDown
 0001:0003076C       TControl.WMMButtonUp
 0001:000305EC       TControl.WMMouseMove
 0001:0003078C       TControl.WMMouseWheel
 0001:0003040C       TControl.WMNCLButtonDown
 0001:00030544       TControl.WMRButtonDblClk
 0001:0003051C       TControl.WMRButtonDown
 0001:0003074C       TControl.WMRButtonUp
 0001:00030824       TControl.WMWindowPosChanged
 0001:0002FFBC       TControl.WndProc
 0001:000301EC       TControl.WriteIsControl
 0001:0002DAC8       TControlActionLink.AssignClient
 0001:0002DAE4       TControlActionLink.DoShowHint
 0001:0002DBD4       TControlActionLink.IsCaptionLinked
 0001:0002DC48       TControlActionLink.IsEnabledLinked
 0001:0002DDC0       TControlActionLink.IsHelpLinked
 0001:0002DC7C       TControlActionLink.IsHintLinked
 0001:0002DCE8       TControlActionLink.IsOnExecuteLinked
 0001:0002DCB4       TControlActionLink.IsVisibleLinked
 0001:0002DD10       TControlActionLink.SetCaption
 0001:0002DD30       TControlActionLink.SetEnabled
 0001:0002DE44       TControlActionLink.SetHelpContext
 0001:0002DE24       TControlActionLink.SetHelpKeyword
 0001:0002DE64       TControlActionLink.SetHelpType
 0001:0002DD50       TControlActionLink.SetHint
 0001:0002DD94       TControlActionLink.SetOnExecute
 0001:0002DD74       TControlActionLink.SetVisible
 0001:0002D884       TControlCanvas.CreateHandle
 0001:0002D858       TControlCanvas.Destroy
 0001:0002D92C       TControlCanvas.FreeHandle
 0001:0002D960       TControlCanvas.SetControl
 0001:0002D978       TControlCanvas.UpdateTextFlags
 0001:000455A4       TControlScrollBar.Assign
 0001:00045700       TControlScrollBar.CalcAutoRange
 0001:000455F4       TControlScrollBar.ChangeBiDiPosition
 0001:00045894       TControlScrollBar.ControlSize
 0001:00045514       TControlScrollBar.Create
 0001:00045E3C       TControlScrollBar.DoSetRange
 0001:0004559C       TControlScrollBar.IsIncrementStored
 0001:00045E68       TControlScrollBar.IsRangeStored
 0001:000457AC       TControlScrollBar.IsScrollBarVisible
 0001:00045914       TControlScrollBar.NeedsScrollBarVisible
 0001:0004598C       TControlScrollBar.ScrollMessage
 0001:00045C8C       TControlScrollBar.SetButtonSize
 0001:00045CD0       TControlScrollBar.SetColor
 0001:00045CEC       TControlScrollBar.SetParentColor
 0001:00045D04       TControlScrollBar.SetPosition
 0001:00045E54       TControlScrollBar.SetRange
 0001:00045DC8       TControlScrollBar.SetSize
 0001:00045E0C       TControlScrollBar.SetStyle
 0001:00045E24       TControlScrollBar.SetThumbSize
 0001:00045E74       TControlScrollBar.SetVisible
 0001:00045F88       TControlScrollBar.Update
 0001:00028414       TConversion.ConvertReadStream
 0001:00028428       TConversion.ConvertWriteStream
 0001:00026664       TCriticalSection.Acquire
 0001:000265F4       TCriticalSection.Create
 0001:00026634       TCriticalSection.Destroy
 0001:0002667C       TCriticalSection.Enter
 0001:00026684       TCriticalSection.Leave
 0001:00026670       TCriticalSection.Release
 0001:0003ADE4       TCustomAction.AssignTo
 0001:0003AD40       TCustomAction.Create
 0001:0003AD94       TCustomAction.Destroy
 0001:0003B2FC       TCustomAction.DoHint
 0001:0003B324       TCustomAction.Execute
 0001:0003B384       TCustomAction.GetSecondaryShortCuts
 0001:0003B3AC       TCustomAction.HandleShortCut
 0001:0003AE90       TCustomAction.SetCaption
 0001:0003AEF0       TCustomAction.SetChecked
 0001:0003AFF8       TCustomAction.SetEnabled
 0001:0003B0D8       TCustomAction.SetHelpContext
 0001:0003B070       TCustomAction.SetHelpKeyword
 0001:0003B130       TCustomAction.SetHint
 0001:0003B190       TCustomAction.SetImageIndex
 0001:0003B2B0       TCustomAction.SetName
 0001:0003B1EC       TCustomAction.SetShortCut
 0001:0003B250       TCustomAction.SetVisible
 0001:0003AAD8       TCustomActionList.AddAction
 0001:0003AB14       TCustomActionList.Change
 0001:0003A900       TCustomActionList.Create
 0001:0003A96C       TCustomActionList.Destroy
 0001:0003AC08       TCustomActionList.ExecuteAction
 0001:0003AA34       TCustomActionList.GetAction
 0001:0003AA48       TCustomActionList.GetActionCount
 0001:0003A9BC       TCustomActionList.GetChildren
 0001:0003AA84       TCustomActionList.ImageListChange
 0001:0003AB7C       TCustomActionList.IsShortCut
 0001:0003AA90       TCustomActionList.Notification
 0001:0003AAF8       TCustomActionList.RemoveAction
 0001:0003AA04       TCustomActionList.SetChildOrder
 0001:0003AA50       TCustomActionList.SetImages
 0001:0003AC28       TCustomActionList.UpdateAction
 0001:00036DD8       TCustomControl.Create
 0001:00036E34       TCustomControl.Destroy
 0001:00036F30       TCustomControl.Paint
 0001:00036E84       TCustomControl.PaintWindow
 0001:00036E64       TCustomControl.WMPaint
 0001:0004B828       TCustomDockForm.CMControlListChange
 0001:0004B880       TCustomDockForm.CMDockNotification
 0001:0004B954       TCustomDockForm.CMUnDockClient
 0001:0004B96C       TCustomDockForm.CMVisibleChanged
 0001:0004B588       TCustomDockForm.Create
 0001:0004B5EC       TCustomDockForm.DoAddDockClient
 0001:0004B6D0       TCustomDockForm.DoRemoveDockClient
 0001:0004B73C       TCustomDockForm.GetSiteInfo
 0001:0004B6F0       TCustomDockForm.Loaded
 0001:0004B768       TCustomDockForm.WMNCHitTest
 0001:0004B790       TCustomDockForm.WMNCLButtonDown
 0001:000496A8       TCustomForm.Activate
 0001:000494AC       TCustomForm.ActiveChanged
 0001:00046A5C       TCustomForm.AfterConstruction
 0001:00047EEC       TCustomForm.AlignControls
 0001:00046C10       TCustomForm.BeforeDestruction
 0001:0004733C       TCustomForm.BeginAutoDrag
 0001:00047340       TCustomForm.ChangeScale
 0001:00047D0C       TCustomForm.ClientWndProc
 0001:0004AA98       TCustomForm.Close
 0001:0004ABA0       TCustomForm.CloseModal
 0001:0004AB3C       TCustomForm.CloseQuery
 0001:0004B18C       TCustomForm.CMActionExecute
 0001:0004B28C       TCustomForm.CMActionUpdate
 0001:0004A324       TCustomForm.CMActivate
 0001:00049DA4       TCustomForm.CMAppSysCommand
 0001:00047F58       TCustomForm.CMBiDiModeChanged
 0001:0004875C       TCustomForm.CMColorChanged
 0001:00048798       TCustomForm.CMCtl3DChanged
 0001:0004A348       TCustomForm.CMDeactivate
 0001:0004A36C       TCustomForm.CMDialogKey
 0001:000487E0       TCustomForm.CMFontChanged
 0001:0004A980       TCustomForm.CMIconChanged
 0001:0004AA6C       TCustomForm.CMIsShortCut
 0001:00048800       TCustomForm.CMMenuChanged
 0001:00047FF0       TCustomForm.CMParentBiDiModeChanged
 0001:0004AA00       TCustomForm.CMParentFontChanged
 0001:0004A9A0       TCustomForm.CMRelease
 0001:0004A408       TCustomForm.CMShowingChanged
 0001:0004A9A8       TCustomForm.CMTextChanged
 0001:0004A9F8       TCustomForm.CMUIActivate
 0001:000468D0       TCustomForm.Create
 0001:00046A94       TCustomForm.CreateNew
 0001:00048BB0       TCustomForm.CreateParams
 0001:00048F10       TCustomForm.CreateWindowHandle
 0001:00048DCC       TCustomForm.CreateWnd
 0001:000496D8       TCustomForm.Deactivate
 0001:0004908C       TCustomForm.DefaultHandler
 0001:000471F8       TCustomForm.DefineProperties
 0001:000491A8       TCustomForm.DefocusControl
 0001:00046C78       TCustomForm.Destroy
 0001:00049048       TCustomForm.DestroyWindowHandle
 0001:000480DC       TCustomForm.Dock
 0001:00047488       TCustomForm.DoClose
 0001:00046D5C       TCustomForm.DoCreate
 0001:00046DD8       TCustomForm.DoDestroy
 0001:00048120       TCustomForm.DoDock
 0001:000474A8       TCustomForm.DoHide
 0001:000474C8       TCustomForm.DoShow
 0001:000491F0       TCustomForm.FocusControl
 0001:00048174       TCustomForm.GetActiveMDIChild
 0001:0004835C       TCustomForm.GetCanvas
 0001:00047570       TCustomForm.GetChildren
 0001:000474E8       TCustomForm.GetClientRect
 0001:000475DC       TCustomForm.GetFloating
 0001:00049728       TCustomForm.GetIconHandle
 0001:000481A8       TCustomForm.GetMDIChildCount
 0001:000481F4       TCustomForm.GetMDIChildren
 0001:00048274       TCustomForm.GetMonitor
 0001:000486BC       TCustomForm.GetPixelsPerInch
 0001:00048720       TCustomForm.GetScaled
 0001:00047318       TCustomForm.GetTextHeight
 0001:0004B424       TCustomForm.HandleCreateException
 0001:0004AC38       TCustomForm.Hide
 0001:000473C0       TCustomForm.IconChanged
 0001:0004B55C       TCustomForm.InitAlphaBlending
 0001:00047454       TCustomForm.IsAutoScrollStored
 0001:0004741C       TCustomForm.IsClientSizeStored
 0001:00048370       TCustomForm.IsForm
 0001:0004742C       TCustomForm.IsFormSizeStored
 0001:00048378       TCustomForm.IsIconStored
 0001:0004B334       TCustomForm.IsShortCut
 0001:00046E38       TCustomForm.Loaded
 0001:000495B4       TCustomForm.MergeMenu
 0001:0004B3EC       TCustomForm.MouseWheelHandler
 0001:00048780       TCustomForm.NormalColor
 0001:00046E74       TCustomForm.Notification
 0001:00049708       TCustomForm.Paint
 0001:00049744       TCustomForm.PaintWindow
 0001:00049800       TCustomForm.PaletteChanged
 0001:0004B3B0       TCustomForm.QueryInterface
 0001:000472A8       TCustomForm.ReadIgnoreFontProperty
 0001:00046F80       TCustomForm.ReadState
 0001:000472C8       TCustomForm.ReadTextHeight
 0001:00048420       TCustomForm.RefreshMDIMenu
 0001:0004ACD4       TCustomForm.Release
 0001:0004B0A0       TCustomForm.RequestAlign
 0001:00049D38       TCustomForm.Resizing
 0001:00049564       TCustomForm.SendCancelMode
 0001:00049500       TCustomForm.SetActive
 0001:000490F0       TCustomForm.SetActiveControl
 0001:0004B50C       TCustomForm.SetAlphaBlend
 0001:0004B520       TCustomForm.SetAlphaBlendValue
 0001:00048078       TCustomForm.SetBorderIcons
 0001:000480A4       TCustomForm.SetBorderStyle
 0001:00047608       TCustomForm.SetChildOrder
 0001:000476F4       TCustomForm.SetClientHeight
 0001:000476C4       TCustomForm.SetClientWidth
 0001:0004AC58       TCustomForm.SetFocus
 0001:00049214       TCustomForm.SetFocusedControl
 0001:000483A0       TCustomForm.SetFormStyle
 0001:00048364       TCustomForm.SetIcon
 0001:0004B434       TCustomForm.SetLayeredAttribs
 0001:000484E8       TCustomForm.SetMenu
 0001:0004849C       TCustomForm.SetObjectMenuItem
 0001:000477D0       TCustomForm.SetParent
 0001:0004769C       TCustomForm.SetParentBiDiMode
 0001:000486D0       TCustomForm.SetPixelsPerInch
 0001:00048704       TCustomForm.SetPosition
 0001:0004872C       TCustomForm.SetScaled
 0001:0004B548       TCustomForm.SetTransparentColor
 0001:0004B534       TCustomForm.SetTransparentColorValue
 0001:00047724       TCustomForm.SetVisible
 0001:000494B0       TCustomForm.SetWindowFocus
 0001:000484C0       TCustomForm.SetWindowMenu
 0001:0004881C       TCustomForm.SetWindowState
 0001:0004885C       TCustomForm.SetWindowToMonitor
 0001:0004AC40       TCustomForm.Show
 0001:0004ACF0       TCustomForm.ShowModal
 0001:0004B038       TCustomForm.UpdateActions
 0001:00047808       TCustomForm.ValidateRename
 0001:00047768       TCustomForm.VisibleChanging
 0001:000477CC       TCustomForm.WantChildKey
 0001:00049D18       TCustomForm.WMActivate
 0001:00049D70       TCustomForm.WMClose
 0001:00049BEC       TCustomForm.WMCommand
 0001:00049B8C       TCustomForm.WMDestroy
 0001:00049FA4       TCustomForm.WMEnterMenuLoop
 0001:00049980       TCustomForm.WMEraseBkgnd
 0001:0004A1CC       TCustomForm.WMGetMinMaxInfo
 0001:0004A06C       TCustomForm.WMHelp
 0001:00049920       TCustomForm.WMIconEraseBkgnd
 0001:00049C20       TCustomForm.WMInitMenuPopup
 0001:00049F20       TCustomForm.WMMDIActivate
 0001:00049C38       TCustomForm.WMMenuChar
 0001:00049C70       TCustomForm.WMMenuSelect
 0001:00049AC8       TCustomForm.WMNCCreate
 0001:00049AFC       TCustomForm.WMNCLButtonDown
 0001:00049F78       TCustomForm.WMNextDlgCtl
 0001:000498A0       TCustomForm.WMPaint
 0001:000499B8       TCustomForm.WMQueryDragIcon
 0001:00049D78       TCustomForm.WMQueryEndSession
 0001:0004B0BC       TCustomForm.WMSettingChange
 0001:00049E88       TCustomForm.WMShowWindow
 0001:00049DFC       TCustomForm.WMSysCommand
 0001:0004A26C       TCustomForm.WMWindowPosChanging
 0001:00047848       TCustomForm.WndProc
 0001:000472FC       TCustomForm.WritePixelsPerInch
 0001:000472E0       TCustomForm.WriteTextHeight
 0001:0003BA00       TCustomImageList.Add
 0001:0003BFD4       TCustomImageList.AddImages
 0001:0003BFF4       TCustomImageList.Assign
 0001:0003C0B4       TCustomImageList.AssignTo
 0001:0003CAC0       TCustomImageList.BeginUpdate
 0001:0003C204       TCustomImageList.Change
 0001:0003C164       TCustomImageList.CheckImage
 0001:0003BB7C       TCustomImageList.Clear
 0001:0003BE2C       TCustomImageList.CopyImages
 0001:0003B618       TCustomImageList.Create
 0001:0003B960       TCustomImageList.CreateImageList
 0001:0003C43C       TCustomImageList.DefineProperties
 0001:0003BAF0       TCustomImageList.Delete
 0001:0003B664       TCustomImageList.Destroy
 0001:0003BBE8       TCustomImageList.DoDraw
 0001:0003BDBC       TCustomImageList.Draw
 0001:0003BDE0       TCustomImageList.Draw
 0001:0003CAC4       TCustomImageList.EndUpdate
 0001:0003C2F0       TCustomImageList.Equal
 0001:0003B928       TCustomImageList.FreeHandle
 0001:0003BBC0       TCustomImageList.GetBkColor
 0001:0003BACC       TCustomImageList.GetCount
 0001:0003B8C4       TCustomImageList.GetHandle
 0001:0003C1F4       TCustomImageList.GetHotSpot
 0001:0003B8D4       TCustomImageList.GetImageHandle
 0001:0003B788       TCustomImageList.HandleAllocated
 0001:0003B790       TCustomImageList.HandleNeeded
 0001:0003B79C       TCustomImageList.InitBitmap
 0001:0003B6D0       TCustomImageList.Initialize
 0001:0003C494       TCustomImageList.ReadD2Stream
 0001:0003C728       TCustomImageList.ReadD3Stream
 0001:0003C8F0       TCustomImageList.ReadData
 0001:0003C298       TCustomImageList.RegisterChanges
 0001:0003BB88       TCustomImageList.SetBkColor
 0001:0003C1DC       TCustomImageList.SetDrawingStyle
 0001:0003B898       TCustomImageList.SetHandle
 0001:0003B860       TCustomImageList.SetNewDimensions
 0001:0003C254       TCustomImageList.UnRegisterChanges
 0001:0003C97C       TCustomImageList.WriteData
 0001:000185EC       TCustomMemoryStream.Read
 0001:00018624       TCustomMemoryStream.Seek
 0001:000185E4       TCustomMemoryStream.SetPointer
 0001:00012968       TCustomVariantType.BinaryOp
 0001:00012974       TCustomVariantType.Cast
 0001:000129AC       TCustomVariantType.CastTo
 0001:00012A38       TCustomVariantType.CastToOle
 0001:000129F4       TCustomVariantType.Compare
 0001:00012A00       TCustomVariantType.CompareOp
 0001:00012A74       TCustomVariantType.Destroy
 0001:00012B54       TCustomVariantType.DispInvoke
 0001:00012B00       TCustomVariantType.IsClear
 0001:00012B04       TCustomVariantType.LeftPromotion
 0001:00012B18       TCustomVariantType.OlePromotion
 0001:00012B78       TCustomVariantType.QueryInterface
 0001:00012B20       TCustomVariantType.RaiseCastError
 0001:00012B30       TCustomVariantType.RaiseDispError
 0001:00012B28       TCustomVariantType.RaiseInvalidOp
 0001:00012B38       TCustomVariantType.RightPromotion
 0001:00012B4C       TCustomVariantType.UnaryOp
 0001:00012B60       TCustomVariantType._AddRef
 0001:00012B6C       TCustomVariantType._Release
 0001:00037788       TDockTree.AdjustDockRect
 0001:0003779C       TDockTree.BeginUpdate
 0001:00039458       TDockTree.ControlVisibilityChanged
 0001:000375CC       TDockTree.Create
 0001:00037734       TDockTree.Destroy
 0001:00039058       TDockTree.DrawSizeSplitter
 0001:000377A0       TDockTree.EndUpdate
 0001:0003780C       TDockTree.FindControlZone
 0001:00037874       TDockTree.ForEachAt
 0001:0003788C       TDockTree.GetControlBounds
 0001:000391D4       TDockTree.GetNextLimit
 0001:00037900       TDockTree.HitTest
 0001:00037910       TDockTree.InsertControl
 0001:00037B20       TDockTree.InsertNewParent
 0001:00037CC8       TDockTree.InsertSibling
 0001:00038000       TDockTree.InternalHitTest
 0001:000380D0       TDockTree.LoadFromStream
 0001:000383B8       TDockTree.PaintDockFrame
 0001:00038494       TDockTree.PaintSite
 0001:000385F8       TDockTree.PositionDockRect
 0001:000387A0       TDockTree.PruneZone
 0001:000387FC       TDockTree.RemoveControl
 0001:00038838       TDockTree.RemoveZone
 0001:00038AB4       TDockTree.ResetBounds
 0001:00038D00       TDockTree.SaveToStream
 0001:00038B90       TDockTree.ScaleZone
 0001:00038ED0       TDockTree.SetNewBounds
 0001:00038EFC       TDockTree.SetReplacingControl
 0001:00038F14       TDockTree.ShiftZone
 0001:00038F44       TDockTree.SplitterMouseDown
 0001:00038FA4       TDockTree.SplitterMouseUp
 0001:00039020       TDockTree.UpdateAll
 0001:00039048       TDockTree.UpdateZone
 0001:00039570       TDockTree.WindowProc
 0001:00036F74       TDockZone.Create
 0001:000374FC       TDockZone.ExpandZoneLimit
 0001:000375C0       TDockZone.FirstVisibleChild
 0001:00036F98       TDockZone.GetChildCount
 0001:00037250       TDockZone.GetControlName
 0001:000370F8       TDockZone.GetHeightWidth
 0001:00036FFC       TDockZone.GetLimitBegin
 0001:00037044       TDockZone.GetLimitSize
 0001:0003708C       TDockZone.GetTopLeft
 0001:00036FC8       TDockZone.GetVisible
 0001:00036FAC       TDockZone.GetVisibleChildCount
 0001:000374C0       TDockZone.GetZoneLimit
 0001:00037598       TDockZone.NextVisible
 0001:000375A4       TDockZone.PrevVisible
 0001:000371A8       TDockZone.ResetChildren
 0001:00037538       TDockZone.ResetZoneLimits
 0001:00037294       TDockZone.SetControlName
 0001:000374E8       TDockZone.SetZoneLimit
 0001:00037348       TDockZone.Update
 0001:0002C430       TDragControlObject.GetDragCursor
 0001:0002C448       TDragControlObject.GetDragImages
 0001:0002C454       TDragControlObject.HideDragImage
 0001:0002C474       TDragControlObject.ShowDragImage
 0001:0002C494       TDragControlObjectEx.BeforeDestruction
 0001:0002C5D0       TDragDockObject.AdjustDockRect
 0001:0002C52C       TDragDockObject.Assign
 0001:0002C498       TDragDockObject.Create
 0001:0002C4FC       TDragDockObject.Destroy
 0001:0002C64C       TDragDockObject.DrawDragDockImage
 0001:0002C588       TDragDockObject.EndDrag
 0001:0002C660       TDragDockObject.EraseDragDockImage
 0001:0002C674       TDragDockObject.GetDragCursor
 0001:0002C680       TDragDockObject.GetFrameWidth
 0001:0002C688       TDragDockObjectEx.BeforeDestruction
 0001:00036C34       TDragImageList.BeginDrag
 0001:00036B08       TDragImageList.CombineDragCursor
 0001:00036C94       TDragImageList.DragLock
 0001:00036D1C       TDragImageList.DragMove
 0001:00036CF8       TDragImageList.DragUnlock
 0001:00036D90       TDragImageList.EndDrag
 0001:00036D78       TDragImageList.HideDragImage
 0001:00036C1C       TDragImageList.SetDragCursor
 0001:00036BD4       TDragImageList.SetDragImage
 0001:00036D60       TDragImageList.ShowDragImage
 0001:0002C370       TDragObject.AfterConstruction
 0001:0002C150       TDragObject.Assign
 0001:0002C360       TDragObject.BeforeDestruction
 0001:0002C190       TDragObject.Capture
 0001:0002C1A8       TDragObject.Finished
 0001:0002C2EC       TDragObject.GetDragCursor
 0001:0002C2E8       TDragObject.GetDragImages
 0001:0002C1B0       TDragObject.GetName
 0001:0002C304       TDragObject.HideDragImage
 0001:0002C308       TDragObject.Instance
 0001:0002C314       TDragObject.MainWndProc
 0001:0002C1D8       TDragObject.ReleaseCapture
 0001:0002C310       TDragObject.ShowDragImage
 0001:0002C1EC       TDragObject.WndProc
 0001:000527D4       Templates
 0002:00002C1C       TemplatesVar
 0002:00000318       TerminateProcList
 0002:0000204E       Test8086
 0002:00000978       TextConversionFormat
 0001:00008814       TextToFloat
 0001:0003DDDC       TextToShortCut
 0001:00018978       TFiler.Create
 0001:000189C0       TFiler.Destroy
 0001:000189E8       TFiler.SetRoot
 0001:00018418       TFileStream.Create
 0001:0001845C       TFileStream.Create
 0001:000185B0       TFileStream.Destroy
 0001:0001EC70       TFont.Assign
 0001:0001EC54       TFont.Changed
 0001:0001EBD8       TFont.Create
 0001:0001EC2C       TFont.Destroy
 0001:0001F0D4       TFont.GetCharset
 0001:0001ED44       TFont.GetData
 0001:0001EDC0       TFont.GetHandle
 0001:0001EF8C       TFont.GetHeight
 0001:0001EFBC       TFont.GetName
 0001:0001F0A4       TFont.GetPitch
 0001:0001F030       TFont.GetSize
 0001:0001F06C       TFont.GetStyle
 0001:0001F0DC       TFont.SetCharset
 0001:0001EDAC       TFont.SetColor
 0001:0001ED5C       TFont.SetData
 0001:0001EF68       TFont.SetHandle
 0001:0001EF94       TFont.SetHeight
 0001:0001EFD4       TFont.SetName
 0001:0001F0AC       TFont.SetPitch
 0001:0001F04C       TFont.SetSize
 0001:0001F078       TFont.SetStyle
 0001:0005BB64       TfrmRenderer.DoGetWindowStyle
 0001:0005BC74       TfrmRenderer.DoInitializeDirectDraw
 0001:0005BBA0       TfrmRenderer.DoPaintWindow
 0001:0005BBC0       TfrmRenderer.DoRenderSample
 0001:0005BA84       TfrmRenderer.DoSetWindowStyle
 0001:0005BB84       TfrmRenderer.DoShowWindow
 0001:0005BCB8       TfrmRenderer.FormCreate
 0001:0005BA48       TfrmRenderer.WndProc
 0001:000211B0       TGraphic.Changed
 0001:00021178       TGraphic.Create
 0001:00021220       TGraphic.DefineProperties
 0001:0002126C       TGraphic.Equals
 0001:000213B4       TGraphic.GetPalette
 0001:000213B8       TGraphic.GetTransparent
 0001:000213BC       TGraphic.LoadFromFile
 0001:00021410       TGraphic.Progress
 0001:00021438       TGraphic.ReadData
 0001:00021444       TGraphic.SaveToFile
 0001:0002149C       TGraphic.SetPalette
 0001:000214A0       TGraphic.SetTransparent
 0001:000214B0       TGraphic.WriteData
 0001:0001E91C       TGraphicsObject.Changed
 0001:0001E930       TGraphicsObject.Lock
 0001:0001E940       TGraphicsObject.Unlock
 0001:00018354       THandleStream.Create
 0001:00018390       THandleStream.Read
 0001:000183B0       THandleStream.Seek
 0001:000183F0       THandleStream.SetSize
 0001:000183DC       THandleStream.SetSize
 0001:000183A0       THandleStream.Write
 0001:00025F40       THelpManager.AssignHelpSelector
 0001:00025A0C       THelpManager.CallSpecialWinHelp
 0001:00025668       THelpManager.Create
 0001:000260E8       THelpManager.Destroy
 0001:0002583C       THelpManager.DoSoftShutDown
 0001:0002586C       THelpManager.DoTableOfContents
 0001:00026044       THelpManager.GetHandle
 0001:00026048       THelpManager.GetHelpFile
 0001:00025F9C       THelpManager.Hook
 0001:000256DC       THelpManager.RegisterViewer
 0001:0002605C       THelpManager.Release
 0001:00025D28       THelpManager.ShowContextHelp
 0001:00025B14       THelpManager.ShowHelp
 0001:00025E3C       THelpManager.ShowTableOfContents
 0001:00025E44       THelpManager.ShowTopicHelp
 0001:000257FC       THelpManager.UnloadAllViewers
 0001:0002562C       THelpViewerNode.Create
 0002:0000098C       ThemeDataNames
 0002:00002A40       ThemeLibrary
 0001:00028EC0       Themes
 0001:000286E4       ThemeServices
 0002:00000984       ThemeServicesClass
 0001:00028FF4       THintAction.Create
 0001:000367CC       THintWindow.ActivateHint
 0001:000369B4       THintWindow.ActivateHintData
 0001:000369DC       THintWindow.CalcHintRect
 0001:00036734       THintWindow.CMTextChanged
 0001:000364E4       THintWindow.Create
 0001:00036550       THintWindow.CreateParams
 0001:000366C8       THintWindow.IsHintMsg
 0001:00036A38       THintWindow.NCPaint
 0001:00036620       THintWindow.Paint
 0001:0003672C       THintWindow.ReleaseHandle
 0001:000365B4       THintWindow.WMNCHitTest
 0001:000365BC       THintWindow.WMNCPaint
 0001:00036AA4       THintWindow.WMPrint
 0002:0000268A       ThousandSeparator
 0002:00002870       ThreadLock
 0002:00000D6C       ThreadStrs
 0001:00023C38       TIcon.Assign
 0001:00023BB4       TIcon.Create
 0001:00023C08       TIcon.Destroy
 0001:00023C98       TIcon.Draw
 0001:00023CD8       TIcon.GetEmpty
 0001:00023CF0       TIcon.GetHandle
 0001:00023D04       TIcon.GetHeight
 0001:00023D18       TIcon.GetWidth
 0001:00023D2C       TIcon.HandleNeeded
 0001:00023DA4       TIcon.ImageNeeded
 0001:00023FF8       TIcon.LoadFromClipboardFormat
 0001:00023E58       TIcon.LoadFromStream
 0001:00023F10       TIcon.NewImage
 0001:0002400C       TIcon.SaveToClipboardFormat
 0001:00023FD0       TIcon.SaveToStream
 0001:00023F84       TIcon.SetHandle
 0001:00023F9C       TIcon.SetHeight
 0001:00023FB4       TIcon.SetTransparent
 0001:00023FB8       TIcon.SetWidth
 0001:00023B6C       TIconImage.Destroy
 0001:00023B9C       TIconImage.FreeHandle
 0002:0000269C       TimeAMString
 0001:0004F60C       timeBeginPeriod
 0001:0005799C       TimeDiff
 0001:0004F614       timeEndPeriod
 0001:0004F61C       timeGetTime
 0001:0004F624       timeKillEvent
 0001:000578FC       TimeKillSynchronousFlagAvailable
 0002:000026A0       TimePMString
 0002:00002698       TimeSeparator
 0001:0004F62C       timeSetEvent
 0002:00000EC0       TIME_FORMAT_MEDIA_TIME
 0001:00015CB4       TIntConst.Create
 0001:00004D94       TInterfacedObject.AfterConstruction
 0001:00004DA0       TInterfacedObject.BeforeDestruction
 0001:00004DB0       TInterfacedObject.NewInstance
 0001:00004DC0       TInterfacedObject.QueryInterface
 0001:00004DE8       TInterfacedObject._AddRef
 0001:00004DFC       TInterfacedObject._Release
 0001:00016A6C       TInterfacedPersistent.AfterConstruction
 0001:00016AFC       TInterfacedPersistent.QueryInterface
 0001:00016ABC       TInterfacedPersistent._AddRef
 0001:00016ADC       TInterfacedPersistent._Release
 0001:000161C8       TList.Add
 0001:000161FC       TList.Clear
 0001:00016214       TList.Delete
 0001:000161A8       TList.Destroy
 0001:000162B0       TList.Error
 0001:00016278       TList.Error
 0001:00016304       TList.Expand
 0001:0001631C       TList.First
 0001:00016324       TList.Get
 0001:0001634C       TList.Grow
 0001:00016380       TList.IndexOf
 0001:000163A0       TList.Insert
 0001:0001640C       TList.Last
 0001:00016534       TList.Notify
 0001:00016418       TList.Put
 0001:00016468       TList.Remove
 0001:00016488       TList.SetCapacity
 0001:000164C4       TList.SetCount
 0001:000053DC       TlsAlloc
 0002:00002674       tlsBuffer
 0001:000053E4       TlsFree
 0001:000053EC       TlsGetValue
 0002:0000009C       TlsIndex
 0002:FFBA1010       TlsLast
 0002:000000BC       TlsProc
 0001:000053F4       TlsSetValue
 0001:0004260C       TMainMenu.GetHandle
 0001:000425E0       TMainMenu.ItemChanged
 0001:00042550       TMainMenu.MenuChanged
 0001:000425A8       TMainMenu.Merge
 0001:00042530       TMainMenu.SetAutoMerge
 0001:000425C4       TMainMenu.Unmerge
 0001:00018674       TMemoryStream.Clear
 0001:00018648       TMemoryStream.Destroy
 0001:0001868C       TMemoryStream.LoadFromStream
 0001:00018718       TMemoryStream.Realloc
 0001:000186C4       TMemoryStream.SetCapacity
 0001:000186EC       TMemoryStream.SetSize
 0001:000187A4       TMemoryStream.Write
 0001:00041F68       TMenu.AdjustBiDiBehavior
 0001:00041740       TMenu.Create
 0001:000417DC       TMenu.Destroy
 0001:000419C8       TMenu.DispatchCommand
 0001:000419E4       TMenu.DispatchPopup
 0001:00041D48       TMenu.DoBiDiModeChanged
 0001:0004201C       TMenu.DoChange
 0001:000423D0       TMenu.DoGetMenuString
 0001:00041928       TMenu.FindItem
 0001:000424F0       TMenu.GetAutoHotkeys
 0001:00042510       TMenu.GetAutoLineReduction
 0001:00041814       TMenu.GetChildren
 0001:00041830       TMenu.GetHandle
 0001:00041958       TMenu.GetHelpContext
 0001:00042088       TMenu.ImageListChange
 0001:00041D40       TMenu.IsBiDiModeStored
 0001:00041AAC       TMenu.IsOwnerDraw
 0001:000420FC       TMenu.IsRightToLeft
 0001:00041C24       TMenu.IsShortCut
 0001:00042034       TMenu.Loaded
 0001:0004204C       TMenu.MenuChanged
 0001:000420D0       TMenu.Notification
 0001:000424C4       TMenu.ParentBiDiModeChanged
 0001:0004249C       TMenu.ParentBiDiModeChanged
 0001:00042258       TMenu.ProcessMenuChar
 0001:00042500       TMenu.SetAutoHotkeys
 0001:00042520       TMenu.SetAutoLineReduction
 0001:00042478       TMenu.SetBiDiMode
 0001:0004183C       TMenu.SetChildOrder
 0001:00042094       TMenu.SetImages
 0001:00041F58       TMenu.SetOwnerDraw
 0001:0004248C       TMenu.SetParentBiDiMode
 0001:00041FE4       TMenu.SetWindowHandle
 0001:00041ED4       TMenu.UpdateImage
 0001:00041878       TMenu.UpdateItems
 0001:0003E05C       TMenuActionLink.AssignClient
 0001:0003E078       TMenuActionLink.IsAutoCheckLinked
 0001:0003E0A0       TMenuActionLink.IsCaptionLinked
 0001:0003E0D8       TMenuActionLink.IsCheckedLinked
 0001:0003E108       TMenuActionLink.IsEnabledLinked
 0001:0003E19C       TMenuActionLink.IsGroupIndexLinked
 0001:0003E138       TMenuActionLink.IsHelpContextLinked
 0001:0003E168       TMenuActionLink.IsHintLinked
 0001:0003E1D8       TMenuActionLink.IsImageIndexLinked
 0001:0003E274       TMenuActionLink.IsOnExecuteLinked
 0001:0003E20C       TMenuActionLink.IsShortCutLinked
 0001:0003E240       TMenuActionLink.IsVisibleLinked
 0001:0003E29C       TMenuActionLink.SetAutoCheck
 0001:0003E2BC       TMenuActionLink.SetCaption
 0001:0003E2DC       TMenuActionLink.SetChecked
 0001:0003E2FC       TMenuActionLink.SetEnabled
 0001:0003E31C       TMenuActionLink.SetHelpContext
 0001:0003E338       TMenuActionLink.SetHint
 0001:0003E35C       TMenuActionLink.SetImageIndex
 0001:0003E3BC       TMenuActionLink.SetOnExecute
 0001:0003E37C       TMenuActionLink.SetShortCut
 0001:0003E39C       TMenuActionLink.SetVisible
 0001:00040ACC       TMenuItem.ActionChange
 0001:00040850       TMenuItem.Add
 0001:0003FF78       TMenuItem.AdvancedDrawItem
 0001:0003E518       TMenuItem.AppendTo
 0001:00040D30       TMenuItem.AssignTo
 0001:00040788       TMenuItem.Click
 0001:0003E3E8       TMenuItem.Create
 0001:0003EA74       TMenuItem.DefineProperties
 0001:00040714       TMenuItem.Delete
 0001:0003E464       TMenuItem.Destroy
 0001:00040BEC       TMenuItem.DoActionChange
 0001:0003EAB8       TMenuItem.DoDrawText
 0001:0003ECC8       TMenuItem.DrawItem
 0001:000404BC       TMenuItem.GetAction
 0001:000404CC       TMenuItem.GetActionLinkClass
 0001:000416E8       TMenuItem.GetAutoHotkeys
 0001:00041714       TMenuItem.GetAutoLineReduction
 0001:00040930       TMenuItem.GetBitmap
 0001:0004059C       TMenuItem.GetChildren
 0001:000404D4       TMenuItem.GetCount
 0001:0003EA28       TMenuItem.GetHandle
 0001:000400AC       TMenuItem.GetImageList
 0001:000404E4       TMenuItem.GetItem
 0001:0004053C       TMenuItem.GetMenuIndex
 0001:00040A28       TMenuItem.GetParentComponent
 0001:00040A90       TMenuItem.GetParentMenu
 0001:00040328       TMenuItem.HasParent
 0001:00040E38       TMenuItem.ImageListChange
 0001:00040838       TMenuItem.IndexOf
 0001:00040650       TMenuItem.InitiateAction
 0001:000409FC       TMenuItem.InitiateActions
 0001:00040660       TMenuItem.Insert
 0001:00041094       TMenuItem.InternalRethinkHotkeys
 0001:00041590       TMenuItem.InternalRethinkLines
 0001:00040C10       TMenuItem.IsCaptionStored
 0001:00040C30       TMenuItem.IsCheckedStored
 0001:00040C50       TMenuItem.IsEnabledStored
 0001:00040C90       TMenuItem.IsHelpContextStored
 0001:00040C70       TMenuItem.IsHintStored
 0001:00040CB0       TMenuItem.IsImageIndexStored
 0001:0004156C       TMenuItem.IsLine
 0001:00040D10       TMenuItem.IsOnClickStored
 0001:00040CD0       TMenuItem.IsShortCutStored
 0001:00040CF0       TMenuItem.IsVisibleStored
 0001:0003E8BC       TMenuItem.Loaded
 0001:00040128       TMenuItem.MeasureItem
 0001:00040894       TMenuItem.MenuChanged
 0001:0003E880       TMenuItem.MergeWith
 0001:00040DA8       TMenuItem.Notification
 0001:0003E7B8       TMenuItem.PopulateMenu
 0001:0003E828       TMenuItem.ReadShortCutText
 0001:0003E8F8       TMenuItem.RebuildHandle
 0001:0004086C       TMenuItem.Remove
 0001:00040958       TMenuItem.SetAction
 0001:0004155C       TMenuItem.SetAutoHotkeys
 0001:000416D8       TMenuItem.SetAutoLineReduction
 0001:000409C8       TMenuItem.SetBitmap
 0001:0004032C       TMenuItem.SetBreak
 0001:0004033C       TMenuItem.SetCaption
 0001:000403AC       TMenuItem.SetChecked
 0001:000405D4       TMenuItem.SetChildOrder
 0001:000405F4       TMenuItem.SetDefault
 0001:00040400       TMenuItem.SetEnabled
 0001:00040478       TMenuItem.SetGroupIndex
 0001:0004052C       TMenuItem.SetImageIndex
 0001:00040554       TMenuItem.SetMenuIndex
 0001:00040A3C       TMenuItem.SetParentComponent
 0001:00040AA0       TMenuItem.SetRadioItem
 0001:00040508       TMenuItem.SetShortCut
 0001:00040DFC       TMenuItem.SetSubMenuImages
 0001:0004051C       TMenuItem.SetVisible
 0001:000408D8       TMenuItem.SubItemChanged
 0001:00040364       TMenuItem.TurnSiblingsOff
 0001:00040E6C       TMenuItem.UpdateItems
 0001:0003E9C8       TMenuItem.VerifyGroupIndex
 0001:00042E04       TMenuItemStack.ClearItem
 0001:0004BA10       TMonitor.GetBoundsRect
 0001:0004B9C0       TMonitor.GetHeight
 0001:0004B9A8       TMonitor.GetLeft
 0001:0004B9DC       TMonitor.GetTop
 0001:0004B9F4       TMonitor.GetWidth
 0001:0004BA40       TMonitor.GetWorkareaRect
 0001:00039958       TMouse.Create
 0001:000399E8       TMouse.Destroy
 0001:00039A18       TMouse.GetCapture
 0001:00039A20       TMouse.GetCursorPos
 0001:00039A30       TMouse.GetMouseData
 0001:00039A4C       TMouse.GetNativeData
 0001:00039A7C       TMouse.GetRegisteredData
 0001:00039AA4       TMouse.SetCapture
 0001:00039ACC       TMouse.SettingChanged
 0001:0000C42C       TMultiReadExclusiveWriteSynchronizer.BeginRead
 0001:0000C330       TMultiReadExclusiveWriteSynchronizer.BeginWrite
 0001:0000C2EC       TMultiReadExclusiveWriteSynchronizer.BlockReaders
 0001:0000C230       TMultiReadExclusiveWriteSynchronizer.Create
 0001:0000C2A4       TMultiReadExclusiveWriteSynchronizer.Destroy
 0001:0000C49C       TMultiReadExclusiveWriteSynchronizer.EndRead
 0001:0000C3DC       TMultiReadExclusiveWriteSynchronizer.EndWrite
 0001:0000C304       TMultiReadExclusiveWriteSynchronizer.UnblockOneWriter
 0001:0000C2F8       TMultiReadExclusiveWriteSynchronizer.UnblockReaders
 0001:0000C310       TMultiReadExclusiveWriteSynchronizer.WaitForReadSignal
 0001:0000C320       TMultiReadExclusiveWriteSynchronizer.WaitForWriteSignal
 0001:000026E0       TObject.AfterConstruction
 0001:000026E4       TObject.BeforeDestruction
 0001:000026C4       TObject.ClassInfo
 0001:000023E0       TObject.ClassName
 0001:000023F4       TObject.ClassNameIs
 0001:0000241C       TObject.ClassParent
 0001:000023D4       TObject.ClassType
 0001:000024F4       TObject.CleanupInstance
 0001:00002460       TObject.Create
 0001:000026DC       TObject.DefaultHandler
 0001:00002480       TObject.Destroy
 0001:000026E8       TObject.Dispatch
 0001:00002760       TObject.FieldAddress
 0001:00002490       TObject.Free
 0001:00002444       TObject.FreeInstance
 0001:00002544       TObject.GetInterface
 0001:000025E4       TObject.GetInterfaceEntry
 0001:000026B0       TObject.InheritsFrom
 0001:0000249C       TObject.InitInstance
 0001:00002458       TObject.InstanceSize
 0001:00002710       TObject.MethodAddress
 0001:00002428       TObject.NewInstance
 0001:000026D4       TObject.SafeCallException
 0001:00024750       TObjectList.Create
 0001:0002478C       TObjectList.GetItem
 0001:000247A0       TObjectList.Insert
 0001:000247A8       TObjectList.Notify
 0001:00004710       ToLongPath
 0001:000270E8       ToolWin
 0001:000247EC       TOrderedList.Create
 0001:00024830       TOrderedList.Destroy
 0001:00024860       TOrderedList.PeekItem
 0001:000247D4       TOrderedList.Pop
 0001:00024874       TOrderedList.PopItem
 0001:000247DC       TOrderedList.Push
 0001:000241E4       TPatternManager.AllocPattern
 0001:00024168       TPatternManager.Create
 0001:00024298       TPatternManager.CreateBitmap
 0001:000241A0       TPatternManager.Destroy
 0001:00024398       TPatternManager.FreePatterns
 0001:000241CC       TPatternManager.Lock
 0001:000241D8       TPatternManager.Unlock
 0001:0001F170       TPen.Assign
 0001:0001F104       TPen.Create
 0001:0001F148       TPen.Destroy
 0001:0001F290       TPen.GetColor
 0001:0001F228       TPen.GetData
 0001:0001F2C0       TPen.GetHandle
 0001:0001F36C       TPen.GetStyle
 0001:0001F39C       TPen.GetWidth
 0001:0001F298       TPen.SetColor
 0001:0001F240       TPen.SetData
 0001:0001F358       TPen.SetMode
 0001:0001F374       TPen.SetStyle
 0001:0001F3A4       TPen.SetWidth
 0001:000168C8       TPersistent.Assign
 0001:000168DC       TPersistent.AssignError
 0001:000169AC       TPersistent.AssignTo
 0001:000169B4       TPersistent.DefineProperties
 0001:0001689C       TPersistent.Destroy
 0001:000169B8       TPersistent.GetNamePath
 0001:00016A68       TPersistent.GetOwner
 0001:00042BAC       TPopupList.Add
 0001:0004261C       TPopupList.MainWndProc
 0001:00042BD4       TPopupList.Remove
 0001:00042668       TPopupList.WndProc
 0001:00042BF0       TPopupMenu.Create
 0001:00042C64       TPopupMenu.Destroy
 0001:00042C98       TPopupMenu.DoPopup
 0001:00042CAC       TPopupMenu.GetHelpContext
 0001:00042D50       TPopupMenu.Popup
 0001:00042CBC       TPopupMenu.SetBiDiModeFromPopupControl
 0001:00042CB4       TPopupMenu.SetHelpContext
 0001:00042D04       TPopupMenu.UseRightToLeftAlignment
 0001:00018AC4       TPropFixup.Create
 0001:00018B1C       TPropFixup.MakeGlobalReference
 0001:00018B64       TPropFixup.ResolveReference
 0001:00018B74       TPropIntfFixup.ResolveReference
 0001:00005FD4       TrackPopupMenu
 0001:0000A664       TranslateDateFormat
 0001:00005FDC       TranslateMDISysAccel
 0001:00005FE4       TranslateMessage
 0001:0000DB64       TranslateResult
 0001:00020194       TransparentStretchBlt
 0001:0004AFC8       TraverseClients
 0001:0004B210       TraverseClients
 0001:0004B110       TraverseClients
 0001:000344C0       TraverseControls
 0001:000190BC       TReader.CheckValue
 0001:00019114       TReader.DefineBinaryProperty
 0001:000190E0       TReader.DefineProperty
 0001:00019080       TReader.Destroy
 0001:00019308       TReader.DoFixupReferences
 0001:000191F0       TReader.EndOfList
 0001:00019204       TReader.Error
 0001:0001B330       TReader.FindAncestorComponent
 0001:0001B428       TReader.FindComponentClass
 0001:00019224       TReader.FindMethod
 0001:00019428       TReader.FlushBuffer
 0001:0001944C       TReader.FreeFixups
 0001:00019488       TReader.GetFieldClass
 0001:0001951C       TReader.GetPosition
 0001:00019534       TReader.NextValue
 0001:00019544       TReader.PropertyError
 0001:00019558       TReader.Read
 0001:000195E0       TReader.ReadBoolean
 0001:000195A4       TReader.ReadBuffer
 0001:000195F4       TReader.ReadChar
 0001:0001964C       TReader.ReadCollection
 0001:00019B0C       TReader.ReadComponent
 0001:00019F10       TReader.ReadCurrency
 0001:00019D48       TReader.ReadData
 0001:00019DB8       TReader.ReadDataInner
 0001:00019F60       TReader.ReadDate
 0001:00019E88       TReader.ReadFloat
 0001:00019FA4       TReader.ReadIdent
 0001:0001A110       TReader.ReadInt64
 0001:0001A0A4       TReader.ReadInteger
 0001:0001A154       TReader.ReadListBegin
 0001:0001A15C       TReader.ReadListEnd
 0001:0001A164       TReader.ReadPrefix
 0001:0001A2C0       TReader.ReadProperty
 0001:0001A644       TReader.ReadPropValue
 0001:0001A9AC       TReader.ReadRootComponent
 0001:0001ACD8       TReader.ReadSet
 0001:0001AD94       TReader.ReadSignature
 0001:00019ECC       TReader.ReadSingle
 0001:0001ADB8       TReader.ReadStr
 0001:0001ADF4       TReader.ReadString
 0001:0001AF94       TReader.ReadValue
 0001:0001B6AC       TReader.ReadVariant
 0001:0001AEB0       TReader.ReadWideString
 0001:0001B3E8       TReader.ReferenceName
 0001:0001B400       TReader.SetName
 0001:0001B49C       TReader.SkipBytes
 0001:0001B288       TReader.SkipComponent
 0001:0001B240       TReader.SkipProperty
 0001:0001AFA8       TReader.SkipSetBody
 0001:0001B0A4       TReader.SkipValue
 0002:00000B10       TreeStreamEndFlag
 0001:00015004       TRegGroup.AddClass
 0001:00015010       TRegGroup.BestClass
 0001:00015070       TRegGroup.BestGroup
 0001:000150E0       TRegGroup.Create
 0001:0001515C       TRegGroup.Destroy
 0001:0001519C       TRegGroup.GetClass
 0001:000151FC       TRegGroup.InGroup
 0001:00015240       TRegGroup.RegisterClass
 0001:000152E8       TRegGroup.Registered
 0001:00015320       TRegGroup.UnregisterModuleClasses
 0001:000153C4       TRegGroups.Activate
 0001:00015410       TRegGroups.Create
 0001:00015484       TRegGroups.Destroy
 0001:000154E0       TRegGroups.FindGroup
 0001:00015524       TRegGroups.GetClass
 0001:000155F8       TRegGroups.GroupWith
 0001:000156C0       TRegGroups.Lock
 0001:000156CC       TRegGroups.RegisterClass
 0001:000156E4       TRegGroups.Registered
 0001:00015728       TRegGroups.StartGroup
 0001:00015778       TRegGroups.Unlock
 0001:00015784       TRegGroups.UnregisterModuleClasses
 0001:0001E0F8       TResourceManager.AllocResource
 0001:0001E314       TResourceManager.AssignResource
 0001:0001E298       TResourceManager.ChangeResource
 0001:0001E080       TResourceManager.Create
 0001:0001E0BC       TResourceManager.Destroy
 0001:0001E1DC       TResourceManager.FreeResource
 0001:0001E0E0       TResourceManager.Lock
 0001:0001E0EC       TResourceManager.Unlock
 0001:000187F4       TResourceStream.Create
 0001:00018928       TResourceStream.Destroy
 0001:000188BC       TResourceStream.Initialize
 0001:00018960       TResourceStream.Write
 0001:000073CC       Trim
 0001:0004F980       TrimPunctuation
 0002:0000278C       TrueBoolStrs
 0001:00008B64       TryEncodeDate
 0001:00008A5C       TryEncodeTime
 0001:0000129C       TryHarder
 0001:00007768       TryStrToBool
 0001:000089FC       TryStrToCurr
 0001:0000A1EC       TryStrToDate
 0001:0000A254       TryStrToDateTime
 0001:00008988       TryStrToFloat
 0001:000089D0       TryStrToFloat
 0001:000089A4       TryStrToFloat
 0001:0000765C       TryStrToInt
 0001:0000767C       TryStrToInt64
 0001:0000A220       TryStrToTime
 0001:0004BE14       TScreen.AddDataModule
 0001:0004BD8C       TScreen.AddForm
 0001:0004C83C       TScreen.AlignForm
 0001:0004C7B4       TScreen.AlignForms
 0001:0004BA70       TScreen.Create
 0001:0004BE2C       TScreen.CreateCursors
 0001:0004BBC8       TScreen.Destroy
 0001:0004BE88       TScreen.DestroyCursors
 0001:0004C3D0       TScreen.DisableAlign
 0001:0004C3D8       TScreen.EnableAlign
 0001:0004C1B0       TScreen.GetCursors
 0001:0004BD38       TScreen.GetCustomFormCount
 0001:0004BD24       TScreen.GetCustomForms
 0001:0004C194       TScreen.GetDataModule
 0001:0004C1A8       TScreen.GetDataModuleCount
 0001:0004C128       TScreen.GetDefaultIME
 0001:0004BCC0       TScreen.GetDesktopHeight
 0001:0004BCB4       TScreen.GetDesktopLeft
 0001:0004BCA8       TScreen.GetDesktopTop
 0001:0004BCCC       TScreen.GetDesktopWidth
 0001:0004BD08       TScreen.GetForm
 0001:0004BD1C       TScreen.GetFormCount
 0001:0004BC90       TScreen.GetHeight
 0001:0004BF28       TScreen.GetImes
 0001:0004C27C       TScreen.GetMetricSettings
 0001:0004BCD8       TScreen.GetMonitor
 0001:0004BCEC       TScreen.GetMonitorCount
 0001:0004BC9C       TScreen.GetWidth
 0001:0004C144       TScreen.IconFontChanged
 0001:0004BF00       TScreen.InsertCursor
 0001:0004C3F8       TScreen.Realign
 0001:0004BE20       TScreen.RemoveDataModule
 0001:0004BDC4       TScreen.RemoveForm
 0001:0004C8C4       TScreen.ResetFonts
 0001:0004C1EC       TScreen.SetCursor
 0001:0004BD40       TScreen.UpdateLastActive
 0001:000467D0       TScrollingWinControl.AdjustClientRect
 0001:000461A4       TScrollingWinControl.AlignControls
 0001:000461C4       TScrollingWinControl.AutoScrollEnabled
 0001:00046474       TScrollingWinControl.AutoScrollInView
 0001:000462FC       TScrollingWinControl.CalcAutoRange
 0001:00046684       TScrollingWinControl.ChangeScale
 0001:00046840       TScrollingWinControl.CMBiDiModeChanged
 0001:000460A0       TScrollingWinControl.Create
 0001:00046154       TScrollingWinControl.CreateParams
 0001:00046164       TScrollingWinControl.CreateWnd
 0001:00046118       TScrollingWinControl.Destroy
 0001:000461E4       TScrollingWinControl.DoFlipChildren
 0001:000466A8       TScrollingWinControl.Resizing
 0001:000465E0       TScrollingWinControl.ScaleScrollBars
 0001:0004648C       TScrollingWinControl.ScrollInView
 0001:00046320       TScrollingWinControl.SetAutoScroll
 0001:0004635C       TScrollingWinControl.SetHorzScrollBar
 0001:0004636C       TScrollingWinControl.SetVertScrollBar
 0001:0004637C       TScrollingWinControl.UpdateScrollBars
 0001:00046788       TScrollingWinControl.WMHScroll
 0001:000466AC       TScrollingWinControl.WMSize
 0001:000467AC       TScrollingWinControl.WMVScroll
 0001:00021874       TSharedImage.Reference
 0001:00021878       TSharedImage.Release
 0001:0003B3B8       TShortCutList.Add
 0001:0003B3E4       TShortCutList.IndexOfShortCut
 0001:0002C05C       TSiteList.AddSite
 0001:0002C0B8       TSiteList.Clear
 0001:0002C000       TSiteList.Find
 0001:0002C0EC       TSiteList.GetTopSite
 0001:0002D9E0       TSizeConstraints.AssignTo
 0001:0002DAB4       TSizeConstraints.Change
 0001:0002D9A4       TSizeConstraints.Create
 0001:0002DA28       TSizeConstraints.SetConstraints
 0001:00024894       TStack.PushItem
 0001:00018200       TStream.CopyFrom
 0001:00017F64       TStream.GetPosition
 0001:00017F98       TStream.GetSize
 0001:00018190       TStream.ReadBuffer
 0001:000182F4       TStream.ReadComponent
 0001:00018120       TStream.Seek
 0001:0001809C       TStream.Seek
 0001:00017F84       TStream.SetPosition
 0001:00017FE4       TStream.SetSize
 0001:00017FFC       TStream.SetSize
 0001:00017FE8       TStream.SetSize64
 0001:000181C8       TStream.WriteBuffer
 0001:0001CCA0       TStreamAdapter.Clone
 0001:0001CBF4       TStreamAdapter.Commit
 0001:0001C9F4       TStreamAdapter.CopyTo
 0001:0001C7BC       TStreamAdapter.Create
 0001:0001C804       TStreamAdapter.Destroy
 0001:0001CC0C       TStreamAdapter.LockRegion
 0001:0001C83C       TStreamAdapter.Read
 0001:0001CC00       TStreamAdapter.Revert
 0001:0001C90C       TStreamAdapter.Seek
 0001:0001C990       TStreamAdapter.SetSize
 0001:0001CC24       TStreamAdapter.Stat
 0001:0001CC18       TStreamAdapter.UnlockRegion
 0001:0001C8A4       TStreamAdapter.Write
 0001:0001796C       TStringList.Add
 0001:00017978       TStringList.AddObject
 0001:000179DC       TStringList.Changed
 0001:000179F8       TStringList.Changing
 0001:00017A14       TStringList.Clear
 0001:00017F48       TStringList.CompareStrings
 0001:00017F10       TStringList.CustomSort
 0001:00017A54       TStringList.Delete
 0001:00017910       TStringList.Destroy
 0001:00017AC0       TStringList.Exchange
 0001:00017B1C       TStringList.ExchangeItems
 0001:00017B40       TStringList.Find
 0001:00017BB8       TStringList.Get
 0001:00017BEC       TStringList.GetCapacity
 0001:00017BF0       TStringList.GetCount
 0001:00017BF4       TStringList.GetObject
 0001:00017C1C       TStringList.Grow
 0001:00017C50       TStringList.IndexOf
 0001:00017C8C       TStringList.Insert
 0001:00017CF0       TStringList.InsertItem
 0001:00017C9C       TStringList.InsertObject
 0001:00017D68       TStringList.Put
 0001:00017DC4       TStringList.PutObject
 0001:00017E04       TStringList.QuickSort
 0001:00017E98       TStringList.SetCapacity
 0001:00017EB4       TStringList.SetSorted
 0001:00017ED4       TStringList.SetUpdateState
 0001:00017F00       TStringList.Sort
 0001:00016BDC       TStrings.Add
 0001:00016C00       TStrings.AddObject
 0001:00016C24       TStrings.AddStrings
 0001:00016CDC       TStrings.Assign
 0001:00016D74       TStrings.BeginUpdate
 0001:000178D0       TStrings.CompareStrings
 0001:00016DE4       TStrings.DefineProperties
 0001:00016BAC       TStrings.Destroy
 0001:00016E30       TStrings.EndUpdate
 0001:00016E44       TStrings.Equals
 0001:00016EF0       TStrings.Error
 0001:00016F28       TStrings.Error
 0001:00016F80       TStrings.Exchange
 0001:00017068       TStrings.GetCapacity
 0001:000178DC       TStrings.GetNameValueSeparator
 0001:00017070       TStrings.GetObject
 0001:00017074       TStrings.GetText
 0001:000170C8       TStrings.GetTextStr
 0001:000171F0       TStrings.IndexOf
 0001:0001727C       TStrings.IndexOfName
 0001:00017350       TStrings.IndexOfObject
 0001:00017384       TStrings.InsertObject
 0001:000173B4       TStrings.LoadFromFile
 0001:00017408       TStrings.LoadFromStream
 0001:000174B4       TStrings.Move
 0001:00017564       TStrings.Put
 0001:00017598       TStrings.PutObject
 0001:0001759C       TStrings.ReadData
 0001:0001764C       TStrings.SaveToFile
 0001:000176A4       TStrings.SaveToStream
 0001:00017700       TStrings.SetCapacity
 0001:000178F4       TStrings.SetNameValueSeparator
 0001:00017704       TStrings.SetStringsAdapter
 0001:00017738       TStrings.SetText
 0001:00017788       TStrings.SetTextStr
 0001:00017848       TStrings.SetUpdateState
 0001:0001784C       TStrings.WriteData
 0001:000265EC       TSynchroObject.Acquire
 0001:000265F0       TSynchroObject.Release
 0001:00028820       TThemeServices.ApplyThemeChange
 0001:00028704       TThemeServices.Create
 0001:00028750       TThemeServices.Destroy
 0001:000287DC       TThemeServices.DoOnThemeChange
 0001:00028834       TThemeServices.DrawEdge
 0001:00028880       TThemeServices.DrawElement
 0001:000288C4       TThemeServices.DrawParentBackground
 0001:00028968       TThemeServices.GetElementDetails
 0001:0002892C       TThemeServices.GetElementDetails
 0001:00028784       TThemeServices.GetTheme
 0001:000287C4       TThemeServices.GetThemesEnabled
 0001:00028CF4       TThemeServices.PaintBorder
 0001:000287F0       TThemeServices.UnloadThemeData
 0001:00028E60       TThemeServices.UpdateThemes
 0001:00016608       TThreadList.Add
 0001:00016538       TThreadList.Create
 0001:0001658C       TThreadList.Destroy
 0001:00016690       TThreadList.LockList
 0001:000166A4       TThreadList.Remove
 0001:000166F4       TThreadList.UnlockList
 0001:0000C1CC       TThreadLocalCounter.Delete
 0001:0000C0B4       TThreadLocalCounter.Destroy
 0001:0000C120       TThreadLocalCounter.HashIndex
 0001:0000C138       TThreadLocalCounter.Open
 0001:0000C1DC       TThreadLocalCounter.Recycle
 0001:000279FC       TTimer.Create
 0001:00027A4C       TTimer.Destroy
 0001:00027B84       TTimer.SetEnabled
 0001:00027B94       TTimer.SetInterval
 0001:00027BA4       TTimer.SetOnTimer
 0001:00027BBC       TTimer.Timer
 0001:00027AF8       TTimer.UpdateTimer
 0001:00027A84       TTimer.WndProc
 0001:0005C6AC       TVideoRenderer.Active
 0001:0005C6D4       TVideoRenderer.CheckMediaType
 0001:0005C54C       TVideoRenderer.Create
 0001:0005C614       TVideoRenderer.CreateFromFactory
 0001:0005C65C       TVideoRenderer.Destroy
 0001:0005C724       TVideoRenderer.DoRenderSample
 0001:0005DBB8       TVideoRenderer.GetCurrentImage
 0001:0005DB04       TVideoRenderer.GetDestinationPosition
 0001:0005C86C       TVideoRenderer.GetIDsOfNames
 0001:0005D594       TVideoRenderer.GetMaxIdealImageSize
 0001:0005D524       TVideoRenderer.GetMinIdealImageSize
 0001:0005DC58       TVideoRenderer.GetMiscFlags
 0001:0005DC30       TVideoRenderer.GetPreferredAspectRatio
 0001:0005D604       TVideoRenderer.GetRestorePosition
 0001:0005DA8C       TVideoRenderer.GetSourcePosition
 0001:0005C840       TVideoRenderer.GetTypeInfo
 0001:0005C824       TVideoRenderer.GetTypeInfoCount
 0001:0005DB90       TVideoRenderer.GetVideoPaletteEntries
 0001:0005DB54       TVideoRenderer.GetVideoSize
 0001:0005D4C0       TVideoRenderer.GetWindowPosition
 0001:0005CC08       TVideoRenderer.get_AutoShow
 0001:0005D6F0       TVideoRenderer.get_AvgTimePerFrame
 0001:0005CD08       TVideoRenderer.get_BackgroundPalette
 0001:0005D754       TVideoRenderer.get_BitErrorRate
 0001:0005D724       TVideoRenderer.get_BitRate
 0001:0005D228       TVideoRenderer.get_BorderColor
 0001:0005C9F4       TVideoRenderer.get_Caption
 0001:0005DA3C       TVideoRenderer.get_DestinationHeight
 0001:0005D94C       TVideoRenderer.get_DestinationLeft
 0001:0005D9EC       TVideoRenderer.get_DestinationTop
 0001:0005D99C       TVideoRenderer.get_DestinationWidth
 0001:0005D278       TVideoRenderer.get_FullScreenMode
 0001:0005D108       TVideoRenderer.get_Height
 0001:0005CE44       TVideoRenderer.get_Left
 0001:0005D1F4       TVideoRenderer.get_MessageDrain
 0001:0005D190       TVideoRenderer.get_Owner
 0001:0005D8FC       TVideoRenderer.get_SourceHeight
 0001:0005D80C       TVideoRenderer.get_SourceLeft
 0001:0005D8AC       TVideoRenderer.get_SourceTop
 0001:0005D85C       TVideoRenderer.get_SourceWidth
 0001:0005D020       TVideoRenderer.get_Top
 0001:0005D7B4       TVideoRenderer.get_VideoHeight
 0001:0005D784       TVideoRenderer.get_VideoWidth
 0001:0005CD64       TVideoRenderer.get_Visible
 0001:0005CF2C       TVideoRenderer.get_Width
 0001:0005CC6C       TVideoRenderer.get_WindowState
 0001:0005CAF4       TVideoRenderer.get_WindowStyle
 0001:0005CBA0       TVideoRenderer.get_WindowStyleEx
 0001:0005D6A0       TVideoRenderer.HideCursor
 0001:0005C6CC       TVideoRenderer.Inactive
 0001:0005C89C       TVideoRenderer.Invoke
 0001:0005D6C8       TVideoRenderer.IsCursorHidden
 0001:0005DC08       TVideoRenderer.IsUsingDefaultDestination
 0001:0005DBE0       TVideoRenderer.IsUsingDefaultSource
 0001:0005D304       TVideoRenderer.NotifyOwnerMessage
 0001:0005C784       TVideoRenderer.OnReceiveFirstSample
 0001:0005CBD8       TVideoRenderer.put_AutoShow
 0001:0005CCE0       TVideoRenderer.put_BackgroundPalette
 0001:0005D250       TVideoRenderer.put_BorderColor
 0001:0005C978       TVideoRenderer.put_Caption
 0001:0005DA14       TVideoRenderer.put_DestinationHeight
 0001:0005D924       TVideoRenderer.put_DestinationLeft
 0001:0005D9C4       TVideoRenderer.put_DestinationTop
 0001:0005D974       TVideoRenderer.put_DestinationWidth
 0001:0005D2A0       TVideoRenderer.put_FullScreenMode
 0001:0005D068       TVideoRenderer.put_Height
 0001:0005CD98       TVideoRenderer.put_Left
 0001:0005D1C4       TVideoRenderer.put_MessageDrain
 0001:0005D150       TVideoRenderer.put_Owner
 0001:0005D8D4       TVideoRenderer.put_SourceHeight
 0001:0005D7E4       TVideoRenderer.put_SourceLeft
 0001:0005D884       TVideoRenderer.put_SourceTop
 0001:0005D834       TVideoRenderer.put_SourceWidth
 0001:0005CF74       TVideoRenderer.put_Top
 0001:0005CD30       TVideoRenderer.put_Visible
 0001:0005CE8C       TVideoRenderer.put_Width
 0001:0005CC38       TVideoRenderer.put_WindowState
 0001:0005CA6C       TVideoRenderer.put_WindowStyle
 0001:0005CB2C       TVideoRenderer.put_WindowStyleEx
 0001:0005DB2C       TVideoRenderer.SetDefaultDestinationPosition
 0001:0005DAB4       TVideoRenderer.SetDefaultSourcePosition
 0001:0005DADC       TVideoRenderer.SetDestinationPosition
 0001:0005C7D4       TVideoRenderer.SetMediaType
 0001:0005DA64       TVideoRenderer.SetSourcePosition
 0001:0005D2C8       TVideoRenderer.SetWindowForeground
 0001:0005D39C       TVideoRenderer.SetWindowPosition
 0001:00035E20       TWinControl.ActionChange
 0001:0003225C       TWinControl.AddBiDiModeExStyle
 0001:00031510       TWinControl.AdjustClientRect
 0001:00035518       TWinControl.AdjustSize
 0001:00031CA8       TWinControl.AlignControl
 0001:00031BA4       TWinControl.AlignControls
 0001:00035E68       TWinControl.AssignTo
 0001:000321F4       TWinControl.Broadcast
 0001:00035A08       TWinControl.CalcConstraints
 0001:00035E98       TWinControl.CanAutoSize
 0001:00035378       TWinControl.CanFocus
 0001:0003597C       TWinControl.CanResize
 0001:00034F44       TWinControl.ChangeScale
 0001:000347B4       TWinControl.CMBiDiModeChanged
 0001:00034A10       TWinControl.CMBorderChanged
 0001:0003488C       TWinControl.CMChanged
 0001:000348A0       TWinControl.CMChildKey
 0001:0003496C       TWinControl.CMColorChanged
 0001:00034B4C       TWinControl.CMControlListChange
 0001:00034A50       TWinControl.CMCtl3DChanged
 0001:000349D0       TWinControl.CMCursorChanged
 0001:0003486C       TWinControl.CMDesignHitTest
 0001:000348BC       TWinControl.CMDialogChar
 0001:000348B4       TWinControl.CMDialogKey
 0001:000340CC       TWinControl.CMDockClient
 0001:00034AF0       TWinControl.CMDrag
 0001:00034924       TWinControl.CMEnabledChanged
 0001:000347EC       TWinControl.CMEnter
 0001:00034860       TWinControl.CMExit
 0001:000341E0       TWinControl.CMFloat
 0001:000348C4       TWinControl.CMFocusChanged
 0001:00034AE0       TWinControl.CMFontChange
 0001:00034994       TWinControl.CMFontChanged
 0001:0003527C       TWinControl.CMInvalidate
 0001:00034A90       TWinControl.CMParentCtl3DChanged
 0001:000329F0       TWinControl.CMRecreateWnd
 0001:0003479C       TWinControl.CMShowHintChanged
 0001:000348FC       TWinControl.CMShowingChanged
 0001:00034AD0       TWinControl.CMSysColorChange
 0001:00034B60       TWinControl.CMSysFontChanged
 0001:00034AE8       TWinControl.CMTimeChange
 0001:000341B8       TWinControl.CMUnDockClient
 0001:000348CC       TWinControl.CMVisibleChanged
 0001:00034AD8       TWinControl.CMWinIniChange
 0001:00034D48       TWinControl.CNChar
 0001:00034C10       TWinControl.CNKeyDown
 0001:00034CF4       TWinControl.CNKeyUp
 0001:00034DF0       TWinControl.CNSysChar
 0001:00034D94       TWinControl.CNSysKeyDown
 0001:00035DE4       TWinControl.ConstrainedResize
 0001:00031F80       TWinControl.ContainsControl
 0001:00032D24       TWinControl.ControlAtPos
 0001:00033FA4       TWinControl.ControlsAligned
 0001:000311D0       TWinControl.Create
 0001:00033FA8       TWinControl.CreateDockManager
 0001:000328D8       TWinControl.CreateHandle
 0001:000322C4       TWinControl.CreateParams
 0001:000325C0       TWinControl.CreateWindowHandle
 0001:000323F0       TWinControl.CreateWnd
 0001:00032970       TWinControl.CustomAlignInsertBefore
 0001:00032974       TWinControl.CustomAlignPosition
 0001:00032FB0       TWinControl.DefaultHandler
 0001:00032778       TWinControl.DefineProperties
 0001:000312F4       TWinControl.Destroy
 0001:00032990       TWinControl.DestroyHandle
 0001:0003282C       TWinControl.DestroyWindowHandle
 0001:000327D4       TWinControl.DestroyWnd
 0001:00031D3C       TWinControl.DisableAlign
 0001:00033D40       TWinControl.DoAddDockClient
 0001:00033D94       TWinControl.DockDrop
 0001:00033E18       TWinControl.DockOver
 0001:00033DE4       TWinControl.DoDockOver
 0001:00033D54       TWinControl.DoEnter
 0001:00033D74       TWinControl.DoExit
 0001:00031D6C       TWinControl.DoFlipChildren
 0001:0003428C       TWinControl.DoKeyDown
 0001:0003443C       TWinControl.DoKeyPress
 0001:00034374       TWinControl.DoKeyUp
 0001:00033D50       TWinControl.DoRemoveDockClient
 0001:00033E58       TWinControl.DoUnDock
 0001:00031D44       TWinControl.EnableAlign
 0001:000357BC       TWinControl.FindNextControl
 0001:000313C4       TWinControl.FixupTabList
 0001:00031E40       TWinControl.FlipChildren
 0001:000353F0       TWinControl.Focused
 0001:00035E60       TWinControl.GetActionLinkClass
 0001:000358F4       TWinControl.GetChildren
 0001:000354E0       TWinControl.GetClientOrigin
 0001:00035500       TWinControl.GetClientRect
 0001:00032198       TWinControl.GetControl
 0001:000321D4       TWinControl.GetControlCount
 0001:0003544C       TWinControl.GetControlExtents
 0001:00035218       TWinControl.GetDeviceContext
 0001:00033ED4       TWinControl.GetDockClientCount
 0001:00033EE8       TWinControl.GetDockClients
 0001:00035438       TWinControl.GetHandle
 0001:0003649C       TWinControl.GetParentBackground
 0001:00033F0C       TWinControl.GetSiteInfo
 0001:000355A8       TWinControl.GetTabOrder
 0001:0003575C       TWinControl.GetTabOrderList
 0001:00033F68       TWinControl.GetVisibleDockClientCount
 0001:00035698       TWinControl.HandleAllocated
 0001:00035414       TWinControl.HandleNeeded
 0001:00031FB4       TWinControl.Insert
 0001:00032048       TWinControl.InsertControl
 0001:0003526C       TWinControl.Invalidate
 0001:00035340       TWinControl.InvalidateFrame
 0001:00032DB8       TWinControl.IsControlMouseMsg
 0001:0003559C       TWinControl.IsCtl3DStored
 0001:00034B7C       TWinControl.IsMenuKey
 0001:00034264       TWinControl.KeyDown
 0001:0003441C       TWinControl.KeyPress
 0001:0003434C       TWinControl.KeyUp
 0001:00032BF4       TWinControl.MainWndProc
 0001:00032234       TWinControl.NotifyControls
 0001:00033244       TWinControl.PaintControls
 0001:000330EC       TWinControl.PaintHandler
 0001:00033474       TWinControl.PaintTo
 0001:0003321C       TWinControl.PaintWindow
 0001:00034700       TWinControl.PaletteChanged
 0001:00032890       TWinControl.PrecedingWindow
 0001:00032600       TWinControl.ReadDesignSize
 0001:00031498       TWinControl.ReadState
 0001:00031D64       TWinControl.Realign
 0001:000329D8       TWinControl.RecreateWnd
 0001:00033EB0       TWinControl.ReloadDockedControl
 0001:00032000       TWinControl.Remove
 0001:0003211C       TWinControl.RemoveControl
 0001:00031F94       TWinControl.RemoveFocus
 0001:00035328       TWinControl.Repaint
 0001:00033CA8       TWinControl.ResetIme
 0001:00034EFC       TWinControl.ScaleControls
 0001:00034FF0       TWinControl.ScrollBy
 0001:000358C8       TWinControl.SelectNext
 0001:00035558       TWinControl.SetBorderWidth
 0001:00034E24       TWinControl.SetBounds
 0001:0003593C       TWinControl.SetChildOrder
 0001:00035578       TWinControl.SetCtl3D
 0001:00034014       TWinControl.SetDockSite
 0001:000353B8       TWinControl.SetFocus
 0001:00033BBC       TWinControl.SetIme
 0001:000364A4       TWinControl.SetParentBackground
 0001:00032B6C       TWinControl.SetParentWindow
 0001:00035628       TWinControl.SetUseDockManager
 0001:000351B8       TWinControl.SetZOrder
 0001:000350E0       TWinControl.SetZOrderPosition
 0001:000350C8       TWinControl.ShowControl
 0001:0003530C       TWinControl.Update
 0001:000356A4       TWinControl.UpdateBounds
 0001:00032B2C       TWinControl.UpdateControlState
 0001:00032A30       TWinControl.UpdateShowing
 0001:000355CC       TWinControl.UpdateTabOrder
 0001:00036408       TWinControl.UpdateUIState
 0001:000344A0       TWinControl.WMChar
 0001:00034618       TWinControl.WMCharToItem
 0001:00033728       TWinControl.WMCommand
 0001:000337FC       TWinControl.WMCompareItem
 0001:0003639C       TWinControl.WMContextMenu
 0001:00033820       TWinControl.WMDeleteItem
 0001:0003468C       TWinControl.WMDestroy
 0001:00033844       TWinControl.WMDrawItem
 0001:0003388C       TWinControl.WMEraseBkgnd
 0001:0003379C       TWinControl.WMFontChange
 0001:000337BC       TWinControl.WMHScroll
 0001:00033BA8       TWinControl.WMIMEEndComp
 0001:00033B94       TWinControl.WMIMEStartComp
 0001:000342F4       TWinControl.WMKeyDown
 0001:000343DC       TWinControl.WMKeyUp
 0001:00033B80       TWinControl.WMKillFocus
 0001:00033868       TWinControl.WMMeasureItem
 0001:00033A58       TWinControl.WMMove
 0001:00036064       TWinControl.WMNCCalcSize
 0001:000346C0       TWinControl.WMNCDestroy
 0001:000346DC       TWinControl.WMNCHitTest
 0001:000360F4       TWinControl.WMNCPaint
 0001:00033748       TWinControl.WMNotify
 0001:000335C8       TWinControl.WMPaint
 0001:0003477C       TWinControl.WMPaletteChanged
 0001:00034638       TWinControl.WMParentNotify
 0001:0003646C       TWinControl.WMPrintClient
 0001:00034758       TWinControl.WMQueryNewPalette
 0001:00033A6C       TWinControl.WMSetCursor
 0001:00033B6C       TWinControl.WMSetFocus
 0001:00033A24       TWinControl.WMSize
 0001:0003376C       TWinControl.WMSysColorChange
 0001:00034570       TWinControl.WMSysCommand
 0001:00034320       TWinControl.WMSysKeyDown
 0001:000343FC       TWinControl.WMSysKeyUp
 0001:000337AC       TWinControl.WMTimeChange
 0001:0003466C       TWinControl.WMVKeyToItem
 0001:000337DC       TWinControl.WMVScroll
 0001:00033914       TWinControl.WMWindowPosChanged
 0001:000339D4       TWinControl.WMWindowPosChanging
 0001:00033788       TWinControl.WMWinIniChange
 0001:00032E4C       TWinControl.WndProc
 0001:00032638       TWinControl.WriteDesignSize
 0001:0003119C       TWinControlActionLink.AssignClient
 0001:000311C0       TWinControlActionLink.IsHelpContextLinked
 0001:000311C8       TWinControlActionLink.SetHelpContext
 0001:000298E0       TWinHelpViewer.CallWinHelp
 0001:0002943C       TWinHelpViewer.CanShowTableOfContents
 0001:00029B3C       TWinHelpViewer.CouldBeUnstableWindow
 0001:00029C40       TWinHelpViewer.Create
 0001:00029C88       TWinHelpViewer.Destroy
 0001:00029850       TWinHelpViewer.DisplayHelpByContext
 0001:000296C8       TWinHelpViewer.DisplayTopic
 0001:00029398       TWinHelpViewer.GetHelpStrings
 0001:0002930C       TWinHelpViewer.GetViewerName
 0001:00029214       TWinHelpViewer.HelpFile
 0001:000292E4       TWinHelpViewer.InternalShutDown
 0001:00029B38       TWinHelpViewer.IsBusyWindow
 0001:00029AB0       TWinHelpViewer.IsNewQuery
 0001:00029B58       TWinHelpViewer.MakeWinHelpHappy
 0001:00029610       TWinHelpViewer.NotifyID
 0001:00029BB4       TWinHelpViewer.RestartWinHelp
 0001:000294C8       TWinHelpViewer.ShowHelp
 0001:00029440       TWinHelpViewer.ShowTableOfContents
 0001:00029630       TWinHelpViewer.ShutDown
 0001:00029614       TWinHelpViewer.SoftShutDown
 0001:000297DC       TWinHelpViewer.UnderstandsContext
 0001:00029320       TWinHelpViewer.UnderstandsKeyword
 0001:00029660       TWinHelpViewer.UnderstandsTopic
 0001:000207E4       TwoBitsFromDIB
 0002:000000E8       TwoDigitYearCenturyWindow
 0001:0001B8B4       TWriter.Write
 0001:0001B918       TWriter.WriteBoolean
 0001:0001B900       TWriter.WriteBuffer
 0001:0001B92C       TWriter.WriteInteger
 0001:0001B9A0       TWriter.WriteListBegin
 0001:0001B9A8       TWriter.WriteListEnd
 0001:0001B9B0       TWriter.WriteMinStr
 0001:0001BA48       TWriter.WriteString
 0001:0001BA9C       TWriter.WriteValue
 0001:00005608       Types
 0001:0001376C       TypInfo
 0001:00050B5C       UInt32x32To64
 0001:0000021C       UnhandledExceptionFilter
 0001:0004CA90       UnhookHintHooks
 0001:00005FEC       UnhookWindowsHookEx
 0001:00004E24       UnicodeToUtf8
 0001:00000C60       UninitAllocator
 0001:0003DED4       UniqueCommand
 0001:000037D8       UniqueString
 0001:0000CBAC       UniUnimplemented
 0001:00006044       UnlockResource
 0001:00005B14       UnrealizeObject
 0001:00005FF4       UnregisterClass
 0001:00015E58       UnregisterFindGlobalComponentProc
 0001:00004C90       UnregisterModule
 0001:00015B14       UnRegisterModuleClasses
 0001:00002E3C       UnsetExceptionHandler
 0001:00001C98       UpCase
 0001:00021940       UpdateDIBColorTable
 0001:00030B24       UpdateFloatingDockSitePos
 0001:00040E44       UpdateItem
 0001:00041850       UpdateItem
 0001:00045E80       UpdateScrollProperties
 0001:00005FFC       UpdateWindow
 0001:000071BC       UpperCase
 0001:000271C8       UrlMon
 0002:00002AD8       UrlMonHandle
 0002:00002ADC       UrlMonInitialized
 0002:00002924       User32Dll
 0001:00026FE8       UseThemes
 0001:000050E4       UTF8Decode
 0001:00005038       UTF8Encode
 0001:00004F00       Utf8ToUnicode
 0002:0000040C       UtilWindowClass
 0001:00027064       UxTheme
 0001:0004EED4       ValidateHintWindow
 0001:0002C6F8       ValidDockTarget
 0002:00000B48       ValidMenuHotkeys
 0001:00045494       ValidParentForm
 0002:00000954       Values
 0002:0000095C       Values
 0002:000027B4       VarAdd
 0002:00000010       VarAddRefProc
 0002:000027CC       VarAnd
 0001:0000DF70       VarArrayClear
 0001:0000E210       VarArrayCopyForEach
 0001:0000DB10       VarArrayCreateError
 0002:000027F0       VarBoolFromStr
 0002:000027FC       VarBstrFromBool
 0002:000027F4       VarBstrFromCy
 0002:000027F8       VarBstrFromDate
 0001:0000E4E8       VarCastAsAny
 0001:0000E5EC       VarCastAsDispatch
 0001:0000E638       VarCastAsInterface
 0001:0000E554       VarCastAsOleStr
 0001:0000E5A0       VarCastAsString
 0001:0000D984       VarCastError
 0001:0000D930       VarCastError
 0001:0000E704       VarCastRare
 0001:0000E684       VarCastViaOS
 0001:0000E0EC       VarClearDeep
 0002:0000000C       VarClearProc
 0002:000027D8       VarCmp
 0001:0000E3F0       VarCopyCopyProc
 0001:0000E3F8       VarCopyDeep
 0002:00000014       VarCopyProc
 0002:000027EC       VarCyFromStr
 0002:000027E8       VarDateFromStr
 0001:000502BC       VarDispInvoke
 0002:00002814       VarDispProc
 0002:000027C0       VarDiv
 0002:000027DC       VarI4FromStr
 0001:0000CB74       VariantChangeType
 0002:000027A8       VariantChangeTypeEx
 0001:0000CB64       VariantClear
 0001:0000CB6C       VariantCopy
 0001:0000CB5C       VariantInit
 0001:00012DC0       Variants
 0002:000027C4       VarIDiv
 0001:0000DA20       VarInvalidOp
 0002:000027C8       VarMod
 0002:000027BC       VarMul
 0002:000027AC       VarNeg
 0002:000027B0       VarNot
 0002:000027D0       VarOr
 0001:0000DA74       VarOverflowError
 0002:000027E0       VarR4FromStr
 0002:000027E4       VarR8FromStr
 0001:0000DDB8       VarResultCheck
 0001:0000DDC4       VarResultCheck
 0002:000027B8       VarSub
 0001:0000FB44       VarToBoolAny
 0001:0000FA3C       VarToBoolAsString
 0001:0000FBA8       VarToBoolCustom
 0001:0000FB04       VarToBoolViaOS
 0001:00010D08       VarToCurrencyAny
 0001:00010C5C       VarToCurrencyAsDouble
 0001:00010BA0       VarToCurrencyAsString
 0001:00010D6C       VarToCurrencyCustom
 0001:00010CBC       VarToCurrencyViaOS
 0001:000107A0       VarToDateAny
 0001:000106F4       VarToDateAsDouble
 0001:00010608       VarToDateAsString
 0001:00010804       VarToDateCustom
 0001:00010754       VarToDateViaOS
 0001:0001004C       VarToDoubleAny
 0001:0000FF3C       VarToDoubleAsString
 0001:000100B0       VarToDoubleCustom
 0001:00010000       VarToDoubleViaOS
 0001:0000F540       VarToInt64Any
 0001:0000F440       VarToInt64AsString
 0001:0000F5AC       VarToInt64Custom
 0001:0000F394       VarToInt64ViaOS
 0001:0000EA8C       VarToIntAny
 0001:0000E99C       VarToIntAsString
 0001:0000EAF0       VarToIntCustom
 0001:0000EA50       VarToIntViaOS
 0001:00011384       VarToLStrAny
 0001:000113E8       VarToLStrCustom
 0002:00000018       VarToLStrProc
 0001:000112B8       VarToLStrViaOS
 0001:00011A60       VarToWStrAny
 0001:00011AC4       VarToWStrCustom
 0002:0000001C       VarToWStrProc
 0001:000119A8       VarToWStrViaOS
 0001:00012744       VarTypeAsText
 0001:0000D348       VarUtils
 0002:000027D4       VarXor
 0001:0000769C       VerifyBoolStrArray
 0001:0000595C       VerQueryValue
 0001:0005DF54       VideoRenderer
 0001:0005DC94       VidRenderer
 0002:00002B08       ViewerName
 0001:0000591C       VirtualAlloc
 0001:00000350       VirtualAlloc
 0001:00000358       VirtualFree
 0001:00005924       VirtualQuery
 0001:000002DC       VirtualQuery
 0001:00057F78       WaitDispatchingMessages
 0001:0000592C       WaitForMultipleObjects
 0001:00005934       WaitForSingleObject
 0001:0001BB08       WaitForSyncEvent
 0001:00006004       WaitMessage
 0002:000003F0       WakeMainThread
 0001:00003408       WCharFromChar
 0002:00000314       WesternGroups
 0001:000040B8       WideCharLenToStrVar
 0001:000002D4       WideCharToMultiByte
 0001:00058A78       WideCompareText
 0002:000000E0       Win32BuildNumber
 0001:0000BFC8       Win32Check
 0002:000000E4       Win32CSDVersion
 0002:000000D8       Win32MajorVersion
 0002:000000DC       Win32MinorVersion
 0001:00039D98       Win32NLSEnableIME
 0002:000000D4       Win32Platform
 0002:00002B24       WindowAtom
 0002:00002B28       WindowAtomString
 0002:00000D20       WindowClass
 0001:000299E0       WindowEnumerationTester
 0001:00006014       WindowFromPoint
 0002:00000AB8       WindowPos
 0001:000062A8       Windows
 0001:00020F6C       WinError
 0001:0000600C       WinHelp
 0002:00002B04       WinHelpTester
 0001:00029D2C       WinHelpViewer
 0001:00027190       WinInet
 0001:000261B4       WinSpool
 0001:000509E8       WMF9
 0002:00000740       WndProcPtrAtom
 0001:00038BCC       WriteControlName
 0001:00003124       WriteErrorMessage
 0001:0000593C       WriteFile
 0001:00000224       WriteFile
 0001:00020F7C       WriteIcon
 0001:00003978       WStrError
 0001:00003998       WStrSet
 0002:00000ED8       wszStreamName
 0001:00024F78       xEnumDisplayMonitors
 0001:00024CFC       xGetMonitorInfo
 0001:00024DD0       xGetMonitorInfoA
 0001:00024EA4       xGetMonitorInfoW
 0001:00024C64       xMonitorFromPoint
 0001:00024B3C       xMonitorFromRect
 0001:00024BCC       xMonitorFromWindow
 0001:0000603C       ZeroMemory
 0001:000060C8       _CreateWindowEx
 0002:0000296C       _FlatSB_GetScrollProp
 0002:00002970       _FlatSB_SetScrollProp
 0001:00024AB4       _GetSystemMetrics
 0002:00002B8C       _ImmGetCompositionString
 0002:00002B70       _ImmGetContext
 0002:00002B78       _ImmGetConversionStatus
 0002:00002B90       _ImmIsIME
 0002:00002B94       _ImmNotifyIME
 0002:00002B74       _ImmReleaseContext
 0002:00002B88       _ImmSetCompositionFont
 0002:00002B84       _ImmSetCompositionWindow
 0002:00002B7C       _ImmSetConversionStatus
 0002:00002B80       _ImmSetOpenStatus
 0002:00002974       _InitializeFlatSB
 0002:00002978       _UninitializeFlatSB
 0002:00002B6C       _WINNLSEnableIME


  Address         Publics by Value

 0002:FFBA1010       TlsLast
 0001:00000204       GetStdHandle
 0001:0000020C       RaiseException
 0001:00000214       RtlUnwind
 0001:0000021C       UnhandledExceptionFilter
 0001:00000224       WriteFile
 0001:0000022C       CharNext
 0001:00000234       ExitProcess
 0001:0000023C       MessageBox
 0001:00000244       FindClose
 0001:0000024C       FindFirstFile
 0001:00000254       FreeLibrary
 0001:0000025C       GetCommandLine
 0001:00000264       GetLocaleInfo
 0001:0000026C       GetModuleFileName
 0001:00000274       GetModuleHandle
 0001:0000027C       GetProcAddress
 0001:00000284       GetStartupInfo
 0001:0000028C       GetThreadLocale
 0001:00000294       LoadLibraryEx
 0001:0000029C       LoadString
 0001:000002A4       lstrcpyn
 0001:000002AC       @strlen
 0001:000002B4       MultiByteToWideChar
 0001:000002BC       RegCloseKey
 0001:000002C4       RegOpenKeyEx
 0001:000002CC       RegQueryValueEx
 0001:000002D4       WideCharToMultiByte
 0001:000002DC       VirtualQuery
 0001:000002E4       SysAllocStringLen
 0001:000002EC       SysReAllocStringLen
 0001:000002F4       SysFreeString
 0001:000002FC       InterlockedIncrement
 0001:00000304       InterlockedDecrement
 0001:0000030C       GetCurrentThreadId
 0001:00000314       GetVersion
 0001:0000031C       GetCmdShow
 0001:00000340       LocalAlloc
 0001:00000348       LocalFree
 0001:00000350       VirtualAlloc
 0001:00000358       VirtualFree
 0001:00000360       InitializeCriticalSection
 0001:00000368       EnterCriticalSection
 0001:00000370       LeaveCriticalSection
 0001:00000378       DeleteCriticalSection
 0001:00000380       GetBlockDesc
 0001:00000404       MakeEmpty
 0001:0000040C       AddBlockAfter
 0001:00000468       DeleteBlock
 0001:0000049C       MergeBlockAfter
 0001:00000524       RemoveBlock
 0001:000005E8       GetSpace
 0001:0000064C       GetSpaceAt
 0001:000006C4       FreeSpace
 0001:0000078C       Commit
 0001:0000084C       Decommit
 0001:00000908       GetCommitted
 0001:000009B0       GetCommittedAt
 0001:00000AF4       FreeCommitted
 0001:00000B88       InitAllocator
 0001:00000C60       UninitAllocator
 0001:00000D60       DeleteFree
 0001:00000DF4       FindCommitted
 0001:00000E38       FillBeforeGap
 0001:00000E74       InternalFreeMem
 0001:00000E98       FillAfterGap
 0001:00000EC0       FillerSizeBeforeGap
 0001:00000F38       FillerSizeAfterGap
 0001:00000F78       DecommitFree
 0001:00001034       InsertFree
 0001:0000112C       FreeCurAlloc
 0001:00001178       MergeCommit
 0001:00001204       NewCommit
 0001:00001230       NewCommitAt
 0001:00001264       SearchSmallBlocks
 0001:0000129C       TryHarder
 0001:000013E4       SysGetMem
 0001:00001590       SysFreeMem
 0001:00001768       ResizeInPlace
 0001:0000196C       SysReallocMem
 0001:00001A38       @GetMem
 0001:00001A68       @FreeMem
 0001:00001A88       @ReallocMem
 0001:00001AD8       ExceptObject
 0001:00001AF8       ExceptAddr
 0001:00001B24       AcquireExceptionObject
 0001:00001B60       RunErrorAt
 0001:00001B6C       ErrorAt
 0001:00001BB8       Error
 0001:00001BC4       @_IOTest
 0001:00001BE4       SetInOutRes
 0001:00001BF4       @Copy
 0001:00001C38       IOResult
 0001:00001C58       Move
 0001:00001C98       UpCase
 0001:00001CA4       Set8087CW
 0001:00001CB4       Get8087CW
 0001:00001CBC       @ROUND
 0001:00001CC8       @AbstractError
 0001:00001CE4       InternalFlush
 0001:00001D2C       Flush
 0001:00001D38       @Close
 0001:00001D90       @PStrNCpy
 0001:00001DAC       @PStrCmp
 0001:00001E30       @AStrCmp
 0001:00001EA0       @FillChar
 0001:00001EC0       @ValLong
 0001:00001F94       @_CToPasStr
 0001:00001FA0       @_CLenToPasStr
 0001:00001FC4       @SetEq
 0001:00001FD8       FPower10
 0001:00001FE0       @Pow10
 0001:000022C4       GetKeyboardType
 0001:000022CC       @isNECWindows
 0001:000022FC       @FpuMaskInit
 0001:000023C0       @FpuInit
 0001:000023CC       @BoundErr
 0001:000023D4       TObject.ClassType
 0001:000023E0       TObject.ClassName
 0001:000023F4       TObject.ClassNameIs
 0001:0000241C       TObject.ClassParent
 0001:00002428       TObject.NewInstance
 0001:00002444       TObject.FreeInstance
 0001:00002458       TObject.InstanceSize
 0001:00002460       TObject.Create
 0001:00002480       TObject.Destroy
 0001:00002490       TObject.Free
 0001:0000249C       TObject.InitInstance
 0001:000024F4       TObject.CleanupInstance
 0001:00002514       InvokeImplGetter
 0001:00002544       TObject.GetInterface
 0001:000025E4       TObject.GetInterfaceEntry
 0001:00002628       @IsClass
 0001:0000264C       @AsClass
 0001:00002668       GetDynaMethod
 0001:00002698       @CallDynaInst
 0001:000026B0       TObject.InheritsFrom
 0001:000026C4       TObject.ClassInfo
 0001:000026D4       TObject.SafeCallException
 0001:000026DC       TObject.DefaultHandler
 0001:000026E0       TObject.AfterConstruction
 0001:000026E4       TObject.BeforeDestruction
 0001:000026E8       TObject.Dispatch
 0001:00002710       TObject.MethodAddress
 0001:00002760       TObject.FieldAddress
 0001:000027B0       @ClassCreate
 0001:00002800       @ClassDestroy
 0001:00002808       @AfterConstruction
 0001:00002818       @BeforeDestruction
 0001:00002828       NotifyReRaise
 0001:00002844       NotifyNonDelphiException
 0001:00002868       NotifyExcept
 0001:00002880       NotifyOnExcept
 0001:00002894       NotifyAnyExcept
 0001:000028A8       CheckJmp
 0001:000028C8       NotifyExceptFinally
 0001:000028F0       NotifyTerminate
 0001:0000290C       NotifyUnhandled
 0001:0000292C       @HandleAnyException
 0001:00002A58       @HandleOnException
 0001:00002BE0       @HandleFinally
 0001:00002C18       @RaiseExcept
 0001:00002C40       @RaiseAgain
 0001:00002C94       @DoneExcept
 0001:00002CC4       @TryFinallyExit
 0001:00002CDC       MapToRunError
 0001:00002D7C       @ExceptionHandler
 0001:00002E1C       SetExceptionHandler
 0001:00002E3C       UnsetExceptionHandler
 0001:00002E64       FinalizeUnits
 0001:00002ED4       InitUnits
 0001:00002F44       @StartLib
 0001:0000300C       @InitResStrings
 0001:00003030       @InitResStringImports
 0001:00003058       @InitImports
 0001:0000307C       @InitWideStrings
 0001:00003098       MakeErrorMessage
 0001:000030F4       ExitDll
 0001:00003124       WriteErrorMessage
 0001:000031B0       @Halt0
 0001:00003290       @Halt
 0001:0000329C       @RunError
 0001:000032A8       @Assert
 0001:000032C8       @LStrClr
 0001:000032EC       @LStrArrayClr
 0001:0000331C       @LStrAsg
 0001:00003360       @LStrLAsg
 0001:0000338C       @NewAnsiString
 0001:000033B8       @LStrFromPCharLen
 0001:000033E8       CharFromWChar
 0001:00003408       WCharFromChar
 0001:00003424       @LStrFromPWCharLen
 0001:000034B0       @LStrFromChar
 0001:000034C0       @LStrFromPChar
 0001:000034F0       @LStrFromPWChar
 0001:0000352C       @LStrFromString
 0001:00003538       @LStrFromArray
 0001:00003550       @LStrFromWStr
 0001:00003564       @LStrToString
 0001:00003588       @LStrLen
 0001:00003590       @LStrCat
 0001:000035D4       @LStrCat3
 0001:00003648       @LStrCatN
 0001:000036D4       @LStrCmp
 0001:00003778       @LStrAddRef
 0001:00003788       @LStrToPChar
 0001:00003794       InternalUniqueString
 0001:000037D8       UniqueString
 0001:000037E0       @UniqueStringA
 0001:000037E8       @LStrCopy
 0001:00003828       @LStrDelete
 0001:00003870       @LStrInsert
 0001:000038CC       @LStrPos
 0001:00003914       @LStrSetLength
 0001:00003978       WStrError
 0001:00003980       @NewWideString
 0001:00003998       WStrSet
 0001:000039A8       @WStrClr
 0001:000039C0       @WStrArrayClr
 0001:000039E4       @WStrAsg
 0001:00003A08       @WStrFromPCharLen
 0001:00003A94       @WStrFromPWCharLen
 0001:00003AB8       @WStrFromPWChar
 0001:00003AF4       @WStrFromLStr
 0001:00003B04       @WStrToPWChar
 0001:00003B14       @WStrLen
 0001:00003B20       @WStrCmp
 0001:00003BA4       @WStrCopy
 0001:00003BF0       @WStrSetLength
 0001:00003C38       @WStrAddRef
 0001:00003C58       @InitializeRecord
 0001:00003C88       @InitializeArray
 0001:00003D1C       @Initialize
 0001:00003D28       @FinalizeRecord
 0001:00003D5C       @VarClr
 0001:00003D74       @FinalizeArray
 0001:00003E60       @Finalize
 0001:00003E6C       @VarCopy
 0001:00003E84       @CopyRecord
 0001:00003FA0       @CopyArray
 0001:00004094       @New
 0001:000040A8       @Dispose
 0001:000040B8       WideCharLenToStrVar
 0001:000040C4       OleStrToStrVar
 0001:000040E8       StringToOleStr
 0001:0000410C       @DispCallByIDError
 0001:00004114       @_llmul
 0001:00004138       @_lldiv
 0001:000041B4       @ValInt64
 0001:000043D8       @DynArrayLength
 0001:000043E0       @DynArrayHigh
 0001:000043E8       CopyArray
 0001:000043F8       FinalizeArray
 0001:00004400       DynArrayClear
 0001:00004408       DynArraySetLength
 0001:000045B4       @DynArraySetLength
 0001:000045C0       @DynArrayClear
 0001:000045FC       @DynArrayAsg
 0001:00004624       FindHInstance
 0001:0000464C       FindClassHInstance
 0001:00004654       DelayLoadResourceModule
 0001:0000469C       FindResourceHInstance
 0001:000046E4       FindBS
 0001:00004710       ToLongPath
 0001:000048E8       LoadResourceModule
 0001:00004B6C       AddModuleUnloadProc
 0001:00004B74       RemoveModuleUnloadProc
 0001:00004B7C       AddModuleUnloadProc
 0001:00004B9C       RemoveModuleUnloadProc
 0001:00004C24       NotifyModuleUnload
 0001:00004C80       RegisterModule
 0001:00004C90       UnregisterModule
 0001:00004D14       @IntfClear
 0001:00004D2C       @IntfCopy
 0001:00004D58       @IntfCast
 0001:00004D88       @IntfAddRef
 0001:00004D94       TInterfacedObject.AfterConstruction
 0001:00004DA0       TInterfacedObject.BeforeDestruction
 0001:00004DB0       TInterfacedObject.NewInstance
 0001:00004DC0       TInterfacedObject.QueryInterface
 0001:00004DE8       TInterfacedObject._AddRef
 0001:00004DFC       TInterfacedObject._Release
 0001:00004E24       UnicodeToUtf8
 0001:00004F00       Utf8ToUnicode
 0001:00005038       UTF8Encode
 0001:000050E4       UTF8Decode
 0001:00005188       AnsiToUtf8
 0001:000051D8       LoadResString
 0001:00005230       LCIDToCodePage
 0001:000052A4       Finalization
 0001:000052F8       System
 0001:000053CC       LocalAlloc
 0001:000053D4       LocalFree
 0001:000053DC       TlsAlloc
 0001:000053E4       TlsFree
 0001:000053EC       TlsGetValue
 0001:000053F4       TlsSetValue
 0001:000053FC       AllocTlsBuffer
 0001:00005408       GetTlsSize
 0001:00005410       InitThreadTLS
 0001:00005454       InitProcessTLS
 0001:00005480       ExitThreadTLS
 0001:000054A8       ExitProcessTLS
 0001:000054CC       @GetTls
 0001:0000550C       InitializeModule
 0001:00005518       @InitLib
 0001:00005560       Finalization
 0001:00005590       SysInit
 0001:00005598       Rect
 0001:000055B4       Point
 0001:000055BC       Bounds
 0001:000055D8       Finalization
 0001:00005608       Types
 0001:000056DC       RegCloseKey
 0001:000056E4       RegCreateKeyEx
 0001:000056EC       RegDeleteKey
 0001:000056F4       RegOpenKeyEx
 0001:000056FC       RegQueryValueEx
 0001:00005704       RegSetValueEx
 0001:0000570C       CloseHandle
 0001:00005714       CompareString
 0001:0000571C       CompareStringA
 0001:00005724       CompareStringW
 0001:0000572C       CreateEvent
 0001:00005734       CreateFile
 0001:0000573C       CreateThread
 0001:00005744       DeleteCriticalSection
 0001:0000574C       EnterCriticalSection
 0001:00005754       EnumCalendarInfoA
 0001:0000575C       FindResource
 0001:00005764       FormatMessage
 0001:0000576C       FreeLibrary
 0001:00005774       InterlockedDecrement
 0001:0000577C       InterlockedExchange
 0001:00005784       InterlockedIncrement
 0001:0000578C       FreeResource
 0001:00005794       GetACP
 0001:0000579C       GetCPInfo
 0001:000057A4       GetCurrentProcessId
 0001:000057AC       GetCurrentThread
 0001:000057B4       GetCurrentThreadId
 0001:000057BC       GetDateFormat
 0001:000057C4       GetDiskFreeSpaceA
 0001:000057CC       GetFullPathName
 0001:000057D4       GetLastError
 0001:000057DC       GetLocalTime
 0001:000057E4       GetLocaleInfo
 0001:000057EC       GetModuleFileName
 0001:000057F4       GetModuleHandle
 0001:000057FC       GetProcAddress
 0001:00005804       GetStdHandle
 0001:0000580C       GetStringTypeEx
 0001:00005814       GetSystemInfo
 0001:0000581C       GetThreadLocale
 0001:00005824       GetThreadPriority
 0001:0000582C       GetTickCount
 0001:00005834       GetVersion
 0001:0000583C       GetVersionEx
 0001:00005844       GlobalAddAtom
 0001:0000584C       GlobalAlloc
 0001:00005854       GlobalDeleteAtom
 0001:0000585C       GlobalFindAtom
 0001:00005864       GlobalFree
 0001:0000586C       GlobalLock
 0001:00005874       GlobalHandle
 0001:0000587C       GlobalReAlloc
 0001:00005884       GlobalUnlock
 0001:0000588C       InitializeCriticalSection
 0001:00005894       LeaveCriticalSection
 0001:0000589C       LoadLibrary
 0001:000058A4       LoadResource
 0001:000058AC       LockResource
 0001:000058B4       MulDiv
 0001:000058BC       MultiByteToWideChar
 0001:000058C4       ReadFile
 0001:000058CC       ResetEvent
 0001:000058D4       SetEndOfFile
 0001:000058DC       SetErrorMode
 0001:000058E4       SetEvent
 0001:000058EC       SetFilePointer
 0001:000058F4       SetLastError
 0001:000058FC       SetThreadLocale
 0001:00005904       SetThreadPriority
 0001:0000590C       SizeofResource
 0001:00005914       Sleep
 0001:0000591C       VirtualAlloc
 0001:00005924       VirtualQuery
 0001:0000592C       WaitForMultipleObjects
 0001:00005934       WaitForSingleObject
 0001:0000593C       WriteFile
 0001:00005944       lstrcpy
 0001:0000594C       GetFileVersionInfo
 0001:00005954       GetFileVersionInfoSize
 0001:0000595C       VerQueryValue
 0001:00005964       BitBlt
 0001:0000596C       CreateBitmap
 0001:00005974       CreateBrushIndirect
 0001:0000597C       CreateCompatibleBitmap
 0001:00005984       CreateCompatibleDC
 0001:0000598C       CreateDIBSection
 0001:00005994       CreateDIBitmap
 0001:0000599C       CreateFontIndirect
 0001:000059A4       CreateHalftonePalette
 0001:000059AC       CreatePalette
 0001:000059B4       CreatePenIndirect
 0001:000059BC       CreateSolidBrush
 0001:000059C4       DeleteDC
 0001:000059CC       DeleteObject
 0001:000059D4       ExcludeClipRect
 0001:000059DC       GetBitmapBits
 0001:000059E4       GetBrushOrgEx
 0001:000059EC       GetClipBox
 0001:000059F4       GetCurrentPositionEx
 0001:000059FC       GetDCOrgEx
 0001:00005A04       GetDIBColorTable
 0001:00005A0C       GetDIBits
 0001:00005A14       GetDeviceCaps
 0001:00005A1C       GetObject
 0001:00005A24       GetPaletteEntries
 0001:00005A2C       GetPixel
 0001:00005A34       GetStockObject
 0001:00005A3C       GetSystemPaletteEntries
 0001:00005A44       GetTextExtentPoint32
 0001:00005A4C       GetTextMetrics
 0001:00005A54       GetWindowOrgEx
 0001:00005A5C       IntersectClipRect
 0001:00005A64       LineTo
 0001:00005A6C       MaskBlt
 0001:00005A74       MoveToEx
 0001:00005A7C       PatBlt
 0001:00005A84       RealizePalette
 0001:00005A8C       RectVisible
 0001:00005A94       RestoreDC
 0001:00005A9C       SaveDC
 0001:00005AA4       SelectObject
 0001:00005AAC       SelectPalette
 0001:00005AB4       SetBkColor
 0001:00005ABC       SetBkMode
 0001:00005AC4       SetBrushOrgEx
 0001:00005ACC       SetDIBColorTable
 0001:00005AD4       SetPixel
 0001:00005ADC       SetROP2
 0001:00005AE4       SetStretchBltMode
 0001:00005AEC       SetTextColor
 0001:00005AF4       SetViewportOrgEx
 0001:00005AFC       SetWindowOrgEx
 0001:00005B04       StretchBlt
 0001:00005B0C       StretchDIBits
 0001:00005B14       UnrealizeObject
 0001:00005B1C       ActivateKeyboardLayout
 0001:00005B24       AdjustWindowRectEx
 0001:00005B2C       AnsiLower
 0001:00005B34       BeginPaint
 0001:00005B3C       CallNextHookEx
 0001:00005B44       CallWindowProc
 0001:00005B4C       CharNext
 0001:00005B54       CharToOemA
 0001:00005B5C       CheckMenuItem
 0001:00005B64       ClientToScreen
 0001:00005B6C       CreateIcon
 0001:00005B74       CreateMenu
 0001:00005B7C       CreatePopupMenu
 0001:00005B84       DefFrameProc
 0001:00005B8C       DefMDIChildProc
 0001:00005B94       DefWindowProc
 0001:00005B9C       DeleteMenu
 0001:00005BA4       DestroyCursor
 0001:00005BAC       DestroyIcon
 0001:00005BB4       DestroyMenu
 0001:00005BBC       DestroyWindow
 0001:00005BC4       DispatchMessage
 0001:00005BCC       DrawEdge
 0001:00005BD4       DrawFrameControl
 0001:00005BDC       DrawIcon
 0001:00005BE4       DrawIconEx
 0001:00005BEC       DrawMenuBar
 0001:00005BF4       DrawText
 0001:00005BFC       EnableMenuItem
 0001:00005C04       EnableScrollBar
 0001:00005C0C       EnableWindow
 0001:00005C14       EndPaint
 0001:00005C1C       EnumThreadWindows
 0001:00005C24       EnumWindows
 0001:00005C2C       EqualRect
 0001:00005C34       FillRect
 0001:00005C3C       FindWindow
 0001:00005C44       FrameRect
 0001:00005C4C       GetActiveWindow
 0001:00005C54       GetCapture
 0001:00005C5C       GetClassInfo
 0001:00005C64       GetClassName
 0001:00005C6C       GetClientRect
 0001:00005C74       GetCursor
 0001:00005C7C       GetCursorPos
 0001:00005C84       GetDC
 0001:00005C8C       GetDCEx
 0001:00005C94       GetDesktopWindow
 0001:00005C9C       GetFocus
 0001:00005CA4       GetForegroundWindow
 0001:00005CAC       GetIconInfo
 0001:00005CB4       GetKeyNameText
 0001:00005CBC       GetKeyState
 0001:00005CC4       GetKeyboardLayout
 0001:00005CCC       GetKeyboardLayoutList
 0001:00005CD4       GetKeyboardState
 0001:00005CDC       GetLastActivePopup
 0001:00005CE4       GetMenu
 0001:00005CEC       GetMenuItemCount
 0001:00005CF4       GetMenuItemID
 0001:00005CFC       GetMenuItemInfo
 0001:00005D04       GetMenuState
 0001:00005D0C       GetMenuString
 0001:00005D14       GetNextWindow
 0001:00005D1C       GetParent
 0001:00005D24       GetProp
 0001:00005D2C       GetQueueStatus
 0001:00005D34       GetScrollInfo
 0001:00005D3C       GetScrollPos
 0001:00005D44       GetScrollRange
 0001:00005D4C       GetSubMenu
 0001:00005D54       GetSysColor
 0001:00005D5C       GetSysColorBrush
 0001:00005D64       GetSystemMenu
 0001:00005D6C       GetSystemMetrics
 0001:00005D74       GetTopWindow
 0001:00005D7C       GetWindow
 0001:00005D84       GetWindowDC
 0001:00005D8C       GetWindowLong
 0001:00005D94       GetWindowPlacement
 0001:00005D9C       GetWindowRect
 0001:00005DA4       GetWindowText
 0001:00005DAC       GetWindowThreadProcessId
 0001:00005DB4       GetWindowThreadProcessId
 0001:00005DBC       InSendMessage
 0001:00005DC4       InflateRect
 0001:00005DCC       InsertMenu
 0001:00005DD4       InsertMenuItem
 0001:00005DDC       IntersectRect
 0001:00005DE4       InvalidateRect
 0001:00005DEC       IsChild
 0001:00005DF4       IsDialogMessage
 0001:00005DFC       IsIconic
 0001:00005E04       IsRectEmpty
 0001:00005E0C       IsWindow
 0001:00005E14       IsWindowEnabled
 0001:00005E1C       IsWindowVisible
 0001:00005E24       IsZoomed
 0001:00005E2C       KillTimer
 0001:00005E34       LoadBitmap
 0001:00005E3C       LoadCursor
 0001:00005E44       LoadIcon
 0001:00005E4C       LoadKeyboardLayout
 0001:00005E54       LoadString
 0001:00005E5C       MapVirtualKey
 0001:00005E64       MapWindowPoints
 0001:00005E6C       MessageBox
 0001:00005E74       MoveWindow
 0001:00005E7C       MsgWaitForMultipleObjects
 0001:00005E84       OemToAnsi
 0001:00005E8C       OffsetRect
 0001:00005E94       PeekMessage
 0001:00005E9C       PostMessage
 0001:00005EA4       PostQuitMessage
 0001:00005EAC       PostThreadMessage
 0001:00005EB4       PtInRect
 0001:00005EBC       RedrawWindow
 0001:00005EC4       RegisterClass
 0001:00005ECC       RegisterClipboardFormat
 0001:00005ED4       RegisterWindowMessage
 0001:00005EDC       ReleaseCapture
 0001:00005EE4       ReleaseDC
 0001:00005EEC       RemoveMenu
 0001:00005EF4       RemoveProp
 0001:00005EFC       ScreenToClient
 0001:00005F04       ScrollWindow
 0001:00005F0C       SendMessage
 0001:00005F14       SetActiveWindow
 0001:00005F1C       SetCapture
 0001:00005F24       SetClassLong
 0001:00005F2C       SetCursor
 0001:00005F34       SetFocus
 0001:00005F3C       SetForegroundWindow
 0001:00005F44       SetMenu
 0001:00005F4C       SetMenuItemInfo
 0001:00005F54       SetParent
 0001:00005F5C       SetProp
 0001:00005F64       SetRect
 0001:00005F6C       SetScrollInfo
 0001:00005F74       SetScrollPos
 0001:00005F7C       SetScrollRange
 0001:00005F84       SetTimer
 0001:00005F8C       SetWindowLong
 0001:00005F94       SetWindowPlacement
 0001:00005F9C       SetWindowPos
 0001:00005FA4       SetWindowsHookEx
 0001:00005FAC       ShowCursor
 0001:00005FB4       ShowOwnedPopups
 0001:00005FBC       ShowScrollBar
 0001:00005FC4       ShowWindow
 0001:00005FCC       SystemParametersInfo
 0001:00005FD4       TrackPopupMenu
 0001:00005FDC       TranslateMDISysAccel
 0001:00005FE4       TranslateMessage
 0001:00005FEC       UnhookWindowsHookEx
 0001:00005FF4       UnregisterClass
 0001:00005FFC       UpdateWindow
 0001:00006004       WaitMessage
 0001:0000600C       WinHelp
 0001:00006014       WindowFromPoint
 0001:0000601C       MakeLong
 0001:00006028       HiWord
 0001:0000602C       GetCurrentTime
 0001:00006034       CopyMemory
 0001:0000603C       ZeroMemory
 0001:00006044       UnlockResource
 0001:00006048       GlobalAllocPtr
 0001:00006058       GlobalReAllocPtr
 0001:00006074       GlobalFreePtr
 0001:00006088       MakeROP4
 0001:00006094       SmallPointToPoint
 0001:000060A8       PointToSmallPoint
 0001:000060C0       MakeWParam
 0001:000060C8       _CreateWindowEx
 0001:000060D0       CreateWindowEx
 0001:00006128       CreateWindow
 0001:00006180       HwndMSWheel
 0001:00006278       Finalization
 0001:000062A8       Windows
 0001:00006588       Finalization
 0001:000065B8       SysConst
 0001:0000715C       DivMod
 0001:00007178       ConvertErrorFmt
 0001:0000719C       AllocMem
 0001:000071BC       UpperCase
 0001:0000720C       LowerCase
 0001:0000725C       CompareStr
 0001:0000728C       CompareMem
 0001:000072AC       CompareText
 0001:00007300       SameText
 0001:00007324       AnsiCompareStr
 0001:0000735C       AnsiCompareText
 0001:00007394       AnsiSameText
 0001:000073AC       AnsiStrLIComp
 0001:000073CC       Trim
 0001:0000741C       IsValidIdent
 0001:00007480       CvtInt
 0001:000074CC       IntToStr
 0001:000074EC       CvtInt64
 0001:000075B8       IntToStr
 0001:000075E0       IntToHex
 0001:00007608       StrToInt
 0001:00007644       StrToIntDef
 0001:0000765C       TryStrToInt
 0001:0000767C       TryStrToInt64
 0001:0000769C       VerifyBoolStrArray
 0001:0000772C       CompareWith
 0001:00007768       TryStrToBool
 0001:00007804       BoolToStr
 0001:00007850       FileOpen
 0001:000078A8       FileCreate
 0001:000078CC       FileCreate
 0001:000078D4       FileRead
 0001:00007900       FileWrite
 0001:0000792C       FileSeek
 0001:00007964       FileClose
 0001:0000796C       AnsiLastChar
 0001:000079A4       LastDelimiter
 0001:000079F4       ExtractFileName
 0001:00007A2C       ExpandFileName
 0001:00007A68       BackfillGetDiskFreeSpaceEx
 0001:00007AE8       StrLen
 0001:00007B00       StrEnd
 0001:00007B14       StrMove
 0001:00007B24       StrCopy
 0001:00007B4C       StrLCopy
 0001:00007B80       StrPCopy
 0001:00007BAC       StrPLCopy
 0001:00007BD4       StrComp
 0001:00007BF8       StrIComp
 0001:00007C38       StrLIComp
 0001:00007C7C       StrScan
 0001:00007C9C       StrPos
 0001:00007CF0       StrAlloc
 0001:00007D04       StrBufSize
 0001:00007D18       StrNew
 0001:00007D4C       StrDispose
 0001:00007D5C       FormatError
 0001:00007DB4       FormatVarToStr
 0001:00007DD8       FormatClearStr
 0001:00007DE4       FormatBuf
 0001:0000815C       StrFmt
 0001:000081A8       StrLFmt
 0001:000081F4       Format
 0001:00008208       FmtStr
 0001:000082D0       PutExponent
 0001:00008314       FloatToText
 0001:000085E8       FloatToDecimal
 0001:00008814       TextToFloat
 0001:00008928       FloatToStr
 0001:00008958       CurrToStr
 0001:00008988       TryStrToFloat
 0001:000089A4       TryStrToFloat
 0001:000089D0       TryStrToFloat
 0001:000089FC       TryStrToCurr
 0001:00008A18       DateTimeToTimeStamp
 0001:00008A5C       TryEncodeTime
 0001:00008ACC       DecodeTime
 0001:00008B28       IsLeapYear
 0001:00008B64       TryEncodeDate
 0001:00008C34       DecodeDateFully
 0001:00008D84       DecodeDate
 0001:00008DA4       DayOfWeek
 0001:00008DCC       CurrentYear
 0001:00008DE0       AppendChars
 0001:00008E24       AppendString
 0001:00008E44       AppendNumber
 0001:00008E90       GetCount
 0001:00008EC0       GetDate
 0001:00008EF8       GetTime
 0001:00008F38       ConvertEraString
 0001:000090A4       ConvertYearString
 0001:000091AC       AppendFormat
 0001:00009984       DateTimeToString
 0001:000099E0       DateTimeToStr
 0001:000099F4       ScanBlanks
 0001:00009A18       ScanNumber
 0001:00009AAC       ScanString
 0001:00009B38       ScanChar
 0001:00009B70       GetDateOrder
 0001:00009BBC       ScanToNumber
 0001:00009C04       GetEraYearOffset
 0001:00009C58       EraToYear
 0001:00009CB4       ScanDate
 0001:00009FF8       ScanTime
 0001:0000A1EC       TryStrToDate
 0001:0000A220       TryStrToTime
 0001:0000A254       TryStrToDateTime
 0001:0000A2E0       SysErrorMessage
 0001:0000A32C       GetLocaleStr
 0001:0000A378       GetLocaleChar
 0001:0000A3A0       LocalGetLocaleStr
 0001:0000A3DC       GetMonthDayNames
 0001:0000A500       EnumEraNames
 0001:0000A53C       EnumEraYearOffsets
 0001:0000A5B4       GetEraNamesAndYearOffsets
 0001:0000A664       TranslateDateFormat
 0001:0000A88C       ConvertAddr
 0001:0000A898       ExceptionErrorMessage
 0001:0000AA30       ShowException
 0001:0000AAF8       Exception.Create
 0001:0000AB34       Exception.CreateFmt
 0001:0000ABB4       Exception.CreateRes
 0001:0000ABF0       Exception.CreateResFmt
 0001:0000AC84       Exception.CreateHelp
 0001:0000ACCC       EHeapException.FreeInstance
 0001:0000ACF8       CreateInOutError
 0001:0000AD78       ErrorHandler
 0001:0000ADCC       CreateAssertException
 0001:0000AE78       RaiseAssertException
 0001:0000AE88       AssertErrorHandler
 0001:0000AEA4       AbstractErrorHandler
 0001:0000AEBC       MapException
 0001:0000AF3C       GetExceptionClass
 0001:0000AF54       CreateAVObject
 0001:0000B128       GetExceptionObject
 0001:0000B1F4       ExceptHandler
 0001:0000B204       InitExceptions
 0001:0000B288       DoneExceptions
 0001:0000B308       InitPlatformId
 0001:0000B378       CheckWin32Version
 0001:0000B398       GetFileVersion
 0001:0000B484       ByteTypeTest
 0001:0000B4FC       ByteType
 0001:0000B520       StrByteType
 0001:0000B538       ByteToCharLen
 0001:0000B560       ByteToCharIndex
 0001:0000B5BC       CountChars
 0001:0000B64C       CharToByteIndex
 0001:0000B6B0       CharToByteLen
 0001:0000B710       StrCharLength
 0001:0000B730       StrNextChar
 0001:0000B744       CharLength
 0001:0000B780       NextCharIndex
 0001:0000B7BC       AnsiPos
 0001:0000B7F8       AnsiStrPos
 0001:0000B8B8       AnsiStrRScan
 0001:0000B900       AnsiStrScan
 0001:0000B948       LCIDToCodePage
 0001:0000B9BC       InitLeadBytes
 0001:0000BA1C       IsWesternGroup
 0001:0000BA34       InitSysLocale
 0001:0000BBAC       GetFormatSettings
 0001:0000BF24       Sleep
 0001:0000BF2C       RaiseLastOSError
 0001:0000BFC8       Win32Check
 0001:0000BFD8       CallTerminateProcs
 0001:0000C004       FreeTerminateProcs
 0001:0000C030       InitDriveSpacePtr
 0001:0000C08C       InterlockedIncrement
 0001:0000C098       InterlockedDecrement
 0001:0000C0A4       InterlockedExchange
 0001:0000C0AC       InterlockedExchangeAdd
 0001:0000C0B4       TThreadLocalCounter.Destroy
 0001:0000C120       TThreadLocalCounter.HashIndex
 0001:0000C138       TThreadLocalCounter.Open
 0001:0000C1CC       TThreadLocalCounter.Delete
 0001:0000C1DC       TThreadLocalCounter.Recycle
 0001:0000C230       TMultiReadExclusiveWriteSynchronizer.Create
 0001:0000C2A4       TMultiReadExclusiveWriteSynchronizer.Destroy
 0001:0000C2EC       TMultiReadExclusiveWriteSynchronizer.BlockReaders
 0001:0000C2F8       TMultiReadExclusiveWriteSynchronizer.UnblockReaders
 0001:0000C304       TMultiReadExclusiveWriteSynchronizer.UnblockOneWriter
 0001:0000C310       TMultiReadExclusiveWriteSynchronizer.WaitForReadSignal
 0001:0000C320       TMultiReadExclusiveWriteSynchronizer.WaitForWriteSignal
 0001:0000C330       TMultiReadExclusiveWriteSynchronizer.BeginWrite
 0001:0000C3DC       TMultiReadExclusiveWriteSynchronizer.EndWrite
 0001:0000C42C       TMultiReadExclusiveWriteSynchronizer.BeginRead
 0001:0000C49C       TMultiReadExclusiveWriteSynchronizer.EndRead
 0001:0000C504       FreeAndNil
 0001:0000C514       Supports
 0001:0000C538       Supports
 0001:0000C5D0       SafeLoadLibrary
 0001:0000C924       Finalization
 0001:0000CAA4       SysUtils
 0001:0000CB24       Finalization
 0001:0000CB54       Messages
 0001:0000CB5C       VariantInit
 0001:0000CB64       VariantClear
 0001:0000CB6C       VariantCopy
 0001:0000CB74       VariantChangeType
 0001:0000CB7C       BackupVariantChangeTypeEx
 0001:0000CBAC       UniUnimplemented
 0001:0000CBB8       BiUnimplemented
 0001:0000CBC4       CmpUnimplemented
 0001:0000CBD0       BackupVarI4FromStr
 0001:0000CC3C       BackupVarR4FromStr
 0001:0000CCA8       BackupVarR8FromStr
 0001:0000CD14       BackupVarDateFromStr
 0001:0000CD80       BackupVarCyFromStr
 0001:0000CDEC       BackupVarBoolFromStr
 0001:0000CE6C       BackupVarBStrFromCy
 0001:0000CEDC       BackupVarBStrFromDate
 0001:0000CF4C       BackupVarBStrFromBool
 0001:0000CFC0       SafeArrayCreate
 0001:0000CFC8       SafeArrayGetLBound
 0001:0000CFD0       SafeArrayGetUBound
 0001:0000CFD8       SafeArrayPtrOfIndex
 0001:0000CFE0       FindProc
 0001:0000D00C       InitializeVarUtils
 0001:0000D318       Finalization
 0001:0000D348       VarUtils
 0001:0000D930       VarCastError
 0001:0000D984       VarCastError
 0001:0000DA20       VarInvalidOp
 0001:0000DA74       VarOverflowError
 0001:0000DB10       VarArrayCreateError
 0001:0000DB64       TranslateResult
 0001:0000DDB8       VarResultCheck
 0001:0000DDC4       VarResultCheck
 0001:0000DDF8       HandleConversionException
 0001:0000DE7C       @DispInvokeError
 0001:0000DED0       @VarNull
 0001:0000DEE4       InBounds
 0001:0000DF14       Increment
 0001:0000DF70       VarArrayClear
 0001:0000E0EC       VarClearDeep
 0001:0000E168       @VarClear
 0001:0000E17C       @VarClr
 0001:0000E184       InBounds
 0001:0000E1B4       Increment
 0001:0000E210       VarArrayCopyForEach
 0001:0000E3F0       VarCopyCopyProc
 0001:0000E3F8       VarCopyDeep
 0001:0000E4A4       @VarCopy
 0001:0000E4E8       VarCastAsAny
 0001:0000E554       VarCastAsOleStr
 0001:0000E5A0       VarCastAsString
 0001:0000E5EC       VarCastAsDispatch
 0001:0000E638       VarCastAsInterface
 0001:0000E684       VarCastViaOS
 0001:0000E704       VarCastRare
 0001:0000E770       @VarCast
 0001:0000E99C       VarToIntAsString
 0001:0000EA50       VarToIntViaOS
 0001:0000EA8C       VarToIntAny
 0001:0000EAF0       VarToIntCustom
 0001:0000EB34       @VarToInteger
 0001:0000EF84       @VarToShortInt
 0001:0000F034       @VarToByte
 0001:0000F0DC       @VarToSmallInt
 0001:0000F1D4       @VarToWord
 0001:0000F2AC       @VarToLongWord
 0001:0000F394       VarToInt64ViaOS
 0001:0000F440       VarToInt64AsString
 0001:0000F540       VarToInt64Any
 0001:0000F5AC       VarToInt64Custom
 0001:0000F5F8       @VarToInt64
 0001:0000FA3C       VarToBoolAsString
 0001:0000FB04       VarToBoolViaOS
 0001:0000FB44       VarToBoolAny
 0001:0000FBA8       VarToBoolCustom
 0001:0000FBF4       @VarToBoolean
 0001:0000FF3C       VarToDoubleAsString
 0001:00010000       VarToDoubleViaOS
 0001:0001004C       VarToDoubleAny
 0001:000100B0       VarToDoubleCustom
 0001:000100FC       @VarToDouble
 0001:00010478       @VarToSingle
 0001:00010608       VarToDateAsString
 0001:000106F4       VarToDateAsDouble
 0001:00010754       VarToDateViaOS
 0001:000107A0       VarToDateAny
 0001:00010804       VarToDateCustom
 0001:00010850       @VarToDate
 0001:00010BA0       VarToCurrencyAsString
 0001:00010C5C       VarToCurrencyAsDouble
 0001:00010CBC       VarToCurrencyViaOS
 0001:00010D08       VarToCurrencyAny
 0001:00010D6C       VarToCurrencyCustom
 0001:00010DB8       @VarToCurrency
 0001:00011184       CurrToWStrViaOS
 0001:000111BC       DateToWStrViaOS
 0001:000111F4       BoolToWStrViaOS
 0001:000112B8       VarToLStrViaOS
 0001:00011384       VarToLStrAny
 0001:000113E8       VarToLStrCustom
 0001:0001146C       @VarToLStr
 0001:000119A8       VarToWStrViaOS
 0001:00011A60       VarToWStrAny
 0001:00011AC4       VarToWStrCustom
 0001:00011B8C       @VarToWStr
 0001:000120E0       AnyToIntf
 0001:00012158       @VarToIntf
 0001:00012224       @VarToDisp
 0001:000122D0       @VarFromInt
 0001:0001230C       @VarFromInteger
 0001:0001232C       @VarFromByte
 0001:0001234C       @VarFromWord
 0001:0001236C       @VarFromLongWord
 0001:0001238C       @VarFromShortInt
 0001:000123AC       @VarFromSmallInt
 0001:000123CC       @VarFromInt64
 0001:000123F8       @VarFromSingle
 0001:0001241C       @VarFromDouble
 0001:00012448       @VarFromCurrency
 0001:00012474       @VarFromDate
 0001:000124A0       @VarFromBool
 0001:000124C8       @VarFromReal
 0001:000124DC       @VarFromTDateTime
 0001:000124F0       @VarFromCurr
 0001:00012504       @VarFromLStr
 0001:00012530       @VarFromWStr
 0001:00012568       @VarFromIntf
 0001:00012594       @VarFromDisp
 0001:000125C0       @VarAddRef
 0001:00012744       VarTypeAsText
 0001:000128B4       SetVarAsError
 0001:000128CC       SetClearVarToEmptyParam
 0001:000128FC       ClearVariantTypeList
 0001:00012968       TCustomVariantType.BinaryOp
 0001:00012974       TCustomVariantType.Cast
 0001:000129AC       TCustomVariantType.CastTo
 0001:000129F4       TCustomVariantType.Compare
 0001:00012A00       TCustomVariantType.CompareOp
 0001:00012A38       TCustomVariantType.CastToOle
 0001:00012A74       TCustomVariantType.Destroy
 0001:00012B00       TCustomVariantType.IsClear
 0001:00012B04       TCustomVariantType.LeftPromotion
 0001:00012B18       TCustomVariantType.OlePromotion
 0001:00012B20       TCustomVariantType.RaiseCastError
 0001:00012B28       TCustomVariantType.RaiseInvalidOp
 0001:00012B30       TCustomVariantType.RaiseDispError
 0001:00012B38       TCustomVariantType.RightPromotion
 0001:00012B4C       TCustomVariantType.UnaryOp
 0001:00012B54       TCustomVariantType.DispInvoke
 0001:00012B60       TCustomVariantType._AddRef
 0001:00012B6C       TCustomVariantType._Release
 0001:00012B78       TCustomVariantType.QueryInterface
 0001:00012BA0       FindCustomVariantType
 0001:00012C58       FindCustomVariantType
 0001:00012D40       Null
 0001:00012D48       Finalization
 0001:00012DC0       Variants
 0001:00012F54       Finalization
 0001:00012F84       RTLConsts
 0001:00012FB8       GetTypeData
 0001:00012FC4       GetEnumNameValue
 0001:00013010       GetEnumValue
 0001:00013074       GetPropInfo
 0001:000130E4       GetOrdProp
 0001:00013158       SetOrdProp
 0001:000131B4       SetShortStrProp
 0001:00013208       SetShortStrPropAsLongStr
 0001:0001323C       AssignLongStr
 0001:00013250       SetLongStrProp
 0001:00013290       SetWideStrPropAsLongStr
 0001:000132E8       SetStrProp
 0001:00013314       SetWideStrProp
 0001:000133E8       SetFloatProp
 0001:000135E0       AssignVariant
 0001:000135F4       SetVariantProp
 0001:00013634       SetMethodProp
 0001:0001366C       SetInt64Prop
 0001:000136A8       SetInterfaceProp
 0001:0001371C       Finalization
 0001:0001376C       TypInfo
 0001:00013840       IsEqualGUID
 0001:00013848       CoInitialize
 0001:00013850       CoUninitialize
 0001:00013858       CoLockObjectExternal
 0001:00013860       CoCreateInstance
 0001:00013868       StringFromCLSID
 0001:00013870       CoTaskMemAlloc
 0001:00013878       CoTaskMemFree
 0001:00013880       SysFreeString
 0001:00013888       LoadTypeLib
 0001:00013890       LoadRegTypeLib
 0001:00013898       GetErrorInfo
 0001:000138A0       Succeeded
 0001:000138AC       Failed
 0001:000138B8       Finalization
 0001:000138E8       ActiveX
 0001:00014EC8       Point
 0001:00014EE0       SmallPoint
 0001:00014EF0       Rect
 0001:00014F18       Bounds
 0001:00014F40       InvalidPoint
 0001:00015004       TRegGroup.AddClass
 0001:00015010       TRegGroup.BestClass
 0001:00015070       TRegGroup.BestGroup
 0001:000150E0       TRegGroup.Create
 0001:0001515C       TRegGroup.Destroy
 0001:0001519C       TRegGroup.GetClass
 0001:000151FC       TRegGroup.InGroup
 0001:00015240       TRegGroup.RegisterClass
 0001:000152E8       TRegGroup.Registered
 0001:00015300       PointerInModule
 0001:00015320       TRegGroup.UnregisterModuleClasses
 0001:000153C4       TRegGroups.Activate
 0001:00015410       TRegGroups.Create
 0001:00015484       TRegGroups.Destroy
 0001:000154E0       TRegGroups.FindGroup
 0001:00015524       TRegGroups.GetClass
 0001:00015568       Error
 0001:000155F8       TRegGroups.GroupWith
 0001:000156C0       TRegGroups.Lock
 0001:000156CC       TRegGroups.RegisterClass
 0001:000156E4       TRegGroups.Registered
 0001:00015728       TRegGroups.StartGroup
 0001:00015778       TRegGroups.Unlock
 0001:00015784       TRegGroups.UnregisterModuleClasses
 0001:000157D4       TClassFinder.Create
 0001:00015900       TClassFinder.Destroy
 0001:00015930       TClassFinder.GetClass
 0001:000159B8       GetFieldClassTable
 0001:000159C4       ClassNotFound
 0001:00015A30       GetClass
 0001:00015A84       FindClass
 0001:00015AA4       RegisterClass
 0001:00015B14       UnRegisterModuleClasses
 0001:00015B60       StartClassGroup
 0001:00015BAC       GroupDescendentsWith
 0001:00015C00       ActivateClassGroup
 0001:00015CB4       TIntConst.Create
 0001:00015CEC       RegisterIntegerConsts
 0001:00015D18       FindIdentToInt
 0001:00015D94       IdentToInt
 0001:00015DD4       IntToIdent
 0001:00015E18       RegisterFindGlobalComponentProc
 0001:00015E58       UnregisterFindGlobalComponentProc
 0001:00015E70       FindGlobalComponent
 0001:00015EB0       IsUniqueGlobalComponentName
 0001:00015ED4       InternalReadComponentRes
 0001:00015F58       BeginGlobalLoading
 0001:00015FB0       NotifyGlobalLoading
 0001:00015FE0       EndGlobalLoading
 0001:0001603C       InitComponent
 0001:000160E4       InitInheritedComponent
 0001:000161A8       TList.Destroy
 0001:000161C8       TList.Add
 0001:000161FC       TList.Clear
 0001:00016214       TList.Delete
 0001:00016274       ReturnAddr
 0001:00016278       TList.Error
 0001:000162B0       TList.Error
 0001:00016304       TList.Expand
 0001:0001631C       TList.First
 0001:00016324       TList.Get
 0001:0001634C       TList.Grow
 0001:00016380       TList.IndexOf
 0001:000163A0       TList.Insert
 0001:0001640C       TList.Last
 0001:00016418       TList.Put
 0001:00016468       TList.Remove
 0001:00016488       TList.SetCapacity
 0001:000164C4       TList.SetCount
 0001:00016534       TList.Notify
 0001:00016538       TThreadList.Create
 0001:0001658C       TThreadList.Destroy
 0001:00016608       TThreadList.Add
 0001:00016690       TThreadList.LockList
 0001:000166A4       TThreadList.Remove
 0001:000166F4       TThreadList.UnlockList
 0001:00016700       TBits.Destroy
 0001:00016730       TBits.Error
 0001:00016748       Min
 0001:00016754       TBits.SetSize
 0001:000167F8       TBits.SetBit
 0001:00016824       TBits.OpenBit
 0001:0001689C       TPersistent.Destroy
 0001:000168C8       TPersistent.Assign
 0001:000168DC       TPersistent.AssignError
 0001:000169AC       TPersistent.AssignTo
 0001:000169B4       TPersistent.DefineProperties
 0001:000169B8       TPersistent.GetNamePath
 0001:00016A68       TPersistent.GetOwner
 0001:00016A6C       TInterfacedPersistent.AfterConstruction
 0001:00016ABC       TInterfacedPersistent._AddRef
 0001:00016ADC       TInterfacedPersistent._Release
 0001:00016AFC       TInterfacedPersistent.QueryInterface
 0001:00016B24       TCollection.Add
 0001:00016B44       TCollection.Clear
 0001:00016BAC       TStrings.Destroy
 0001:00016BDC       TStrings.Add
 0001:00016C00       TStrings.AddObject
 0001:00016C24       TStrings.AddStrings
 0001:00016CDC       TStrings.Assign
 0001:00016D74       TStrings.BeginUpdate
 0001:00016D8C       DoWrite
 0001:00016DE4       TStrings.DefineProperties
 0001:00016E30       TStrings.EndUpdate
 0001:00016E44       TStrings.Equals
 0001:00016EEC       ReturnAddr
 0001:00016EF0       TStrings.Error
 0001:00016F28       TStrings.Error
 0001:00016F80       TStrings.Exchange
 0001:00017068       TStrings.GetCapacity
 0001:00017070       TStrings.GetObject
 0001:00017074       TStrings.GetText
 0001:000170C8       TStrings.GetTextStr
 0001:000171F0       TStrings.IndexOf
 0001:0001727C       TStrings.IndexOfName
 0001:00017350       TStrings.IndexOfObject
 0001:00017384       TStrings.InsertObject
 0001:000173B4       TStrings.LoadFromFile
 0001:00017408       TStrings.LoadFromStream
 0001:000174B4       TStrings.Move
 0001:00017564       TStrings.Put
 0001:00017598       TStrings.PutObject
 0001:0001759C       TStrings.ReadData
 0001:0001764C       TStrings.SaveToFile
 0001:000176A4       TStrings.SaveToStream
 0001:00017700       TStrings.SetCapacity
 0001:00017704       TStrings.SetStringsAdapter
 0001:00017738       TStrings.SetText
 0001:00017788       TStrings.SetTextStr
 0001:00017848       TStrings.SetUpdateState
 0001:0001784C       TStrings.WriteData
 0001:000178D0       TStrings.CompareStrings
 0001:000178DC       TStrings.GetNameValueSeparator
 0001:000178F4       TStrings.SetNameValueSeparator
 0001:00017910       TStringList.Destroy
 0001:0001796C       TStringList.Add
 0001:00017978       TStringList.AddObject
 0001:000179DC       TStringList.Changed
 0001:000179F8       TStringList.Changing
 0001:00017A14       TStringList.Clear
 0001:00017A54       TStringList.Delete
 0001:00017AC0       TStringList.Exchange
 0001:00017B1C       TStringList.ExchangeItems
 0001:00017B40       TStringList.Find
 0001:00017BB8       TStringList.Get
 0001:00017BEC       TStringList.GetCapacity
 0001:00017BF0       TStringList.GetCount
 0001:00017BF4       TStringList.GetObject
 0001:00017C1C       TStringList.Grow
 0001:00017C50       TStringList.IndexOf
 0001:00017C8C       TStringList.Insert
 0001:00017C9C       TStringList.InsertObject
 0001:00017CF0       TStringList.InsertItem
 0001:00017D68       TStringList.Put
 0001:00017DC4       TStringList.PutObject
 0001:00017E04       TStringList.QuickSort
 0001:00017E98       TStringList.SetCapacity
 0001:00017EB4       TStringList.SetSorted
 0001:00017ED4       TStringList.SetUpdateState
 0001:00017EEC       StringListCompareStrings
 0001:00017F00       TStringList.Sort
 0001:00017F10       TStringList.CustomSort
 0001:00017F48       TStringList.CompareStrings
 0001:00017F64       TStream.GetPosition
 0001:00017F84       TStream.SetPosition
 0001:00017F98       TStream.GetSize
 0001:00017FE4       TStream.SetSize
 0001:00017FE8       TStream.SetSize64
 0001:00017FFC       TStream.SetSize
 0001:00018050       RaiseException
 0001:0001809C       TStream.Seek
 0001:00018120       TStream.Seek
 0001:00018190       TStream.ReadBuffer
 0001:000181C8       TStream.WriteBuffer
 0001:00018200       TStream.CopyFrom
 0001:000182F4       TStream.ReadComponent
 0001:00018354       THandleStream.Create
 0001:00018390       THandleStream.Read
 0001:000183A0       THandleStream.Write
 0001:000183B0       THandleStream.Seek
 0001:000183DC       THandleStream.SetSize
 0001:000183F0       THandleStream.SetSize
 0001:00018418       TFileStream.Create
 0001:0001845C       TFileStream.Create
 0001:000185B0       TFileStream.Destroy
 0001:000185E4       TCustomMemoryStream.SetPointer
 0001:000185EC       TCustomMemoryStream.Read
 0001:00018624       TCustomMemoryStream.Seek
 0001:00018648       TMemoryStream.Destroy
 0001:00018674       TMemoryStream.Clear
 0001:0001868C       TMemoryStream.LoadFromStream
 0001:000186C4       TMemoryStream.SetCapacity
 0001:000186EC       TMemoryStream.SetSize
 0001:00018718       TMemoryStream.Realloc
 0001:000187A4       TMemoryStream.Write
 0001:000187F4       TResourceStream.Create
 0001:0001884C       Error
 0001:000188BC       TResourceStream.Initialize
 0001:00018928       TResourceStream.Destroy
 0001:00018960       TResourceStream.Write
 0001:00018978       TFiler.Create
 0001:000189C0       TFiler.Destroy
 0001:000189E8       TFiler.SetRoot
 0001:00018AC4       TPropFixup.Create
 0001:00018B1C       TPropFixup.MakeGlobalReference
 0001:00018B64       TPropFixup.ResolveReference
 0001:00018B74       TPropIntfFixup.ResolveReference
 0001:00018BF8       FindNestedComponent
 0001:00018CC0       AddFinished
 0001:00018CF8       AddNotFinished
 0001:00018D40       GlobalFixupReferences
 0001:00018EE8       RemoveFixupReferences
 0001:00018F94       RemoveFixups
 0001:00019018       ReadError
 0001:00019030       PropValueError
 0001:0001903C       PropertyNotFound
 0001:00019068       EnumValue
 0001:00019080       TReader.Destroy
 0001:000190BC       TReader.CheckValue
 0001:000190E0       TReader.DefineProperty
 0001:00019114       TReader.DefineBinaryProperty
 0001:000191F0       TReader.EndOfList
 0001:00019204       TReader.Error
 0001:00019224       TReader.FindMethod
 0001:0001928C       RemoveGlobalFixup
 0001:00019308       TReader.DoFixupReferences
 0001:00019428       TReader.FlushBuffer
 0001:0001944C       TReader.FreeFixups
 0001:00019488       TReader.GetFieldClass
 0001:0001951C       TReader.GetPosition
 0001:00019534       TReader.NextValue
 0001:00019544       TReader.PropertyError
 0001:00019558       TReader.Read
 0001:000195A4       TReader.ReadBuffer
 0001:000195E0       TReader.ReadBoolean
 0001:000195F4       TReader.ReadChar
 0001:0001964C       TReader.ReadCollection
 0001:0001971C       AddSubComponentsToLoaded
 0001:00019758       CheckSubComponents
 0001:000197D0       SetSubComponentState
 0001:00019838       ComponentCreated
 0001:00019858       Recover
 0001:000198B8       CreateComponent
 0001:000199C8       SetCompName
 0001:00019A68       FindExistingComponent
 0001:00019B0C       TReader.ReadComponent
 0001:00019D48       TReader.ReadData
 0001:00019DB8       TReader.ReadDataInner
 0001:00019E88       TReader.ReadFloat
 0001:00019ECC       TReader.ReadSingle
 0001:00019F10       TReader.ReadCurrency
 0001:00019F60       TReader.ReadDate
 0001:00019FA4       TReader.ReadIdent
 0001:0001A0A4       TReader.ReadInteger
 0001:0001A110       TReader.ReadInt64
 0001:0001A154       TReader.ReadListBegin
 0001:0001A15C       TReader.ReadListEnd
 0001:0001A164       TReader.ReadPrefix
 0001:0001A1A4       HandleException
 0001:0001A2A4       PropPathError
 0001:0001A2C0       TReader.ReadProperty
 0001:0001A4A0       SetIntIdent
 0001:0001A4E8       SetObjectIdent
 0001:0001A528       SetVariantReference
 0001:0001A584       SetInterfaceReference
 0001:0001A644       TReader.ReadPropValue
 0001:0001A94C       FindUniqueName
 0001:0001A9AC       TReader.ReadRootComponent
 0001:0001ACD8       TReader.ReadSet
 0001:0001AD94       TReader.ReadSignature
 0001:0001ADB8       TReader.ReadStr
 0001:0001ADF4       TReader.ReadString
 0001:0001AEB0       TReader.ReadWideString
 0001:0001AF94       TReader.ReadValue
 0001:0001AFA8       TReader.SkipSetBody
 0001:0001AFF0       SkipList
 0001:0001B018       SkipBinary
 0001:0001B048       SkipCollection
 0001:0001B0A4       TReader.SkipValue
 0001:0001B240       TReader.SkipProperty
 0001:0001B288       TReader.SkipComponent
 0001:0001B330       TReader.FindAncestorComponent
 0001:0001B3E8       TReader.ReferenceName
 0001:0001B400       TReader.SetName
 0001:0001B428       TReader.FindComponentClass
 0001:0001B49C       TReader.SkipBytes
 0001:0001B4E4       ReadCustomVariant
 0001:0001B6AC       TReader.ReadVariant
 0001:0001B8B4       TWriter.Write
 0001:0001B900       TWriter.WriteBuffer
 0001:0001B918       TWriter.WriteBoolean
 0001:0001B92C       TWriter.WriteInteger
 0001:0001B9A0       TWriter.WriteListBegin
 0001:0001B9A8       TWriter.WriteListEnd
 0001:0001B9B0       TWriter.WriteMinStr
 0001:0001BA48       TWriter.WriteString
 0001:0001BA9C       TWriter.WriteValue
 0001:0001BAB0       InitThreadSynchronization
 0001:0001BAE4       DoneThreadSynchronization
 0001:0001BAFC       ResetSyncEvent
 0001:0001BB08       WaitForSyncEvent
 0001:0001BB24       CheckSynchronize
 0001:0001BCC4       TComponent.Create
 0001:0001BD10       TComponent.Destroy
 0001:0001BD88       TComponent.BeforeDestruction
 0001:0001BD94       TComponent.FreeNotification
 0001:0001BDE8       TComponent.ReadLeft
 0001:0001BDFC       TComponent.ReadTop
 0001:0001BE10       TComponent.WriteLeft
 0001:0001BE1C       TComponent.WriteTop
 0001:0001BE28       TComponent.Insert
 0001:0001BE54       TComponent.Remove
 0001:0001BE7C       TComponent.InsertComponent
 0001:0001BED4       TComponent.RemoveComponent
 0001:0001BF0C       TComponent.DestroyComponents
 0001:0001BF64       TComponent.Destroying
 0001:0001BFA0       TComponent.RemoveNotification
 0001:0001BFC4       TComponent.RemoveFreeNotification
 0001:0001BFE0       TComponent.Notification
 0001:0001C03C       TComponent.DefineProperties
 0001:0001C0C4       TComponent.HasParent
 0001:0001C0C8       TComponent.GetChildren
 0001:0001C0D0       TComponent.GetChildOwner
 0001:0001C0D4       TComponent.GetChildParent
 0001:0001C0D8       TComponent.GetNamePath
 0001:0001C0EC       TComponent.GetOwner
 0001:0001C0F0       TComponent.SetChildOrder
 0001:0001C0F4       TComponent.GetParentComponent
 0001:0001C0F8       TComponent.SetParentComponent
 0001:0001C0FC       TComponent.Updating
 0001:0001C108       TComponent.Updated
 0001:0001C114       TComponent.Loaded
 0001:0001C120       TComponent.PaletteCreated
 0001:0001C124       TComponent.ReadState
 0001:0001C12C       TComponent.WriteState
 0001:0001C134       TComponent.ValidateRename
 0001:0001C1B4       TComponent.ValidateContainer
 0001:0001C1C8       TComponent.ValidateInsert
 0001:0001C1CC       TComponent.FindComponent
 0001:0001C21C       TComponent.SetName
 0001:0001C2A8       TComponent.ChangeName
 0001:0001C2BC       TComponent.GetComponent
 0001:0001C2E8       TComponent.GetComponentCount
 0001:0001C2F8       TComponent.SetComponentIndex
 0001:0001C34C       TComponent.SetDesigning
 0001:0001C39C       TComponent.SetReference
 0001:0001C3E4       TComponent.ExecuteAction
 0001:0001C40C       TComponent.UpdateAction
 0001:0001C434       TComponent.SafeCallException
 0001:0001C44C       TComponent.UpdateRegistry
 0001:0001C454       TComponent.QueryInterface
 0001:0001C494       TComponent._AddRef
 0001:0001C4B4       TComponent._Release
 0001:0001C4D4       TComponent.IntfGetComponent
 0001:0001C4D8       TBasicActionLink.Create
 0001:0001C51C       TBasicActionLink.AssignClient
 0001:0001C520       TBasicActionLink.Destroy
 0001:0001C554       TBasicActionLink.Change
 0001:0001C56C       TBasicActionLink.Execute
 0001:0001C588       TBasicActionLink.SetAction
 0001:0001C5B4       TBasicActionLink.IsOnExecuteLinked
 0001:0001C5B8       TBasicActionLink.SetOnExecute
 0001:0001C5C0       TBasicActionLink.Update
 0001:0001C5CC       TBasicAction.Create
 0001:0001C610       TBasicAction.Destroy
 0001:0001C668       TBasicAction.HandlesTarget
 0001:0001C66C       TBasicAction.ExecuteTarget
 0001:0001C670       TBasicAction.Notification
 0001:0001C698       TBasicAction.UpdateTarget
 0001:0001C69C       TBasicAction.Execute
 0001:0001C6B8       TBasicAction.Update
 0001:0001C6D4       TBasicAction.SetOnExecute
 0001:0001C730       TBasicAction.Change
 0001:0001C744       TBasicAction.RegisterChanges
 0001:0001C750       TBasicAction.UnRegisterChanges
 0001:0001C790       TBasicAction.SetActionComponent
 0001:0001C7BC       TStreamAdapter.Create
 0001:0001C804       TStreamAdapter.Destroy
 0001:0001C83C       TStreamAdapter.Read
 0001:0001C8A4       TStreamAdapter.Write
 0001:0001C90C       TStreamAdapter.Seek
 0001:0001C990       TStreamAdapter.SetSize
 0001:0001C9F4       TStreamAdapter.CopyTo
 0001:0001CBF4       TStreamAdapter.Commit
 0001:0001CC00       TStreamAdapter.Revert
 0001:0001CC0C       TStreamAdapter.LockRegion
 0001:0001CC18       TStreamAdapter.UnlockRegion
 0001:0001CC24       TStreamAdapter.Stat
 0001:0001CCA0       TStreamAdapter.Clone
 0001:0001CCB8       FreeIntConstList
 0001:0001CD24       ModuleUnload
 0001:0001CD2C       StdWndProc
 0001:0001CD4C       CalcJmpOffset
 0001:0001CD54       MakeObjectInstance
 0001:0001CDEC       FreeObjectInstance
 0001:0001CE10       AllocateHWnd
 0001:0001CEC4       DeallocateHWnd
 0001:0001CEEC       Finalization
 0001:0001CF9C       Classes
 0001:0001D030       Min
 0001:0001D038       Min
 0001:0001D078       Max
 0001:0001D080       Finalization
 0001:0001D0B0       Math
 0001:0001D310       Finalization
 0001:0001D340       Consts
 0001:0001DFF8       InternalDeletePalette
 0001:0001E06C       GetHashCode
 0001:0001E080       TResourceManager.Create
 0001:0001E0BC       TResourceManager.Destroy
 0001:0001E0E0       TResourceManager.Lock
 0001:0001E0EC       TResourceManager.Unlock
 0001:0001E0F8       TResourceManager.AllocResource
 0001:0001E1DC       TResourceManager.FreeResource
 0001:0001E298       TResourceManager.ChangeResource
 0001:0001E314       TResourceManager.AssignResource
 0001:0001E384       ClearColor
 0001:0001E400       PaletteChanged
 0001:0001E8EC       ColorToRGB
 0001:0001E8FC       ColorToIdent
 0001:0001E90C       IdentToColor
 0001:0001E91C       TGraphicsObject.Changed
 0001:0001E930       TGraphicsObject.Lock
 0001:0001E940       TGraphicsObject.Unlock
 0001:0001EB04       CharsetToIdent
 0001:0001EB14       IdentToCharset
 0001:0001EB24       GetFontData
 0001:0001EBD8       TFont.Create
 0001:0001EC2C       TFont.Destroy
 0001:0001EC54       TFont.Changed
 0001:0001EC70       TFont.Assign
 0001:0001ED44       TFont.GetData
 0001:0001ED5C       TFont.SetData
 0001:0001EDAC       TFont.SetColor
 0001:0001EDC0       TFont.GetHandle
 0001:0001EF68       TFont.SetHandle
 0001:0001EF8C       TFont.GetHeight
 0001:0001EF94       TFont.SetHeight
 0001:0001EFBC       TFont.GetName
 0001:0001EFD4       TFont.SetName
 0001:0001F030       TFont.GetSize
 0001:0001F04C       TFont.SetSize
 0001:0001F06C       TFont.GetStyle
 0001:0001F078       TFont.SetStyle
 0001:0001F0A4       TFont.GetPitch
 0001:0001F0AC       TFont.SetPitch
 0001:0001F0D4       TFont.GetCharset
 0001:0001F0DC       TFont.SetCharset
 0001:0001F104       TPen.Create
 0001:0001F148       TPen.Destroy
 0001:0001F170       TPen.Assign
 0001:0001F228       TPen.GetData
 0001:0001F240       TPen.SetData
 0001:0001F290       TPen.GetColor
 0001:0001F298       TPen.SetColor
 0001:0001F2C0       TPen.GetHandle
 0001:0001F358       TPen.SetMode
 0001:0001F36C       TPen.GetStyle
 0001:0001F374       TPen.SetStyle
 0001:0001F39C       TPen.GetWidth
 0001:0001F3A4       TPen.SetWidth
 0001:0001F3D0       TBrush.Create
 0001:0001F410       TBrush.Destroy
 0001:0001F438       TBrush.Assign
 0001:0001F4E0       TBrush.GetData
 0001:0001F4FC       TBrush.SetData
 0001:0001F54C       TBrush.SetBitmap
 0001:0001F570       TBrush.GetColor
 0001:0001F578       TBrush.SetColor
 0001:0001F5AC       TBrush.GetHandle
 0001:0001F68C       TBrush.GetStyle
 0001:0001F694       TBrush.SetStyle
 0001:0001F6C8       TCanvas.Create
 0001:0001F78C       TCanvas.Destroy
 0001:0001F7E8       TCanvas.CopyRect
 0001:0001F870       TCanvas.Draw
 0001:0001F91C       TCanvas.FillRect
 0001:0001F958       TCanvas.LineTo
 0001:0001F990       TCanvas.Lock
 0001:0001F9B8       TCanvas.MoveTo
 0001:0001F9E4       TCanvas.StretchDraw
 0001:0001FA20       TCanvas.TextExtent
 0001:0001FA64       TCanvas.TextWidth
 0001:0001FA80       TCanvas.TextHeight
 0001:0001FAA0       TCanvas.TryLock
 0001:0001FAFC       TCanvas.Unlock
 0001:0001FB24       TCanvas.SetFont
 0001:0001FB34       TCanvas.SetPen
 0001:0001FB40       TCanvas.SetBrush
 0001:0001FB4C       TCanvas.GetPenPos
 0001:0001FB70       TCanvas.SetPenPos
 0001:0001FB90       TCanvas.GetPixel
 0001:0001FBBC       TCanvas.SetPixel
 0001:0001FC04       TCanvas.GetHandle
 0001:0001FC24       TCanvas.DeselectHandles
 0001:0001FC80       TCanvas.CreateHandle
 0001:0001FC84       TCanvas.SetHandle
 0001:0001FCD8       TCanvas.RequiredState
 0001:0001FD4C       TCanvas.Changing
 0001:0001FD60       TCanvas.Changed
 0001:0001FD74       TCanvas.CreateFont
 0001:0001FDA0       TCanvas.CreatePen
 0001:0001FDD0       TCanvas.CreateBrush
 0001:0001FE4C       TCanvas.FontChanged
 0001:0001FE6C       TCanvas.PenChanged
 0001:0001FE8C       TCanvas.BrushChanged
 0001:0001FEAC       InvalidOperation
 0001:0001FEC4       InvalidGraphic
 0001:0001FEDC       InvalidBitmap
 0001:0001FEE8       InvalidIcon
 0001:0001FEF4       OutOfResources
 0001:0001FF48       GDIError
 0001:0001FFF0       GDICheck
 0001:00020000       DupBits
 0001:00020160       GetDInColors
 0001:00020180       BytesPerScanline
 0001:00020194       TransparentStretchBlt
 0001:00020428       RGBTripleToQuad
 0001:00020470       RGBQuadToTriple
 0001:000204E4       ByteSwapColors
 0001:0002053C       CreateSystemPalette
 0001:00020654       SystemPaletteOverride
 0001:000206EC       PaletteFromDIBColorTable
 0001:00020790       PaletteToDIBColorTable
 0001:000207E4       TwoBitsFromDIB
 0001:000209A8       AdjustColor
 0001:000209B4       BetterSize
 0001:00020A44       ReadIcon
 0001:00020D58       InitializeBitmapInfoHeader
 0001:00020E3C       InternalGetDIBSizes
 0001:00020EA0       GetDIBSizes
 0001:00020EA8       InternalGetDIB
 0001:00020F58       GetDIB
 0001:00020F6C       WinError
 0001:00020F70       CheckBool
 0001:00020F7C       WriteIcon
 0001:00021178       TGraphic.Create
 0001:000211B0       TGraphic.Changed
 0001:000211C8       DoWrite
 0001:00021220       TGraphic.DefineProperties
 0001:0002126C       TGraphic.Equals
 0001:000213B4       TGraphic.GetPalette
 0001:000213B8       TGraphic.GetTransparent
 0001:000213BC       TGraphic.LoadFromFile
 0001:00021410       TGraphic.Progress
 0001:00021438       TGraphic.ReadData
 0001:00021444       TGraphic.SaveToFile
 0001:0002149C       TGraphic.SetPalette
 0001:000214A0       TGraphic.SetTransparent
 0001:000214B0       TGraphic.WriteData
 0001:00021558       FreeMemoryContexts
 0001:00021604       DeselectBitmap
 0001:00021680       TBitmapCanvas.Create
 0001:000216BC       TBitmapCanvas.Destroy
 0001:000216E8       TBitmapCanvas.FreeContext
 0001:00021788       TBitmapCanvas.CreateHandle
 0001:00021874       TSharedImage.Reference
 0001:00021878       TSharedImage.Release
 0001:00021898       TBitmapImage.Destroy
 0001:000218F4       TBitmapImage.FreeHandle
 0001:00021940       UpdateDIBColorTable
 0001:000219FC       FixupBitFields
 0001:00021A48       CopyBitmap
 0001:000220AC       CopyPalette
 0001:00022110       CopyBitmapAsMask
 0001:0002231C       TBitmap.Create
 0001:00022384       TBitmap.Destroy
 0001:000223C0       TBitmap.Assign
 0001:000224B8       TBitmap.CopyImage
 0001:00022578       TBitmap.Changing
 0001:0002259C       TBitmap.Changed
 0001:000225A8       TBitmap.Dormant
 0001:0002261C       TBitmap.Draw
 0001:0002286C       TBitmap.FreeImage
 0001:000228D0       TBitmap.GetEmpty
 0001:000228EC       TBitmap.GetCanvas
 0001:00022934       TBitmap.GetHandle
 0001:00022958       TBitmap.GetHandleType
 0001:00022984       TBitmap.GetHeight
 0001:00022994       TBitmap.GetMaskHandle
 0001:000229A8       TBitmap.GetMonochrome
 0001:000229C4       TBitmap.GetPalette
 0001:000229D8       TBitmap.GetTransparentColor
 0001:00022A20       TBitmap.GetWidth
 0001:00022A28       TBitmap.DIBNeeded
 0001:00022A9C       TBitmap.FreeContext
 0001:00022AAC       TBitmap.HandleNeeded
 0001:00022B4C       TBitmap.MaskHandleNeeded
 0001:00022BAC       TBitmap.PaletteNeeded
 0001:00022C64       TBitmap.LoadFromClipboardFormat
 0001:00022CE8       TBitmap.LoadFromStream
 0001:00022D0C       TBitmap.NewImage
 0001:00022E0C       TBitmap.ReadData
 0001:00022E34       TBitmap.ReadDIB
 0001:0002339C       TBitmap.ReadStream
 0001:0002340C       TBitmap.SetHandle
 0001:000234D0       TBitmap.SetHandleType
 0001:00023608       TBitmap.SetHeight
 0001:0002365C       TBitmap.SetMonochrome
 0001:000236DC       TBitmap.SetPalette
 0001:000237B0       TBitmap.SetWidth
 0001:00023804       TBitmap.WriteData
 0001:0002380C       TBitmap.WriteStream
 0001:00023AC4       TBitmap.SaveToStream
 0001:00023ACC       TBitmap.SaveToClipboardFormat
 0001:00023B6C       TIconImage.Destroy
 0001:00023B9C       TIconImage.FreeHandle
 0001:00023BB4       TIcon.Create
 0001:00023C08       TIcon.Destroy
 0001:00023C38       TIcon.Assign
 0001:00023C98       TIcon.Draw
 0001:00023CD8       TIcon.GetEmpty
 0001:00023CF0       TIcon.GetHandle
 0001:00023D04       TIcon.GetHeight
 0001:00023D18       TIcon.GetWidth
 0001:00023D2C       TIcon.HandleNeeded
 0001:00023DA4       TIcon.ImageNeeded
 0001:00023E58       TIcon.LoadFromStream
 0001:00023F10       TIcon.NewImage
 0001:00023F84       TIcon.SetHandle
 0001:00023F9C       TIcon.SetHeight
 0001:00023FB4       TIcon.SetTransparent
 0001:00023FB8       TIcon.SetWidth
 0001:00023FD0       TIcon.SaveToStream
 0001:00023FF8       TIcon.LoadFromClipboardFormat
 0001:0002400C       TIcon.SaveToClipboardFormat
 0001:00024020       InitScreenLogPixels
 0001:00024058       GetDefFontCharSet
 0001:0002409C       InitDefFontData
 0001:00024168       TPatternManager.Create
 0001:000241A0       TPatternManager.Destroy
 0001:000241CC       TPatternManager.Lock
 0001:000241D8       TPatternManager.Unlock
 0001:000241E4       TPatternManager.AllocPattern
 0001:00024298       TPatternManager.CreateBitmap
 0001:00024398       TPatternManager.FreePatterns
 0001:00024418       AllocPatternBitmap
 0001:00024450       Finalization
 0001:00024524       Graphics
 0001:00024750       TObjectList.Create
 0001:0002478C       TObjectList.GetItem
 0001:000247A0       TObjectList.Insert
 0001:000247A8       TObjectList.Notify
 0001:000247D4       TOrderedList.Pop
 0001:000247DC       TOrderedList.Push
 0001:000247EC       TOrderedList.Create
 0001:00024830       TOrderedList.Destroy
 0001:00024860       TOrderedList.PeekItem
 0001:00024874       TOrderedList.PopItem
 0001:00024894       TStack.PushItem
 0001:000248A0       Finalization
 0001:000248D0       Contnrs
 0001:000248D8       ImageList_Create
 0001:000248E0       ImageList_Destroy
 0001:000248E8       ImageList_GetImageCount
 0001:000248F0       ImageList_Add
 0001:000248F8       ImageList_ReplaceIcon
 0001:00024900       ImageList_SetBkColor
 0001:00024908       ImageList_GetBkColor
 0001:00024910       ImageList_AddIcon
 0001:0002491C       ImageList_Draw
 0001:00024924       ImageList_DrawEx
 0001:0002492C       ImageList_Remove
 0001:00024934       ImageList_BeginDrag
 0001:0002493C       ImageList_EndDrag
 0001:00024944       ImageList_DragEnter
 0001:0002494C       ImageList_DragLeave
 0001:00024954       ImageList_DragMove
 0001:0002495C       ImageList_SetDragCursorImage
 0001:00024964       ImageList_DragShowNolock
 0001:0002496C       ImageList_GetDragImage
 0001:00024974       ImageList_Read
 0001:0002497C       ImageList_Write
 0001:00024984       ImageList_GetIconSize
 0001:0002498C       ImageList_SetIconSize
 0001:00024994       Finalization
 0001:000249C4       CommCtrl
 0001:000249CC       InitAnApi
 0001:00024AB4       _GetSystemMetrics
 0001:00024B3C       xMonitorFromRect
 0001:00024BCC       xMonitorFromWindow
 0001:00024C64       xMonitorFromPoint
 0001:00024CFC       xGetMonitorInfo
 0001:00024DD0       xGetMonitorInfoA
 0001:00024EA4       xGetMonitorInfoW
 0001:00024F78       xEnumDisplayMonitors
 0001:000250A8       InitMultiMonStubs
 0001:00025114       Finalization
 0001:00025144       MultiMon
 0001:00025154       Finalization
 0001:00025184       Imm
 0001:00025550       RegisterViewer
 0001:000255D4       GetHelpSystem
 0001:0002562C       THelpViewerNode.Create
 0001:00025668       THelpManager.Create
 0001:000256DC       THelpManager.RegisterViewer
 0001:000257FC       THelpManager.UnloadAllViewers
 0001:0002583C       THelpManager.DoSoftShutDown
 0001:0002586C       THelpManager.DoTableOfContents
 0001:00025A0C       THelpManager.CallSpecialWinHelp
 0001:00025B14       THelpManager.ShowHelp
 0001:00025D28       THelpManager.ShowContextHelp
 0001:00025E3C       THelpManager.ShowTableOfContents
 0001:00025E44       THelpManager.ShowTopicHelp
 0001:00025F40       THelpManager.AssignHelpSelector
 0001:00025F9C       THelpManager.Hook
 0001:00026044       THelpManager.GetHandle
 0001:00026048       THelpManager.GetHelpFile
 0001:0002605C       THelpManager.Release
 0001:000260E8       THelpManager.Destroy
 0001:0002613C       Finalization
 0001:0002617C       HelpIntfs
 0001:00026184       Finalization
 0001:000261B4       WinSpool
 0001:000261BC       Finalization
 0001:000261F8       Printers
 0001:00026200       FlatSB_SetScrollProp
 0001:00026234       InitializeFlatSB
 0001:0002625C       InitFlatSB
 0001:000264E0       Finalization
 0001:00026510       FlatSB
 0001:000265EC       TSynchroObject.Acquire
 0001:000265F0       TSynchroObject.Release
 0001:000265F4       TCriticalSection.Create
 0001:00026634       TCriticalSection.Destroy
 0001:00026664       TCriticalSection.Acquire
 0001:00026670       TCriticalSection.Release
 0001:0002667C       TCriticalSection.Enter
 0001:00026684       TCriticalSection.Leave
 0001:0002668C       Finalization
 0001:000266BC       SyncObjs
 0001:000266C4       FreeThemeLibrary
 0001:00026884       InitThemeLibrary
 0001:00026FE8       UseThemes
 0001:00027010       Finalization
 0001:00027064       UxTheme
 0001:00027080       Finalization
 0001:000270B0       RichEdit
 0001:000270B8       Finalization
 0001:000270E8       ToolWin
 0001:000270F0       Finalization
 0001:00027120       ShellAPI
 0001:00027128       Finalization
 0001:00027158       RegStr
 0001:00027160       Finalization
 0001:00027190       WinInet
 0001:00027198       Finalization
 0001:000271C8       UrlMon
 0001:000271D0       Finalization
 0001:00027200       ShlObj
 0001:00027208       Finalization
 0001:00027238       CommDlg
 0001:00027240       Finalization
 0001:00027270       Dlgs
 0001:000273E4       TCommonDialog.Create
 0001:0002742C       TCommonDialog.Destroy
 0001:00027460       TCommonDialog.MessageHook
 0001:00027488       TCommonDialog.DefaultHandler
 0001:000274C0       TCommonDialog.MainWndProc
 0001:0002750C       TCommonDialog.WndProc
 0001:00027514       TCommonDialog.WMDestroy
 0001:0002752C       TCommonDialog.WMInitDialog
 0001:00027544       TCommonDialog.WMNCDestroy
 0001:00027558       TCommonDialog.TaskModalDialog
 0001:0002762C       TCommonDialog.DoClose
 0001:00027640       TCommonDialog.DoShow
 0001:000276F8       InitGlobals
 0001:0002784C       Finalization
 0001:000278A8       Dialogs
 0001:000279FC       TTimer.Create
 0001:00027A4C       TTimer.Destroy
 0001:00027A84       TTimer.WndProc
 0001:00027AF8       TTimer.UpdateTimer
 0001:00027B84       TTimer.SetEnabled
 0001:00027B94       TTimer.SetInterval
 0001:00027BA4       TTimer.SetOnTimer
 0001:00027BBC       TTimer.Timer
 0001:00027EC4       Finalization
 0001:00027F0C       ExtCtrls
 0001:00027F3C       Finalization
 0001:00027F6C       ComStrs
 0001:00027F74       Finalization
 0001:00027FB0       Clipbrd
 0001:00028008       Finalization
 0001:00028038       StrUtils
 0001:00028040       DestroyLocals
 0001:000280D8       Finalization
 0001:00028110       Buttons
 0001:00028138       Finalization
 0001:00028168       ExtDlgs
 0001:00028188       Finalization
 0001:000281D0       IniFiles
 0001:000281F0       Finalization
 0001:00028238       Registry
 0001:00028254       Finalization
 0001:000282A4       Mapi
 0001:000282AC       Finalization
 0001:000282FC       ExtActns
 0001:00028304       Finalization
 0001:00028334       ListActns
 0001:000283DC       GetComCtlVersion
 0001:00028414       TConversion.ConvertReadStream
 0001:00028428       TConversion.ConvertWriteStream
 0001:0002843C       Finalization
 0001:000284B4       ComCtrls
 0001:000286E4       ThemeServices
 0001:00028704       TThemeServices.Create
 0001:00028750       TThemeServices.Destroy
 0001:00028784       TThemeServices.GetTheme
 0001:000287C4       TThemeServices.GetThemesEnabled
 0001:000287DC       TThemeServices.DoOnThemeChange
 0001:000287F0       TThemeServices.UnloadThemeData
 0001:00028820       TThemeServices.ApplyThemeChange
 0001:00028834       TThemeServices.DrawEdge
 0001:00028880       TThemeServices.DrawElement
 0001:000288C4       TThemeServices.DrawParentBackground
 0001:0002892C       TThemeServices.GetElementDetails
 0001:00028968       TThemeServices.GetElementDetails
 0001:00028CF4       TThemeServices.PaintBorder
 0001:00028E60       TThemeServices.UpdateThemes
 0001:00028E7C       Finalization
 0001:00028EC0       Themes
 0001:00028EC8       Finalization
 0001:00028EF8       StdCtrls
 0001:00028FF4       THintAction.Create
 0001:00029030       Finalization
 0001:00029060       StdActns
 0001:00029214       TWinHelpViewer.HelpFile
 0001:000292E4       TWinHelpViewer.InternalShutDown
 0001:0002930C       TWinHelpViewer.GetViewerName
 0001:00029320       TWinHelpViewer.UnderstandsKeyword
 0001:00029398       TWinHelpViewer.GetHelpStrings
 0001:0002943C       TWinHelpViewer.CanShowTableOfContents
 0001:00029440       TWinHelpViewer.ShowTableOfContents
 0001:000294C8       TWinHelpViewer.ShowHelp
 0001:00029610       TWinHelpViewer.NotifyID
 0001:00029614       TWinHelpViewer.SoftShutDown
 0001:00029630       TWinHelpViewer.ShutDown
 0001:00029660       TWinHelpViewer.UnderstandsTopic
 0001:000296C8       TWinHelpViewer.DisplayTopic
 0001:000297DC       TWinHelpViewer.UnderstandsContext
 0001:00029850       TWinHelpViewer.DisplayHelpByContext
 0001:000298E0       TWinHelpViewer.CallWinHelp
 0001:000299E0       WindowEnumerationTester
 0001:00029A3C       DialogEnumerationTester
 0001:00029A94       FindWinHelp
 0001:00029AB0       TWinHelpViewer.IsNewQuery
 0001:00029B38       TWinHelpViewer.IsBusyWindow
 0001:00029B3C       TWinHelpViewer.CouldBeUnstableWindow
 0001:00029B58       TWinHelpViewer.MakeWinHelpHappy
 0001:00029BB4       TWinHelpViewer.RestartWinHelp
 0001:00029C40       TWinHelpViewer.Create
 0001:00029C88       TWinHelpViewer.Destroy
 0001:00029CB4       Finalization
 0001:00029D2C       WinHelpViewer
 0001:0002BB78       InitWndProc
 0001:0002BC30       ObjectFromHWnd
 0001:0002BC64       FindControl
 0001:0002BCC0       SendAppMessage
 0001:0002BE84       CursorToIdent
 0001:0002BE94       IdentToCursor
 0001:0002BEA4       GetShortHint
 0001:0002BEE8       GetLongHint
 0001:0002BF2C       GetCaptureControl
 0001:0002BF54       SetCaptureControl
 0001:0002C000       TSiteList.Find
 0001:0002C034       GetTopParent
 0001:0002C05C       TSiteList.AddSite
 0001:0002C0B8       TSiteList.Clear
 0001:0002C0EC       TSiteList.GetTopSite
 0001:0002C150       TDragObject.Assign
 0001:0002C190       TDragObject.Capture
 0001:0002C1A8       TDragObject.Finished
 0001:0002C1B0       TDragObject.GetName
 0001:0002C1D8       TDragObject.ReleaseCapture
 0001:0002C1EC       TDragObject.WndProc
 0001:0002C2E8       TDragObject.GetDragImages
 0001:0002C2EC       TDragObject.GetDragCursor
 0001:0002C304       TDragObject.HideDragImage
 0001:0002C308       TDragObject.Instance
 0001:0002C310       TDragObject.ShowDragImage
 0001:0002C314       TDragObject.MainWndProc
 0001:0002C360       TDragObject.BeforeDestruction
 0001:0002C370       TDragObject.AfterConstruction
 0001:0002C380       TBaseDragControlObject.Create
 0001:0002C3A4       TBaseDragControlObject.Assign
 0001:0002C3D0       TBaseDragControlObject.EndDrag
 0001:0002C3FC       TBaseDragControlObject.Finished
 0001:0002C430       TDragControlObject.GetDragCursor
 0001:0002C448       TDragControlObject.GetDragImages
 0001:0002C454       TDragControlObject.HideDragImage
 0001:0002C474       TDragControlObject.ShowDragImage
 0001:0002C494       TDragControlObjectEx.BeforeDestruction
 0001:0002C498       TDragDockObject.Create
 0001:0002C4FC       TDragDockObject.Destroy
 0001:0002C52C       TDragDockObject.Assign
 0001:0002C588       TDragDockObject.EndDrag
 0001:0002C5AC       AbsMin
 0001:0002C5D0       TDragDockObject.AdjustDockRect
 0001:0002C64C       TDragDockObject.DrawDragDockImage
 0001:0002C660       TDragDockObject.EraseDragDockImage
 0001:0002C674       TDragDockObject.GetDragCursor
 0001:0002C680       TDragDockObject.GetFrameWidth
 0001:0002C688       TDragDockObjectEx.BeforeDestruction
 0001:0002C68C       IsBeforeTargetWindow
 0001:0002C6F8       ValidDockTarget
 0001:0002C890       IsSiteChildOfClient
 0001:0002C8D4       GetDockSiteAtPos
 0001:0002CA30       RegisterDockSite
 0001:0002CA90       DragMessage
 0001:0002CAE8       IsDelphiHandle
 0001:0002CB48       DragFindWindow
 0001:0002CB74       DragFindTarget
 0001:0002CBC4       DoDragOver
 0001:0002CC00       GetDropCtl
 0001:0002CC94       DragTo
 0001:0002CF64       DragInit
 0001:0002D0D4       DragInitControl
 0001:0002D298       CheckUndock
 0001:0002D30C       DragDone
 0001:0002D5E4       CancelDrag
 0001:0002D5FC       FindVCLWindow
 0001:0002D630       FindDragTarget
 0001:0002D678       ListAdd
 0001:0002D6A0       ListRemove
 0001:0002D6C0       MoveWindowOrg
 0001:0002D6F0       FreeDeviceContext
 0001:0002D7AC       FreeDeviceContexts
 0001:0002D858       TControlCanvas.Destroy
 0001:0002D884       TControlCanvas.CreateHandle
 0001:0002D92C       TControlCanvas.FreeHandle
 0001:0002D960       TControlCanvas.SetControl
 0001:0002D978       TControlCanvas.UpdateTextFlags
 0001:0002D9A4       TSizeConstraints.Create
 0001:0002D9E0       TSizeConstraints.AssignTo
 0001:0002DA28       TSizeConstraints.SetConstraints
 0001:0002DAB4       TSizeConstraints.Change
 0001:0002DAC8       TControlActionLink.AssignClient
 0001:0002DAE4       TControlActionLink.DoShowHint
 0001:0002DBD4       TControlActionLink.IsCaptionLinked
 0001:0002DC48       TControlActionLink.IsEnabledLinked
 0001:0002DC7C       TControlActionLink.IsHintLinked
 0001:0002DCB4       TControlActionLink.IsVisibleLinked
 0001:0002DCE8       TControlActionLink.IsOnExecuteLinked
 0001:0002DD10       TControlActionLink.SetCaption
 0001:0002DD30       TControlActionLink.SetEnabled
 0001:0002DD50       TControlActionLink.SetHint
 0001:0002DD74       TControlActionLink.SetVisible
 0001:0002DD94       TControlActionLink.SetOnExecute
 0001:0002DDC0       TControlActionLink.IsHelpLinked
 0001:0002DE24       TControlActionLink.SetHelpKeyword
 0001:0002DE44       TControlActionLink.SetHelpContext
 0001:0002DE64       TControlActionLink.SetHelpType
 0001:0002DE84       TControl.Create
 0001:0002DF5C       TControl.Destroy
 0001:0002E010       TControl.GetDragImages
 0001:0002E014       TControl.GetEnabled
 0001:0002E018       TControl.GetPalette
 0001:0002E01C       TControl.HasParent
 0001:0002E024       TControl.GetParentComponent
 0001:0002E028       TControl.SetParentComponent
 0001:0002E050       TControl.PaletteChanged
 0001:0002E0C8       TControl.GetAction
 0001:0002E0D8       TControl.SetAnchors
 0001:0002E0F8       TControl.SetAction
 0001:0002E174       TControl.IsAnchorsStored
 0001:0002E18C       TControl.SetDragMode
 0001:0002E190       TControl.RequestAlign
 0001:0002E1A0       TControl.Resize
 0001:0002E1C0       TControl.ReadState
 0001:0002E254       TControl.Notification
 0001:0002E298       TControl.SetAlign
 0001:0002E340       TControl.SetBounds
 0001:0002E3D8       TControl.UpdateAnchorRules
 0001:0002E4F4       TControl.SetLeft
 0001:0002E518       TControl.SetTop
 0001:0002E540       TControl.SetWidth
 0001:0002E564       TControl.SetHeight
 0001:0002E588       TControl.Dock
 0001:0002E694       TControl.DoDock
 0001:0002E6EC       TControl.SetHelpContext
 0001:0002E700       TControl.SetHelpKeyword
 0001:0002E724       TControl.GetBoundsRect
 0001:0002E744       TControl.SetBoundsRect
 0001:0002E770       TControl.GetClientRect
 0001:0002E788       TControl.GetClientWidth
 0001:0002E7A0       TControl.SetClientWidth
 0001:0002E7CC       TControl.GetClientHeight
 0001:0002E7E4       TControl.SetClientHeight
 0001:0002E80C       TControl.GetClientOrigin
 0001:0002E89C       TControl.ClientToScreen
 0001:0002E8C8       TControl.ScreenToClient
 0001:0002E8F4       TControl.SendCancelMode
 0001:0002E924       TControl.SendDockNotification
 0001:0002E990       TControl.ChangeScale
 0001:0002EB44       TControl.SetAutoSize
 0001:0002EB5C       TControl.SetName
 0001:0002EC00       TControl.SetClientSize
 0001:0002EC48       TControl.SetParent
 0001:0002EC94       TControl.SetVisible
 0001:0002ECD0       TControl.SetEnabled
 0001:0002ECE8       TControl.GetTextLen
 0001:0002ECF8       TControl.GetTextBuf
 0001:0002ED04       TControl.GetUndockHeight
 0001:0002ED18       TControl.GetUndockWidth
 0001:0002ED2C       TControl.SetPopupMenu
 0001:0002ED50       TControl.SetTextBuf
 0001:0002ED74       TControl.GetText
 0001:0002EDA4       TControl.SetText
 0001:0002EE08       TControl.SetBiDiMode
 0001:0002EE24       TControl.FontChanged
 0001:0002EE68       TControl.SetFont
 0001:0002EE78       TControl.IsFontStored
 0001:0002EE8C       TControl.IsShowHintStored
 0001:0002EE98       TControl.IsBiDiModeStored
 0001:0002EEA0       TControl.SetParentFont
 0001:0002EEC4       TControl.SetShowHint
 0001:0002EEE8       TControl.SetColor
 0001:0002EF04       TControl.IsColorStored
 0001:0002EF0C       TControl.SetParentColor
 0001:0002EF30       TControl.SetParentBiDiMode
 0001:0002EF54       TControl.SetCursor
 0001:0002EF70       TControl.GetMouseCapture
 0001:0002EF80       TControl.SetMouseCapture
 0001:0002EFA8       TControl.BringToFront
 0001:0002EFB8       TControl.SetZOrderPosition
 0001:0002F038       TControl.SetZOrder
 0001:0002F05C       TControl.GetDeviceContext
 0001:0002F104       BackgroundClipped
 0001:0002F190       TControl.InvalidateControl
 0001:0002F21C       TControl.Invalidate
 0001:0002F22C       TControl.MouseWheelHandler
 0001:0002F270       TControl.Update
 0001:0002F284       TControl.Repaint
 0001:0002F37C       TControl.GetControlsAlignment
 0001:0002F380       TControl.UseRightToLeftReading
 0001:0002F398       TControl.UseRightToLeftAlignment
 0001:0002F3B0       TControl.UseRightToLeftScrollBar
 0001:0002F3CC       TControl.BeginAutoDrag
 0001:0002F3E4       TControl.BeginDrag
 0001:0002F4A8       TControl.DragCanceled
 0001:0002F4AC       TControl.Dragging
 0001:0002F4B8       TControl.DragOver
 0001:0002F4F4       TControl.DragDrop
 0001:0002F520       TControl.DoStartDrag
 0001:0002F540       TControl.DoEndDrag
 0001:0002F56C       TControl.PositionDockRect
 0001:0002F63C       TControl.DockTrackNoTarget
 0001:0002F650       TControl.DoEndDock
 0001:0002F67C       TControl.DoStartDock
 0001:0002F69C       TControl.DoMouseWheel
 0001:0002F760       TControl.DoMouseWheelDown
 0001:0002F7AC       TControl.DoMouseWheelUp
 0001:0002F7F8       TControl.DefaultDockImage
 0001:0002F924       TControl.DrawDragDockImage
 0001:0002F938       TControl.EraseDragDockImage
 0001:0002F94C       TControl.DoDragMsg
 0001:0002FA3C       TControl.ManualDock
 0001:0002FC1C       TControl.ManualFloat
 0001:0002FCB0       TControl.DoConstraintsChange
 0001:0002FCBC       TControl.CanAutoSize
 0001:0002FCC0       TControl.CanResize
 0001:0002FCF0       TControl.DoCanAutoSize
 0001:0002FD5C       TControl.DoCanResize
 0001:0002FD8C       TControl.ConstrainedResize
 0001:0002FDBC       TControl.CalcCursorPos
 0001:0002FDE8       TControl.DesignWndProc
 0001:0002FE1C       TControl.DoConstrainedResize
 0001:0002FEF0       TControl.Perform
 0001:0002FF24       TControl.CalcDockSizes
 0001:0002FF94       TControl.UpdateBoundsRect
 0001:0002FFB8       TControl.VisibleChanging
 0001:0002FFBC       TControl.WndProc
 0001:00030150       TControl.DefaultHandler
 0001:000301D8       TControl.ReadIsControl
 0001:000301EC       TControl.WriteIsControl
 0001:000301F8       DoWriteIsControl
 0001:00030228       TControl.DefineProperties
 0001:00030278       TControl.Click
 0001:000302E4       TControl.DblClick
 0001:00030304       TControl.MouseDown
 0001:0003033C       TControl.DoMouseDown
 0001:000303C0       TControl.WMLButtonDown
 0001:0003040C       TControl.WMNCLButtonDown
 0001:00030428       TControl.WMLButtonDblClk
 0001:0003047C       TControl.GetPopupMenu
 0001:00030480       TControl.CheckNewSize
 0001:0003051C       TControl.WMRButtonDown
 0001:00030544       TControl.WMRButtonDblClk
 0001:0003056C       TControl.WMMButtonDown
 0001:00030594       TControl.WMMButtonDblClk
 0001:000305BC       TControl.MouseMove
 0001:000305EC       TControl.WMMouseMove
 0001:00030664       TControl.MouseUp
 0001:0003069C       TControl.DoMouseUp
 0001:000306D4       TControl.WMLButtonUp
 0001:0003074C       TControl.WMRButtonUp
 0001:0003076C       TControl.WMMButtonUp
 0001:0003078C       TControl.WMMouseWheel
 0001:000307E4       TControl.WMCancelMode
 0001:00030824       TControl.WMWindowPosChanged
 0001:000308D4       TControl.CMVisibleChanged
 0001:000308FC       TControl.CMEnabledChanged
 0001:00030904       TControl.CMFontChanged
 0001:0003090C       TControl.CMColorChanged
 0001:00030914       TControl.CMParentColorChanged
 0001:00030944       TControl.CMParentBiDiModeChanged
 0001:00030968       TControl.CMMouseWheel
 0001:000309C4       TControl.CMBiDiModeChanged
 0001:000309E4       TControl.CMParentShowHintChanged
 0001:00030A0C       TControl.CMParentFontChanged
 0001:00030A3C       TControl.CMSysFontChanged
 0001:00030A60       TControl.CMHitTest
 0001:00030A68       TControl.CMMouseEnter
 0001:00030A80       TControl.CMMouseLeave
 0001:00030A98       TControl.CMDesignHitTest
 0001:00030AA0       TControl.CreateFloatingDockSite
 0001:00030B24       UpdateFloatingDockSitePos
 0001:00030BB0       TControl.CMFloat
 0001:00030C10       TControl.ActionChange
 0001:00030D0C       TControl.DoActionChange
 0001:00030D30       TControl.GetActionLinkClass
 0001:00030D38       TControl.IsEnabledStored
 0001:00030D58       TControl.IsHintStored
 0001:00030D78       TControl.IsHelpContextStored
 0001:00030D98       TControl.IsVisibleStored
 0001:00030DB8       TControl.Loaded
 0001:00030DF0       TControl.AssignTo
 0001:00030E9C       MinVar
 0001:00030ED8       TControl.GetDockEdge
 0001:00030F88       TControl.GetFloating
 0001:00030FB4       TControl.GetFloatingDockSiteClass
 0001:00030FBC       TControl.AdjustSize
 0001:00030FDC       TControl.DrawTextBiDiModeFlagsReadingOnly
 0001:00030FF8       TControl.InitiateAction
 0001:00031008       TControl.CMHintShow
 0001:00031034       TControl.WMContextMenu
 0001:0003115C       TControl.DoContextPopup
 0001:00031190       TControl.SetConstraints
 0001:0003119C       TWinControlActionLink.AssignClient
 0001:000311C0       TWinControlActionLink.IsHelpContextLinked
 0001:000311C8       TWinControlActionLink.SetHelpContext
 0001:000311D0       TWinControl.Create
 0001:000312F4       TWinControl.Destroy
 0001:000313C4       TWinControl.FixupTabList
 0001:00031498       TWinControl.ReadState
 0001:00031510       TWinControl.AdjustClientRect
 0001:00031514       InsertBefore
 0001:000315A0       DoPosition
 0001:000319E0       DoAlign
 0001:00031B50       AlignWork
 0001:00031BA4       TWinControl.AlignControls
 0001:00031CA8       TWinControl.AlignControl
 0001:00031D3C       TWinControl.DisableAlign
 0001:00031D44       TWinControl.EnableAlign
 0001:00031D64       TWinControl.Realign
 0001:00031D6C       TWinControl.DoFlipChildren
 0001:00031E40       TWinControl.FlipChildren
 0001:00031F80       TWinControl.ContainsControl
 0001:00031F94       TWinControl.RemoveFocus
 0001:00031FB4       TWinControl.Insert
 0001:00032000       TWinControl.Remove
 0001:00032048       TWinControl.InsertControl
 0001:0003211C       TWinControl.RemoveControl
 0001:00032198       TWinControl.GetControl
 0001:000321D4       TWinControl.GetControlCount
 0001:000321F4       TWinControl.Broadcast
 0001:00032234       TWinControl.NotifyControls
 0001:0003225C       TWinControl.AddBiDiModeExStyle
 0001:000322C4       TWinControl.CreateParams
 0001:000323F0       TWinControl.CreateWnd
 0001:000325C0       TWinControl.CreateWindowHandle
 0001:00032600       TWinControl.ReadDesignSize
 0001:00032638       TWinControl.WriteDesignSize
 0001:0003268C       PointsEqual
 0001:000326A0       DoWriteDesignSize
 0001:00032778       TWinControl.DefineProperties
 0001:000327D4       TWinControl.DestroyWnd
 0001:0003282C       TWinControl.DestroyWindowHandle
 0001:00032890       TWinControl.PrecedingWindow
 0001:000328D8       TWinControl.CreateHandle
 0001:00032970       TWinControl.CustomAlignInsertBefore
 0001:00032974       TWinControl.CustomAlignPosition
 0001:00032990       TWinControl.DestroyHandle
 0001:000329D8       TWinControl.RecreateWnd
 0001:000329F0       TWinControl.CMRecreateWnd
 0001:00032A30       TWinControl.UpdateShowing
 0001:00032B2C       TWinControl.UpdateControlState
 0001:00032B6C       TWinControl.SetParentWindow
 0001:00032BF4       TWinControl.MainWndProc
 0001:00032C6C       GetControlAtPos
 0001:00032D24       TWinControl.ControlAtPos
 0001:00032DB8       TWinControl.IsControlMouseMsg
 0001:00032E4C       TWinControl.WndProc
 0001:00032FB0       TWinControl.DefaultHandler
 0001:000330B8       DoControlMsg
 0001:000330EC       TWinControl.PaintHandler
 0001:0003321C       TWinControl.PaintWindow
 0001:00033244       TWinControl.PaintControls
 0001:00033474       TWinControl.PaintTo
 0001:000335C8       TWinControl.WMPaint
 0001:00033728       TWinControl.WMCommand
 0001:00033748       TWinControl.WMNotify
 0001:0003376C       TWinControl.WMSysColorChange
 0001:00033788       TWinControl.WMWinIniChange
 0001:0003379C       TWinControl.WMFontChange
 0001:000337AC       TWinControl.WMTimeChange
 0001:000337BC       TWinControl.WMHScroll
 0001:000337DC       TWinControl.WMVScroll
 0001:000337FC       TWinControl.WMCompareItem
 0001:00033820       TWinControl.WMDeleteItem
 0001:00033844       TWinControl.WMDrawItem
 0001:00033868       TWinControl.WMMeasureItem
 0001:0003388C       TWinControl.WMEraseBkgnd
 0001:00033914       TWinControl.WMWindowPosChanged
 0001:000339D4       TWinControl.WMWindowPosChanging
 0001:00033A24       TWinControl.WMSize
 0001:00033A58       TWinControl.WMMove
 0001:00033A6C       TWinControl.WMSetCursor
 0001:00033B6C       TWinControl.WMSetFocus
 0001:00033B80       TWinControl.WMKillFocus
 0001:00033B94       TWinControl.WMIMEStartComp
 0001:00033BA8       TWinControl.WMIMEEndComp
 0001:00033BBC       TWinControl.SetIme
 0001:00033CA8       TWinControl.ResetIme
 0001:00033D40       TWinControl.DoAddDockClient
 0001:00033D50       TWinControl.DoRemoveDockClient
 0001:00033D54       TWinControl.DoEnter
 0001:00033D74       TWinControl.DoExit
 0001:00033D94       TWinControl.DockDrop
 0001:00033DE4       TWinControl.DoDockOver
 0001:00033E18       TWinControl.DockOver
 0001:00033E58       TWinControl.DoUnDock
 0001:00033EB0       TWinControl.ReloadDockedControl
 0001:00033ED4       TWinControl.GetDockClientCount
 0001:00033EE8       TWinControl.GetDockClients
 0001:00033F0C       TWinControl.GetSiteInfo
 0001:00033F68       TWinControl.GetVisibleDockClientCount
 0001:00033FA4       TWinControl.ControlsAligned
 0001:00033FA8       TWinControl.CreateDockManager
 0001:00034014       TWinControl.SetDockSite
 0001:000340CC       TWinControl.CMDockClient
 0001:000341B8       TWinControl.CMUnDockClient
 0001:000341E0       TWinControl.CMFloat
 0001:00034264       TWinControl.KeyDown
 0001:0003428C       TWinControl.DoKeyDown
 0001:000342F4       TWinControl.WMKeyDown
 0001:00034320       TWinControl.WMSysKeyDown
 0001:0003434C       TWinControl.KeyUp
 0001:00034374       TWinControl.DoKeyUp
 0001:000343DC       TWinControl.WMKeyUp
 0001:000343FC       TWinControl.WMSysKeyUp
 0001:0003441C       TWinControl.KeyPress
 0001:0003443C       TWinControl.DoKeyPress
 0001:000344A0       TWinControl.WMChar
 0001:000344C0       TraverseControls
 0001:00034570       TWinControl.WMSysCommand
 0001:00034618       TWinControl.WMCharToItem
 0001:00034638       TWinControl.WMParentNotify
 0001:0003466C       TWinControl.WMVKeyToItem
 0001:0003468C       TWinControl.WMDestroy
 0001:000346C0       TWinControl.WMNCDestroy
 0001:000346DC       TWinControl.WMNCHitTest
 0001:00034700       TWinControl.PaletteChanged
 0001:00034758       TWinControl.WMQueryNewPalette
 0001:0003477C       TWinControl.WMPaletteChanged
 0001:0003479C       TWinControl.CMShowHintChanged
 0001:000347B4       TWinControl.CMBiDiModeChanged
 0001:000347EC       TWinControl.CMEnter
 0001:00034860       TWinControl.CMExit
 0001:0003486C       TWinControl.CMDesignHitTest
 0001:0003488C       TWinControl.CMChanged
 0001:000348A0       TWinControl.CMChildKey
 0001:000348B4       TWinControl.CMDialogKey
 0001:000348BC       TWinControl.CMDialogChar
 0001:000348C4       TWinControl.CMFocusChanged
 0001:000348CC       TWinControl.CMVisibleChanged
 0001:000348FC       TWinControl.CMShowingChanged
 0001:00034924       TWinControl.CMEnabledChanged
 0001:0003496C       TWinControl.CMColorChanged
 0001:00034994       TWinControl.CMFontChanged
 0001:000349D0       TWinControl.CMCursorChanged
 0001:00034A10       TWinControl.CMBorderChanged
 0001:00034A50       TWinControl.CMCtl3DChanged
 0001:00034A90       TWinControl.CMParentCtl3DChanged
 0001:00034AD0       TWinControl.CMSysColorChange
 0001:00034AD8       TWinControl.CMWinIniChange
 0001:00034AE0       TWinControl.CMFontChange
 0001:00034AE8       TWinControl.CMTimeChange
 0001:00034AF0       TWinControl.CMDrag
 0001:00034B4C       TWinControl.CMControlListChange
 0001:00034B60       TWinControl.CMSysFontChanged
 0001:00034B7C       TWinControl.IsMenuKey
 0001:00034C10       TWinControl.CNKeyDown
 0001:00034CF4       TWinControl.CNKeyUp
 0001:00034D48       TWinControl.CNChar
 0001:00034D94       TWinControl.CNSysKeyDown
 0001:00034DF0       TWinControl.CNSysChar
 0001:00034E24       TWinControl.SetBounds
 0001:00034EFC       TWinControl.ScaleControls
 0001:00034F44       TWinControl.ChangeScale
 0001:00034FF0       TWinControl.ScrollBy
 0001:000350C8       TWinControl.ShowControl
 0001:000350E0       TWinControl.SetZOrderPosition
 0001:000351B8       TWinControl.SetZOrder
 0001:00035218       TWinControl.GetDeviceContext
 0001:0003526C       TWinControl.Invalidate
 0001:0003527C       TWinControl.CMInvalidate
 0001:0003530C       TWinControl.Update
 0001:00035328       TWinControl.Repaint
 0001:00035340       TWinControl.InvalidateFrame
 0001:00035378       TWinControl.CanFocus
 0001:000353B8       TWinControl.SetFocus
 0001:000353F0       TWinControl.Focused
 0001:00035414       TWinControl.HandleNeeded
 0001:00035438       TWinControl.GetHandle
 0001:0003544C       TWinControl.GetControlExtents
 0001:000354E0       TWinControl.GetClientOrigin
 0001:00035500       TWinControl.GetClientRect
 0001:00035518       TWinControl.AdjustSize
 0001:00035558       TWinControl.SetBorderWidth
 0001:00035578       TWinControl.SetCtl3D
 0001:0003559C       TWinControl.IsCtl3DStored
 0001:000355A8       TWinControl.GetTabOrder
 0001:000355CC       TWinControl.UpdateTabOrder
 0001:00035628       TWinControl.SetUseDockManager
 0001:00035698       TWinControl.HandleAllocated
 0001:000356A4       TWinControl.UpdateBounds
 0001:0003575C       TWinControl.GetTabOrderList
 0001:000357BC       TWinControl.FindNextControl
 0001:000358C8       TWinControl.SelectNext
 0001:000358F4       TWinControl.GetChildren
 0001:0003593C       TWinControl.SetChildOrder
 0001:0003597C       TWinControl.CanResize
 0001:00035984       DoCalcConstraints
 0001:00035A08       TWinControl.CalcConstraints
 0001:00035DE4       TWinControl.ConstrainedResize
 0001:00035E20       TWinControl.ActionChange
 0001:00035E60       TWinControl.GetActionLinkClass
 0001:00035E68       TWinControl.AssignTo
 0001:00035E98       TWinControl.CanAutoSize
 0001:00036064       TWinControl.WMNCCalcSize
 0001:000360F4       TWinControl.WMNCPaint
 0001:0003639C       TWinControl.WMContextMenu
 0001:00036408       TWinControl.UpdateUIState
 0001:0003646C       TWinControl.WMPrintClient
 0001:0003649C       TWinControl.GetParentBackground
 0001:000364A4       TWinControl.SetParentBackground
 0001:000364E4       THintWindow.Create
 0001:00036550       THintWindow.CreateParams
 0001:000365B4       THintWindow.WMNCHitTest
 0001:000365BC       THintWindow.WMNCPaint
 0001:00036620       THintWindow.Paint
 0001:000366C8       THintWindow.IsHintMsg
 0001:0003672C       THintWindow.ReleaseHandle
 0001:00036734       THintWindow.CMTextChanged
 0001:000367CC       THintWindow.ActivateHint
 0001:000369B4       THintWindow.ActivateHintData
 0001:000369DC       THintWindow.CalcHintRect
 0001:00036A38       THintWindow.NCPaint
 0001:00036AA4       THintWindow.WMPrint
 0001:00036AC8       ClientToWindow
 0001:00036B08       TDragImageList.CombineDragCursor
 0001:00036BD4       TDragImageList.SetDragImage
 0001:00036C1C       TDragImageList.SetDragCursor
 0001:00036C34       TDragImageList.BeginDrag
 0001:00036C94       TDragImageList.DragLock
 0001:00036CF8       TDragImageList.DragUnlock
 0001:00036D1C       TDragImageList.DragMove
 0001:00036D60       TDragImageList.ShowDragImage
 0001:00036D78       TDragImageList.HideDragImage
 0001:00036D90       TDragImageList.EndDrag
 0001:00036DD8       TCustomControl.Create
 0001:00036E34       TCustomControl.Destroy
 0001:00036E64       TCustomControl.WMPaint
 0001:00036E84       TCustomControl.PaintWindow
 0001:00036F30       TCustomControl.Paint
 0001:00036F34       NextVisibleZone
 0001:00036F50       IsOrientationSet
 0001:00036F74       TDockZone.Create
 0001:00036F98       TDockZone.GetChildCount
 0001:00036FAC       TDockZone.GetVisibleChildCount
 0001:00036FC8       TDockZone.GetVisible
 0001:00036FFC       TDockZone.GetLimitBegin
 0001:00037044       TDockZone.GetLimitSize
 0001:0003708C       TDockZone.GetTopLeft
 0001:000370F8       TDockZone.GetHeightWidth
 0001:000371A8       TDockZone.ResetChildren
 0001:00037250       TDockZone.GetControlName
 0001:00037294       TDockZone.SetControlName
 0001:00037318       ParentNotLast
 0001:00037348       TDockZone.Update
 0001:000374C0       TDockZone.GetZoneLimit
 0001:000374E8       TDockZone.SetZoneLimit
 0001:000374EC       GetLastChildZone
 0001:000374FC       TDockZone.ExpandZoneLimit
 0001:00037538       TDockZone.ResetZoneLimits
 0001:00037598       TDockZone.NextVisible
 0001:000375A4       TDockZone.PrevVisible
 0001:000375C0       TDockZone.FirstVisibleChild
 0001:000375CC       TDockTree.Create
 0001:00037734       TDockTree.Destroy
 0001:00037788       TDockTree.AdjustDockRect
 0001:0003779C       TDockTree.BeginUpdate
 0001:000377A0       TDockTree.EndUpdate
 0001:000377B4       DoFindControlZone
 0001:0003780C       TDockTree.FindControlZone
 0001:00037838       DoForEach
 0001:00037874       TDockTree.ForEachAt
 0001:0003788C       TDockTree.GetControlBounds
 0001:00037900       TDockTree.HitTest
 0001:00037910       TDockTree.InsertControl
 0001:00037B20       TDockTree.InsertNewParent
 0001:00037CC8       TDockTree.InsertSibling
 0001:00037D40       DoFindZone
 0001:00037F6C       FindControlAtPos
 0001:00038000       TDockTree.InternalHitTest
 0001:00038088       ReadControlName
 0001:000380D0       TDockTree.LoadFromStream
 0001:000382D8       DrawCloseButton
 0001:00038330       DrawGrabberLine
 0001:000383B8       TDockTree.PaintDockFrame
 0001:00038494       TDockTree.PaintSite
 0001:000385F8       TDockTree.PositionDockRect
 0001:0003876C       DoPrune
 0001:000387A0       TDockTree.PruneZone
 0001:000387FC       TDockTree.RemoveControl
 0001:00038838       TDockTree.RemoveZone
 0001:00038AB4       TDockTree.ResetBounds
 0001:00038B90       TDockTree.ScaleZone
 0001:00038BCC       WriteControlName
 0001:00038C44       DoSaveZone
 0001:00038D00       TDockTree.SaveToStream
 0001:00038E48       DoSetNewBounds
 0001:00038ED0       TDockTree.SetNewBounds
 0001:00038EFC       TDockTree.SetReplacingControl
 0001:00038F14       TDockTree.ShiftZone
 0001:00038F44       TDockTree.SplitterMouseDown
 0001:00038FA4       TDockTree.SplitterMouseUp
 0001:00039020       TDockTree.UpdateAll
 0001:00039048       TDockTree.UpdateZone
 0001:00039058       TDockTree.DrawSizeSplitter
 0001:00039144       DoGetNextLimit
 0001:000391D4       TDockTree.GetNextLimit
 0001:00039224       GetDockAlign
 0001:000392A0       HideZone
 0001:00039320       ShowZone
 0001:00039458       TDockTree.ControlVisibilityChanged
 0001:000394E0       CalcSplitterPos
 0001:00039570       TDockTree.WindowProc
 0001:00039958       TMouse.Create
 0001:000399E8       TMouse.Destroy
 0001:00039A18       TMouse.GetCapture
 0001:00039A20       TMouse.GetCursorPos
 0001:00039A30       TMouse.GetMouseData
 0001:00039A4C       TMouse.GetNativeData
 0001:00039A7C       TMouse.GetRegisteredData
 0001:00039AA4       TMouse.SetCapture
 0001:00039ACC       TMouse.SettingChanged
 0001:00039B30       InitIMM32
 0001:00039D98       Win32NLSEnableIME
 0001:00039DB4       SetImeMode
 0001:00039E90       Imm32IsIME
 0001:00039EA4       DoneControls
 0001:00039F2C       InitControls
 0001:0003A0F8       Finalization
 0001:0003A160       Controls
 0001:0003A6E4       TContainedAction.Destroy
 0001:0003A718       TContainedAction.GetIndex
 0001:0003A730       TContainedAction.IsCategoryStored
 0001:0003A734       TContainedAction.GetParentComponent
 0001:0003A744       TContainedAction.HasParent
 0001:0003A754       TContainedAction.ReadState
 0001:0003A788       TContainedAction.SetIndex
 0001:0003A7D0       TContainedAction.SetCategory
 0001:0003A7FC       TContainedAction.SetActionList
 0001:0003A824       TContainedAction.SetParentComponent
 0001:0003A850       TContainedAction.Execute
 0001:0003A8A8       TContainedAction.Update
 0001:0003A900       TCustomActionList.Create
 0001:0003A96C       TCustomActionList.Destroy
 0001:0003A9BC       TCustomActionList.GetChildren
 0001:0003AA04       TCustomActionList.SetChildOrder
 0001:0003AA34       TCustomActionList.GetAction
 0001:0003AA48       TCustomActionList.GetActionCount
 0001:0003AA50       TCustomActionList.SetImages
 0001:0003AA84       TCustomActionList.ImageListChange
 0001:0003AA90       TCustomActionList.Notification
 0001:0003AAD8       TCustomActionList.AddAction
 0001:0003AAF8       TCustomActionList.RemoveAction
 0001:0003AB14       TCustomActionList.Change
 0001:0003AB7C       TCustomActionList.IsShortCut
 0001:0003AC08       TCustomActionList.ExecuteAction
 0001:0003AC28       TCustomActionList.UpdateAction
 0001:0003AC48       TActionLink.IsCaptionLinked
 0001:0003AC5C       TActionLink.IsCheckedLinked
 0001:0003AC70       TActionLink.IsEnabledLinked
 0001:0003AC84       TActionLink.IsGroupIndexLinked
 0001:0003AC98       TActionLink.IsHelpContextLinked
 0001:0003ACAC       TActionLink.IsHelpLinked
 0001:0003ACC0       TActionLink.IsHintLinked
 0001:0003ACD4       TActionLink.IsImageIndexLinked
 0001:0003ACE8       TActionLink.IsShortCutLinked
 0001:0003ACFC       TActionLink.IsVisibleLinked
 0001:0003AD10       TActionLink.SetAutoCheck
 0001:0003AD14       TActionLink.SetCaption
 0001:0003AD18       TActionLink.SetChecked
 0001:0003AD1C       TActionLink.SetEnabled
 0001:0003AD20       TActionLink.SetGroupIndex
 0001:0003AD24       TActionLink.SetHelpContext
 0001:0003AD28       TActionLink.SetHelpKeyword
 0001:0003AD2C       TActionLink.SetHelpType
 0001:0003AD30       TActionLink.SetHint
 0001:0003AD34       TActionLink.SetImageIndex
 0001:0003AD38       TActionLink.SetShortCut
 0001:0003AD3C       TActionLink.SetVisible
 0001:0003AD40       TCustomAction.Create
 0001:0003AD94       TCustomAction.Destroy
 0001:0003ADE4       TCustomAction.AssignTo
 0001:0003AE90       TCustomAction.SetCaption
 0001:0003AEF0       TCustomAction.SetChecked
 0001:0003AFF8       TCustomAction.SetEnabled
 0001:0003B070       TCustomAction.SetHelpKeyword
 0001:0003B0D8       TCustomAction.SetHelpContext
 0001:0003B130       TCustomAction.SetHint
 0001:0003B190       TCustomAction.SetImageIndex
 0001:0003B1EC       TCustomAction.SetShortCut
 0001:0003B250       TCustomAction.SetVisible
 0001:0003B2B0       TCustomAction.SetName
 0001:0003B2FC       TCustomAction.DoHint
 0001:0003B324       TCustomAction.Execute
 0001:0003B384       TCustomAction.GetSecondaryShortCuts
 0001:0003B3AC       TCustomAction.HandleShortCut
 0001:0003B3B8       TShortCutList.Add
 0001:0003B3E4       TShortCutList.IndexOfShortCut
 0001:0003B428       Finalization
 0001:0003B458       ActnList
 0001:0003B5D8       GetRGBColor
 0001:0003B5F8       GetColor
 0001:0003B618       TCustomImageList.Create
 0001:0003B664       TCustomImageList.Destroy
 0001:0003B6D0       TCustomImageList.Initialize
 0001:0003B788       TCustomImageList.HandleAllocated
 0001:0003B790       TCustomImageList.HandleNeeded
 0001:0003B79C       TCustomImageList.InitBitmap
 0001:0003B860       TCustomImageList.SetNewDimensions
 0001:0003B898       TCustomImageList.SetHandle
 0001:0003B8C4       TCustomImageList.GetHandle
 0001:0003B8D4       TCustomImageList.GetImageHandle
 0001:0003B928       TCustomImageList.FreeHandle
 0001:0003B960       TCustomImageList.CreateImageList
 0001:0003BA00       TCustomImageList.Add
 0001:0003BACC       TCustomImageList.GetCount
 0001:0003BAF0       TCustomImageList.Delete
 0001:0003BB7C       TCustomImageList.Clear
 0001:0003BB88       TCustomImageList.SetBkColor
 0001:0003BBC0       TCustomImageList.GetBkColor
 0001:0003BBE8       TCustomImageList.DoDraw
 0001:0003BDBC       TCustomImageList.Draw
 0001:0003BDE0       TCustomImageList.Draw
 0001:0003BE2C       TCustomImageList.CopyImages
 0001:0003BFD4       TCustomImageList.AddImages
 0001:0003BFF4       TCustomImageList.Assign
 0001:0003C0B4       TCustomImageList.AssignTo
 0001:0003C164       TCustomImageList.CheckImage
 0001:0003C1DC       TCustomImageList.SetDrawingStyle
 0001:0003C1F4       TCustomImageList.GetHotSpot
 0001:0003C204       TCustomImageList.Change
 0001:0003C254       TCustomImageList.UnRegisterChanges
 0001:0003C298       TCustomImageList.RegisterChanges
 0001:0003C2AC       StreamsEqual
 0001:0003C2F0       TCustomImageList.Equal
 0001:0003C3E0       DoWrite
 0001:0003C43C       TCustomImageList.DefineProperties
 0001:0003C494       TCustomImageList.ReadD2Stream
 0001:0003C728       TCustomImageList.ReadD3Stream
 0001:0003C8F0       TCustomImageList.ReadData
 0001:0003C97C       TCustomImageList.WriteData
 0001:0003CAC0       TCustomImageList.BeginUpdate
 0001:0003CAC4       TCustomImageList.EndUpdate
 0001:0003CAE4       TChangeLink.Destroy
 0001:0003CB18       TChangeLink.Change
 0001:0003CB30       Finalization
 0001:0003CB60       ImgList
 0001:0003DA98       FindPopupControl
 0001:0003DAC8       ReturnAddr
 0001:0003DAD0       Error
 0001:0003DAF0       ShortCut
 0001:0003DB28       GetSpecialName
 0001:0003DB7C       ShortCutToText
 0001:0003DD80       CompareFront
 0001:0003DDDC       TextToShortCut
 0001:0003DED4       UniqueCommand
 0001:0003DEF4       Iterate
 0001:0003DF54       IterateMenus
 0001:0003E05C       TMenuActionLink.AssignClient
 0001:0003E078       TMenuActionLink.IsAutoCheckLinked
 0001:0003E0A0       TMenuActionLink.IsCaptionLinked
 0001:0003E0D8       TMenuActionLink.IsCheckedLinked
 0001:0003E108       TMenuActionLink.IsEnabledLinked
 0001:0003E138       TMenuActionLink.IsHelpContextLinked
 0001:0003E168       TMenuActionLink.IsHintLinked
 0001:0003E19C       TMenuActionLink.IsGroupIndexLinked
 0001:0003E1D8       TMenuActionLink.IsImageIndexLinked
 0001:0003E20C       TMenuActionLink.IsShortCutLinked
 0001:0003E240       TMenuActionLink.IsVisibleLinked
 0001:0003E274       TMenuActionLink.IsOnExecuteLinked
 0001:0003E29C       TMenuActionLink.SetAutoCheck
 0001:0003E2BC       TMenuActionLink.SetCaption
 0001:0003E2DC       TMenuActionLink.SetChecked
 0001:0003E2FC       TMenuActionLink.SetEnabled
 0001:0003E31C       TMenuActionLink.SetHelpContext
 0001:0003E338       TMenuActionLink.SetHint
 0001:0003E35C       TMenuActionLink.SetImageIndex
 0001:0003E37C       TMenuActionLink.SetShortCut
 0001:0003E39C       TMenuActionLink.SetVisible
 0001:0003E3BC       TMenuActionLink.SetOnExecute
 0001:0003E3E8       TMenuItem.Create
 0001:0003E464       TMenuItem.Destroy
 0001:0003E518       TMenuItem.AppendTo
 0001:0003E79C       AddIn
 0001:0003E7B8       TMenuItem.PopulateMenu
 0001:0003E828       TMenuItem.ReadShortCutText
 0001:0003E880       TMenuItem.MergeWith
 0001:0003E8BC       TMenuItem.Loaded
 0001:0003E8F8       TMenuItem.RebuildHandle
 0001:0003E9C8       TMenuItem.VerifyGroupIndex
 0001:0003EA28       TMenuItem.GetHandle
 0001:0003EA74       TMenuItem.DefineProperties
 0001:0003EAB8       TMenuItem.DoDrawText
 0001:0003ECC8       TMenuItem.DrawItem
 0001:0003ED08       NormalDraw
 0001:0003F630       BiDiDraw
 0001:0003FF78       TMenuItem.AdvancedDrawItem
 0001:000400AC       TMenuItem.GetImageList
 0001:000400DC       GetMenuSize
 0001:00040128       TMenuItem.MeasureItem
 0001:00040328       TMenuItem.HasParent
 0001:0004032C       TMenuItem.SetBreak
 0001:0004033C       TMenuItem.SetCaption
 0001:00040364       TMenuItem.TurnSiblingsOff
 0001:000403AC       TMenuItem.SetChecked
 0001:00040400       TMenuItem.SetEnabled
 0001:00040478       TMenuItem.SetGroupIndex
 0001:000404BC       TMenuItem.GetAction
 0001:000404CC       TMenuItem.GetActionLinkClass
 0001:000404D4       TMenuItem.GetCount
 0001:000404E4       TMenuItem.GetItem
 0001:00040508       TMenuItem.SetShortCut
 0001:0004051C       TMenuItem.SetVisible
 0001:0004052C       TMenuItem.SetImageIndex
 0001:0004053C       TMenuItem.GetMenuIndex
 0001:00040554       TMenuItem.SetMenuIndex
 0001:0004059C       TMenuItem.GetChildren
 0001:000405D4       TMenuItem.SetChildOrder
 0001:000405F4       TMenuItem.SetDefault
 0001:00040650       TMenuItem.InitiateAction
 0001:00040660       TMenuItem.Insert
 0001:00040714       TMenuItem.Delete
 0001:00040788       TMenuItem.Click
 0001:00040838       TMenuItem.IndexOf
 0001:00040850       TMenuItem.Add
 0001:0004086C       TMenuItem.Remove
 0001:00040894       TMenuItem.MenuChanged
 0001:000408D8       TMenuItem.SubItemChanged
 0001:00040930       TMenuItem.GetBitmap
 0001:00040958       TMenuItem.SetAction
 0001:000409C8       TMenuItem.SetBitmap
 0001:000409FC       TMenuItem.InitiateActions
 0001:00040A28       TMenuItem.GetParentComponent
 0001:00040A3C       TMenuItem.SetParentComponent
 0001:00040A90       TMenuItem.GetParentMenu
 0001:00040AA0       TMenuItem.SetRadioItem
 0001:00040ACC       TMenuItem.ActionChange
 0001:00040BEC       TMenuItem.DoActionChange
 0001:00040C10       TMenuItem.IsCaptionStored
 0001:00040C30       TMenuItem.IsCheckedStored
 0001:00040C50       TMenuItem.IsEnabledStored
 0001:00040C70       TMenuItem.IsHintStored
 0001:00040C90       TMenuItem.IsHelpContextStored
 0001:00040CB0       TMenuItem.IsImageIndexStored
 0001:00040CD0       TMenuItem.IsShortCutStored
 0001:00040CF0       TMenuItem.IsVisibleStored
 0001:00040D10       TMenuItem.IsOnClickStored
 0001:00040D30       TMenuItem.AssignTo
 0001:00040DA8       TMenuItem.Notification
 0001:00040DFC       TMenuItem.SetSubMenuImages
 0001:00040E38       TMenuItem.ImageListChange
 0001:00040E44       UpdateItem
 0001:00040E6C       TMenuItem.UpdateItems
 0001:00040E80       IfHotkeyAvailable
 0001:00040EB0       CopyToBest
 0001:00040F34       InsertHotkeyFarEastFormat
 0001:00041094       TMenuItem.InternalRethinkHotkeys
 0001:0004155C       TMenuItem.SetAutoHotkeys
 0001:0004156C       TMenuItem.IsLine
 0001:00041590       TMenuItem.InternalRethinkLines
 0001:000416D8       TMenuItem.SetAutoLineReduction
 0001:000416E8       TMenuItem.GetAutoHotkeys
 0001:00041714       TMenuItem.GetAutoLineReduction
 0001:00041740       TMenu.Create
 0001:000417DC       TMenu.Destroy
 0001:00041814       TMenu.GetChildren
 0001:00041830       TMenu.GetHandle
 0001:0004183C       TMenu.SetChildOrder
 0001:00041850       UpdateItem
 0001:00041878       TMenu.UpdateItems
 0001:00041890       Find
 0001:00041928       TMenu.FindItem
 0001:00041958       TMenu.GetHelpContext
 0001:000419C8       TMenu.DispatchCommand
 0001:000419E4       TMenu.DispatchPopup
 0001:00041AAC       TMenu.IsOwnerDraw
 0001:00041AC0       NthParentOf
 0001:00041AD0       DoClick
 0001:00041C24       TMenu.IsShortCut
 0001:00041D40       TMenu.IsBiDiModeStored
 0001:00041D48       TMenu.DoBiDiModeChanged
 0001:00041E04       BuildImage
 0001:00041ED4       TMenu.UpdateImage
 0001:00041F58       TMenu.SetOwnerDraw
 0001:00041F68       TMenu.AdjustBiDiBehavior
 0001:00041FE4       TMenu.SetWindowHandle
 0001:0004201C       TMenu.DoChange
 0001:00042034       TMenu.Loaded
 0001:0004204C       TMenu.MenuChanged
 0001:00042088       TMenu.ImageListChange
 0001:00042094       TMenu.SetImages
 0001:000420D0       TMenu.Notification
 0001:000420FC       TMenu.IsRightToLeft
 0001:00042114       IsAccelChar
 0001:00042170       IsInitialChar
 0001:00042258       TMenu.ProcessMenuChar
 0001:000423D0       TMenu.DoGetMenuString
 0001:00042478       TMenu.SetBiDiMode
 0001:0004248C       TMenu.SetParentBiDiMode
 0001:0004249C       TMenu.ParentBiDiModeChanged
 0001:000424C4       TMenu.ParentBiDiModeChanged
 0001:000424F0       TMenu.GetAutoHotkeys
 0001:00042500       TMenu.SetAutoHotkeys
 0001:00042510       TMenu.GetAutoLineReduction
 0001:00042520       TMenu.SetAutoLineReduction
 0001:00042530       TMainMenu.SetAutoMerge
 0001:00042550       TMainMenu.MenuChanged
 0001:000425A8       TMainMenu.Merge
 0001:000425C4       TMainMenu.Unmerge
 0001:000425E0       TMainMenu.ItemChanged
 0001:0004260C       TMainMenu.GetHandle
 0001:0004261C       TPopupList.MainWndProc
 0001:00042668       TPopupList.WndProc
 0001:00042BAC       TPopupList.Add
 0001:00042BD4       TPopupList.Remove
 0001:00042BF0       TPopupMenu.Create
 0001:00042C64       TPopupMenu.Destroy
 0001:00042C98       TPopupMenu.DoPopup
 0001:00042CAC       TPopupMenu.GetHelpContext
 0001:00042CB4       TPopupMenu.SetHelpContext
 0001:00042CBC       TPopupMenu.SetBiDiModeFromPopupControl
 0001:00042D04       TPopupMenu.UseRightToLeftAlignment
 0001:00042D50       TPopupMenu.Popup
 0001:00042E04       TMenuItemStack.ClearItem
 0001:00042E40       DrawMenuItem
 0001:00042F28       StripHotkey
 0001:00042FC0       GetHotkey
 0001:00043024       AnsiSameCaption
 0001:00043120       Finalization
 0001:00043190       Menus
 0001:00044FA4       SaveFocusState
 0001:00044FB4       RestoreFocusState
 0001:00044FBC       ShowMDIClientEdge
 0001:00045008       DoneApplication
 0001:00045040       DoDisableWindow
 0001:00045090       DisableTaskWindows
 0001:00045144       EnableTaskWindows
 0001:00045194       DoFindWindow
 0001:000451F8       FindTopMostWindow
 0001:00045234       SendFocusMessage
 0001:00045254       CheckTaskWindow
 0001:00045274       ForegroundTask
 0001:000452A0       FindGlobalComponent
 0001:00045320       KeysToShiftState
 0001:00045374       KeyDataToShiftState
 0001:000453B0       KeyboardStateToShiftState
 0001:000453FC       IsAccel
 0001:0004546C       GetParentForm
 0001:00045494       ValidParentForm
 0001:00045514       TControlScrollBar.Create
 0001:0004559C       TControlScrollBar.IsIncrementStored
 0001:000455A4       TControlScrollBar.Assign
 0001:000455F4       TControlScrollBar.ChangeBiDiPosition
 0001:0004562C       ProcessHorz
 0001:00045698       ProcessVert
 0001:00045700       TControlScrollBar.CalcAutoRange
 0001:000457AC       TControlScrollBar.IsScrollBarVisible
 0001:000457E4       ScrollBarVisible
 0001:00045818       Adjustment
 0001:00045894       TControlScrollBar.ControlSize
 0001:00045914       TControlScrollBar.NeedsScrollBarVisible
 0001:0004592C       GetRealScrollPosition
 0001:0004598C       TControlScrollBar.ScrollMessage
 0001:00045C8C       TControlScrollBar.SetButtonSize
 0001:00045CD0       TControlScrollBar.SetColor
 0001:00045CEC       TControlScrollBar.SetParentColor
 0001:00045D04       TControlScrollBar.SetPosition
 0001:00045DC8       TControlScrollBar.SetSize
 0001:00045E0C       TControlScrollBar.SetStyle
 0001:00045E24       TControlScrollBar.SetThumbSize
 0001:00045E3C       TControlScrollBar.DoSetRange
 0001:00045E54       TControlScrollBar.SetRange
 0001:00045E68       TControlScrollBar.IsRangeStored
 0001:00045E74       TControlScrollBar.SetVisible
 0001:00045E80       UpdateScrollProperties
 0001:00045F88       TControlScrollBar.Update
 0001:000460A0       TScrollingWinControl.Create
 0001:00046118       TScrollingWinControl.Destroy
 0001:00046154       TScrollingWinControl.CreateParams
 0001:00046164       TScrollingWinControl.CreateWnd
 0001:000461A4       TScrollingWinControl.AlignControls
 0001:000461C4       TScrollingWinControl.AutoScrollEnabled
 0001:000461E4       TScrollingWinControl.DoFlipChildren
 0001:000462FC       TScrollingWinControl.CalcAutoRange
 0001:00046320       TScrollingWinControl.SetAutoScroll
 0001:0004635C       TScrollingWinControl.SetHorzScrollBar
 0001:0004636C       TScrollingWinControl.SetVertScrollBar
 0001:0004637C       TScrollingWinControl.UpdateScrollBars
 0001:00046474       TScrollingWinControl.AutoScrollInView
 0001:0004648C       TScrollingWinControl.ScrollInView
 0001:000465E0       TScrollingWinControl.ScaleScrollBars
 0001:00046684       TScrollingWinControl.ChangeScale
 0001:000466A8       TScrollingWinControl.Resizing
 0001:000466AC       TScrollingWinControl.WMSize
 0001:00046788       TScrollingWinControl.WMHScroll
 0001:000467AC       TScrollingWinControl.WMVScroll
 0001:000467D0       TScrollingWinControl.AdjustClientRect
 0001:00046840       TScrollingWinControl.CMBiDiModeChanged
 0001:000468D0       TCustomForm.Create
 0001:00046A5C       TCustomForm.AfterConstruction
 0001:00046A94       TCustomForm.CreateNew
 0001:00046C10       TCustomForm.BeforeDestruction
 0001:00046C78       TCustomForm.Destroy
 0001:00046D5C       TCustomForm.DoCreate
 0001:00046DD8       TCustomForm.DoDestroy
 0001:00046E38       TCustomForm.Loaded
 0001:00046E74       TCustomForm.Notification
 0001:00046F80       TCustomForm.ReadState
 0001:000471F8       TCustomForm.DefineProperties
 0001:000472A8       TCustomForm.ReadIgnoreFontProperty
 0001:000472C8       TCustomForm.ReadTextHeight
 0001:000472E0       TCustomForm.WriteTextHeight
 0001:000472FC       TCustomForm.WritePixelsPerInch
 0001:00047318       TCustomForm.GetTextHeight
 0001:0004733C       TCustomForm.BeginAutoDrag
 0001:00047340       TCustomForm.ChangeScale
 0001:000473C0       TCustomForm.IconChanged
 0001:0004741C       TCustomForm.IsClientSizeStored
 0001:0004742C       TCustomForm.IsFormSizeStored
 0001:00047454       TCustomForm.IsAutoScrollStored
 0001:00047488       TCustomForm.DoClose
 0001:000474A8       TCustomForm.DoHide
 0001:000474C8       TCustomForm.DoShow
 0001:000474E8       TCustomForm.GetClientRect
 0001:00047570       TCustomForm.GetChildren
 0001:000475DC       TCustomForm.GetFloating
 0001:00047608       TCustomForm.SetChildOrder
 0001:0004769C       TCustomForm.SetParentBiDiMode
 0001:000476C4       TCustomForm.SetClientWidth
 0001:000476F4       TCustomForm.SetClientHeight
 0001:00047724       TCustomForm.SetVisible
 0001:00047768       TCustomForm.VisibleChanging
 0001:000477CC       TCustomForm.WantChildKey
 0001:000477D0       TCustomForm.SetParent
 0001:00047808       TCustomForm.ValidateRename
 0001:00047848       TCustomForm.WndProc
 0001:00047C80       Default
 0001:00047CCC       MaximizedChildren
 0001:00047D0C       TCustomForm.ClientWndProc
 0001:00047EEC       TCustomForm.AlignControls
 0001:00047F58       TCustomForm.CMBiDiModeChanged
 0001:00047FF0       TCustomForm.CMParentBiDiModeChanged
 0001:00048078       TCustomForm.SetBorderIcons
 0001:000480A4       TCustomForm.SetBorderStyle
 0001:000480DC       TCustomForm.Dock
 0001:00048120       TCustomForm.DoDock
 0001:00048174       TCustomForm.GetActiveMDIChild
 0001:000481A8       TCustomForm.GetMDIChildCount
 0001:000481F4       TCustomForm.GetMDIChildren
 0001:00048244       EnumMonitorsProc
 0001:00048274       TCustomForm.GetMonitor
 0001:0004835C       TCustomForm.GetCanvas
 0001:00048364       TCustomForm.SetIcon
 0001:00048370       TCustomForm.IsForm
 0001:00048378       TCustomForm.IsIconStored
 0001:000483A0       TCustomForm.SetFormStyle
 0001:00048420       TCustomForm.RefreshMDIMenu
 0001:0004849C       TCustomForm.SetObjectMenuItem
 0001:000484C0       TCustomForm.SetWindowMenu
 0001:000484E8       TCustomForm.SetMenu
 0001:000486BC       TCustomForm.GetPixelsPerInch
 0001:000486D0       TCustomForm.SetPixelsPerInch
 0001:00048704       TCustomForm.SetPosition
 0001:00048720       TCustomForm.GetScaled
 0001:0004872C       TCustomForm.SetScaled
 0001:0004875C       TCustomForm.CMColorChanged
 0001:00048780       TCustomForm.NormalColor
 0001:00048798       TCustomForm.CMCtl3DChanged
 0001:000487E0       TCustomForm.CMFontChanged
 0001:00048800       TCustomForm.CMMenuChanged
 0001:0004881C       TCustomForm.SetWindowState
 0001:0004885C       TCustomForm.SetWindowToMonitor
 0001:00048BB0       TCustomForm.CreateParams
 0001:00048DCC       TCustomForm.CreateWnd
 0001:00048F10       TCustomForm.CreateWindowHandle
 0001:00049048       TCustomForm.DestroyWindowHandle
 0001:0004908C       TCustomForm.DefaultHandler
 0001:000490F0       TCustomForm.SetActiveControl
 0001:000491A8       TCustomForm.DefocusControl
 0001:000491F0       TCustomForm.FocusControl
 0001:00049214       TCustomForm.SetFocusedControl
 0001:000494AC       TCustomForm.ActiveChanged
 0001:000494B0       TCustomForm.SetWindowFocus
 0001:00049500       TCustomForm.SetActive
 0001:00049564       TCustomForm.SendCancelMode
 0001:000495B4       TCustomForm.MergeMenu
 0001:0004965C       DoNestedActivation
 0001:000496A8       TCustomForm.Activate
 0001:000496D8       TCustomForm.Deactivate
 0001:00049708       TCustomForm.Paint
 0001:00049728       TCustomForm.GetIconHandle
 0001:00049744       TCustomForm.PaintWindow
 0001:00049800       TCustomForm.PaletteChanged
 0001:000498A0       TCustomForm.WMPaint
 0001:00049920       TCustomForm.WMIconEraseBkgnd
 0001:00049980       TCustomForm.WMEraseBkgnd
 0001:000499B8       TCustomForm.WMQueryDragIcon
 0001:000499CC       ModifySystemMenu
 0001:00049AC8       TCustomForm.WMNCCreate
 0001:00049AFC       TCustomForm.WMNCLButtonDown
 0001:00049B8C       TCustomForm.WMDestroy
 0001:00049BEC       TCustomForm.WMCommand
 0001:00049C20       TCustomForm.WMInitMenuPopup
 0001:00049C38       TCustomForm.WMMenuChar
 0001:00049C70       TCustomForm.WMMenuSelect
 0001:00049D18       TCustomForm.WMActivate
 0001:00049D38       TCustomForm.Resizing
 0001:00049D70       TCustomForm.WMClose
 0001:00049D78       TCustomForm.WMQueryEndSession
 0001:00049DA4       TCustomForm.CMAppSysCommand
 0001:00049DFC       TCustomForm.WMSysCommand
 0001:00049E88       TCustomForm.WMShowWindow
 0001:00049F20       TCustomForm.WMMDIActivate
 0001:00049F78       TCustomForm.WMNextDlgCtl
 0001:00049FA4       TCustomForm.WMEnterMenuLoop
 0001:00049FC0       GetMenuHelpContext
 0001:0004A000       ControlHasHelp
 0001:0004A038       GetHelpInfo
 0001:0004A06C       TCustomForm.WMHelp
 0001:0004A1CC       TCustomForm.WMGetMinMaxInfo
 0001:0004A240       HandleEdge
 0001:0004A26C       TCustomForm.WMWindowPosChanging
 0001:0004A324       TCustomForm.CMActivate
 0001:0004A348       TCustomForm.CMDeactivate
 0001:0004A36C       TCustomForm.CMDialogKey
 0001:0004A408       TCustomForm.CMShowingChanged
 0001:0004A980       TCustomForm.CMIconChanged
 0001:0004A9A0       TCustomForm.CMRelease
 0001:0004A9A8       TCustomForm.CMTextChanged
 0001:0004A9F8       TCustomForm.CMUIActivate
 0001:0004AA00       TCustomForm.CMParentFontChanged
 0001:0004AA6C       TCustomForm.CMIsShortCut
 0001:0004AA98       TCustomForm.Close
 0001:0004AB3C       TCustomForm.CloseQuery
 0001:0004ABA0       TCustomForm.CloseModal
 0001:0004AC38       TCustomForm.Hide
 0001:0004AC40       TCustomForm.Show
 0001:0004AC58       TCustomForm.SetFocus
 0001:0004ACD4       TCustomForm.Release
 0001:0004ACF0       TCustomForm.ShowModal
 0001:0004AFC8       TraverseClients
 0001:0004B038       TCustomForm.UpdateActions
 0001:0004B0A0       TCustomForm.RequestAlign
 0001:0004B0BC       TCustomForm.WMSettingChange
 0001:0004B0E0       ProcessExecute
 0001:0004B110       TraverseClients
 0001:0004B18C       TCustomForm.CMActionExecute
 0001:0004B1E0       ProcessUpdate
 0001:0004B210       TraverseClients
 0001:0004B28C       TCustomForm.CMActionUpdate
 0001:0004B2E0       DispatchShortCut
 0001:0004B334       TCustomForm.IsShortCut
 0001:0004B3B0       TCustomForm.QueryInterface
 0001:0004B3EC       TCustomForm.MouseWheelHandler
 0001:0004B424       TCustomForm.HandleCreateException
 0001:0004B434       TCustomForm.SetLayeredAttribs
 0001:0004B50C       TCustomForm.SetAlphaBlend
 0001:0004B520       TCustomForm.SetAlphaBlendValue
 0001:0004B534       TCustomForm.SetTransparentColorValue
 0001:0004B548       TCustomForm.SetTransparentColor
 0001:0004B55C       TCustomForm.InitAlphaBlending
 0001:0004B588       TCustomDockForm.Create
 0001:0004B5EC       TCustomDockForm.DoAddDockClient
 0001:0004B6D0       TCustomDockForm.DoRemoveDockClient
 0001:0004B6F0       TCustomDockForm.Loaded
 0001:0004B73C       TCustomDockForm.GetSiteInfo
 0001:0004B768       TCustomDockForm.WMNCHitTest
 0001:0004B790       TCustomDockForm.WMNCLButtonDown
 0001:0004B828       TCustomDockForm.CMControlListChange
 0001:0004B880       TCustomDockForm.CMDockNotification
 0001:0004B954       TCustomDockForm.CMUnDockClient
 0001:0004B96C       TCustomDockForm.CMVisibleChanged
 0001:0004B9A8       TMonitor.GetLeft
 0001:0004B9C0       TMonitor.GetHeight
 0001:0004B9DC       TMonitor.GetTop
 0001:0004B9F4       TMonitor.GetWidth
 0001:0004BA10       TMonitor.GetBoundsRect
 0001:0004BA40       TMonitor.GetWorkareaRect
 0001:0004BA70       TScreen.Create
 0001:0004BBC8       TScreen.Destroy
 0001:0004BC90       TScreen.GetHeight
 0001:0004BC9C       TScreen.GetWidth
 0001:0004BCA8       TScreen.GetDesktopTop
 0001:0004BCB4       TScreen.GetDesktopLeft
 0001:0004BCC0       TScreen.GetDesktopHeight
 0001:0004BCCC       TScreen.GetDesktopWidth
 0001:0004BCD8       TScreen.GetMonitor
 0001:0004BCEC       TScreen.GetMonitorCount
 0001:0004BD08       TScreen.GetForm
 0001:0004BD1C       TScreen.GetFormCount
 0001:0004BD24       TScreen.GetCustomForms
 0001:0004BD38       TScreen.GetCustomFormCount
 0001:0004BD40       TScreen.UpdateLastActive
 0001:0004BD8C       TScreen.AddForm
 0001:0004BDC4       TScreen.RemoveForm
 0001:0004BE14       TScreen.AddDataModule
 0001:0004BE20       TScreen.RemoveDataModule
 0001:0004BE2C       TScreen.CreateCursors
 0001:0004BE88       TScreen.DestroyCursors
 0001:0004BF00       TScreen.InsertCursor
 0001:0004BF28       TScreen.GetImes
 0001:0004C128       TScreen.GetDefaultIME
 0001:0004C144       TScreen.IconFontChanged
 0001:0004C194       TScreen.GetDataModule
 0001:0004C1A8       TScreen.GetDataModuleCount
 0001:0004C1B0       TScreen.GetCursors
 0001:0004C1EC       TScreen.SetCursor
 0001:0004C27C       TScreen.GetMetricSettings
 0001:0004C3D0       TScreen.DisableAlign
 0001:0004C3D8       TScreen.EnableAlign
 0001:0004C3F8       TScreen.Realign
 0001:0004C400       InsertBefore
 0001:0004C460       DoPosition
 0001:0004C610       DoAlign
 0001:0004C75C       AlignWork
 0001:0004C7B4       TScreen.AlignForms
 0001:0004C83C       TScreen.AlignForm
 0001:0004C8C4       TScreen.ResetFonts
 0001:0004C8D0       GetHint
 0001:0004C908       GetHintControl
 0001:0004C928       HintTimerProc
 0001:0004C97C       HintMouseThread
 0001:0004C9D8       HintGetMsgHook
 0001:0004CA1C       HookHintHooks
 0001:0004CA90       UnhookHintHooks
 0001:0004CAEC       GetAnimation
 0001:0004CB1C       SetAnimation
 0001:0004CB44       ShowWinNoAnimate
 0001:0004CB84       TApplication.Create
 0001:0004CD84       TApplication.Destroy
 0001:0004CEA0       TApplication.CreateHandle
 0001:0004D050       TApplication.ControlDestroyed
 0001:0004D0B0       GetTopMostWindows
 0001:0004D120       TApplication.DoNormalizeTopMosts
 0001:0004D1D0       TApplication.ModalStarted
 0001:0004D1FC       TApplication.ModalFinished
 0001:0004D228       TApplication.NormalizeTopMosts
 0001:0004D230       TApplication.NormalizeAllTopMosts
 0001:0004D238       TApplication.RestoreTopMosts
 0001:0004D2A4       TApplication.UseRightToLeftReading
 0001:0004D2BC       TApplication.UseRightToLeftAlignment
 0001:0004D2D4       TApplication.CheckIniChange
 0001:0004D32C       TApplication.SettingChange
 0001:0004D398       Default
 0001:0004D3D4       DrawAppIcon
 0001:0004D420       TApplication.WndProc
 0001:0004DB20       TApplication.GetIconHandle
 0001:0004DB3C       TApplication.Minimize
 0001:0004DBEC       TApplication.Restore
 0001:0004DCEC       TApplication.BringToFront
 0001:0004DD28       TApplication.GetTitle
 0001:0004DD74       TApplication.IsDlgMsg
 0001:0004DD98       TApplication.IsMDIMsg
 0001:0004DDE8       TApplication.IsKeyMsg
 0001:0004DEA0       TApplication.IsHintMsg
 0001:0004DED4       TApplication.IsShortCut
 0001:0004DF40       TApplication.ProcessMessage
 0001:0004DFD8       TApplication.HandleMessage
 0001:0004DFFC       TApplication.HookMainWindow
 0001:0004E058       TApplication.UnhookMainWindow
 0001:0004E0E4       TApplication.Terminate
 0001:0004E0F8       TApplication.HandleException
 0001:0004E188       TApplication.MessageBox
 0001:0004E2F0       TApplication.ShowException
 0001:0004E3C8       TApplication.InvokeHelp
 0001:0004E530       DoOnHelp
 0001:0004E598       TApplication.HelpKeyword
 0001:0004E628       TApplication.HelpContext
 0001:0004E6B0       TApplication.HelpCommand
 0001:0004E6B8       TApplication.SetShowHint
 0001:0004E708       TApplication.DoActionIdle
 0001:0004E76C       TApplication.DoMouseIdle
 0001:0004E7E4       TApplication.Idle
 0001:0004E904       TApplication.NotifyForms
 0001:0004E940       TApplication.IconChanged
 0001:0004E9A4       TApplication.SetHint
 0001:0004EA38       SetVisible
 0001:0004EA94       TApplication.UpdateVisible
 0001:0004EB1C       TApplication.ValidateHelpSystem
 0001:0004EB44       TApplication.StartHintTimer
 0001:0004EB88       TApplication.StopHintTimer
 0001:0004EBB0       TApplication.HintMouseMessage
 0001:0004ECC0       TApplication.HintTimerExpired
 0001:0004ECF8       TApplication.HideHint
 0001:0004ED3C       TApplication.CancelHint
 0001:0004ED64       FindScanline
 0001:0004ED74       GetCursorHeightMargin
 0001:0004EED4       ValidateHintWindow
 0001:0004EF34       MultiLineWidth
 0001:0004EFF8       TApplication.ActivateHint
 0001:0004F38C       TApplication.GetCurrentHelpFile
 0001:0004F3C8       TApplication.DispatchAction
 0001:0004F458       TApplication.ExecuteAction
 0001:0004F480       TApplication.UpdateAction
 0001:0004F4A8       InitProcs
 0001:0004F4F4       TApplication.WakeMainThread
 0001:0004F504       TApplication.HookSynchronizeWakeup
 0001:0004F514       TApplication.UnhookSynchronizeWakeup
 0001:0004F534       Finalization
 0001:0004F590       Forms
 0001:0004F5D4       Finalization
 0001:0004F604       DirectDraw
 0001:0004F60C       timeBeginPeriod
 0001:0004F614       timeEndPeriod
 0001:0004F61C       timeGetTime
 0001:0004F624       timeKillEvent
 0001:0004F62C       timeSetEvent
 0001:0004F634       Finalization
 0001:0004F664       MMSystem
 0001:0004F66C       Finalization
 0001:0004F69C       DXTypes
 0001:0004F6E0       Finalization
 0001:0004F710       DirectSound
 0001:0004F718       Finalization
 0001:0004F748       Direct3D9
 0001:0004F778       Finalization
 0001:0004F7A8       ComConst
 0001:0004F980       TrimPunctuation
 0001:0004F9D0       EOleSysError.Create
 0001:0004FAA0       EOleException.Create
 0001:0004FB38       OleError
 0001:0004FB54       OleCheck
 0001:0004FB6C       GUIDToString
 0001:0004FB98       CreateRegKey
 0001:0004FC30       DeleteRegKey
 0001:0004FC48       LoadComExProcs
 0001:0004FD4C       SafeCallError
 0001:0004FE4C       DispatchInvoke
 0001:00050190       RaiseNameException
 0001:000501C4       GetIDsOfNames
 0001:000502A4       RaiseException
 0001:000502BC       VarDispInvoke
 0001:00050358       DispCallError
 0001:0005042C       DispatchInvokeError
 0001:00050438       ClearExcepInfo
 0001:00050448       DispCall
 0001:0005052C       DispCallByID
 0001:00050608       InitComObj
 0001:00050680       Finalization
 0001:00050700       ComObj
 0001:00050980       Finalization
 0001:000509B0       DirectShow9
 0001:000509B8       Finalization
 0001:000509E8       WMF9
 0001:000509F0       FreeAndNil
 0001:00050A00       DeleteMediaType
 0001:00050A18       CopyMediaType
 0001:00050AEC       FreeMediaType
 0001:00050B40       EnlargedUnsignedDivide
 0001:00050B5C       UInt32x32To64
 0001:00050B60       llMulDiv
 0001:0005105C       Finalization
 0001:000510A4       DSUtil
 0001:00052650       TBCMediaType.MatchesPartial
 0001:000526F4       TBCMediaType.IsPartiallySpecified
 0001:00052728       TBCMediaType.InitMediaType
 0001:0005274C       AMGetWideString
 0001:000527D4       Templates
 0001:000527F4       DllGetClassObject
 0001:0005283C       DllCanUnloadNow
 0001:00052858       DllRegisterServer
 0001:00052874       DllUnregisterServer
 0001:00052890       TBCClassFactory.CreateFilter
 0001:00052944       TBCClassFactory.CreateInstance
 0001:000529C8       TBCClassFactory.UpdateRegistry
 0001:00052B78       TBCClassFactory.RegisterFilter
 0001:00052D60       TBCClassFactory.RegisterFilter
 0001:00052E38       TBCClassFactory._AddRef
 0001:00052E4C       TBCClassFactory._Release
 0001:00052E60       TBCClassFactory.LockServer
 0001:00052EA0       TBCClassFactory.QueryInterface
 0001:00052EC8       TBCFilterTemplate.AddObjectFactory
 0001:00052ED4       TBCFilterTemplate.Create
 0001:00052EFC       TBCFilterTemplate.Destroy
 0001:00052F40       TBCFilterTemplate.GetFactoryFromClassID
 0001:00052F70       TBCFilterTemplate.RegisterServer
 0001:00053084       TBCBaseObject.Create
 0001:000530F8       TBCBaseObject.Destroy
 0001:00053120       TBCBaseObject.FreeInstance
 0001:00053130       TBCBaseObject.NewInstance
 0001:00053148       TBCUnknown.QueryInterface
 0001:00053174       TBCUnknown._AddRef
 0001:00053198       TBCUnknown._Release
 0001:000531BC       TBCUnknown.NonDelegatingQueryInterface
 0001:000531E4       TBCUnknown.NonDelegatingAddRef
 0001:000531F8       TBCUnknown.NonDelegatingRelease
 0001:00053220       TBCUnknown.GetOwner
 0001:00053234       TBCUnknown.Create
 0001:000532C0       TBCUnknown.CreateFromFactory
 0001:00053304       TBCBaseFilter.Create
 0001:00053438       TBCBaseFilter.CreateFromFactory
 0001:00053490       TBCBaseFilter.destroy
 0001:000534D0       TBCBaseFilter.EnumPins
 0001:00053518       TBCBaseFilter.FindPin
 0001:00053674       TBCBaseFilter.GetClassID
 0001:00053690       TBCBaseFilter.GetPinVersion
 0001:00053694       TBCBaseFilter.GetState
 0001:000536A8       TBCBaseFilter.GetSyncSource
 0001:00053708       TBCBaseFilter.IsActive
 0001:0005376C       TBCBaseFilter.JoinFilterGraph
 0001:000538C8       TBCBaseFilter.NotifyEvent
 0001:00053954       TBCBaseFilter.Pause
 0001:00053A04       TBCBaseFilter.QueryFilterInfo
 0001:00053A94       TBCBaseFilter.QueryVendorInfo
 0001:00053AA0       TBCBaseFilter.Register
 0001:00053BCC       TBCBaseFilter.Run
 0001:00053CBC       TBCBaseFilter.SetSyncSource
 0001:00053D44       TBCBaseFilter.Stop
 0001:00053DF8       TBCBaseFilter.StreamTime
 0001:00053E3C       TBCBaseFilter.Unregister
 0001:00053F68       TBCEnumPins.Create
 0001:000540BC       TBCEnumPins.Destroy
 0001:000540F4       TBCEnumPins.Clone
 0001:00054158       TBCEnumPins.Next
 0001:000542C4       TBCEnumPins.Skip
 0001:00054300       TBCEnumPins.Reset
 0001:00054334       TBCEnumPins.Refresh
 0001:00054360       TBCEnumPins.AreWeOutOfSync
 0001:00054378       TBCBasePin.Active
 0001:0005437C       TBCBasePin.AgreeMediaType
 0001:00054518       TBCBasePin.AttemptConnection
 0001:000546E4       TBCBasePin.BreakConnect
 0001:000546E8       TBCBasePin.CheckConnect
 0001:000547DC       TBCBasePin.CompleteConnect
 0001:0005480C       TBCBasePin.Connect
 0001:00054970       TBCBasePin.ConnectedTo
 0001:000549A4       TBCBasePin.ConnectionMediaType
 0001:00054A40       TBCBasePin.Create
 0001:00054BE4       TBCBasePin.destroy
 0001:00054CA0       TBCBasePin.Disconnect
 0001:00054D08       TBCBasePin.DisconnectInternal
 0001:00054DB4       TBCBasePin.DisplayPinInfo
 0001:00054DDC       TBCBasePin.DisplayTypeInfo
 0001:00054E04       TBCBasePin.EndOfStream
 0001:00054E10       TBCBasePin.EnumMediaTypes
 0001:00054E58       TBCBasePin.GetMediaType
 0001:00054E60       TBCBasePin.GetMediaTypeVersion
 0001:00054E64       TBCBasePin.Inactive
 0001:00054E6C       TBCBasePin.IsConnected
 0001:00054E74       TBCBasePin.IsStopped
 0001:00054E80       TBCBasePin.NewSegment
 0001:00054EC4       TBCBasePin.NonDelegatingAddRef
 0001:00054F50       TBCBasePin.NonDelegatingRelease
 0001:00054FDC       TBCBasePin.Notify
 0001:00055020       TBCBasePin.QueryAccept
 0001:00055048       TBCBasePin.QueryDirection
 0001:0005505C       TBCBasePin.QueryId
 0001:00055074       TBCBasePin.QueryInternalConnections
 0001:0005508C       TBCBasePin.QueryPinInfo
 0001:00055100       TBCBasePin.ReceiveConnection
 0001:0005533C       TBCBasePin.Run
 0001:00055348       TBCBasePin.SetMediaType
 0001:00055368       TBCBasePin.SetSink
 0001:000553F4       TBCBasePin.TryMediaTypes
 0001:0005558C       TBCEnumMediaTypes.AreWeOutOfSync
 0001:000555A4       TBCEnumMediaTypes.Clone
 0001:00055608       TBCEnumMediaTypes.Create
 0001:000556D8       TBCEnumMediaTypes.Destroy
 0001:00055708       TBCEnumMediaTypes.Next
 0001:00055810       TBCEnumMediaTypes.Reset
 0001:00055830       TBCEnumMediaTypes.Skip
 0001:00055884       TBCBaseInputPin.BeginFlush
 0001:00055948       TBCBaseInputPin.BreakConnect
 0001:00055980       TBCBaseInputPin.CheckStreaming
 0001:00055A28       TBCBaseInputPin.Create
 0001:00055AEC       TBCBaseInputPin.Destroy
 0001:00055B28       TBCBaseInputPin.EndFlush
 0001:00055BF4       TBCBaseInputPin.GetAllocator
 0001:00055D10       TBCBaseInputPin.GetAllocatorRequirements
 0001:00055D1C       TBCBaseInputPin.Inactive
 0001:00055D44       TBCBaseInputPin.Notify
 0001:00055D84       TBCBaseInputPin.NotifyAllocator
 0001:00055E24       TBCBaseInputPin.Receive
 0001:00056060       TBCBaseInputPin.ReceiveCanBlock
 0001:000561F4       TBCBaseInputPin.ReceiveMultiple
 0001:00056234       TBCBaseInputPin.SampleProps
 0001:000562B4       TBCCritSec.Create
 0001:000562EC       TBCCritSec.CritCheckIn
 0001:000562F0       TBCCritSec.Destroy
 0001:00056314       TBCCritSec.Lock
 0001:00056320       TBCCritSec.UnLock
 0001:0005632C       TBCBasePropertyPage.Activate
 0001:00056394       TBCBasePropertyPage.Apply
 0001:000563E0       TBCBasePropertyPage.Deactivate
 0001:00056444       TBCBasePropertyPage.GetPageInfo
 0001:000564DC       TBCBasePropertyPage.Help
 0001:000564E8       TBCBasePropertyPage.IsPageDirty
 0001:00056504       TBCBasePropertyPage.Move
 0001:0005654C       TBCBasePropertyPage.SetObjects
 0001:0005659C       TBCBasePropertyPage.SetPageSite
 0001:000565E4       TBCBasePropertyPage.Show
 0001:00056648       TBCBasePropertyPage.TranslateAccelerator
 0001:00056654       TBCBasePropertyPage.Create
 0001:000566FC       TBCBasePropertyPage.Destroy
 0001:00056734       TBCBaseDispatch.GetIDsOfNames
 0001:000567B0       TBCBaseDispatch.GetTypeInfo
 0001:000568A0       TBCBaseDispatch.GetTypeInfoCount
 0001:000568B4       TBCMediaPosition.Create
 0001:00056950       TBCMediaPosition.Destroy
 0001:00056980       TBCMediaPosition.GetIDsOfNames
 0001:000569AC       TBCMediaPosition.GetTypeInfo
 0001:000569D4       TBCMediaPosition.GetTypeInfoCount
 0001:000569EC       TBCMediaPosition.Invoke
 0001:00056A8C       TBCPosPassThru.CheckCapabilities
 0001:00056AF8       TBCPosPassThru.ConvertTimeFormat
 0001:00056B70       TBCPosPassThru.Create
 0001:00056C80       TBCPosPassThru.GetAvailable
 0001:00056CF0       TBCPosPassThru.GetCapabilities
 0001:00056D5C       TBCPosPassThru.GetCurrentPosition
 0001:00056DEC       TBCPosPassThru.GetDuration
 0001:00056E58       TBCPosPassThru.GetMediaTime
 0001:00056E60       TBCPosPassThru.GetPeerSeeking
 0001:00056F14       TBCPosPassThru.GetPositions
 0001:00056F84       TBCPosPassThru.GetPreroll
 0001:00056FF0       TBCPosPassThru.GetRate
 0001:0005705C       TBCPosPassThru.GetStopPosition
 0001:000570C8       TBCPosPassThru.GetTimeFormat
 0001:00057134       TBCPosPassThru.IsFormatSupported
 0001:000571A0       TBCPosPassThru.IsUsingTimeFormat
 0001:0005720C       TBCPosPassThru.QueryPreferredFormat
 0001:00057278       TBCPosPassThru.SetPositions
 0001:000572F0       TBCPosPassThru.SetRate
 0001:00057374       TBCPosPassThru.SetTimeFormat
 0001:000573E0       TBCRendererPosPassThru.Create
 0001:000574B4       TBCRendererPosPassThru.destroy
 0001:000574E4       TBCRendererPosPassThru.EOS
 0001:0005757C       TBCRendererPosPassThru.GetMediaTime
 0001:0005762C       TBCRendererPosPassThru.RegisterMediaTime
 0001:00057784       TBCRendererPosPassThru.ResetMediaTime
 0001:000577FC       TBCAMEvent.Create
 0001:00057848       TBCAMEvent.destroy
 0001:000578E4       TBCAMEvent.Reset
 0001:000578F0       TBCAMEvent.SetEv
 0001:000578FC       TimeKillSynchronousFlagAvailable
 0001:0005793C       CompatibleTimeSetEvent
 0001:00057998       MSR_INTEGER
 0001:0005799C       TimeDiff
 0001:000579DC       TBCBaseRenderer.Create
 0001:00057B4C       TBCBaseRenderer.Destroy
 0001:00057C74       TBCBaseRenderer.GetMediaPositionInterface
 0001:00057DE0       TBCBaseRenderer.JoinFilterGraph
 0001:00057E4C       TBCBaseRenderer.NonDelegatingQueryInterface
 0001:00057E98       TBCBaseRenderer.SourceThreadCanWait
 0001:00057EB4       TBCBaseRenderer.WaitForRenderTime
 0001:00057F24       TBCBaseRenderer.WaitForReceiveToComplete
 0001:00057F74       TBCBaseRenderer.GetRealState
 0001:00057F78       WaitDispatchingMessages
 0001:00058158       TBCBaseRenderer.GetState
 0001:00058190       TBCBaseRenderer.CompleteStateChange
 0001:000581D8       TBCBaseRenderer.OnReceiveFirstSample
 0001:00058200       TBCBaseRenderer.Ready
 0001:0005820C       TBCBaseRenderer.NotReady
 0001:00058218       TBCBaseRenderer.Stop
 0001:000583D4       TBCBaseRenderer.Pause
 0001:00058618       TBCBaseRenderer.Run
 0001:0005889C       TBCBaseRenderer.GetPinCount
 0001:000588A4       TBCBaseRenderer.GetPin
 0001:000589E4       DumbItDownFor95
 0001:00058A78       WideCompareText
 0001:00058ADC       TBCBaseRenderer.FindPin
 0001:00058BF4       TBCBaseRenderer.EndOfStream
 0001:00058C28       TBCBaseRenderer.BeginFlush
 0001:00058C60       TBCBaseRenderer.EndFlush
 0001:00058CF0       TBCBaseRenderer.CompleteConnect
 0001:00058D60       TBCBaseRenderer.Active
 0001:00058D64       TBCBaseRenderer.Inactive
 0001:00058D84       TBCBaseRenderer.SetMediaType
 0001:00058D88       TBCBaseRenderer.BreakConnect
 0001:00058E00       TBCBaseRenderer.GetSampleTimes
 0001:00058F24       TBCBaseRenderer.ShouldDrawSampleNow
 0001:00058F58       TBCBaseRenderer.SignalTimerFired
 0001:00058F60       TBCBaseRenderer.CancelNotification
 0001:00059024       TBCBaseRenderer.ScheduleSample
 0001:000591AC       TBCBaseRenderer.Render
 0001:0005922C       TBCBaseRenderer.HaveCurrentSample
 0001:00059288       TBCBaseRenderer.GetCurrentSample
 0001:000592E4       TBCBaseRenderer.PrepareReceive
 0001:00059620       TBCBaseRenderer.Receive
 0001:000598F8       TBCBaseRenderer.ClearPendingSample
 0001:00059960       EndOfStreamTimer
 0001:00059970       TBCBaseRenderer.TimerCallback
 0001:000599D8       TBCBaseRenderer.SendEndOfStream
 0001:00059A90       TBCBaseRenderer.NotifyEndOfStream
 0001:00059C28       TBCBaseRenderer.ResetEndOfStream
 0001:00059CAC       TBCBaseRenderer.ResetEndOfStreamTimer
 0001:00059CCC       TBCBaseRenderer.StartStreaming
 0001:00059E44       TBCBaseRenderer.StopStreaming
 0001:00059EC0       TBCBaseRenderer.SetRepaintStatus
 0001:00059F18       TBCBaseRenderer.OnRenderStart
 0001:00059F40       TBCBaseRenderer.OnRenderEnd
 0001:00059F68       TBCBaseRenderer.OnStartStreaming
 0001:00059F6C       TBCBaseRenderer.OnStopStreaming
 0001:00059F70       TBCBaseRenderer.OnWaitStart
 0001:00059F74       TBCBaseRenderer.OnWaitEnd
 0001:00059F78       TBCBaseRenderer.PrepareRender
 0001:00059F7C       TBCRendererInputPin.Create
 0001:0005A098       TBCRendererInputPin.EndOfStream
 0001:0005A158       TBCRendererInputPin.BeginFlush
 0001:0005A224       TBCRendererInputPin.EndFlush
 0001:0005A2CC       TBCRendererInputPin.Receive
 0001:0005A440       TBCRendererInputPin.InheritedReceive
 0001:0005A490       TBCRendererInputPin.BreakConnect
 0001:0005A4C0       TBCRendererInputPin.CompleteConnect
 0001:0005A530       TBCRendererInputPin.QueryId
 0001:0005A550       TBCRendererInputPin.CheckMediaType
 0001:0005A560       TBCRendererInputPin.Active
 0001:0005A570       TBCRendererInputPin.Inactive
 0001:0005A584       TBCRendererInputPin.SetMediaType
 0001:0005A5BC       TBCBaseVideoRenderer.Create
 0001:0005A66C       TBCBaseVideoRenderer.Destroy
 0001:0005A6FC       TBCBaseVideoRenderer.ResetStreamingTimes
 0001:0005A7FC       TBCBaseVideoRenderer.PreparePerformanceData
 0001:0005A80C       TBCBaseVideoRenderer.RecordFrameLateness
 0001:0005A940       TBCBaseVideoRenderer.ThrottleWait
 0001:0005A978       TBCBaseVideoRenderer.OnDirectRender
 0001:0005A9D8       TBCBaseVideoRenderer.OnRenderStart
 0001:0005AA28       TBCBaseVideoRenderer.OnRenderEnd
 0001:0005AAA4       TBCBaseVideoRenderer.SetSink
 0001:0005AAF8       TBCBaseVideoRenderer.Notify
 0001:0005AB6C       TBCBaseVideoRenderer.SendQuality
 0001:0005ADB4       TBCBaseVideoRenderer.ShouldDrawSampleNow
 0001:0005B1E4       TBCBaseVideoRenderer.ScheduleSample
 0001:0005B240       TBCBaseVideoRenderer.get_FramesDroppedInRenderer
 0001:0005B2A8       TBCBaseVideoRenderer.get_FramesDrawn
 0001:0005B310       TBCBaseVideoRenderer.get_AvgFrameRate
 0001:0005B428       TBCBaseVideoRenderer.get_AvgSyncOffset
 0001:0005B4D4       isqrt
 0001:0005B540       TBCBaseVideoRenderer.GetStdDev
 0001:0005B698       TBCBaseVideoRenderer.get_DevSyncOffset
 0001:0005B6CC       TBCBaseVideoRenderer.get_Jitter
 0001:0005B700       TBCBaseVideoRenderer.NonDelegatingQueryInterface
 0001:0005B77C       TBCBaseVideoRenderer.JoinFilterGraph
 0001:0005B814       Finalization
 0001:0005B860       BaseClass
 0001:0005B9F4       PossiblyEatMessage
 0001:0005BA48       TfrmRenderer.WndProc
 0001:0005BA84       TfrmRenderer.DoSetWindowStyle
 0001:0005BB64       TfrmRenderer.DoGetWindowStyle
 0001:0005BB84       TfrmRenderer.DoShowWindow
 0001:0005BBA0       TfrmRenderer.DoPaintWindow
 0001:0005BBC0       TfrmRenderer.DoRenderSample
 0001:0005BC74       TfrmRenderer.DoInitializeDirectDraw
 0001:0005BCB8       TfrmRenderer.FormCreate
 0001:0005BCC4       Finalization
 0001:0005BCF4       formRenderer
 0001:0005C524       CheckConnected
 0001:0005C54C       TVideoRenderer.Create
 0001:0005C614       TVideoRenderer.CreateFromFactory
 0001:0005C65C       TVideoRenderer.Destroy
 0001:0005C6AC       TVideoRenderer.Active
 0001:0005C6CC       TVideoRenderer.Inactive
 0001:0005C6D4       TVideoRenderer.CheckMediaType
 0001:0005C724       TVideoRenderer.DoRenderSample
 0001:0005C784       TVideoRenderer.OnReceiveFirstSample
 0001:0005C7D4       TVideoRenderer.SetMediaType
 0001:0005C824       TVideoRenderer.GetTypeInfoCount
 0001:0005C840       TVideoRenderer.GetTypeInfo
 0001:0005C86C       TVideoRenderer.GetIDsOfNames
 0001:0005C89C       TVideoRenderer.Invoke
 0001:0005C978       TVideoRenderer.put_Caption
 0001:0005C9F4       TVideoRenderer.get_Caption
 0001:0005CA6C       TVideoRenderer.put_WindowStyle
 0001:0005CAF4       TVideoRenderer.get_WindowStyle
 0001:0005CB2C       TVideoRenderer.put_WindowStyleEx
 0001:0005CBA0       TVideoRenderer.get_WindowStyleEx
 0001:0005CBD8       TVideoRenderer.put_AutoShow
 0001:0005CC08       TVideoRenderer.get_AutoShow
 0001:0005CC38       TVideoRenderer.put_WindowState
 0001:0005CC6C       TVideoRenderer.get_WindowState
 0001:0005CCE0       TVideoRenderer.put_BackgroundPalette
 0001:0005CD08       TVideoRenderer.get_BackgroundPalette
 0001:0005CD30       TVideoRenderer.put_Visible
 0001:0005CD64       TVideoRenderer.get_Visible
 0001:0005CD98       TVideoRenderer.put_Left
 0001:0005CE44       TVideoRenderer.get_Left
 0001:0005CE8C       TVideoRenderer.put_Width
 0001:0005CF2C       TVideoRenderer.get_Width
 0001:0005CF74       TVideoRenderer.put_Top
 0001:0005D020       TVideoRenderer.get_Top
 0001:0005D068       TVideoRenderer.put_Height
 0001:0005D108       TVideoRenderer.get_Height
 0001:0005D150       TVideoRenderer.put_Owner
 0001:0005D190       TVideoRenderer.get_Owner
 0001:0005D1C4       TVideoRenderer.put_MessageDrain
 0001:0005D1F4       TVideoRenderer.get_MessageDrain
 0001:0005D228       TVideoRenderer.get_BorderColor
 0001:0005D250       TVideoRenderer.put_BorderColor
 0001:0005D278       TVideoRenderer.get_FullScreenMode
 0001:0005D2A0       TVideoRenderer.put_FullScreenMode
 0001:0005D2C8       TVideoRenderer.SetWindowForeground
 0001:0005D304       TVideoRenderer.NotifyOwnerMessage
 0001:0005D39C       TVideoRenderer.SetWindowPosition
 0001:0005D4C0       TVideoRenderer.GetWindowPosition
 0001:0005D524       TVideoRenderer.GetMinIdealImageSize
 0001:0005D594       TVideoRenderer.GetMaxIdealImageSize
 0001:0005D604       TVideoRenderer.GetRestorePosition
 0001:0005D6A0       TVideoRenderer.HideCursor
 0001:0005D6C8       TVideoRenderer.IsCursorHidden
 0001:0005D6F0       TVideoRenderer.get_AvgTimePerFrame
 0001:0005D724       TVideoRenderer.get_BitRate
 0001:0005D754       TVideoRenderer.get_BitErrorRate
 0001:0005D784       TVideoRenderer.get_VideoWidth
 0001:0005D7B4       TVideoRenderer.get_VideoHeight
 0001:0005D7E4       TVideoRenderer.put_SourceLeft
 0001:0005D80C       TVideoRenderer.get_SourceLeft
 0001:0005D834       TVideoRenderer.put_SourceWidth
 0001:0005D85C       TVideoRenderer.get_SourceWidth
 0001:0005D884       TVideoRenderer.put_SourceTop
 0001:0005D8AC       TVideoRenderer.get_SourceTop
 0001:0005D8D4       TVideoRenderer.put_SourceHeight
 0001:0005D8FC       TVideoRenderer.get_SourceHeight
 0001:0005D924       TVideoRenderer.put_DestinationLeft
 0001:0005D94C       TVideoRenderer.get_DestinationLeft
 0001:0005D974       TVideoRenderer.put_DestinationWidth
 0001:0005D99C       TVideoRenderer.get_DestinationWidth
 0001:0005D9C4       TVideoRenderer.put_DestinationTop
 0001:0005D9EC       TVideoRenderer.get_DestinationTop
 0001:0005DA14       TVideoRenderer.put_DestinationHeight
 0001:0005DA3C       TVideoRenderer.get_DestinationHeight
 0001:0005DA64       TVideoRenderer.SetSourcePosition
 0001:0005DA8C       TVideoRenderer.GetSourcePosition
 0001:0005DAB4       TVideoRenderer.SetDefaultSourcePosition
 0001:0005DADC       TVideoRenderer.SetDestinationPosition
 0001:0005DB04       TVideoRenderer.GetDestinationPosition
 0001:0005DB2C       TVideoRenderer.SetDefaultDestinationPosition
 0001:0005DB54       TVideoRenderer.GetVideoSize
 0001:0005DB90       TVideoRenderer.GetVideoPaletteEntries
 0001:0005DBB8       TVideoRenderer.GetCurrentImage
 0001:0005DBE0       TVideoRenderer.IsUsingDefaultSource
 0001:0005DC08       TVideoRenderer.IsUsingDefaultDestination
 0001:0005DC30       TVideoRenderer.GetPreferredAspectRatio
 0001:0005DC58       TVideoRenderer.GetMiscFlags
 0001:0005DC64       Finalization
 0001:0005DC94       VidRenderer
 0001:0005DCEC       Finalization
 0001:0005DF54       VideoRenderer
 0002:00000000       ExitCode
 0002:00000004       ErrorAddr
 0002:00000008       FileMode
 0002:0000000C       VarClearProc
 0002:00000010       VarAddRefProc
 0002:00000014       VarCopyProc
 0002:00000018       VarToLStrProc
 0002:0000001C       VarToWStrProc
 0002:00000020       Default8087CW
 0002:00000024       HeapAllocFlags
 0002:00000028       DebugHook
 0002:0000002C       JITEnable
 0002:00000030       NoErrMsg
 0002:00000034       LibModuleList
 0002:00000038       ModuleUnloadList
 0002:0000003C       MemoryManager
 0002:00000048       reMap
 0002:00000064       errCaption
 0002:0000006C       runErrMsg
 0002:0000008C       dig
 0002:0000009C       TlsIndex
 0002:000000A0       PtrToNil
 0002:000000A4       Module
 0002:000000BC       TlsProc
 0002:000000CC       EmptyStr
 0002:000000D0       EmptyWideStr
 0002:000000D4       Win32Platform
 0002:000000D8       Win32MajorVersion
 0002:000000DC       Win32MinorVersion
 0002:000000E0       Win32BuildNumber
 0002:000000E4       Win32CSDVersion
 0002:000000E8       TwoDigitYearCenturyWindow
 0002:000000EC       MonthDays
 0002:0000011C       LeadBytes
 0002:0000013C       HexDisplayPrefix
 0002:00000140       GetDiskFreeSpaceEx
 0002:00000144       cSimpleBoolStrs
 0002:0000014C       AccessMode
 0002:00000158       ShareMode
 0002:0000016C       FormatErrorStrs
 0002:00000174       FCon1E18
 0002:00000180       DCon10
 0002:00000184       CWNear
 0002:00000188       FMSecsPerDay
 0002:0000018C       IMSecsPerDay
 0002:00000190       Format
 0002:00000194       DefShortMonthNames
 0002:000001C4       DefLongMonthNames
 0002:000001F4       DefShortDayNames
 0002:00000210       DefLongDayNames
 0002:0000022C       ErrorMap
 0002:00000264       ExceptMap
 0002:00000314       WesternGroups
 0002:00000318       TerminateProcList
 0002:0000031C       CResult
 0002:00000324       NullStrictConvert
 0002:00000328       NullAsStringValue
 0002:0000032C       PackVarCreation
 0002:00000330       BooleanToStringRule
 0002:00000334       CInvalidCustomVariantType
 0002:00000338       CRangeToType
 0002:0000034C       CText
 0002:000003A0       CRelationshipToBoolean
 0002:000003B4       BooleanIdents
 0002:000003BC       DotSep
 0002:000003C0       GUID_NULL
 0002:000003D0       AddDataModule
 0002:000003D8       RemoveDataModule
 0002:000003E0       ApplicationHandleException
 0002:000003E8       ApplicationShowException
 0002:000003F0       WakeMainThread
 0002:000003F8       FilerSignature
 0002:000003FC       NilMethod
 0002:00000404       SyncList
 0002:00000408       BlockCode
 0002:0000040C       UtilWindowClass
 0002:00000434       DefFontData
 0002:00000460       DDBsOnly
 0002:00000464       Colors
 0002:00000604       FontCharsets
 0002:00000694       DefPenData
 0002:000006A4       PenStyles
 0002:000006B4       DefBrushData
 0002:000006C4       PenModes
 0002:000006E4       ClipboardFormats
 0002:000006E8       FileFormats
 0002:000006EC       BitmapCanvasList
 0002:000006F0       DIBPalSizes
 0002:000006F4       PalSize
 0002:000006F8       Pal16
 0002:00000738       FPrinter
 0002:0000073C       CreationControl
 0002:00000740       WndProcPtrAtom
 0002:00000744       Captions
 0002:00000758       ButtonNames
 0002:00000784       ButtonCaptions
 0002:000007B0       ColorToPretyName
 0002:00000928       BitBtnCaptions
 0002:00000954       Values
 0002:0000095C       Values
 0002:00000964       MAPIDLL
 0002:00000968       MAPIModule
 0002:0000096C       RTFConversionFormat
 0002:00000978       TextConversionFormat
 0002:00000984       ThemeServicesClass
 0002:00000988       Copyright
 0002:0000098C       ThemeDataNames
 0002:000009EC       AnimateWindowProc
 0002:000009F0       CreationControl
 0002:000009F4       DefaultDockTreeClass
 0002:000009F8       AnchorAlign
 0002:00000A00       Cursors
 0002:00000AB0       CaptureControl
 0002:00000AB4       ShowFlags
 0002:00000AB8       WindowPos
 0002:00000ABC       InnerStyles
 0002:00000ACC       OuterStyles
 0002:00000ADC       EdgeStyles
 0002:00000AEC       Ctl3DStyles
 0002:00000AF4       AnimationStyle
 0002:00000B00       OrientArray
 0002:00000B08       MakeLast
 0002:00000B10       TreeStreamEndFlag
 0002:00000B14       SizeCursors
 0002:00000B1C       IMM32DLL
 0002:00000B20       ModeMap
 0002:00000B28       DrawingStyles
 0002:00000B38       Images
 0002:00000B40       Mask
 0002:00000B48       ValidMenuHotkeys
 0002:00000B4C       cMenuAutoFlagToItem
 0002:00000B50       cItemAutoFlagToMenu
 0002:00000B54       cBooleanToItemAutoFlag
 0002:00000B58       cItemAutoFlagToBoolean
 0002:00000B5C       MenuKeyCaps
 0002:00000BA4       Checks
 0002:00000BAC       Enables
 0002:00000BB4       Breaks
 0002:00000BC0       Separators
 0002:00000BC8       IBreaks
 0002:00000BD4       IChecks
 0002:00000BDC       IDefaults
 0002:00000BE4       IEnables
 0002:00000BEC       IRadios
 0002:00000BF4       ISeparators
 0002:00000BFC       IRTL
 0002:00000C04       IOwnerDraw
 0002:00000C0C       Alignments
 0002:00000C14       EdgeStyle
 0002:00000C1C       Alignments
 0002:00000C24       Flags
 0002:00000C30       Buttons
 0002:00000C34       HintWindowClass
 0002:00000C38       SetLayeredWindowAttributes
 0002:00000C3C       FocusMessages
 0002:00000C40       FocusCount
 0002:00000C44       TaskActiveWindow
 0002:00000C48       TaskFirstWindow
 0002:00000C4C       TaskFirstTopMost
 0002:00000C50       TaskWindowList
 0002:00000C54       SysConsts
 0002:00000C5C       SysConsts
 0002:00000C64       Props
 0002:00000C8C       Styles
 0002:00000C98       ShowCommands
 0002:00000CA4       ShowCommands
 0002:00000CB0       ShowCommands
 0002:00000CBC       cUseAlpha
 0002:00000CC4       cUseColorKey
 0002:00000CCC       CursorMap
 0002:00000D20       WindowClass
 0002:00000D48       AppVisible
 0002:00000D4C       ShowFlags
 0002:00000D50       CoCreateInstanceEx
 0002:00000D54       CoInitializeEx
 0002:00000D58       CoAddRefServerProcess
 0002:00000D5C       CoReleaseServerProcess
 0002:00000D60       CoResumeClassObjects
 0002:00000D64       CoSuspendClassObjects
 0002:00000D68       CoInitFlags
 0002:00000D6C       ThreadStrs
 0002:00000D80       IID_IBaseFilter
 0002:00000D90       IID_IMediaSample2
 0002:00000DA0       IID_IMemAllocator
 0002:00000DB0       IID_IMemInputPin
 0002:00000DC0       IID_IMediaSeeking
 0002:00000DD0       IID_IQualityControl
 0002:00000DE0       IID_IMediaEventSink
 0002:00000DF0       LIBID_QuartzTypeLib
 0002:00000E00       IID_IMediaPosition
 0002:00000E10       IID_IVideoWindow
 0002:00000E20       IID_IQualProp
 0002:00000E30       GUID_NULL
 0002:00000E40       MEDIATYPE_Video
 0002:00000E50       MEDIASUBTYPE_RGB24
 0002:00000E60       CLSID_FilterMapper
 0002:00000E70       CLSID_VideoRenderer
 0002:00000E80       CLSID_LegacyAmFilterCategory
 0002:00000E90       CLSID_FilterMapper2
 0002:00000EA0       CLSID_MemoryAllocator
 0002:00000EB0       FORMAT_VideoInfo
 0002:00000EC0       TIME_FORMAT_MEDIA_TIME
 0002:00000ED0       MAX_TIME
 0002:00000ED8       wszStreamName
 0002:00000EDC       IsCheckedVersion
 0002:00000EE0       IsTimeKillSynchronousFlagAvailable
 0002:00000EE4       MsgId
 0002:00000EE8       CLSID_DelphiVideoRenderer
 0002:00002000       DispCallByIDProc
 0002:00002004       ExceptProc
 0002:00002008       ErrorProc
 0002:0000200C       ExceptClsProc
 0002:00002010       ExceptObjProc
 0002:00002014       RaiseExceptionProc
 0002:00002018       RTLUnwindProc
 0002:0000201C       ExceptionClass
 0002:00002020       SafeCallErrorProc
 0002:00002024       AssertErrorProc
 0002:00002028       ExitProcessProc
 0002:0000202C       AbstractErrorProc
 0002:00002030       MainInstance
 0002:00002034       MainThreadID
 0002:00002038       IsLibrary
 0002:0000203C       CmdShow
 0002:00002040       CmdLine
 0002:00002044       InitProc
 0002:00002048       ExitProc
 0002:0000204C       IsConsole
 0002:0000204D       IsMultiThread
 0002:0000204E       Test8086
 0002:00002050       Input
 0002:0000221C       Output
 0002:000023E8       ErrOutput
 0002:000025B4       AllocMemCount
 0002:000025B8       AllocMemSize
 0002:000025BC       .5
 0002:000025C0       DefaultUserCodePage
 0002:000025C4       initialized
 0002:000025C8       heapErrorCode
 0002:000025CC       heapLock
 0002:000025E4       blockDescBlockList
 0002:000025E8       blockDescFreeList
 0002:000025EC       spaceRoot
 0002:000025FC       decommittedRoot
 0002:0000260C       avail
 0002:00002618       rover
 0002:0000261C       remBytes
 0002:00002620       curAlloc
 0002:00002624       smallTab
 0002:00002628       committedRoot
 0002:00002638       InitContext
 0002:00002664       ModuleIsLib
 0002:00002665       ModuleIsCpp
 0002:00002668       HInstance
 0002:0000266C       DllProc
 0002:00002670       .1
 0002:00002674       tlsBuffer
 0002:00002678       .1
 0002:0000267C       .3
 0002:00002680       .1
 0002:00002684       CurrencyString
 0002:00002688       CurrencyFormat
 0002:00002689       NegCurrFormat
 0002:0000268A       ThousandSeparator
 0002:0000268B       DecimalSeparator
 0002:0000268C       CurrencyDecimals
 0002:0000268D       DateSeparator
 0002:00002690       ShortDateFormat
 0002:00002694       LongDateFormat
 0002:00002698       TimeSeparator
 0002:0000269C       TimeAMString
 0002:000026A0       TimePMString
 0002:000026A4       ShortTimeFormat
 0002:000026A8       LongTimeFormat
 0002:000026AC       ShortMonthNames
 0002:000026DC       LongMonthNames
 0002:0000270C       ShortDayNames
 0002:00002728       LongDayNames
 0002:00002744       SysLocale
 0002:00002752       ListSeparator
 0002:00002754       EraNames
 0002:00002770       EraYearOffsets
 0002:0000278C       TrueBoolStrs
 0002:00002790       FalseBoolStrs
 0002:00002794       .35
 0002:00002798       OutOfMemory
 0002:0000279C       InvalidPointer
 0002:000027A0       FLanguages
 0002:000027A4       .1
 0002:000027A8       VariantChangeTypeEx
 0002:000027AC       VarNeg
 0002:000027B0       VarNot
 0002:000027B4       VarAdd
 0002:000027B8       VarSub
 0002:000027BC       VarMul
 0002:000027C0       VarDiv
 0002:000027C4       VarIDiv
 0002:000027C8       VarMod
 0002:000027CC       VarAnd
 0002:000027D0       VarOr
 0002:000027D4       VarXor
 0002:000027D8       VarCmp
 0002:000027DC       VarI4FromStr
 0002:000027E0       VarR4FromStr
 0002:000027E4       VarR8FromStr
 0002:000027E8       VarDateFromStr
 0002:000027EC       VarCyFromStr
 0002:000027F0       VarBoolFromStr
 0002:000027F4       VarBstrFromCy
 0002:000027F8       VarBstrFromDate
 0002:000027FC       VarBstrFromBool
 0002:00002800       .5
 0002:00002804       EmptyParam
 0002:00002814       VarDispProc
 0002:00002818       ClearAnyProc
 0002:0000281C       ChangeAnyProc
 0002:00002820       RefAnyProc
 0002:00002824       .81
 0002:00002828       LVarTypes
 0002:0000282C       LVarTypeSync
 0002:00002844       .1
 0002:00002848       .6
 0002:0000284C       .3
 0002:00002850       GlobalNameSpace
 0002:00002854       IsUniqueGlobalComponentNameProc
 0002:00002858       SyncEvent
 0002:0000285C       .45
 0002:00002860       IntConstList
 0002:00002864       RegGroups
 0002:00002868       FindGlobalComponentProcs
 0002:0000286C       GlobalFixupList
 0002:00002870       ThreadLock
 0002:00002888       InstBlockList
 0002:0000288C       InstFreeList
 0002:00002890       .2
 0002:00002894       .1
 0002:00002898       SystemPalette16
 0002:0000289C       .12
 0002:000028A0       ScreenLogPixels
 0002:000028A4       StockPen
 0002:000028A8       StockBrush
 0002:000028AC       StockFont
 0002:000028B0       StockIcon
 0002:000028B4       BitmapImageLock
 0002:000028CC       CounterLock
 0002:000028E4       FontManager
 0002:000028E8       PenManager
 0002:000028EC       BrushManager
 0002:000028F0       CanvasList
 0002:000028F4       PatternManager
 0002:000028F8       .21
 0002:000028FC       .1
 0002:00002900       GetSystemMetrics
 0002:00002904       MonitorFromWindow
 0002:00002908       MonitorFromRect
 0002:0000290C       MonitorFromPoint
 0002:00002910       GetMonitorInfo
 0002:00002914       GetMonitorInfoA
 0002:00002918       GetMonitorInfoW
 0002:0000291C       EnumDisplayMonitors
 0002:00002920       .1
 0002:00002924       User32Dll
 0002:00002928       InitApis
 0002:00002930       MMAvailable
 0002:00002934       .1
 0002:00002938       .2
 0002:0000293C       HelpManager
 0002:00002940       .3
 0002:00002944       .3
 0002:00002948       FlatSB_EnableScrollBar
 0002:0000294C       FlatSB_ShowScrollBar
 0002:00002950       FlatSB_GetScrollRange
 0002:00002954       FlatSB_GetScrollInfo
 0002:00002958       FlatSB_GetScrollPos
 0002:0000295C       FlatSB_SetScrollPos
 0002:00002960       FlatSB_SetScrollInfo
 0002:00002964       FlatSB_SetScrollRange
 0002:00002968       .1
 0002:0000296C       _FlatSB_GetScrollProp
 0002:00002970       _FlatSB_SetScrollProp
 0002:00002974       _InitializeFlatSB
 0002:00002978       _UninitializeFlatSB
 0002:0000297C       .6
 0002:00002980       OpenThemeData
 0002:00002984       CloseThemeData
 0002:00002988       DrawThemeBackground
 0002:0000298C       DrawThemeText
 0002:00002990       GetThemeBackgroundContentRect
 0002:00002994       GetThemeBackgroundExtent
 0002:00002998       GetThemePartSize
 0002:0000299C       GetThemeTextExtent
 0002:000029A0       GetThemeTextMetrics
 0002:000029A4       GetThemeBackgroundRegion
 0002:000029A8       HitTestThemeBackground
 0002:000029AC       DrawThemeEdge
 0002:000029B0       DrawThemeIcon
 0002:000029B4       IsThemePartDefined
 0002:000029B8       IsThemeBackgroundPartiallyTransparent
 0002:000029BC       GetThemeColor
 0002:000029C0       GetThemeMetric
 0002:000029C4       GetThemeString
 0002:000029C8       GetThemeBool
 0002:000029CC       GetThemeInt
 0002:000029D0       GetThemeEnumValue
 0002:000029D4       GetThemePosition
 0002:000029D8       GetThemeFont
 0002:000029DC       GetThemeRect
 0002:000029E0       GetThemeMargins
 0002:000029E4       GetThemeIntList
 0002:000029E8       GetThemePropertyOrigin
 0002:000029EC       SetWindowTheme
 0002:000029F0       GetThemeFilename
 0002:000029F4       GetThemeSysColor
 0002:000029F8       GetThemeSysColorBrush
 0002:000029FC       GetThemeSysBool
 0002:00002A00       GetThemeSysSize
 0002:00002A04       GetThemeSysFont
 0002:00002A08       GetThemeSysString
 0002:00002A0C       GetThemeSysInt
 0002:00002A10       IsThemeActive
 0002:00002A14       IsAppThemed
 0002:00002A18       GetWindowTheme
 0002:00002A1C       EnableThemeDialogTexture
 0002:00002A20       IsThemeDialogTextureEnabled
 0002:00002A24       GetThemeAppProperties
 0002:00002A28       SetThemeAppProperties
 0002:00002A2C       GetCurrentThemeName
 0002:00002A30       GetThemeDocumentationProperty
 0002:00002A34       DrawThemeParentBackground
 0002:00002A38       EnableTheming
 0002:00002A3C       .1
 0002:00002A40       ThemeLibrary
 0002:00002A44       ReferenceCount
 0002:00002A48       Lock
 0002:00002A4C       .1
 0002:00002A50       .4
 0002:00002A54       .1
 0002:00002A58       .1
 0002:00002A5C       .1
 0002:00002A60       .1
 0002:00002A64       .1
 0002:00002A68       .1
 0002:00002A6C       .1
 0002:00002A70       .11
 0002:00002A74       HelpMsg
 0002:00002A78       FindMsg
 0002:00002A7C       .12
 0002:00002A80       .1
 0002:00002A84       CF_PICTURE
 0002:00002A86       CF_COMPONENT
 0002:00002A88       .2
 0002:00002A8C       FClipboard
 0002:00002A90       .1
 0002:00002A94       .4
 0002:00002A98       BitBtnGlyphs
 0002:00002AC4       .3
 0002:00002AC8       .8
 0002:00002ACC       .5
 0002:00002AD0       .1
 0002:00002AD4       .72
 0002:00002AD8       UrlMonHandle
 0002:00002ADC       UrlMonInitialized
 0002:00002AE0       .8
 0002:00002AE4       .36
 0002:00002AE8       ShellModule
 0002:00002AEC       FRichEditModule
 0002:00002AF0       ComCtlVersion
 0002:00002AF4       .2
 0002:00002AF8       InternalServices
 0002:00002AFC       .42
 0002:00002B00       .73
 0002:00002B04       WinHelpTester
 0002:00002B08       ViewerName
 0002:00002B0C       .1
 0002:00002B10       HelpViewer
 0002:00002B14       HelpViewerIntf
 0002:00002B18       Mouse
 0002:00002B1C       NewStyleControls
 0002:00002B20       .72
 0002:00002B24       WindowAtom
 0002:00002B26       ControlAtom
 0002:00002B28       WindowAtomString
 0002:00002B2C       ControlAtomString
 0002:00002B30       RM_GetObjectInstance
 0002:00002B34       DragControl
 0002:00002B38       DragObject
 0002:00002B3C       DragInternalObject
 0002:00002B40       DragCapture
 0002:00002B44       DragStartPos
 0002:00002B4C       DragSaveCursor
 0002:00002B50       DragThreshold
 0002:00002B54       ActiveDrag
 0002:00002B58       DragImageList
 0002:00002B5C       DockSiteList
 0002:00002B60       QualifyingSites
 0002:00002B64       DragSave
 0002:00002B68       CanvasList
 0002:00002B6C       _WINNLSEnableIME
 0002:00002B70       _ImmGetContext
 0002:00002B74       _ImmReleaseContext
 0002:00002B78       _ImmGetConversionStatus
 0002:00002B7C       _ImmSetConversionStatus
 0002:00002B80       _ImmSetOpenStatus
 0002:00002B84       _ImmSetCompositionWindow
 0002:00002B88       _ImmSetCompositionFont
 0002:00002B8C       _ImmGetCompositionString
 0002:00002B90       _ImmIsIME
 0002:00002B94       _ImmNotifyIME
 0002:00002B98       .8
 0002:00002B9C       .3
 0002:00002BA0       CachedComCtrlVer
 0002:00002BA4       ImageListWriteExProc
 0002:00002BA8       PopupList
 0002:00002BAC       ShortCutItems
 0002:00002BB0       .9
 0002:00002BB4       CommandPool
 0002:00002BB8       Application
 0002:00002BBC       Screen
 0002:00002BC0       .41
 0002:00002BC4       RM_TaskbarCreated
 0002:00002BC8       HintThreadID
 0002:00002BCC       HintDoneEvent
 0002:00002BD0       HintHook
 0002:00002BD4       HintThread
 0002:00002BD8       .1
 0002:00002BDC       .7
 0002:00002BE0       .1
 0002:00002BE4       .1
 0002:00002BE8       .1
 0002:00002BEC       .1
 0002:00002BF0       .41
 0002:00002BF4       OleUninitializing
 0002:00002BF8       ComClassManagerVar
 0002:00002BFC       SaveInitProc
 0002:00002C00       NeedToUninitialize
 0002:00002C04       .31
 0002:00002C08       .1
 0002:00002C0C       .11
 0002:00002C10       .74
 0002:00002C14       ObjectCount
 0002:00002C18       FactoryCount
 0002:00002C1C       TemplatesVar
 0002:00002C20       .2
 0002:00002C24       .2


Line numbers for DirectDraw(DirectDraw.pas) segment .text

  7161 0001:0004F604  7161 0001:0004F60B

Line numbers for DXTypes(DXTypes.pas) segment .text

    67 0001:0004F69C    67 0001:0004F6A3

Line numbers for DirectSound(DirectSound.pas) segment .text

  2426 0001:0004F710  2426 0001:0004F717

Line numbers for Direct3D9(Direct3D9.pas) segment .text

  4942 0001:0004F748  4942 0001:0004F74F

Line numbers for DirectShow9(DirectShow9.pas) segment .text

 31878 0001:000409B7

Line numbers for WMF9(WMF9.pas) segment .text

 15611 0001:000509B8 15611 0001:000509E4 15586 0001:000509E8 15606 0001:000509EF

Line numbers for DSUtil(DSUtil.pas) segment .text

  1097 0001:000509F0  1098 0001:000509F2  1099 0001:000509F6  1100 0001:000509FD
  1223 0001:00050A00  1225 0001:00050A03  1226 0001:00050A07  1227 0001:00050A0E
  1228 0001:00050A14  1256 0001:00050A18  1259 0001:00050A1F  1261 0001:00050A37
  1262 0001:00050A45  1264 0001:00050A4B  1265 0001:00050A65  1266 0001:00050A73
  1267 0001:00050A77  1269 0001:00050A7E  1271 0001:00050A8B  1272 0001:00050A9A
  1275 0001:00050AEC  1276 0001:00050AEF  1278 0001:00050AF5  1280 0001:00050AFE
  1281 0001:00050B03  1283 0001:00050B08  1284 0001:00050B16  4174 0001:00050B40
  4175 0001:00050B43  4176 0001:00050B46  4177 0001:00050B49  4178 0001:00050B4C
  4179 0001:00050B4F  4180 0001:00050B51  4181 0001:00050B53  4183 0001:00050B55
  4197 0001:00050B5C  4198 0001:00050B5E  4214 0001:00050B60  4215 0001:00050B6F
  4216 0001:00050B8D  4217 0001:00050BAC  4218 0001:00050BCA  4219 0001:00050BE9
  4220 0001:00050C07  4221 0001:00050C26  4223 0001:00050C50  4225 0001:00050C62
  4229 0001:00050C9A  4230 0001:00050CA0  4232 0001:00050CC2  4234 0001:00050CD2
  4236 0001:00050CD6  4237 0001:00050CFB  4238 0001:00050D21  4241 0001:00050D37
  4242 0001:00050D49  4243 0001:00050D6F  4246 0001:00050D83  4247 0001:00050DA1
  4249 0001:00050DA6  4250 0001:00050DAC  4252 0001:00050DB1  4253 0001:00050DD6
  4255 0001:00050DDC  4256 0001:00050DE2  4258 0001:00050DE7  4260 0001:00050E05
  4262 0001:00050E0B  4263 0001:00050E1A  4264 0001:00050E28  4265 0001:00050E38
  4266 0001:00050E48  4270 0001:00050E64  4272 0001:00050E83  4274 0001:00050E97
  4275 0001:00050EAE  4276 0001:00050EBC  4279 0001:00050EC1  4281 0001:00050ECD
  4282 0001:00050EE3  4283 0001:00050EFF  4284 0001:00050F0B  4287 0001:00050F10
  4288 0001:00050F1C  4290 0001:00050F22  4291 0001:00050F27  4292 0001:00050F2D
  4293 0001:00050F33  4294 0001:00050F45  4295 0001:00050F5A  4296 0001:00050F5F
  4297 0001:00050F6F  4298 0001:00050F8B  4299 0001:00050F97  4302 0001:00050F9C
  4304 0001:00050FAA  4306 0001:00050FAF  4307 0001:00050FC1  4308 0001:00050FD3
  4309 0001:00050FDC  4310 0001:00050FEC  4312 0001:00051000  4313 0001:00051012
  4304 0001:00051024  4317 0001:00051027  4318 0001:00051040  4319 0001:00051052
  5015 0001:000510A4  5015 0001:000510B7

Line numbers for BaseClass(BaseClass.pas) segment .text

   106 0001:0005117C   144 0001:00051240   265 0001:00051394   416 0001:000515D0
   466 0001:000519B4  1307 0001:00051F20  2887 0001:00052650  2888 0001:00052658
  2889 0001:0005265A  2892 0001:00052677  2895 0001:0005269D  2897 0001:000526B0
  2898 0001:000526C3  2899 0001:000526CD  2902 0001:000526E9  2903 0001:000526ED
  2906 0001:000526F4  2907 0001:000526F7  2908 0001:0005271E  2909 0001:00052722
  2910 0001:00052724  2918 0001:00052728  2919 0001:0005272B  2920 0001:00052737
  2921 0001:00052740  2922 0001:00052747  2934 0001:0005274C  2935 0001:0005276D
  2937 0001:00052771  2938 0001:00052776  2941 0001:00052778  2942 0001:00052785
  2943 0001:0005278D  2945 0001:00052792  2946 0001:00052797  2948 0001:00052799
  2949 0001:000527AC  2950 0001:000527CD  3021 0001:000527D4  3022 0001:000527EE
  3023 0001:000527F3  3028 0001:000527F4  3029 0001:000527FC  3030 0001:0005280B
  3031 0001:0005280F  3032 0001:0005281F  3034 0001:00052823  3037 0001:0005282A
  3038 0001:0005282E  3040 0001:00052833  3044 0001:0005283C  3045 0001:0005284E
  3046 0001:00052856  3050 0001:00052858  3051 0001:00052870  3055 0001:00052874
  3056 0001:0005288C  3063 0001:00052890  3064 0001:000528BE  3065 0001:000528CA
  3066 0001:000528CD  3067 0001:000528D8  3068 0001:000528E6  3069 0001:000528F4
  3070 0001:000528FA  3071 0001:00052900  3072 0001:0005293A  3087 0001:00052944
  3088 0001:0005294F  3090 0001:00052953  3091 0001:00052958  3093 0001:0005295A
  3094 0001:0005295E  3096 0001:00052965  3097 0001:00052970  3098 0001:00052987
  3102 0001:00052996  3103 0001:000529A5  3104 0001:000529B2  3106 0001:000529C1
  3112 0001:000529C8  3113 0001:000529FF  3114 0001:00052A0A  3115 0001:00052A29
  3117 0001:00052A31  3118 0001:00052A59  3119 0001:00052A70  3120 0001:00052A9B
  3123 0001:00052AB4  3124 0001:00052AC1  3126 0001:00052B16  3135 0001:00052B78
  3136 0001:00052B9F  3137 0001:00052BBB  3139 0001:00052BC5  3140 0001:00052BEE
  3142 0001:00052BF6  3144 0001:00052C08  3145 0001:00052C16  3146 0001:00052C2A
  3147 0001:00052C37  3155 0001:00052CA0  3157 0001:00052CA8  3159 0001:00052CC2
  3163 0001:00052D1C  3164 0001:00052D20  3157 0001:00052D23  3165 0001:00052D28
  3167 0001:00052D2C  3168 0001:00052D30  3142 0001:00052D31  3171 0001:00052D59
  3176 0001:00052D60  3177 0001:00052D8B  3181 0001:00052DA5  3183 0001:00052DB7
  3185 0001:00052DBD  3186 0001:00052DC4  3187 0001:00052DCA  3188 0001:00052DD0
  3189 0001:00052DD6  3192 0001:00052E31  3195 0001:00052E38  3196 0001:00052E3B
  3197 0001:00052E45  3200 0001:00052E4C  3201 0001:00052E4F  3202 0001:00052E59
  3205 0001:00052E60  3206 0001:00052E6B  3207 0001:00052E7D  3208 0001:00052E8D
  3209 0001:00052E99  3212 0001:00052EA0  3213 0001:00052EA7  3214 0001:00052EC1
  3220 0001:00052EC8  3221 0001:00052ECE  3222 0001:00052ED1  3225 0001:00052ED4
  3226 0001:00052EE0  3227 0001:00052EF8  3231 0001:00052EFC  3234 0001:00052F0B
  3235 0001:00052F0D  3236 0001:00052F13  3232 0001:00052F1A  3238 0001:00052F21
  3239 0001:00052F38  3243 0001:00052F40  3244 0001:00052F45  3245 0001:00052F47
  3246 0001:00052F4A  3248 0001:00052F4E  3250 0001:00052F5C  3251 0001:00052F5E
  3253 0001:00052F60  3246 0001:00052F63  3255 0001:00052F69  3265 0001:00052F70
  3266 0001:00052F8E  3271 0001:00052F90  3272 0001:00052FB6  3274 0001:00052FDC
  3275 0001:00052FDF  3277 0001:00052FE3  3278 0001:00052FEC  3279 0001:00052FF2
  3280 0001:00053003  3281 0001:00053012  3282 0001:00053020  3275 0001:00053023
  3284 0001:00053027  3285 0001:0005302F  3286 0001:0005305E  3291 0001:00053084
  3295 0001:000530B3  3296 0001:000530F2  3299 0001:000530F8  3303 0001:00053103
  3304 0001:0005311A  3308 0001:00053120  3309 0001:00053125  3310 0001:0005312F
  3313 0001:00053130  3314 0001:00053131  3315 0001:00053138  3316 0001:00053144
  3326 0001:00053148  3327 0001:00053155  3328 0001:0005315B  3330 0001:00053167
  3331 0001:0005316F  3334 0001:00053174  3335 0001:0005317A  3336 0001:00053180
  3337 0001:0005318B  3338 0001:00053191  3341 0001:00053198  3342 0001:0005319E
  3343 0001:000531A4  3344 0001:000531AF  3345 0001:000531B5  3349 0001:000531BC
  3350 0001:000531C3  3351 0001:000531DD  3354 0001:000531E4  3355 0001:000531EA
  3356 0001:000531F3  3359 0001:000531F8  3360 0001:00053200  3361 0001:0005320B
  3362 0001:0005321A  3365 0001:00053220  3366 0001:00053226  3367 0001:00053230
  3370 0001:00053234  3371 0001:0005326B  3372 0001:00053277  3373 0001:000532B9
  3377 0001:000532C0  3378 0001:000532D5  3379 0001:000532FC  3385 0001:00053304
  3386 0001:0005333C  3387 0001:0005334C  3388 0001:00053352  3389 0001:00053360
  3390 0001:00053365  3391 0001:0005336D  3392 0001:00053375  3393 0001:0005337D
  3394 0001:00053385  3395 0001:0005338C  3396 0001:000533E2  3406 0001:00053438
  3407 0001:00053450  3408 0001:00053488  3411 0001:00053490  3412 0001:0005349B
  3413 0001:000534A3  3414 0001:000534AB  3415 0001:000534B3  3416 0001:000534CA
  3419 0001:000534D0  3421 0001:000534E3  3422 0001:00053503  3423 0001:00053511
  3429 0001:00053518  3431 0001:0005353F  3432 0001:0005354A  3433 0001:00053558
  3435 0001:0005356A  3436 0001:00053576  3437 0001:0005358E  3441 0001:000535A6
  3442 0001:000535BA  3443 0001:000535BF  3445 0001:000535C6  3433 0001:000535C7
  3446 0001:000535CA  3447 0001:000535D2  3449 0001:000535E6  3451 0001:00053619
  3454 0001:00053674  3455 0001:0005367C  3456 0001:00053688  3457 0001:0005368A
  3466 0001:00053690  3467 0001:00053693  3471 0001:00053694  3472 0001:0005369A
  3473 0001:000536A2  3474 0001:000536A4  3477 0001:000536A8  3478 0001:000536B7
  3479 0001:000536C2  3480 0001:000536D0  3482 0001:000536EB  3483 0001:000536ED
  3485 0001:00053702  3493 0001:00053708  3494 0001:00053711  3495 0001:0005371C
  3496 0001:0005372A  3498 0001:00053750  3500 0001:00053766  3509 0001:0005376C
  3510 0001:0005378A  3511 0001:00053795  3514 0001:000537A3  3515 0001:000537AC
  3517 0001:000537B5  3519 0001:000537DB  3526 0001:00053808  3529 0001:00053810
  3530 0001:0005381B  3531 0001:0005382C  3533 0001:0005383E  3535 0001:00053871
  3541 0001:000538C8  3543 0001:000538E4  3545 0001:000538EA  3546 0001:000538FF
  3547 0001:0005390A  3548 0001:0005391B  3551 0001:00053925  3552 0001:00053949
  3558 0001:00053954  3559 0001:0005395B  3560 0001:00053966  3561 0001:00053974
  3563 0001:0005397D  3565 0001:0005398F  3568 0001:0005399B  3570 0001:000539A6
  3571 0001:000539B0  3573 0001:000539C3  3563 0001:000539C4  3576 0001:000539C7
  3577 0001:000539D1  3579 0001:000539E3  3581 0001:000539F9  3586 0001:00053A04
  3587 0001:00053A1D  3588 0001:00053A22  3589 0001:00053A2E  3591 0001:00053A3A
  3592 0001:00053A4F  3595 0001:00053A57  3597 0001:00053A77  3598 0001:00053A7C
  3599 0001:00053A8A  3600 0001:00053A8C  3603 0001:00053A94  3604 0001:00053A97
  3605 0001:00053A9C  3634 0001:00053AA0  3635 0001:00053ABB  3636 0001:00053ABD
  3637 0001:00053AC2  3638 0001:00053AD1  3644 0001:00053AD9  3645 0001:00053AFF
  3646 0001:00053B25  3647 0001:00053B2E  3648 0001:00053B34  3649 0001:00053B44
  3650 0001:00053B52  3651 0001:00053B5F  3652 0001:00053B67  3654 0001:00053B6F
  3655 0001:00053BA3  3661 0001:00053BCC  3662 0001:00053BD3  3663 0001:00053BDE
  3665 0001:00053BEC  3666 0001:00053BFB  3668 0001:00053C04  3669 0001:00053C10
  3672 0001:00053C26  3674 0001:00053C2F  3676 0001:00053C41  3679 0001:00053C4D
  3681 0001:00053C58  3682 0001:00053C68  3684 0001:00053C7B  3674 0001:00053C7C
  3686 0001:00053C7F  3687 0001:00053C89  3689 0001:00053C9B  3691 0001:00053CB1
  3694 0001:00053CBC  3695 0001:00053CD6  3696 0001:00053CE1  3697 0001:00053CEF
  3699 0001:00053D0A  3700 0001:00053D0C  3702 0001:00053D3E  3709 0001:00053D44
  3710 0001:00053D4B  3711 0001:00053D56  3712 0001:00053D64  3714 0001:00053D69
  3716 0001:00053D72  3718 0001:00053D84  3724 0001:00053D90  3726 0001:00053D9B
  3727 0001:00053DA4  3729 0001:00053DBE  3716 0001:00053DBF  3731 0001:00053DC2
  3733 0001:00053DD7  3735 0001:00053DED  3738 0001:00053DF8  3742 0001:00053DFF
  3744 0001:00053E05  3745 0001:00053E0A  3748 0001:00053E0C  3749 0001:00053E18
  3751 0001:00053E23  3752 0001:00053E33  3753 0001:00053E37  3764 0001:00053E3C
  3765 0001:00053E57  3766 0001:00053E59  3767 0001:00053E5E  3768 0001:00053E6D
  3774 0001:00053E75  3775 0001:00053E9B  3776 0001:00053EC1  3777 0001:00053ECA
  3778 0001:00053ED0  3779 0001:00053EE0  3780 0001:00053EEE  3781 0001:00053EFB
  3782 0001:00053F03  3784 0001:00053F0B  3785 0001:00053F3F  3791 0001:00053F68
  3792 0001:00053F85  3793 0001:00053F8A  3794 0001:00053F8F  3795 0001:00053F92
  3798 0001:00053FA1  3801 0001:00053FBB  3804 0001:00053FC4  3806 0001:00053FC8
  3807 0001:00053FD3  3811 0001:00053FE0  3812 0001:00053FFC  3813 0001:00054002
  3814 0001:00054008  3815 0001:0005400E  3816 0001:00054016  3817 0001:00054020
  3818 0001:0005402F  3817 0001:00054047  3820 0001:00054063  3823 0001:000540BC
  3824 0001:000540C7  3825 0001:000540CF  3826 0001:000540D8  3827 0001:000540EF
  3830 0001:000540F4  3831 0001:00054108  3833 0001:0005410A  3835 0001:00054115
  3836 0001:0005411C  3840 0001:00054123  3841 0001:00054143  3843 0001:0005414F
  3854 0001:00054158  3855 0001:0005416F  3856 0001:00054175  3858 0001:0005417E
  3860 0001:00054184  3861 0001:0005418B  3863 0001:00054190  3869 0001:00054192
  3870 0001:0005419D  3873 0001:000541A3  3874 0001:000541BB  3876 0001:000541C1
  3877 0001:000541C8  3887 0001:000541CD  3890 0001:000541D3  3891 0001:000541D6
  3892 0001:000541E4  3897 0001:000541E8  3898 0001:00054200  3899 0001:00054207
  3903 0001:00054209  3906 0001:00054216  3907 0001:0005421E  3908 0001:00054235
  3909 0001:00054236  3910 0001:00054240  3887 0001:00054243  3914 0001:00054249
  3916 0001:00054254  3917 0001:0005426A  3921 0001:000542C4  3923 0001:000542CF
  3925 0001:000542DA  3926 0001:000542DF  3933 0001:000542E1  3934 0001:000542E7
  3936 0001:000542EB  3937 0001:000542F0  3940 0001:000542F2  3941 0001:000542F5
  3942 0001:000542F7  3945 0001:00054300  3946 0001:00054307  3947 0001:00054312
  3948 0001:0005431D  3949 0001:00054322  3950 0001:0005432A  3951 0001:0005432C
  3954 0001:00054334  3955 0001:0005433B  3956 0001:00054346  3957 0001:00054351
  3958 0001:00054356  3959 0001:00054358  3962 0001:00054360  3963 0001:00054363
  3964 0001:00054376  3974 0001:00054378  3975 0001:0005437A  3990 0001:0005437C
  3991 0001:000543A8  3994 0001:000543C2  3999 0001:000543D4  4000 0001:000543E3
  4005 0001:000543E8  4006 0001:000543EF  4008 0001:000543F1  4009 0001:000543FA
  4010 0001:00054410  4012 0001:00054421  4014 0001:0005442C  4015 0001:00054446
  4016 0001:00054459  4017 0001:00054461  4019 0001:0005446C  4020 0001:0005446E
  4025 0001:00054470  4027 0001:00054488  4030 0001:0005448B  4006 0001:0005448C
  4031 0001:00054495  4032 0001:000544BF  4035 0001:00054518  4041 0001:0005453C
  4045 0001:0005455C  4046 0001:00054568  4053 0001:00054573  4054 0001:0005459B
  4057 0001:000545A0  4061 0001:000545AC  4062 0001:000545B7  4066 0001:000545BB
  4067 0001:000545C6  4068 0001:000545D1  4071 0001:000545DC  4072 0001:000545F4
  4075 0001:000545FF  4076 0001:0005460B  4082 0001:00054616  4093 0001:00054621
  4094 0001:0005463C  4103 0001:00054641  4106 0001:00054665  4107 0001:0005468C
  4114 0001:000546E4  4115 0001:000546E6  4123 0001:000546E8  4125 0001:0005470A
  4126 0001:00054717  4127 0001:00054737  4130 0001:00054757  4131 0001:00054766
  4132 0001:00054787  4138 0001:000547DC  4139 0001:000547EE  4140 0001:00054807
  4150 0001:0005480C  4151 0001:00054827  4152 0001:00054832  4153 0001:00054840
  4155 0001:0005484B  4160 0001:00054854  4162 0001:0005485B  4167 0001:00054865
  4169 0001:0005487A  4170 0001:00054881  4178 0001:00054888  4179 0001:00054898
  4186 0001:000548A3  4187 0001:000548C8  4188 0001:000548CB  4193 0001:000548D2
  4195 0001:000548E4  4197 0001:00054917  4202 0001:00054970  4205 0001:00054983
  4206 0001:0005498D  4207 0001:00054992  4208 0001:00054996  4209 0001:0005499B
  4212 0001:000549A4  4213 0001:000549B6  4214 0001:000549C1  4216 0001:000549CF
  4218 0001:000549DB  4219 0001:000549E9  4223 0001:000549F0  4224 0001:000549FD
  4225 0001:00054A07  4226 0001:00054A11  4230 0001:00054A25  4232 0001:00054A3B
  4237 0001:00054A40  4238 0001:00054A81  4239 0001:00054A8F  4240 0001:00054A92
  4241 0001:00054A95  4242 0001:00054AA0  4243 0001:00054AA8  4244 0001:00054AAE
  4245 0001:00054AB2  4246 0001:00054ABA  4247 0001:00054AC1  4248 0001:00054AD5
  4249 0001:00054AEB  4250 0001:00054AEF  4251 0001:00054AF3  4259 0001:00054B05
  4260 0001:00054B0D  4261 0001:00054B1A  4262 0001:00054B32  4263 0001:00054B88
  4266 0001:00054BE4  4270 0001:00054BEF  4271 0001:00054C09  4272 0001:00054C11
  4273 0001:00054C2E  4274 0001:00054C36  4275 0001:00054C4D  4280 0001:00054CA0
  4281 0001:00054CA4  4282 0001:00054CAF  4284 0001:00054CBD  4285 0001:00054CC9
  4286 0001:00054CD2  4288 0001:00054CEB  4290 0001:00054D01  4293 0001:00054D08
  4294 0001:00054D10  4295 0001:00054D30  4297 0001:00054D36  4298 0001:00054D3F
  4306 0001:00054D4A  4307 0001:00054D52  4308 0001:00054D54  4312 0001:00054D56
  4313 0001:00054D5D  4332 0001:00054DB4  4334 0001:00054DDA  4337 0001:00054DDC
  4344 0001:00054E02  4349 0001:00054E04  4350 0001:00054E07  4351 0001:00054E09
  4361 0001:00054E10  4363 0001:00054E23  4364 0001:00054E43  4365 0001:00054E4F
  4366 0001:00054E51  4376 0001:00054E58  4377 0001:00054E5D  4390 0001:00054E60
  4391 0001:00054E63  4399 0001:00054E64  4400 0001:00054E68  4401 0001:00054E6A
  4412 0001:00054E6C  4413 0001:00054E73  4417 0001:00054E74  4418 0001:00054E7E
  4427 0001:00054E80  4428 0001:00054E86  4429 0001:00054E98  4430 0001:00054EAA
  4431 0001:00054EBC  4432 0001:00054EBE  4435 0001:00054EC4  4436 0001:00054ECB
  4437 0001:00054EEF  4438 0001:00054EF8  4441 0001:00054F50  4442 0001:00054F57
  4443 0001:00054F7B  4444 0001:00054F84  4447 0001:00054FDC  4451 0001:00054FF6
  4452 0001:0005501A  4460 0001:00055020  4464 0001:00055027  4465 0001:00055031
  4466 0001:00055043  4469 0001:00055048  4470 0001:0005504E  4471 0001:00055056
  4472 0001:00055058  4475 0001:0005505C  4476 0001:00055062  4477 0001:0005506D
  4481 0001:00055074  4482 0001:00055082  4483 0001:00055087  4488 0001:0005508C
  4489 0001:000550A4  4490 0001:000550B5  4492 0001:000550C1  4493 0001:000550D8
  4495 0001:000550E9  4496 0001:000550EF  4497 0001:000550F5  4498 0001:000550F7
  4505 0001:00055100  4506 0001:0005511E  4507 0001:00055129  4509 0001:00055137
  4511 0001:00055140  4512 0001:00055147  4516 0001:00055151  4518 0001:00055166
  4519 0001:0005516D  4522 0001:00055177  4523 0001:00055185  4527 0001:00055191
  4528 0001:000551B6  4534 0001:000551C0  4535 0001:000551CD  4540 0001:000551D3
  4544 0001:000551F8  4547 0001:00055216  4548 0001:0005521D  4552 0001:00055227
  4553 0001:00055235  4554 0001:00055242  4556 0001:0005524E  4557 0001:0005525C
  4559 0001:00055268  4560 0001:0005526D  4567 0001:00055274  4571 0001:0005527F
  4573 0001:000552B1  4575 0001:000552E4  4582 0001:0005533C  4583 0001:0005533F
  4584 0001:00055341  4602 0001:00055348  4603 0001:0005534E  4604 0001:00055356
  4605 0001:00055360  4606 0001:00055362  4609 0001:00055368  4610 0001:00055382
  4611 0001:0005538D  4612 0001:0005539B  4613 0001:000553A9  4615 0001:000553BB
  4617 0001:000553EE  4632 0001:000553F4  4634 0001:00055423  4635 0001:0005542E
  4637 0001:0005543D  4640 0001:00055442  4649 0001:00055444  4650 0001:00055459
  4652 0001:0005545D  4653 0001:00055461  4654 0001:00055466  4655 0001:00055468
  4658 0001:0005546D  4659 0001:00055487  4662 0001:000554A1  4664 0001:000554B3
  4666 0001:000554C3  4670 0001:000554F1  4672 0001:000554F5  4673 0001:000554FA
  4674 0001:00055502  4642 0001:0005550A  4676 0001:00055531  4687 0001:0005558C
  4688 0001:0005558F  4689 0001:000555A2  4696 0001:000555A4  4697 0001:000555B8
  4699 0001:000555BA  4701 0001:000555C5  4702 0001:000555CC  4703 0001:000555D1
  4707 0001:000555D3  4708 0001:000555F3  4710 0001:000555FF  4714 0001:00055608
  4715 0001:00055622  4716 0001:00055627  4722 0001:0005562A  4725 0001:00055642
  4729 0001:0005564B  4731 0001:0005564F  4732 0001:0005565A  4735 0001:0005565C
  4736 0001:00055662  4737 0001:00055681  4745 0001:000556D8  4749 0001:000556E3
  4750 0001:000556EC  4751 0001:00055703  4768 0001:00055708  4770 0001:00055714
  4772 0001:0005571F  4773 0001:00055726  4776 0001:0005572B  4777 0001:00055731
  4780 0001:0005573A  4782 0001:00055740  4783 0001:00055747  4786 0001:0005574C
  4794 0001:0005574E  4795 0001:00055761  4797 0001:00055767  4798 0001:0005576F
  4799 0001:00055772  4800 0001:00055784  4811 0001:0005578A  4812 0001:00055797
  4816 0001:000557A0  4819 0001:000557B5  4820 0001:000557BD  4821 0001:000557C5
  4823 0001:000557CD  4824 0001:000557CE  4795 0001:000557D1  4826 0001:000557D7
  4827 0001:000557E5  4828 0001:000557F0  4829 0001:00055807  4838 0001:00055810
  4839 0001:00055817  4843 0001:0005581C  4844 0001:00055827  4845 0001:00055829
  4851 0001:00055830  4852 0001:0005583C  4855 0001:00055841  4857 0001:00055845
  4858 0001:00055847  4861 0001:00055849  4863 0001:00055854  4864 0001:00055859
  4867 0001:0005585B  4870 0001:0005585E  4871 0001:0005587A  5144 0001:00055884
  5147 0001:00055888  5148 0001:00055893  5151 0001:000558A1  5153 0001:000558C1
  5156 0001:000558CB  5158 0001:000558DD  5161 0001:000558F3  5164 0001:00055948
  5166 0001:0005594C  5171 0001:00055955  5172 0001:00055963  5173 0001:0005596E
  5175 0001:00055979  5176 0001:0005597D  5181 0001:00055980  5183 0001:00055983
  5185 0001:000559A2  5186 0001:000559B4  5187 0001:000559C4  5188 0001:000559D1
  5189 0001:000559D3  5196 0001:00055A28  5197 0001:00055A5F  5198 0001:00055A7D
  5199 0001:00055A88  5200 0001:00055A8F  5201 0001:00055A96  5202 0001:00055AE2
  5205 0001:00055AEC  5206 0001:00055AF7  5207 0001:00055B0B  5208 0001:00055B22
  5217 0001:00055B28  5220 0001:00055B2C  5221 0001:00055B37  5223 0001:00055B45
  5228 0001:00055B65  5230 0001:00055B6F  5231 0001:00055B76  5233 0001:00055B88
  5235 0001:00055B9E  5248 0001:00055BF4  5249 0001:00055C03  5250 0001:00055C0E
  5251 0001:00055C1C  5253 0001:00055C28  5255 0001:00055C4E  5257 0001:00055C61
  5258 0001:00055C81  5259 0001:00055C92  5261 0001:00055CA4  5263 0001:00055CBA
  5271 0001:00055D10  5272 0001:00055D13  5273 0001:00055D18  5280 0001:00055D1C
  5281 0001:00055D20  5283 0001:00055D29  5284 0001:00055D2E  5286 0001:00055D2F
  5287 0001:00055D36  5288 0001:00055D42  5291 0001:00055D44  5295 0001:00055D5E
  5296 0001:00055D7F  5305 0001:00055D84  5306 0001:00055D9E  5307 0001:00055DA9
  5308 0001:00055DB7  5312 0001:00055DC7  5313 0001:00055DD7  5315 0001:00055DE9
  5317 0001:00055E1C  5364 0001:00055E24  5365 0001:00055E44  5367 0001:00055E5E
  5368 0001:00055E67  5371 0001:00055E6F  5373 0001:00055E8F  5374 0001:00055EA3
  5375 0001:00055EAB  5380 0001:00055EBF  5381 0001:00055EC9  5382 0001:00055ED1
  5383 0001:00055ED9  5384 0001:00055EE1  5385 0001:00055EEE  5386 0001:00055EF5
  5387 0001:00055F02  5388 0001:00055F09  5389 0001:00055F16  5390 0001:00055F1D
  5391 0001:00055F3D  5392 0001:00055F51  5393 0001:00055F65  5394 0001:00055F6C
  5395 0001:00055F7C  5396 0001:00055F8B  5401 0001:00055F9A  5403 0001:00055FA7
  5404 0001:00055FA9  5410 0001:00055FAB  5412 0001:00055FBA  5416 0001:00055FBE
  5417 0001:00055FC2  5418 0001:00055FC8  5419 0001:00055FDC  5420 0001:00056008
  5431 0001:00056060  5434 0001:0005607F  5435 0001:0005608A  5436 0001:0005608F
  5438 0001:000560A2  5439 0001:000560B2  5440 0001:000560BE  5441 0001:000560CD
  5443 0001:000560D7  5444 0001:000560E8  5446 0001:000560F3  5447 0001:0005610D
  5448 0001:00056110  5449 0001:00056129  5450 0001:00056131  5452 0001:0005613C
  5453 0001:00056147  5454 0001:0005614F  5456 0001:00056152  5457 0001:00056154
  5463 0001:00056156  5464 0001:00056158  5468 0001:0005615A  5436 0001:0005615D
  5469 0001:00056164  5470 0001:0005619A  5478 0001:000561F4  5479 0001:00056200
  5480 0001:00056202  5481 0001:00056206  5482 0001:00056207  5484 0001:0005620B
  5486 0001:0005621F  5487 0001:00056223  5488 0001:00056225  5482 0001:00056226
  5490 0001:0005622C  5493 0001:00056234  5494 0001:00056238  5495 0001:00056255
  5496 0001:00056261  6403 0001:000562B4  6404 0001:000562C6  6414 0001:000562E6
  6421 0001:000562EC  6423 0001:000562EE  6435 0001:000562F0  6436 0001:000562FB
  6437 0001:0005630F  6451 0001:00056314  6463 0001:0005631D  6478 0001:00056320
  6479 0001:00056329  8176 0001:0005632C  8178 0001:00056337  8180 0001:00056341
  8181 0001:00056346  8186 0001:00056348  8188 0001:0005634F  8189 0001:00056354
  8192 0001:00056356  8193 0001:0005635C  8194 0001:00056379  8195 0001:00056383
  8196 0001:0005638B  8199 0001:00056394  8206 0001:0005639C  8208 0001:000563A8
  8209 0001:000563AD  8212 0001:000563AF  8214 0001:000563B5  8215 0001:000563B7
  8220 0001:000563B9  8221 0001:000563C6  8222 0001:000563D7  8226 0001:000563E0
  8227 0001:000563E8  8229 0001:000563EF  8230 0001:000563F4  8235 0001:000563F6
  8236 0001:00056407  8242 0001:0005640D  8243 0001:0005641E  8249 0001:0005643B
  8250 0001:0005643D  8253 0001:00056444  8254 0001:00056461  8255 0001:00056467
  8256 0001:00056488  8257 0001:0005648D  8258 0001:00056492  8259 0001:00056497
  8260 0001:000564A0  8261 0001:000564A9  8262 0001:000564D2  8265 0001:000564DC
  8266 0001:000564DF  8267 0001:000564E4  8270 0001:000564E8  8271 0001:000564EE
  8272 0001:000564FD  8275 0001:00056504  8276 0001:00056510  8278 0001:00056517
  8279 0001:0005651C  8282 0001:0005651E  8289 0001:00056541  8290 0001:00056543
  8294 0001:0005654C  8295 0001:00056558  8297 0001:0005655D  8299 0001:00056561
  8300 0001:00056566  8303 0001:00056568  8304 0001:0005656C  8305 0001:00056579
  8308 0001:0005657B  8311 0001:0005657F  8312 0001:00056583  8313 0001:0005658E
  8319 0001:00056590  8320 0001:00056595  8324 0001:0005659C  8325 0001:000565A7
  8327 0001:000565AB  8329 0001:000565B1  8330 0001:000565B6  8332 0001:000565B8
  8336 0001:000565C4  8338 0001:000565CA  8339 0001:000565CF  8341 0001:000565D1
  8343 0001:000565D9  8344 0001:000565DB  8347 0001:000565E4  8348 0001:000565EE
  8350 0001:000565F4  8351 0001:000565F9  8354 0001:000565FB  8356 0001:00056609
  8357 0001:0005660E  8360 0001:00056610  8361 0001:0005662C  8362 0001:0005663E
  8363 0001:00056640  8366 0001:00056648  8367 0001:0005664B  8368 0001:00056650
  8371 0001:00056654  8372 0001:0005668B  8373 0001:0005669B  8374 0001:000566A1
  8375 0001:000566A8  8376 0001:000566B0  8377 0001:000566B4  8378 0001:000566F4
  8381 0001:000566FC  8382 0001:00056707  8384 0001:0005670E  8385 0001:00056713
  8387 0001:00056718  8388 0001:0005672F  8443 0001:00056734  8446 0001:0005674B
  8447 0001:00056766  8448 0001:00056771  8449 0001:000567A7  8455 0001:000567B0
  8457 0001:000567C8  8459 0001:000567CE  8460 0001:000567D3  8464 0001:000567D8
  8466 0001:000567DE  8467 0001:000567FC  8469 0001:00056807  8470 0001:0005681C
  8472 0001:00056827  8473 0001:0005683F  8474 0001:00056847  8476 0001:00056852
  8477 0001:0005685D  8478 0001:0005687E  8481 0001:000568A0  8482 0001:000568A3
  8483 0001:000568AC  8484 0001:000568AE  8583 0001:000568B4  8584 0001:000568EB
  8585 0001:000568FB  8586 0001:00056946  8596 0001:00056950  8597 0001:0005695B
  8598 0001:00056963  8599 0001:0005697A  8603 0001:00056980  8604 0001:00056986
  8605 0001:000569A6  8609 0001:000569AC  8610 0001:000569B2  8611 0001:000569CE
  8614 0001:000569D4  8615 0001:000569DA  8616 0001:000569E7  8622 0001:000569EC
  8624 0001:00056A04  8626 0001:00056A17  8627 0001:00056A1C  8629 0001:00056A1E
  8630 0001:00056A35  8631 0001:00056A40  8632 0001:00056A84  8658 0001:00056A8C
  8659 0001:00056AA3  8660 0001:00056AB6  8661 0001:00056AC1  8662 0001:00056AEF
  8667 0001:00056AF8  8668 0001:00056B0F  8669 0001:00056B22  8670 0001:00056B2D
  8671 0001:00056B69  8675 0001:00056B70  8676 0001:00056BAF  8677 0001:00056BC9
  8678 0001:00056BD9  8679 0001:00056C28  8730 0001:00056C80  8731 0001:00056C97
  8732 0001:00056CAA  8733 0001:00056CB5  8734 0001:00056CE7  8738 0001:00056CF0
  8739 0001:00056D07  8740 0001:00056D1A  8741 0001:00056D25  8742 0001:00056D53
  8748 0001:00056D5C  8749 0001:00056D7A  8750 0001:00056D89  8751 0001:00056D94
  8754 0001:00056D98  8755 0001:00056DAB  8756 0001:00056DB6  8758 0001:00056DE4
  8762 0001:00056DEC  8763 0001:00056E03  8764 0001:00056E16  8765 0001:00056E21
  8766 0001:00056E4F  8771 0001:00056E58  8772 0001:00056E5D  8800 0001:00056E60
  8801 0001:00056E8A  8803 0001:00056E92  8804 0001:00056EA6  8806 0001:00056EB1
  8807 0001:00056EB6  8810 0001:00056EB8  8811 0001:00056ED1  8812 0001:00056ED9
  8814 0001:00056EE4  8815 0001:00056EE9  8818 0001:00056EEB  8819 0001:00056F0C
  8823 0001:00056F14  8824 0001:00056F2B  8825 0001:00056F3E  8826 0001:00056F49
  8827 0001:00056F7B  8831 0001:00056F84  8832 0001:00056F9B  8833 0001:00056FAE
  8834 0001:00056FB9  8835 0001:00056FE7  8839 0001:00056FF0  8840 0001:00057007
  8841 0001:0005701A  8842 0001:00057025  8843 0001:00057053  8847 0001:0005705C
  8848 0001:00057073  8849 0001:00057086  8850 0001:00057091  8851 0001:000570BF
  8855 0001:000570C8  8856 0001:000570DF  8857 0001:000570F2  8858 0001:000570FD
  8859 0001:0005712B  8863 0001:00057134  8864 0001:0005714B  8865 0001:0005715E
  8866 0001:00057169  8867 0001:00057197  8871 0001:000571A0  8872 0001:000571B7
  8873 0001:000571CA  8874 0001:000571D5  8875 0001:00057203  8917 0001:0005720C
  8918 0001:00057223  8919 0001:00057236  8920 0001:00057241  8921 0001:0005726F
  8926 0001:00057278  8927 0001:0005728F  8928 0001:000572A2  8929 0001:000572AD
  8930 0001:000572E7  8934 0001:000572F0  8935 0001:00057307  8937 0001:00057315
  8938 0001:0005731A  8940 0001:0005731C  8941 0001:0005732F  8942 0001:0005733A
  8943 0001:0005736A  8947 0001:00057374  8948 0001:0005738B  8949 0001:0005739E
  8950 0001:000573A9  8951 0001:000573D7  8963 0001:000573E0  8964 0001:0005741F
  8965 0001:00057437  8966 0001:00057445  8967 0001:00057453  8968 0001:00057457
  8969 0001:000574AA  8972 0001:000574B4  8973 0001:000574BF  8974 0001:000574C7
  8975 0001:000574DE  8983 0001:000574E4  8984 0001:000574ED  8987 0001:000574FF
  8988 0001:0005750F  8990 0001:0005751B  8991 0001:00057526  8992 0001:00057534
  8993 0001:00057543  8995 0001:0005755F  8999 0001:00057575  9003 0001:0005757C
  9004 0001:0005758B  9005 0001:00057596  9006 0001:000575A4  9008 0001:000575AD
  9009 0001:000575B4  9012 0001:000575BB  9013 0001:000575D9  9014 0001:000575E5
  9016 0001:00057610  9018 0001:00057626  9025 0001:0005762C  9026 0001:0005764E
  9027 0001:00057668  9028 0001:00057673  9030 0001:00057681  9031 0001:00057695
  9033 0001:000576A1  9034 0001:000576BE  9036 0001:000576C5  9037 0001:000576D4
  9038 0001:000576E3  9039 0001:000576EA  9041 0001:000576FC  9043 0001:0005772F
  9064 0001:00057784  9065 0001:0005778D  9066 0001:00057798  9067 0001:000577A6
  9068 0001:000577B7  9069 0001:000577C8  9070 0001:000577CF  9072 0001:000577E1
  9074 0001:000577F7  9084 0001:000577FC  9085 0001:00057815  9086 0001:00057843
  9089 0001:00057848  9090 0001:00057854  9091 0001:0005785B  9092 0001:00057879
  9093 0001:00057890  9097 0001:000578E4  9098 0001:000578ED  9102 0001:000578F0
  9103 0001:000578F9 10708 0001:000578FC 10709 0001:00057902 10710 0001:00057909
 10714 0001:00057913 10717 0001:00057930 10718 0001:00057932 10739 0001:0005793C
 10740 0001:0005794A 10745 0001:0005794D 10747 0001:00057956 10748 0001:00057964
 10751 0001:0005796E 10752 0001:00057977 10755 0001:0005797D 10756 0001:0005798D
 10855 0001:00057998 10867 0001:0005799C 10868 0001:0005799F 10869 0001:000579B2
 10871 0001:000579B9 10872 0001:000579CC 10874 0001:000579D3 10875 0001:000579D6
 10881 0001:000579DC 10882 0001:00057A19 10883 0001:00057A28 10884 0001:00057A3A
 10886 0001:00057A4C 10888 0001:00057A6F 10889 0001:00057A80 10890 0001:00057A91
 10891 0001:00057A95 10892 0001:00057A9A 10893 0001:00057AAB 10894 0001:00057AAF
 10895 0001:00057AB3 10896 0001:00057AB7 10897 0001:00057ABF 10898 0001:00057AC4
 10899 0001:00057ACF 10900 0001:00057AD4 10901 0001:00057ADB 10902 0001:00057AEF
 10903 0001:00057AF6 10905 0001:00057AFE 10911 0001:00057B41 10920 0001:00057B4C
 10921 0001:00057B57 10922 0001:00057B71 10923 0001:00057B8E 10924 0001:00057B98
 10928 0001:00057BA2 10929 0001:00057BA8 10933 0001:00057BB0 10934 0001:00057BB6
 10938 0001:00057BBE 10942 0001:00057BDB 10943 0001:00057BE6 10945 0001:00057BF1
 10946 0001:00057BF9 10947 0001:00057C01 10949 0001:00057C09 10950 0001:00057C20
 10959 0001:00057C74 10960 0001:00057C9E 10961 0001:00057CAC 10962 0001:00057CBA
 10966 0001:00057CC4 10968 0001:00057CD2 10971 0001:00057CDC 10979 0001:00057CE1
 10981 0001:00057D21 10983 0001:00057D25 10984 0001:00057D2C 10986 0001:00057D33
 10988 0001:00057D3F 10989 0001:00057D4A 10990 0001:00057D51 10994 0001:00057D58
 10997 0001:00057D64 10999 0001:00057D81 11001 0001:00057DB7 11006 0001:00057DE0
 11007 0001:00057DFD 11009 0001:00057E09 11010 0001:00057E12 11012 0001:00057E17
 11013 0001:00057E46 11020 0001:00057E4C 11023 0001:00057E5B 11024 0001:00057E7B
 11025 0001:00057E88 11027 0001:00057E90 11037 0001:00057E98 11038 0001:00057E9C
 11040 0001:00057EA7 11041 0001:00057EAF 11042 0001:00057EB1 11147 0001:00057EB4
 11148 0001:00057EBB 11149 0001:00057EC4 11151 0001:00057ECE 11155 0001:00057ED3
 11156 0001:00057EDA 11158 0001:00057EE2 11156 0001:00057EF7 11165 0001:00057EFF
 11169 0001:00057F06 11171 0001:00057F0A 11172 0001:00057F0F 11175 0001:00057F11
 11176 0001:00057F18 11177 0001:00057F1C 11190 0001:00057F24 11192 0001:00057F2A
 11196 0001:00057F33 11198 0001:00057F45 11199 0001:00057F4C 11206 0001:00057F4E
 11208 0001:00057F5E 11209 0001:00057F6F 11231 0001:00057F74 11232 0001:00057F77
 11261 0001:00057F78 11262 0001:00057F87 11263 0001:00057F8B 11264 0001:00057F93
 11265 0001:00057F98 11267 0001:00057F9D 11268 0001:00057FA0 11269 0001:00057FA6
 11270 0001:00057FB2 11273 0001:00057FBA 11274 0001:00057FC0 11276 0001:00057FC7
 11280 0001:00057FCC 11281 0001:00057FDC 11284 0001:00057FE6 11285 0001:00057FE9
 11286 0001:00057FEE 11288 0001:00057FF3 11289 0001:00057FF9 11291 0001:00058000
 11293 0001:00058005 11295 0001:00058015 11298 0001:0005802E 11300 0001:00058036
 11299 0001:0005803F 11304 0001:0005805A 11306 0001:0005806B 11308 0001:00058077
 11311 0001:0005807C 11312 0001:00058081 11313 0001:00058086 11315 0001:0005808D
 11316 0001:00058090 11319 0001:00058093 11323 0001:0005809D 11324 0001:000580AB
 11327 0001:000580B1 11329 0001:000580BE 11334 0001:000580C2 11336 0001:000580C7
 11339 0001:000580CD 11342 0001:000580DC 11345 0001:000580EF 11346 0001:000580F8
 11349 0001:00058109 11355 0001:00058129 11359 0001:0005813E 11360 0001:00058140
 11368 0001:00058158 11369 0001:0005815F 11370 0001:0005817A 11372 0001:00058181
 11374 0001:00058183 11375 0001:0005818B 11385 0001:00058190 11387 0001:00058196
 11393 0001:000581BA 11394 0001:000581C1 11395 0001:000581C3 11398 0001:000581C6
 11399 0001:000581CD 11400 0001:000581D2 11408 0001:000581D8 11410 0001:000581FE
 11414 0001:00058200 11415 0001:00058208 11419 0001:0005820C 11420 0001:00058214
 11436 0001:00058218 11437 0001:0005821C 11438 0001:00058227 11441 0001:00058235
 11443 0001:0005823E 11444 0001:00058243 11449 0001:0005824D 11454 0001:0005825C
 11455 0001:00058264 11456 0001:00058269 11459 0001:00058273 11465 0001:0005827C
 11466 0001:0005828B 11470 0001:0005829D 11471 0001:000582A7 11472 0001:000582B2
 11473 0001:000582BC 11474 0001:000582C7 11477 0001:000582D2 11478 0001:000582F4
 11479 0001:00058320 11481 0001:00058340 11482 0001:00058348 11483 0001:00058350
 11485 0001:00058357 11488 0001:00058369 11490 0001:0005837F 11505 0001:000583D4
 11506 0001:000583DA 11507 0001:000583E5 11508 0001:000583F3 11509 0001:000583F9
 11513 0001:0005841C 11515 0001:00058425 11516 0001:00058435 11521 0001:0005843F
 11526 0001:0005844E 11527 0001:00058458 11528 0001:00058468 11533 0001:00058472
 11534 0001:0005847D 11539 0001:00058488 11540 0001:0005848B 11545 0001:00058495
 11546 0001:0005849F 11547 0001:000584AA 11548 0001:000584B4 11549 0001:000584BF
 11554 0001:000584C7 11555 0001:000584D6 11558 0001:000584E8 11559 0001:0005850A
 11560 0001:00058536 11561 0001:00058556 11569 0001:00058579 11571 0001:0005857D
 11572 0001:00058584 11575 0001:0005858F 11578 0001:000585A9 11580 0001:000585BF
 11598 0001:00058618 11599 0001:00058633 11600 0001:0005863E 11601 0001:0005864C
 11605 0001:00058654 11607 0001:00058659 11608 0001:0005865E 11613 0001:00058668
 11616 0001:00058677 11617 0001:0005868F 11618 0001:000586A2 11620 0001:000586AA
 11621 0001:000586B4 11622 0001:000586B9 11625 0001:000586C3 11629 0001:000586CB
 11630 0001:000586DC 11635 0001:000586E7 11636 0001:000586EA 11640 0001:000586F4
 11641 0001:00058717 11642 0001:00058721 11645 0001:0005872B 11646 0001:0005874D
 11647 0001:00058779 11648 0001:00058799 11654 0001:000587BC 11655 0001:000587CB
 11663 0001:000587DD 11665 0001:000587E1 11666 0001:000587E8 11669 0001:000587F3
 11672 0001:0005880E 11674 0001:00058841 11680 0001:0005889C 11681 0001:000588A1
 11688 0001:000588A4 11689 0001:000588B0 11690 0001:000588BE 11692 0001:000588CC
 11694 0001:000588E4 11696 0001:000588E8 11697 0001:000588ED 11702 0001:000588F7
 11707 0001:00058900 11709 0001:00058905 11710 0001:00058925 11712 0001:00058929
 11713 0001:0005892E 11716 0001:00058935 11718 0001:00058941 11719 0001:0005894C
 11720 0001:00058951 11724 0001:00058958 11726 0001:0005896E 11728 0001:00058987
 11733 0001:000589E4 11734 0001:00058A02 11735 0001:00058A0C 11736 0001:00058A16
 11738 0001:00058A6E 11741 0001:00058A78 11742 0001:00058A7F 11743 0001:00058A86
 11745 0001:00058AB7 11747 0001:00058AC3 11749 0001:00058AD5 11753 0001:00058ADC
 11755 0001:00058AFE 11757 0001:00058B05 11758 0001:00058B0A 11762 0001:00058B0C
 11765 0001:00058B28 11766 0001:00058B45 11768 0001:00058B61 11772 0001:00058B65
 11773 0001:00058B6D 11775 0001:00058B91 11783 0001:00058BF4 11786 0001:00058BF7
 11788 0001:00058BFD 11789 0001:00058BFF 11794 0001:00058C01 11795 0001:00058C05
 11797 0001:00058C0B 11798 0001:00058C0D 11805 0001:00058C0F 11811 0001:00058C16
 11812 0001:00058C1C 11814 0001:00058C23 11815 0001:00058C25 11820 0001:00058C28
 11823 0001:00058C2B 11824 0001:00058C31 11826 0001:00058C38 11827 0001:00058C41
 11828 0001:00058C4B 11830 0001:00058C55 11832 0001:00058C5C 11833 0001:00058C5E
 11838 0001:00058C60 11840 0001:00058C63 11841 0001:00058C6A 11845 0001:00058C6F
 11846 0001:00058C90 11847 0001:00058C99 11848 0001:00058C9B 11853 0001:00058CF0
 11861 0001:00058D05 11863 0001:00058D09 11865 0001:00058D15 11866 0001:00058D21
 11869 0001:00058D2C 11872 0001:00058D37 11874 0001:00058D40 11875 0001:00058D59
 11881 0001:00058D60 11882 0001:00058D62 11887 0001:00058D64 11888 0001:00058D67
 11889 0001:00058D6E 11893 0001:00058D73 11895 0001:00058D7D 11896 0001:00058D7F
 11902 0001:00058D84 11903 0001:00058D86 11912 0001:00058D88 11915 0001:00058D8B
 11916 0001:00058D94 11920 0001:00058D9F 11922 0001:00058DAB 11923 0001:00058DB0
 11927 0001:00058DB2 11929 0001:00058DC1 11930 0001:00058DC6 11933 0001:00058DC8
 11934 0001:00058DD1 11935 0001:00058DDB 11936 0001:00058DE5 11938 0001:00058DE9
 11939 0001:00058DEF 11941 0001:00058DF9 11942 0001:00058DFB 11951 0001:00058E00
 11952 0001:00058E24 11953 0001:00058E3E 11959 0001:00058E58 11961 0001:00058E6F
 11963 0001:00058E84 11964 0001:00058E89 11970 0001:00058E8B 11971 0001:00058E8D
 11978 0001:00058E8F 11979 0001:00058E95 11981 0001:00058E99 11982 0001:00058ECC
 11990 0001:00058F24 11991 0001:00058F36 11992 0001:00058F52 12000 0001:00058F58
 12001 0001:00058F5D 12015 0001:00058F60 12016 0001:00058F64 12017 0001:00058F84
 12021 0001:00058F89 12023 0001:00058F8D 12024 0001:00058F97 12025 0001:00058F9E
 12030 0001:00058FB8 12031 0001:00058FC0 12032 0001:00058FC4 12034 0001:00058FC9
 12035 0001:00058FCE 12047 0001:00059024 12050 0001:00059047 12052 0001:0005904D
 12053 0001:0005904F 12061 0001:00059054 12062 0001:00059067 12064 0001:00059072
 12065 0001:00059074 12072 0001:00059079 12076 0001:0005907D 12077 0001:00059085
 12078 0001:00059087 12081 0001:0005908C 12082 0001:000590A6 12083 0001:000590C0
 12090 0001:000590E9 12096 0001:0005910B 12098 0001:00059116 12099 0001:00059118
 12106 0001:0005911A 12107 0001:00059134 12108 0001:00059155 12116 0001:000591AC
 12121 0001:000591CC 12123 0001:000591D2 12124 0001:000591D7 12131 0001:000591D9
 12133 0001:000591DF 12134 0001:000591E4 12139 0001:000591E6 12140 0001:000591F0
 12141 0001:000591FD 12143 0001:00059207 12144 0001:00059228 12149 0001:0005922C
 12150 0001:00059235 12151 0001:00059243 12152 0001:00059251 12155 0001:00059269
 12157 0001:00059282 12165 0001:00059288 12166 0001:00059292 12167 0001:000592A0
 12172 0001:000592AE 12174 0001:000592C8 12176 0001:000592DE 12190 0001:000592E4
 12191 0001:00059307 12192 0001:00059312 12193 0001:00059320 12202 0001:0005932A
 12203 0001:0005933F 12205 0001:00059343 12206 0001:0005934D 12207 0001:00059354
 12216 0001:0005935E 12218 0001:0005936F 12219 0001:00059382 12221 0001:0005938D
 12222 0001:00059390 12223 0001:0005939A 12227 0001:000593A4 12228 0001:000593B2
 12229 0001:000593C0 12230 0001:000593E0 12231 0001:00059403 12232 0001:00059426
 12238 0001:00059443 12240 0001:0005945E 12241 0001:00059466 12242 0001:00059470
 12243 0001:00059477 12247 0001:00059486 12248 0001:00059490 12252 0001:00059498
 12254 0001:000594B0 12255 0001:000594DC 12256 0001:000594FE 12257 0001:00059508
 12258 0001:0005950F 12262 0001:0005951E 12270 0001:0005953F 12273 0001:0005954D
 12274 0001:00059556 12276 0001:00059560 12279 0001:00059572 12283 0001:00059595
 12285 0001:000595C8 12294 0001:00059620 12295 0001:00059642 12299 0001:0005965C
 12300 0001:0005966D 12301 0001:00059694 12303 0001:000596A0 12304 0001:000596AD
 12305 0001:000596B2 12310 0001:000596B7 12312 0001:000596C4 12315 0001:000596CC
 12318 0001:000596D6 12319 0001:000596E1 12320 0001:000596EF 12322 0001:000596F8
 12323 0001:000596FD 12326 0001:00059707 12327 0001:00059711 12328 0001:0005971F
 12329 0001:0005972D 12331 0001:00059745 12334 0001:00059768 12337 0001:0005977B
 12343 0001:00059783 12344 0001:0005978E 12346 0001:0005979A 12347 0001:000597A4
 12348 0001:000597A9 12351 0001:000597AE 12357 0001:000597B6 12360 0001:000597C0
 12361 0001:000597CB 12364 0001:000597D9 12366 0001:000597E2 12367 0001:000597E7
 12369 0001:000597F1 12370 0001:000597FF 12373 0001:0005980D 12374 0001:0005981E
 12376 0001:00059829 12378 0001:00059831 12379 0001:0005983C 12382 0001:0005984E
 12385 0001:00059871 12387 0001:000598A4 12396 0001:000598F8 12397 0001:00059901
 12398 0001:0005990F 12399 0001:0005991D 12400 0001:00059926 12401 0001:00059931
 12403 0001:00059943 12405 0001:0005995C 12413 0001:00059960 12414 0001:00059963
 12419 0001:00059966 12425 0001:0005996B 12431 0001:00059970 12434 0001:00059977
 12435 0001:00059985 12438 0001:00059993 12440 0001:0005999F 12442 0001:000599AA
 12447 0001:000599BF 12449 0001:000599D5 12466 0001:000599D8 12470 0001:000599E0
 12472 0001:000599F5 12473 0001:000599F7 12477 0001:000599FC 12479 0001:00059A02
 12480 0001:00059A09 12485 0001:00059A0B 12486 0001:00059A24 12489 0001:00059A32
 12502 0001:00059A50 12504 0001:00059A55 12505 0001:00059A5C 12509 0001:00059A5E
 12519 0001:00059A7A 12521 0001:00059A7E 12522 0001:00059A85 12525 0001:00059A87
 12526 0001:00059A89 12533 0001:00059A90 12534 0001:00059AAC 12535 0001:00059ABA
 12536 0001:00059AC8 12537 0001:00059AE5 12541 0001:00059B05 12543 0001:00059B0E
 12544 0001:00059B2E 12545 0001:00059B33 12549 0001:00059B3A 12556 0001:00059B45
 12557 0001:00059B4F 12558 0001:00059B54 12564 0001:00059B5B 12565 0001:00059B73
 12566 0001:00059B89 12569 0001:00059B9E 12571 0001:00059BD4 12582 0001:00059C28
 12583 0001:00059C31 12584 0001:00059C39 12585 0001:00059C47 12586 0001:00059C55
 12587 0001:00059C5C 12588 0001:00059C63 12590 0001:00059C7A 12592 0001:00059C8C
 12594 0001:00059CA5 12599 0001:00059CAC 12603 0001:00059CAF 12605 0001:00059CB9
 12606 0001:00059CBF 12608 0001:00059CC7 12617 0001:00059CCC 12618 0001:00059CD5
 12619 0001:00059CE3 12620 0001:00059CF1 12622 0001:00059CFA 12623 0001:00059CFF
 12628 0001:00059D09 12630 0001:00059D10 12631 0001:00059D17 12634 0001:00059D1F
 12635 0001:00059D4B 12639 0001:00059D6D 12641 0001:00059D76 12642 0001:00059D81
 12647 0001:00059D88 12648 0001:00059DA5 12649 0001:00059DB7 12651 0001:00059DC2
 12654 0001:00059DD4 12656 0001:00059DED 12664 0001:00059E44 12665 0001:00059E4D
 12666 0001:00059E5B 12667 0001:00059E69 12669 0001:00059E70 12671 0001:00059E79
 12672 0001:00059E80 12673 0001:00059E88 12675 0001:00059E8F 12678 0001:00059EA1
 12680 0001:00059EBA 12691 0001:00059EC0 12692 0001:00059ECA 12693 0001:00059ED8
 12694 0001:00059EE6 12696 0001:00059EFC 12698 0001:00059F12 12812 0001:00059F18
 12825 0001:00059F3E 12836 0001:00059F40 12844 0001:00059F66 12848 0001:00059F68
 12849 0001:00059F6A 12853 0001:00059F6C 12854 0001:00059F6E 12859 0001:00059F70
 12864 0001:00059F74 12869 0001:00059F78 12875 0001:00059F7C 12877 0001:00059FAA
 12878 0001:00059FD0 12879 0001:00059FD8 12880 0001:0005A026 12885 0001:0005A098
 12886 0001:0005A09C 12887 0001:0005A0AD 12888 0001:0005A0C1 12891 0001:0005A0CF
 12892 0001:0005A0DA 12893 0001:0005A0E0 12897 0001:0005A0E7 12898 0001:0005A0FB
 12899 0001:0005A107 12902 0001:0005A120 12903 0001:0005A134 12905 0001:0005A150
 12914 0001:0005A158 12915 0001:0005A15C 12916 0001:0005A16D 12917 0001:0005A17B
 12918 0001:0005A18F 12919 0001:0005A19D 12920 0001:0005A1A6 12922 0001:0005A1C4
 12924 0001:0005A1E0 12926 0001:0005A201 12928 0001:0005A21D 12933 0001:0005A224
 12934 0001:0005A228 12935 0001:0005A239 12936 0001:0005A24D 12937 0001:0005A25B
 12938 0001:0005A26F 12939 0001:0005A27B 12941 0001:0005A294 12942 0001:0005A2A8
 12944 0001:0005A2C4 12951 0001:0005A2CC 12952 0001:0005A2E7 12953 0001:0005A2FE
 12963 0001:0005A30E 12964 0001:0005A31F 12969 0001:0005A32D 12976 0001:0005A36D
 12977 0001:0005A385 12978 0001:0005A399 12979 0001:0005A3A7 12981 0001:0005A3BC
 12983 0001:0005A3CE 12985 0001:0005A3EA 12988 0001:0005A3FE 12991 0001:0005A417
 12992 0001:0005A439 12995 0001:0005A440 12996 0001:0005A45D 12997 0001:0005A488
 13002 0001:0005A490 13003 0001:0005A494 13004 0001:0005A4A4 13005 0001:0005A4AF
 13006 0001:0005A4BA 13011 0001:0005A4C0 13012 0001:0005A4E1 13013 0001:0005A4F4
 13014 0001:0005A4FF 13015 0001:0005A52A 13020 0001:0005A530 13022 0001:0005A533
 13024 0001:0005A540 13030 0001:0005A550 13031 0001:0005A55E 13037 0001:0005A560
 13038 0001:0005A56E 13050 0001:0005A570 13051 0001:0005A574 13052 0001:0005A582
 13057 0001:0005A584 13058 0001:0005A58B 13059 0001:0005A596 13060 0001:0005A5A1
 13061 0001:0005A5B5 13080 0001:0005A5BC 13083 0001:0005A5F4 13086 0001:0005A60C
 13087 0001:0005A614 13088 0001:0005A61C 13090 0001:0005A623 13113 0001:0005A661
 13118 0001:0005A66C 13119 0001:0005A677 13123 0001:0005A691 13125 0001:0005A6A8
 13150 0001:0005A6FC 13151 0001:0005A6FF 13152 0001:0005A713 13153 0001:0005A71E
 13154 0001:0005A726 13155 0001:0005A730 13156 0001:0005A738 13157 0001:0005A740
 13158 0001:0005A748 13159 0001:0005A750 13160 0001:0005A758 13161 0001:0005A760
 13162 0001:0005A774 13163 0001:0005A788 13164 0001:0005A79C 13165 0001:0005A7A4
 13166 0001:0005A7AC 13167 0001:0005A7C0 13168 0001:0005A7C8 13169 0001:0005A7D0
 13170 0001:0005A7DA 13171 0001:0005A7E2 13176 0001:0005A7F6 13177 0001:0005A7F8
 13267 0001:0005A7FC 13268 0001:0005A802 13269 0001:0005A808 13282 0001:0005A80C
 13284 0001:0005A812 13297 0001:0005A81E 13298 0001:0005A82E 13299 0001:0005A837
 13300 0001:0005A83B 13301 0001:0005A83F 13303 0001:0005A846 13307 0001:0005A84B
 13309 0001:0005A854 13310 0001:0005A863 13315 0001:0005A874 13317 0001:0005A87D
 13322 0001:0005A889 13323 0001:0005A895 13324 0001:0005A89A 13325 0001:0005A8AB
 13326 0001:0005A8D5 13328 0001:0005A8E4 13329 0001:0005A8EA 13334 0001:0005A940
 13335 0001:0005A944 13337 0001:0005A94E 13338 0001:0005A95A 13342 0001:0005A963
 13345 0001:0005A96C 13346 0001:0005A973 13357 0001:0005A978 13358 0001:0005A98D
 13359 0001:0005A995 13363 0001:0005A99F 13364 0001:0005A9B5 13365 0001:0005A9D1
 13373 0001:0005A9D8 13374 0001:0005A9ED 13375 0001:0005AA03 13376 0001:0005AA23
 13386 0001:0005AA28 13392 0001:0005AA3C 13395 0001:0005AA4D 13397 0001:0005AA67
 13398 0001:0005AA7C 13399 0001:0005AA82 13400 0001:0005AA9E 13403 0001:0005AAA4
 13404 0001:0005AAC1 13405 0001:0005AACF 13406 0001:0005AAF0 13410 0001:0005AAF8
 13446 0001:0005AB15 13447 0001:0005AB20 13451 0001:0005AB2A 13452 0001:0005AB43
 13453 0001:0005AB64 13498 0001:0005AB6C 13511 0001:0005AB8D 13513 0001:0005AB99
 13514 0001:0005ABA3 13516 0001:0005ABAA 13517 0001:0005ABB6 13519 0001:0005ABBD
 13521 0001:0005ABC4 13523 0001:0005ABCB 13525 0001:0005ABD3 13531 0001:0005ABE3
 13532 0001:0005ABFF 13533 0001:0005AC07 13536 0001:0005AC10 13540 0001:0005AC31
 13546 0001:0005AC3B 13549 0001:0005AC44 13550 0001:0005AC50 13556 0001:0005AC62
 13558 0001:0005AC69 13559 0001:0005AC72 13576 0001:0005AC79 13585 0001:0005AC93
 13591 0001:0005AC9C 13592 0001:0005ACA4 13593 0001:0005ACB2 13597 0001:0005ACCC
 13598 0001:0005ACE5 13599 0001:0005ACF0 13601 0001:0005ACFE 13602 0001:0005AD07
 13604 0001:0005AD2F 13605 0001:0005AD5B 13631 0001:0005ADB4 13634 0001:0005ADDB
 13645 0001:0005ADF5 13647 0001:0005AE08 13648 0001:0005AE13 13653 0001:0005AE20
 13656 0001:0005AE32 13665 0001:0005AE3F 13674 0001:0005AE4B 13675 0001:0005AE61
 13682 0001:0005AE64 13684 0001:0005AE79 13688 0001:0005AE84 13694 0001:0005AE8E
 13695 0001:0005AE9E 13700 0001:0005AEB2 13701 0001:0005AEB8 13720 0001:0005AEBE
 13729 0001:0005AEE6 13730 0001:0005AEEA 13731 0001:0005AEF4 13732 0001:0005AF04
 13734 0001:0005AF0C 13740 0001:0005AF1C 13741 0001:0005AF20 13743 0001:0005AF26
 13744 0001:0005AF28 13746 0001:0005AF3D 13747 0001:0005AF55 13748 0001:0005AF68
 13749 0001:0005AF76 13751 0001:0005AF7C 13752 0001:0005AF85 13754 0001:0005AF92
 13756 0001:0005AF9B 13781 0001:0005AFE8 13786 0001:0005AFEA 13788 0001:0005AFF0
 13796 0001:0005AFF4 13803 0001:0005B017 13824 0001:0005B019 13825 0001:0005B021
 13827 0001:0005B023 13829 0001:0005B027 13838 0001:0005B02F 13841 0001:0005B048
 13849 0001:0005B064 13851 0001:0005B071 13852 0001:0005B083 13853 0001:0005B08B
 13854 0001:0005B091 13858 0001:0005B098 13865 0001:0005B09E 13871 0001:0005B0A6
 13872 0001:0005B0AC 13873 0001:0005B0B4 13874 0001:0005B0BE 13876 0001:0005B0C7
 13877 0001:0005B0CC 13878 0001:0005B0D0 13880 0001:0005B0D4 13882 0001:0005B0D9
 13886 0001:0005B0DF 13889 0001:0005B0E4 13891 0001:0005B100 13895 0001:0005B114
 13897 0001:0005B126 13899 0001:0005B12A 13902 0001:0005B145 13903 0001:0005B148
 13906 0001:0005B154 13913 0001:0005B156 13931 0001:0005B15C 13932 0001:0005B166
 13933 0001:0005B18A 13945 0001:0005B1E4 13948 0001:0005B205 13949 0001:0005B211
 13950 0001:0005B215 13954 0001:0005B23A 13967 0001:0005B240 13969 0001:0005B248
 13971 0001:0005B24C 13972 0001:0005B253 13975 0001:0005B255 13976 0001:0005B260
 13977 0001:0005B26E 13978 0001:0005B279 13980 0001:0005B28B 13982 0001:0005B2A1
 13989 0001:0005B2A8 13991 0001:0005B2B0 13993 0001:0005B2B4 13994 0001:0005B2BB
 13997 0001:0005B2BD 13998 0001:0005B2C8 13999 0001:0005B2D6 14000 0001:0005B2E1
 14002 0001:0005B2F3 14004 0001:0005B309 14013 0001:0005B310 14015 0001:0005B319
 14017 0001:0005B31D 14018 0001:0005B324 14021 0001:0005B329 14022 0001:0005B334
 14023 0001:0005B342 14026 0001:0005B34B 14029 0001:0005B35D 14031 0001:0005B366
 14033 0001:0005B36A 14034 0001:0005B36E 14038 0001:0005B390 14039 0001:0005B3A7
 14041 0001:0005B3B9 14043 0001:0005B3CF 14050 0001:0005B428 14052 0001:0005B431
 14054 0001:0005B435 14055 0001:0005B43C 14058 0001:0005B441 14059 0001:0005B44C
 14060 0001:0005B45A 14062 0001:0005B463 14063 0001:0005B467 14064 0001:0005B46C
 14068 0001:0005B473 14069 0001:0005B481 14071 0001:0005B487 14072 0001:0005B4A3
 14074 0001:0005B4B5 14076 0001:0005B4CB 14099 0001:0005B4D4 14100 0001:0005B4D7
 14102 0001:0005B4DC 14103 0001:0005B4E4 14107 0001:0005B4EB 14106 0001:0005B4F1
 14109 0001:0005B4F9 14110 0001:0005B4FD 14114 0001:0005B501 14115 0001:0005B512
 14116 0001:0005B516 14117 0001:0005B527 14118 0001:0005B52B 14121 0001:0005B53C
 14122 0001:0005B53E 14133 0001:0005B540 14135 0001:0005B54F 14137 0001:0005B553
 14138 0001:0005B55A 14141 0001:0005B55F 14142 0001:0005B56A 14143 0001:0005B578
 14145 0001:0005B581 14146 0001:0005B585 14147 0001:0005B58A 14155 0001:0005B594
 14156 0001:0005B599 14166 0001:0005B59F 14167 0001:0005B5D0 14169 0001:0005B5E7
 14170 0001:0005B60B 14172 0001:0005B615 14175 0001:0005B627 14177 0001:0005B63D
 14183 0001:0005B698 14186 0001:0005B69E 14187 0001:0005B6C5 14193 0001:0005B6CC
 14197 0001:0005B6D2 14198 0001:0005B6FB 14204 0001:0005B700 14207 0001:0005B70F
 14208 0001:0005B71F 14209 0001:0005B732 14211 0001:0005B736 14212 0001:0005B73D
 14213 0001:0005B74D 14214 0001:0005B760 14216 0001:0005B764 14218 0001:0005B76B
 14219 0001:0005B773 14228 0001:0005B77C 14232 0001:0005B79B 14236 0001:0005B7A7
 14237 0001:0005B7BC 14238 0001:0005B7CD 14241 0001:0005B7D5 14242 0001:0005B80C
 15556 0001:0005B814 15557 0001:0005B82D 15558 0001:0005B840 15575 0001:0005B85C
 15540 0001:0005B860 15555 0001:0005B867

Line numbers for formRenderer(formRenderer.pas) segment .text

    58 0001:0005B9F4    59 0001:0005B9FB    61 0001:0005BA08    97 0001:0005BA2A
    98 0001:0005BA3C    99 0001:0005BA3E   103 0001:0005BA40   104 0001:0005BA42
   107 0001:0005BA48   108 0001:0005BA4E   110 0001:0005BA69   113 0001:0005BA70
   114 0001:0005BA75   118 0001:0005BA78   119 0001:0005BA81   125 0001:0005BA84
   128 0001:0005BA90   129 0001:0005BA9F   130 0001:0005BAA4   134 0001:0005BAAD
   139 0001:0005BAB3   140 0001:0005BACB   141 0001:0005BACD   146 0001:0005BAD2
   155 0001:0005BAF9   160 0001:0005BB11   162 0001:0005BB20   164 0001:0005BB39
   171 0001:0005BB5A   172 0001:0005BB5C   175 0001:0005BB64   176 0001:0005BB6D
   177 0001:0005BB7D   178 0001:0005BB7F   181 0001:0005BB84   182 0001:0005BB8A
   183 0001:0005BB98   184 0001:0005BB9A   187 0001:0005BBA0   188 0001:0005BBA6
   189 0001:0005BBBC   194 0001:0005BBC0   195 0001:0005BBE2   197 0001:0005BBEF
   198 0001:0005BBFB   203 0001:0005BC45   204 0001:0005BC6E   207 0001:0005BC74
   208 0001:0005BC79   209 0001:0005BC88   210 0001:0005BC91   211 0001:0005BC9A
   212 0001:0005BCA7   213 0001:0005BCB4   217 0001:0005BCB8   218 0001:0005BCC0
   220 0001:0005BCF4   220 0001:0005BCFB

Line numbers for VidRenderer(VidRenderer.pas) segment .text

   134 0001:0005BCFC   139 0001:0005C524   140 0001:0005C52A   142 0001:0005C535
   143 0001:0005C53B   146 0001:0005C540   147 0001:0005C544   149 0001:0005C546
   152 0001:0005C54C   153 0001:0005C577   154 0001:0005C594   155 0001:0005C5A6
   156 0001:0005C5BA   157 0001:0005C5F5   162 0001:0005C614   163 0001:0005C62A
   164 0001:0005C655   167 0001:0005C65C   168 0001:0005C667   169 0001:0005C67B
   170 0001:0005C68F   171 0001:0005C6A6   174 0001:0005C6AC   175 0001:0005C6AF
   176 0001:0005C6C3   177 0001:0005C6CA   181 0001:0005C6CC   182 0001:0005C6D1
   185 0001:0005C6D4   186 0001:0005C6D7   188 0001:0005C6DB   189 0001:0005C6E0
   192 0001:0005C6E2   196 0001:0005C718   197 0001:0005C71D   200 0001:0005C71F
   201 0001:0005C721   204 0001:0005C724   205 0001:0005C744   207 0001:0005C74A
   208 0001:0005C74F   211 0001:0005C751   212 0001:0005C75F   213 0001:0005C780
   216 0001:0005C784   217 0001:0005C7A4   218 0001:0005C7CE   223 0001:0005C7D4
   224 0001:0005C7D8   226 0001:0005C7DC   227 0001:0005C7E1   230 0001:0005C7E4
   231 0001:0005C7EA   233 0001:0005C7F0   234 0001:0005C7F5   237 0001:0005C7F8
   238 0001:0005C80B   239 0001:0005C81C   240 0001:0005C81E   243 0001:0005C824
   244 0001:0005C82A   245 0001:0005C83A   248 0001:0005C840   249 0001:0005C846
   250 0001:0005C865   253 0001:0005C86C   254 0001:0005C872   255 0001:0005C895
   260 0001:0005C89C   261 0001:0005C8B6   263 0001:0005C8C9   264 0001:0005C8CE
   267 0001:0005C8D0   269 0001:0005C8E7   271 0001:0005C8F2   273 0001:0005C930
   274 0001:0005C95F   277 0001:0005C978   278 0001:0005C99D   279 0001:0005C9AC
   280 0001:0005C9ED   283 0001:0005C9F4   284 0001:0005CA1C   285 0001:0005CA2B
   286 0001:0005CA64   289 0001:0005CA6C   290 0001:0005CA78   293 0001:0005CA87
   300 0001:0005CAC9   301 0001:0005CAD0   304 0001:0005CAD2   305 0001:0005CAEA
   308 0001:0005CAF4   309 0001:0005CAFC   310 0001:0005CB0B   311 0001:0005CB24
   314 0001:0005CB2C   315 0001:0005CB38   318 0001:0005CB47   320 0001:0005CB62
   327 0001:0005CB68   330 0001:0005CB70   331 0001:0005CB73   333 0001:0005CB77
   334 0001:0005CB7C   338 0001:0005CB7E   339 0001:0005CB96   342 0001:0005CBA0
   343 0001:0005CBA8   344 0001:0005CBB7   345 0001:0005CBD0   348 0001:0005CBD8
   349 0001:0005CBE0   350 0001:0005CBEF   351 0001:0005CBFF   354 0001:0005CC08
   355 0001:0005CC10   356 0001:0005CC1F   357 0001:0005CC31   360 0001:0005CC38
   361 0001:0005CC40   362 0001:0005CC4F   363 0001:0005CC63   366 0001:0005CC6C
   367 0001:0005CC79   369 0001:0005CC88   375 0001:0005CC8C   378 0001:0005CC98
   380 0001:0005CCA9   383 0001:0005CCAE   385 0001:0005CCC3   390 0001:0005CCC8
   395 0001:0005CCCD   397 0001:0005CCD0   398 0001:0005CCD8   401 0001:0005CCE0
   402 0001:0005CCE8   403 0001:0005CCF7   404 0001:0005CD01   407 0001:0005CD08
   408 0001:0005CD10   409 0001:0005CD1F   410 0001:0005CD29   413 0001:0005CD30
   414 0001:0005CD38   415 0001:0005CD47   416 0001:0005CD5C   419 0001:0005CD64
   420 0001:0005CD6C   421 0001:0005CD7B   422 0001:0005CD90   429 0001:0005CD98
   430 0001:0005CDA3   433 0001:0005CDB6   435 0001:0005CDCB   436 0001:0005CDDB
   442 0001:0005CDE9   443 0001:0005CDEF   444 0001:0005CDF5   446 0001:0005CDFA
   454 0001:0005CE24   455 0001:0005CE31   456 0001:0005CE39   461 0001:0005CE44
   462 0001:0005CE4E   464 0001:0005CE5D   465 0001:0005CE72   466 0001:0005CE7A
   467 0001:0005CE82   474 0001:0005CE8C   475 0001:0005CE97   481 0001:0005CEA6
   483 0001:0005CEBB   484 0001:0005CECB   487 0001:0005CED9   488 0001:0005CEDF
   494 0001:0005CEE4   502 0001:0005CF0E   503 0001:0005CF1B   504 0001:0005CF23
   509 0001:0005CF2C   510 0001:0005CF36   511 0001:0005CF45   512 0001:0005CF5A
   513 0001:0005CF65   514 0001:0005CF6D   521 0001:0005CF74   522 0001:0005CF7F
   525 0001:0005CF92   527 0001:0005CFA7   528 0001:0005CFB7   535 0001:0005CFC5
   536 0001:0005CFCB   537 0001:0005CFD1   539 0001:0005CFD6   547 0001:0005D000
   548 0001:0005D00D   549 0001:0005D015   554 0001:0005D020   555 0001:0005D02A
   556 0001:0005D039   557 0001:0005D04E   558 0001:0005D056   559 0001:0005D05E
   566 0001:0005D068   567 0001:0005D073   573 0001:0005D082   575 0001:0005D097
   576 0001:0005D0A7   578 0001:0005D0B5   579 0001:0005D0BB   581 0001:0005D0C0
   589 0001:0005D0EA   590 0001:0005D0F7   591 0001:0005D0FF   596 0001:0005D108
   597 0001:0005D112   599 0001:0005D121   600 0001:0005D136   601 0001:0005D141
   602 0001:0005D149   605 0001:0005D150   606 0001:0005D158   607 0001:0005D167
   610 0001:0005D175   614 0001:0005D182   615 0001:0005D18A   618 0001:0005D190
   619 0001:0005D198   620 0001:0005D1A7   621 0001:0005D1BB   624 0001:0005D1C4
   625 0001:0005D1CC   626 0001:0005D1DB   627 0001:0005D1ED   630 0001:0005D1F4
   631 0001:0005D1FC   632 0001:0005D20B   633 0001:0005D21F   636 0001:0005D228
   637 0001:0005D230   638 0001:0005D23F   639 0001:0005D249   642 0001:0005D250
   643 0001:0005D258   644 0001:0005D267   645 0001:0005D271   648 0001:0005D278
   649 0001:0005D280   650 0001:0005D28F   651 0001:0005D299   654 0001:0005D2A0
   655 0001:0005D2A8   656 0001:0005D2B7   657 0001:0005D2C1   660 0001:0005D2C8
   661 0001:0005D2D0   662 0001:0005D2DF   663 0001:0005D2FB   666 0001:0005D304
   667 0001:0005D310   670 0001:0005D31F   680 0001:0005D349   682 0001:0005D358
   683 0001:0005D35D   685 0001:0005D35F   691 0001:0005D37B   693 0001:0005D395
   699 0001:0005D39C   700 0001:0005D3A5   703 0001:0005D3B8   705 0001:0005D3BD
   706 0001:0005D3E6   713 0001:0005D412   717 0001:0005D42E   718 0001:0005D43E
   719 0001:0005D446   724 0001:0005D4C0   725 0001:0005D4CA   729 0001:0005D4D9
   733 0001:0005D4EE   734 0001:0005D4F6   735 0001:0005D4FE   736 0001:0005D508
   738 0001:0005D512   739 0001:0005D51A   745 0001:0005D524   746 0001:0005D52E
   749 0001:0005D53D   750 0001:0005D549   752 0001:0005D54F   753 0001:0005D556
   756 0001:0005D558   757 0001:0005D56F   758 0001:0005D57A   759 0001:0005D585
   760 0001:0005D58D   766 0001:0005D594   767 0001:0005D59E   770 0001:0005D5AD
   771 0001:0005D5B9   773 0001:0005D5BF   774 0001:0005D5C6   777 0001:0005D5C8
   778 0001:0005D5DF   779 0001:0005D5EA   780 0001:0005D5F5   781 0001:0005D5FD
   787 0001:0005D604   788 0001:0005D60E   792 0001:0005D61D   793 0001:0005D624
   797 0001:0005D639   799 0001:0005D64C   801 0001:0005D65B   802 0001:0005D661
   803 0001:0005D664   804 0001:0005D66A   810 0001:0005D66D   811 0001:0005D675
   812 0001:0005D67D   813 0001:0005D687   815 0001:0005D691   816 0001:0005D699
   819 0001:0005D6A0   820 0001:0005D6A8   821 0001:0005D6B7   822 0001:0005D6C1
   825 0001:0005D6C8   826 0001:0005D6D0   827 0001:0005D6DF   828 0001:0005D6E9
   831 0001:0005D6F0   832 0001:0005D6F8   833 0001:0005D707   834 0001:0005D713
   835 0001:0005D71B   838 0001:0005D724   839 0001:0005D72C   840 0001:0005D73B
   841 0001:0005D746   842 0001:0005D74E   845 0001:0005D754   846 0001:0005D75C
   847 0001:0005D76B   848 0001:0005D776   849 0001:0005D77E   852 0001:0005D784
   853 0001:0005D78C   854 0001:0005D79B   855 0001:0005D7A6   856 0001:0005D7AE
   859 0001:0005D7B4   860 0001:0005D7BC   861 0001:0005D7CB   862 0001:0005D7D6
   863 0001:0005D7DE   866 0001:0005D7E4   867 0001:0005D7EC   868 0001:0005D7FB
   869 0001:0005D805   872 0001:0005D80C   873 0001:0005D814   874 0001:0005D823
   875 0001:0005D82D   878 0001:0005D834   879 0001:0005D83C   880 0001:0005D84B
   881 0001:0005D855   884 0001:0005D85C   885 0001:0005D864   886 0001:0005D873
   887 0001:0005D87D   890 0001:0005D884   891 0001:0005D88C   892 0001:0005D89B
   893 0001:0005D8A5   896 0001:0005D8AC   897 0001:0005D8B4   898 0001:0005D8C3
   899 0001:0005D8CD   902 0001:0005D8D4   903 0001:0005D8DC   904 0001:0005D8EB
   905 0001:0005D8F5   908 0001:0005D8FC   909 0001:0005D904   910 0001:0005D913
   911 0001:0005D91D   914 0001:0005D924   915 0001:0005D92C   916 0001:0005D93B
   917 0001:0005D945   920 0001:0005D94C   921 0001:0005D954   922 0001:0005D963
   923 0001:0005D96D   926 0001:0005D974   927 0001:0005D97C   928 0001:0005D98B
   929 0001:0005D995   932 0001:0005D99C   933 0001:0005D9A4   934 0001:0005D9B3
   935 0001:0005D9BD   938 0001:0005D9C4   939 0001:0005D9CC   940 0001:0005D9DB
   941 0001:0005D9E5   944 0001:0005D9EC   945 0001:0005D9F4   946 0001:0005DA03
   947 0001:0005DA0D   950 0001:0005DA14   951 0001:0005DA1C   952 0001:0005DA2B
   953 0001:0005DA35   956 0001:0005DA3C   957 0001:0005DA44   958 0001:0005DA53
   959 0001:0005DA5D   962 0001:0005DA64   963 0001:0005DA6C   964 0001:0005DA7B
   965 0001:0005DA85   968 0001:0005DA8C   969 0001:0005DA94   970 0001:0005DAA3
   971 0001:0005DAAD   974 0001:0005DAB4   975 0001:0005DABC   976 0001:0005DACB
   977 0001:0005DAD5   980 0001:0005DADC   981 0001:0005DAE4   982 0001:0005DAF3
   983 0001:0005DAFD   986 0001:0005DB04   987 0001:0005DB0C   988 0001:0005DB1B
   989 0001:0005DB25   992 0001:0005DB2C   993 0001:0005DB34   994 0001:0005DB43
   995 0001:0005DB4D   998 0001:0005DB54   999 0001:0005DB5C  1000 0001:0005DB6B
  1001 0001:0005DB76  1002 0001:0005DB81  1003 0001:0005DB89  1006 0001:0005DB90
  1007 0001:0005DB98  1008 0001:0005DBA7  1009 0001:0005DBB1  1012 0001:0005DBB8
  1013 0001:0005DBC0  1014 0001:0005DBCF  1015 0001:0005DBD9  1018 0001:0005DBE0
  1019 0001:0005DBE8  1020 0001:0005DBF7  1021 0001:0005DC01  1024 0001:0005DC08
  1025 0001:0005DC10  1026 0001:0005DC1F  1027 0001:0005DC29  1030 0001:0005DC30
  1031 0001:0005DC38  1032 0001:0005DC47  1033 0001:0005DC51  1036 0001:0005DC58
  1037 0001:0005DC5B  1038 0001:0005DC60  1040 0001:0005DC94  1042 0001:0005DC9D
  1047 0001:0005DCC9

Line numbers for VideoRenderer(E:\VCL\DSPACK234\Demos\D6-D7\Filters\RGB24 Video Renderer\VideoRenderer.dpr) segment .text

    34 0001:0005DF54    35 0001:0005DF64

Bound resource files

c:\program files\borland\delphi7\Lib\Buttons.res
c:\program files\borland\delphi7\Lib\ExtDlgs.res
c:\program files\borland\delphi7\Lib\Controls.res
formRenderer.dfm
VideoRenderer.drf


Program entry point at 0001:0005DF54
